** EXPERIMENTAL (HLL) ** Open Watcom Linker Version 1.6beta1 Limited Availability
Portions Copyright (c) 1985-2002 Sybase, Inc. All Rights Reserved.
Created on:       11/09/21 06:32:12
Executable Image: .libs/php5.dll
creating an OS/2 EMX dynamic link library


                        +------------+
                        |   Groups   |
                        +------------+

Group                           Address              Size
=====                           =======              ====

CGROUP                          0001:00000000        00814a80
DGROUP                          0002:00000000        00022440



                        +--------------+
                        |   Segments   |
                        +--------------+

Segment                Class          Group          Address         Size
=======                =====          =====          =======         ====

TEXT32                 CODE           CGROUP         0001:00000000   00814a78
________TEXT           CODE           CGROUP         0001:00814a80   00000000
DATA32                 DATA           DGROUP         0002:00000000   00008de0
SET1__os2dll           DATA           DGROUP         0002:00008de0   00000004
SET2__os2dll           DATA           DGROUP         0002:00008de4   00000000
SET3__os2dll           DATA           DGROUP         0002:00008de4   00000004
SET1___CTOR_LIST__     DATA           DGROUP         0002:00008de8   00000004
SET2___CTOR_LIST__     DATA           DGROUP         0002:00008dec   00000000
SET3___CTOR_LIST__     DATA           DGROUP         0002:00008dec   00000004
SET1___DTOR_LIST__     DATA           DGROUP         0002:00008df0   00000004
SET2___DTOR_LIST__     DATA           DGROUP         0002:00008df4   00000000
SET3___DTOR_LIST__     DATA           DGROUP         0002:00008df4   00000004
SET1___crtinit1__      DATA           DGROUP         0002:00008df8   00000004
SET2___crtinit1__      DATA           DGROUP         0002:00008dfc   00000000
SET3___crtinit1__      DATA           DGROUP         0002:00008dfc   00000004
SET1___crtexit1__      DATA           DGROUP         0002:00008e00   00000004
SET2___crtexit1__      DATA           DGROUP         0002:00008e04   00000000
SET3___crtexit1__      DATA           DGROUP         0002:00008e04   00000004
SET1___eh_frame__      DATA           DGROUP         0002:00008e08   00000004
SET2___eh_frame__      DATA           DGROUP         0002:00008e0c   0000002c
SET3___eh_frame__      DATA           DGROUP         0002:00008e38   00000004
SET1___eh_init__       DATA           DGROUP         0002:00008e3c   00000004
SET2___eh_init__       DATA           DGROUP         0002:00008e40   00000004
SET3___eh_init__       DATA           DGROUP         0002:00008e44   00000004
SET1___eh_term__       DATA           DGROUP         0002:00008e48   00000004
SET2___eh_term__       DATA           DGROUP         0002:00008e4c   00000004
SET3___eh_term__       DATA           DGROUP         0002:00008e50   00000004
SET1___fork_parent1__  DATA           DGROUP         0002:00008e54   00000004
SET2___fork_parent1__  DATA           DGROUP         0002:00008e58   00000000
SET3___fork_parent1__  DATA           DGROUP         0002:00008e58   00000004
SET1___fork_child1__   DATA           DGROUP         0002:00008e5c   00000004
SET2___fork_child1__   DATA           DGROUP         0002:00008e60   00000000
SET3___fork_child1__   DATA           DGROUP         0002:00008e60   00000004
________DATA           DATA           DGROUP         0002:00008e70   00000000
BSS32                  BSS            DGROUP         0002:00008e70   00017300
c_common               BSS            DGROUP         0002:00020170   000022d0
________BSS            BSS            DGROUP         0002:00022440   00000000


                        +----------------+
                        |   Memory Map   |
                        +----------------+

* = unreferenced symbol
+ = symbol only referenced locally

Address        Symbol
=======        ======

Module: U:\usr\lib\dll0.obj({standard input})
0001:00000000* __text
0002:00000000* __data
0002:00000000* ___data_start
0002:00008e70* ___bss_start
0002:00008de0+ __os2dll
0002:00008de8  ___CTOR_LIST__
0002:00008df0  ___DTOR_LIST__
0002:00008df8* ___crtinit1__
0002:00008e00* ___crtexit1__
0002:00008e08  ___eh_frame__
0002:00008e3c  ___eh_init__
0002:00008e48  ___eh_term__
0002:00008e54+ ___fork_parent1__
0002:00008e5c+ ___fork_child1__
Module: U:\dev\php-5.3.8\ext\date\php_date.o(php_date.o)
0002:00020170  _date_globals_id
0002:00020180  _php_date_global_timezone_db
0002:00020190  _date_ce_interval
0002:000201a0  _date_ce_date
0002:000201b0  _date_ce_timezone
0002:000201c0  _php_date_global_timezone_db_enabled
0002:000201d0  _date_ce_period
0001:00000241  _zm_activate_date
0001:0000028f  _zif_timezone_version_get
0001:000002f6  _zif_date_default_timezone_set
0001:00000402  _zif_timezone_abbreviations_list
0001:00000691  _zif_timezone_identifiers_list
0001:00000b3d  _zim_DatePeriod___construct
0001:00000fd2  _zif_date_timestamp_get
0001:00001105  _zif_date_interval_format
0001:0000170d  _zim_DateInterval___construct
0001:0000194b  _zif_timezone_location_get
0001:00001a8f  _zif_timezone_offset_get
0001:00001bf2  _zif_date_offset_get
0001:00001d28  _zif_timezone_name_from_abbr
0001:00001de4  _zif_timezone_name_get
0001:00002190  _zim_DateTimeZone___construct
0001:000023ec  _zif_date_get_last_errors
0001:0000244a  _zif_time
0001:00002531  _zif_date_interval_create_from_date_string
0001:00002626  _zif_timezone_open
0001:000026d7  _zif_date_diff
0001:00002835  _zif_date_timezone_get
0001:000029a5  _date_object_period_get_iterator
0001:00002a15  _zif_checkdate
0001:00002dc1  _zm_info_date
0001:00002e86  _zm_shutdown_date
0001:0000c100  _date_funcs_date
0001:0000c2d0  _date_funcs_timezone
0001:0000c390  _date_funcs_interval
0001:000056a8  _date_interval_read_property
0001:00005d26  _date_interval_write_property
0001:0000c3e0  _date_funcs_period
0001:00003b03  _zm_startup_date
0001:0000467f  _zm_deactivate_date
0001:0000471d  _zif_date_timestamp_set
0001:00004827  _zif_date_date_set
0001:00004949  _zif_date_time_set
0001:00004a6d  _zif_date_isodate_set
0001:00004c25  _zif_date_modify
0001:00004f12  _zif_date_add
0001:00005218  _zif_date_sub
0001:00005553  _zif_date_timezone_set
0001:0000621d  _php_date_get_date_ce
0001:00006227  _php_date_get_timezone_ce
0001:0000626f  _get_timezone_info
0001:00006390  _zif_date_sun_info
0001:00006eb7  _zif_date_sunset
0001:00006ed3  _zif_date_sunrise
0001:00006eef  _zif_date_default_timezone_get
0001:00006f7d  _zif_localtime
0001:000072a0  _zif_strtotime
0001:0000752d  _php_date_full_day_name
0001:000075b4  _zif_getdate
0001:00007841  _php_date_short_day_name
0001:00008b3d  _zif_date_format
0001:00008f2e  _php_format_date
0001:00008fca  _zif_timezone_transitions_get
0001:00009908  _zif_gmdate
0001:00009924  _zif_date
0001:00009940  _php_idate
0001:00009f34  _zif_idate
0001:0000a003  _php_date_set_tzdb
0001:0000a03c  _php_parse_date
0001:0000a153  _php_mktime
0001:0000a430  _zif_gmmktime
0001:0000a46e  _zif_mktime
0001:0000a4ac  _php_strftime
0001:0000a739  _zif_gmstrftime
0001:0000a777  _zif_strftime
0001:0000a7b5  _php_date_instantiate
0001:0000a7f0  _php_date_initialize
0001:0000ad79  _zim_DateTime___wakeup
0001:0000adb8  _zim_DateTime___set_state
0001:0000ae6e  _zim_DateTime___construct
0001:0000af4c  _zif_date_create_from_format
0001:0000b04e  _zif_date_create
0001:0000b1b7  _php_date_do_return_parsed_time
0001:0000b858  _zif_date_parse_from_format
0001:0000b91d  _zif_date_parse
0001:0000bca0  _date_functions
0002:000000b0  _date_period_it_funcs
0002:00000050  _date_module_entry
Module: U:\dev\php-5.3.8\ext\date\lib\astro.o(astro.o)
0001:0000db90  _timelib_astro_rise_set_altitude
0001:0000e16e  _timelib_ts_to_juliandate
Module: U:\dev\php-5.3.8\ext\date\lib\dow.o(dow.o)
0001:0000e3d0  _timelib_day_of_week
0001:0000e40a  _timelib_iso_day_of_week
0001:0000e444  _timelib_day_of_year
0001:0000e4de  _timelib_days_in_month
0001:0000e555  _timelib_isoweek_from_date
0001:0000e86d  _timelib_daynr_from_weeknr
0001:0000e91f  _timelib_valid_time
0001:0000e982  _timelib_valid_date
Module: U:\dev\php-5.3.8\ext\date\lib\parse_date.o(parse_date.o)
0001:0000fdc9  _timelib_strtotime
0001:0002aa97  _timelib_parse_from_format
0001:0002bd8a  _timelib_fill_holes
0001:0002c0e6  _timelib_timezone_id_from_abbr
0001:0002c107  _timelib_timezone_abbreviations_list
Module: U:\dev\php-5.3.8\ext\date\lib\parse_tz.o(parse_tz.o)
0001:000370ae  _timelib_dump_tzinfo
0001:000372a4  _timelib_builtin_db
0001:000372ae  _timelib_timezone_builtin_identifiers_list
0001:00039ce0  _timezonedb_idx_builtin
0001:000372c1  _timelib_timezone_id_is_valid
0001:000372d7  _timelib_parse_tzfile
0001:000378d5  _timelib_timestamp_is_in_dst
0001:00037903  _timelib_get_time_zone_info
0001:00037a51  _timelib_get_current_offset
0001:0003aed0  _timelib_timezone_db_data_builtin
0001:00079e20  _timezonedb_builtin
Module: U:\dev\php-5.3.8\ext\date\lib\timelib.o(timelib.o)
0001:00079e40  _timelib_time_ctor
0001:00079e5c  _timelib_rel_time_ctor
0001:00079e78  _timelib_time_clone
0001:00079ec0  _timelib_rel_time_clone
0001:00079eda  _timelib_time_tz_abbr_update
0001:00079f57  _timelib_time_dtor
0001:00079f84  _timelib_rel_time_dtor
0001:00079f99  _timelib_time_offset_ctor
0001:00079fb5  _timelib_time_offset_dtor
0001:00079fe2  _timelib_tzinfo_ctor
0001:0007a014  _timelib_tzinfo_clone
0001:0007a11f  _timelib_tzinfo_dtor
0001:0007a1ce  _timelib_get_tz_abbr_ptr
0001:0007a1fb  _timelib_error_container_dtor
0001:0007a274  _timelib_date_to_int
0001:0007a2c2  _timelib_decimal_hour_to_hms
0001:0007a44b  _timelib_dump_date
0001:0007a817  _timelib_dump_rel_time
Module: U:\dev\php-5.3.8\ext\date\lib\tm2unixtime.o(tm2unixtime.o)
0001:0007b205  _timelib_do_rel_normalize
0001:0007ba95  _timelib_update_ts
Module: U:\dev\php-5.3.8\ext\date\lib\unixtime2tm.o(unixtime2tm.o)
0001:0007c680  _timelib_unixtime2gmt
0001:0007cd00  _timelib_update_from_sse
0001:0007cdfd  _timelib_unixtime2local
0001:0007cf0f  _timelib_set_timezone
0001:0007cf8b  _timelib_apply_localtime
Module: U:\dev\php-5.3.8\ext\date\lib\parse_iso_intervals.o(parse_iso_intervals.o)
0001:0007d2d7  _timelib_strtointerval
Module: U:\dev\php-5.3.8\ext\date\lib\interval.o(interval.o)
0001:0007e4f0  _timelib_diff
Module: U:\dev\php-5.3.8\ext\ereg\ereg.o(ereg.o)
0002:000201e0  _ereg_globals_id
0001:0007e8d4  _zm_shutdown_ereg
0001:0007e8dd  _zif_sql_regcase
0001:0007eda7  _zm_info_ereg
0001:0007edd4  _zm_startup_ereg
0001:0007f057  _zif_spliti
0001:0007f073  _zif_split
0001:0007f4dd  _zif_eregi
0001:0007f504  _zif_ereg
0001:0007f52b  _php_ereg_replace
0001:0007fcbf  _zif_eregi_replace
0001:0007fcdb  _zif_ereg_replace
0001:0007fd40  _ereg_functions
0002:00000130  _ereg_module_entry
Module: U:\dev\php-5.3.8\ext\ereg\regex\regcomp.o(regcomp.o)
0001:00082075  _php_regcomp
Module: U:\dev\php-5.3.8\ext\ereg\regex\regexec.o(regexec.o)
0001:0008509c  _php_regexec
Module: U:\dev\php-5.3.8\ext\ereg\regex\regerror.o(regerror.o)
0001:000861ee  _php_regerror
Module: U:\dev\php-5.3.8\ext\ereg\regex\regfree.o(regfree.o)
0001:000866d0  _php_regfree
Module: U:\dev\php-5.3.8\ext\libxml\libxml.o(libxml.o)
0001:0008784b  _php_libxml_structured_error_handler
0001:00087830  _php_libxml_error_handler
0001:0008785c  _php_libxml_issue_error
0001:000878b4  _php_libxml_ctx_error
0001:000878d2  _php_libxml_ctx_warning
0001:000878f0  _php_libxml_initialize
0001:00087f92  _php_libxml_shutdown
0001:00087fdc  _php_libxml_switch_context
0001:00087ff7  _php_libxml_xmlCheckUTF8
0001:000880c3  _php_libxml_register_export
0001:0008811a  _php_libxml_import_node
0001:00088188  _php_libxml_decrement_node_ptr
0001:000881dc  _php_libxml_increment_node_ptr
0001:00088264  _php_libxml_increment_doc_ref
0001:000882b8  _php_libxml_decrement_doc_ref
0001:000884ac  _php_libxml_node_free_resource
0001:00088574  _php_libxml_node_decrement_resource
0002:00000190  _libxml_module_entry
Module: U:\dev\php-5.3.8\ext\pcre\pcrelib\pcre_chartables.o(pcre_chartables.o)
0001:00088830  _php__pcre_default_tables
Module: U:\dev\php-5.3.8\ext\pcre\pcrelib\pcre_ucd.o(pcre_ucd.o)
0001:00088c70  _php__pcre_ucd_records
0001:00089ca0  _php__pcre_ucd_stage1
0001:0008bea0  _php__pcre_ucd_stage2
Module: U:\dev\php-5.3.8\ext\pcre\pcrelib\pcre_compile.o(pcre_compile.o)
0001:000999f6  __pcre_find_bracket
0001:0009f4b0  _php_pcre_compile2
0001:0009fed9  _php_pcre_compile
Module: U:\dev\php-5.3.8\ext\pcre\pcrelib\pcre_config.o(pcre_config.o)
0001:000a0e20  _php_pcre_config
Module: U:\dev\php-5.3.8\ext\pcre\pcrelib\pcre_exec.o(pcre_exec.o)
0001:000a11b1  _php_pcre_exec
Module: U:\dev\php-5.3.8\ext\pcre\pcrelib\pcre_fullinfo.o(pcre_fullinfo.o)
0001:000b79c0  _php_pcre_fullinfo
Module: U:\dev\php-5.3.8\ext\pcre\pcrelib\pcre_get.o(pcre_get.o)
0001:000b7bc0  _php_pcre_get_stringnumber
0001:000b7cb0  _php_pcre_get_stringtable_entries
0001:000b7f00  _php_pcre_copy_substring
0001:000b7f5b  _php_pcre_copy_named_substring
0001:000b7fb6  _php_pcre_get_substring_list
0001:000b806a  _php_pcre_free_substring_list
0001:000b8078  _php_pcre_get_substring
0001:000b80e6  _php_pcre_get_named_substring
0001:000b8135  _php_pcre_free_substring
Module: U:\dev\php-5.3.8\ext\pcre\pcrelib\pcre_globals.o(pcre_globals.o)
0002:000001f0  _php_pcre_malloc
0002:000001f4  _php_pcre_free
0002:000001f8  _php_pcre_stack_malloc
0002:000001fc  _php_pcre_stack_free
0002:000090b0  _php_pcre_callout
Module: U:\dev\php-5.3.8\ext\pcre\pcrelib\pcre_info.o(pcre_info.o)
0001:000b8150  _php_pcre_info
Module: U:\dev\php-5.3.8\ext\pcre\pcrelib\pcre_maketables.o(pcre_maketables.o)
0001:000b81ed  _php_pcre_maketables
Module: U:\dev\php-5.3.8\ext\pcre\pcrelib\pcre_newline.o(pcre_newline.o)
0001:000b8560  _php__pcre_is_newline
0001:000b870c  _php__pcre_was_newline
Module: U:\dev\php-5.3.8\ext\pcre\pcrelib\pcre_ord2utf8.o(pcre_ord2utf8.o)
0001:000b88f0  _php__pcre_ord2utf8
Module: U:\dev\php-5.3.8\ext\pcre\pcrelib\pcre_refcount.o(pcre_refcount.o)
0001:000b8960  _php_pcre_refcount
Module: U:\dev\php-5.3.8\ext\pcre\pcrelib\pcre_study.o(pcre_study.o)
0001:000b9a48  _php_pcre_study
Module: U:\dev\php-5.3.8\ext\pcre\pcrelib\pcre_tables.o(pcre_tables.o)
0001:000b9c30  _php__pcre_OP_lengths
0001:000b9cb0  _php__pcre_utf8_table1
0001:000b9cc8  _php__pcre_utf8_table1_size
0001:000b9cd0  _php__pcre_utf8_table2
0001:000b9cf0  _php__pcre_utf8_table3
0001:000b9d10  _php__pcre_utf8_table4
0001:000b9d50  _php__pcre_ucp_gentype
0001:000b9dd0  _php__pcre_utt_names
0001:000ba180  _php__pcre_utt
0001:000ba4ac  _php__pcre_utt_size
Module: U:\dev\php-5.3.8\ext\pcre\pcrelib\pcre_try_flipped.o(pcre_try_flipped.o)
0001:000ba4d1  _php__pcre_try_flipped
Module: U:\dev\php-5.3.8\ext\pcre\pcrelib\pcre_valid_utf8.o(pcre_valid_utf8.o)
0001:000ba640  _php__pcre_valid_utf8
Module: U:\dev\php-5.3.8\ext\pcre\pcrelib\pcre_version.o(pcre_version.o)
0001:000ba7a0  _php_pcre_version
Module: U:\dev\php-5.3.8\ext\pcre\pcrelib\pcre_xclass.o(pcre_xclass.o)
0001:000ba7b0  _php__pcre_xclass
Module: U:\dev\php-5.3.8\ext\pcre\php_pcre.o(php_pcre.o)
0002:000201f0  _pcre_globals_id
0001:000bbbdc  _pcre_get_compiled_regex_cache
0001:000bc31c  _pcre_get_compiled_regex
0001:000bc381  _pcre_get_compiled_regex_ex
0001:000bc451  _php_pcre_match_impl
0001:000bd17f  _php_pcre_replace_impl
0001:000bdede  _php_pcre_replace
0001:000beabe  _php_pcre_split_impl
0001:000bf1d3  _php_pcre_grep_impl
0002:00000200  _pcre_module_entry
Module: U:\dev\php-5.3.8\ext\sqlite3\sqlite3.o(sqlite3.o)
0002:00020200  _php_sqlite3_sc_entry
0002:00020210  _php_sqlite3_stmt_entry
0002:00020220  _php_sqlite3_result_entry
0002:00020230  _sqlite3_globals_id
0001:000bfe37  _zm_info_sqlite3
0001:000bfead  _zm_shutdown_sqlite3
0001:000bfff0  _zm_startup_sqlite3
0001:000c09de  _zim_sqlite3result___construct
0001:000c0a0f  _zim_sqlite3stmt_close
0001:000c0a7e  _zim_sqlite3_enableExceptions
0001:000c0bcc  _zim_sqlite3result_finalize
0001:000c0c7d  _zim_sqlite3result_reset
0001:000c0d43  _zim_sqlite3stmt_reset
0001:000c0dde  _zim_sqlite3result_columnType
0001:000c0e93  _zim_sqlite3result_columnName
0001:000c0f96  _zim_sqlite3_lastErrorMsg
0001:000c11b8  _zim_sqlite3result_fetchArray
0001:000c136e  _zim_sqlite3result_numColumns
0001:000c13f5  _zim_sqlite3stmt_readOnly
0001:000c1482  _zim_sqlite3stmt_clear
0001:000c151b  _zim_sqlite3stmt_paramCount
0001:000c1596  _zim_sqlite3_openBlob
0001:000c17e0  _zim_sqlite3_querySingle
0001:000c1ab5  _zim_sqlite3_exec
0001:000c1b9f  _zim_sqlite3_escapeString
0001:000c1c56  _zim_sqlite3_changes
0001:000c1db4  _zim_sqlite3_loadExtension
0001:000c2103  _zim_sqlite3_busyTimeout
0001:000c21c8  _zim_sqlite3_lastErrorCode
0001:000c2246  _zim_sqlite3_lastInsertRowID
0001:000c22e0  _zim_sqlite3_version
0001:000c238d  _zim_sqlite3_close
0001:000c257a  _zim_sqlite3_open
0001:000c29e8  _zim_sqlite3stmt_bindValue
0001:000c2b0e  _zim_sqlite3stmt_bindParam
0001:000c2d2a  _zim_sqlite3stmt_execute
0001:000c3112  _zim_sqlite3stmt___construct
0001:000c32c8  _zim_sqlite3_prepare
0001:000c3427  _zim_sqlite3_query
0001:000c3701  _zim_sqlite3_createFunction
0001:000c38ec  _zim_sqlite3_createAggregate
0002:00000260  _sqlite3_module_entry
Module: U:\dev\php-5.3.8\ext\sqlite3\libsqlite\sqlite3.o(sqlite3.o)
0002:00020240  _doclist
0001:000c4970  _sqlite3_compileoption_get
0001:000c4dd6  _sqlite3_vfs_unregister
0001:000c4e5a  _sqlite3_mutex_free
0001:000c4e71  _sqlite3_mutex_enter
0001:000c4e88  _sqlite3_mutex_try
0001:000c4ea1  _sqlite3_mutex_leave
0001:000c4ef4  _sqlite3_release_memory
0001:000c53df  _sqlite3_free
0001:000c5993  _sqlite3_strnicmp
0001:000c5a00  _sqlite3_compileoption_used
0001:000c7c8e  _sqlite3_enable_shared_cache
0001:000c81cc  _sqlite3_backup_remaining
0001:000c81d7  _sqlite3_backup_pagecount
0001:000c84d2  _sqlite3_sql
0001:000c8ab7  _sqlite3_expired
0001:000c8ad1  _sqlite3_value_double
0001:000c8ae0  _sqlite3_value_int
0001:000c8aed  _sqlite3_value_int64
0001:000c8af9  _sqlite3_value_type
0001:000c8b05  _sqlite3_result_null
0001:000c8b17  _sqlite3_result_error_nomem
0001:000c8b3d  _sqlite3_user_data
0001:000c8b4a  _sqlite3_context_db_handle
0001:000c8b55  _sqlite3_get_auxdata
0001:000c8b7f  _sqlite3_aggregate_count
0001:000c8b8d  _sqlite3_column_count
0001:000c8b9f  _sqlite3_data_count
0001:000c8c36  _sqlite3_column_name
0001:000c8c54  _sqlite3_column_name16
0001:000c8c72  _sqlite3_column_decltype
0001:000c8c90  _sqlite3_column_decltype16
0001:000c8cae  _sqlite3_column_database_name
0001:000c8ccc  _sqlite3_column_database_name16
0001:000c8cea  _sqlite3_column_table_name
0001:000c8d08  _sqlite3_column_table_name16
0001:000c8d26  _sqlite3_column_origin_name
0001:000c8d44  _sqlite3_column_origin_name16
0001:000c8d62  _sqlite3_bind_parameter_count
0001:000c8d74  _sqlite3_bind_parameter_name
0001:000c8d9e  _sqlite3_db_handle
0001:000c8dae  _sqlite3_next_stmt
0001:000c8df6  _sqlite3_stmt_status
0001:000c8e84  _sqlite3_blob_bytes
0001:000c9644  _sqlite3_set_authorizer
0001:000ca502  _sqlite3_free_table
0001:000cb432  _sqlite3_complete
0001:000cb94d  _sqlite3_libversion
0001:000cb995  _sqlite3_sourceid
0001:000cb99f  _sqlite3_libversion_number
0001:000cb9a9  _sqlite3_threadsafe
0001:000cbb56  _sqlite3_db_mutex
0001:000cbb9c  _sqlite3_last_insert_rowid
0001:000cbbaa  _sqlite3_changes
0001:000cbbb5  _sqlite3_total_changes
0001:000cbc59  _sqlite3_busy_handler
0001:000cbccb  _sqlite3_progress_handler
0001:000cbd4e  _sqlite3_busy_timeout
0001:000cbe23  _sqlite3_interrupt
0001:000cbe35  _sqlite3_trace
0001:000cbea1  _sqlite3_profile
0001:000cbf0d  _sqlite3_commit_hook
0001:000cbf79  _sqlite3_update_hook
0001:000cbfe5  _sqlite3_rollback_hook
0001:000cc051  _sqlite3_wal_autocheckpoint
0001:000cc0f8  _sqlite3_wal_hook
0001:000cc164  _sqlite3_limit
0001:000cc19c  _sqlite3_collation_needed
0001:000cc20e  _sqlite3_collation_needed16
0001:000cc280  _sqlite3_get_autocommit
0001:000cc28c  _sqlite3_thread_cleanup
0001:000cc291  _sqlite3_extended_result_codes
0001:000cd3e0  _sqlite3_file_control
0001:000cd53b  _sqlite3_db_config
0001:000ce739  _sqlite3_result_int64
0001:000ce7a0  _sqlite3_result_int
0001:000cea8b  _sqlite3_result_zeroblob
0001:000ceb1b  _sqlite3_result_double
0001:000cebac  _sqlite3_clear_bindings
0001:000d1409  _sqlite3_transfer_bindings
0001:000d1b0a  _sqlite3_bind_parameter_index
0001:000d2d88  _sqlite3_value_numeric_type
0001:000e72df  _sqlite3_value_text
0001:000e71d9  _sqlite3_value_text16
0001:001334c6  _sqlite3_version
0001:000d4d26  _sqlite3_db_status
0001:000d5f3a  _sqlite3_memory_alarm
0001:000d5f5d  _convertCpPathToUtf8
0001:000d5fee  _sqlite3_os_end
0001:000d602e  _sqlite3_stmt_readonly
0001:000d6043  _sqlite3_enable_load_extension
0001:000d608e  _sqlite3_vtab_on_conflict
0001:000d60be  _sqlite3_config
0001:000e13a5  _sqlite3_log
0001:000d631f  _sqlite3_initialize
0001:000dcaa3  _sqlite3_malloc
0001:000ef677  _sqlite3_os_init
0001:000d685a  _sqlite3_reset_auto_extension
0001:000d68e7  _sqlite3_shutdown
0001:000d699a  _sqlite3_realloc
0001:000d7427  _sqlite3_result_value
0001:000d7725  _sqlite3_result_error_toobig
0001:000d7805  _sqlite3_result_error_code
0001:000d7891  _sqlite3_result_text16le
0001:000d78b0  _sqlite3_result_text16be
0001:000d78cf  _sqlite3_result_text16
0001:000d78f1  _sqlite3_result_text
0001:000d7ae1  _sqlite3_result_blob
0001:000d7b03  _sqlite3_result_error16
0001:000d7b30  _sqlite3_result_error
0001:000d7f5b  _sqlite3_aggregate_context
0001:000da243  _sqlite3_set_auxdata
0001:000dc9de  _sqlite3_auto_extension
0001:000ddbe3  _sqlite3_create_module_v2
0001:000ddc04  _sqlite3_create_module
0001:000ddce7  _sqlite3_column_type
0001:000ddd0a  _sqlite3_column_value
0001:000ddd3e  _sqlite3_column_int64
0001:000ddd70  _sqlite3_column_int
0001:000ddd9f  _sqlite3_column_double
0001:000e2619  _sqlite3_create_collation16
0001:000e26ab  _sqlite3_create_collation_v2
0001:000e2714  _sqlite3_create_collation
0001:000e2a1b  _sqlite3_overload_function
0001:000e2ae3  _sqlite3_create_function16
0001:000e2b7b  _sqlite3_create_function_v2
0001:000e2c83  _sqlite3_create_function
0001:000e2ccf  _sqlite3_vtab_config
0001:000e2d89  _sqlite3_status
0001:000e2df8  _sqlite3_memory_highwater
0001:000e2e25  _sqlite3_memory_used
0001:000e2ed6  _sqlite3_extended_errcode
0001:000e2f38  _sqlite3_errcode
0001:000e3396  _sqlite3_bind_zeroblob
0001:000e34e2  _sqlite3_bind_text16
0001:000e350f  _sqlite3_bind_text
0001:000e353c  _sqlite3_bind_blob
0001:000e3569  _sqlite3_bind_null
0001:000e359f  _sqlite3_bind_int64
0001:000e3617  _sqlite3_bind_int
0001:000e363d  _sqlite3_bind_double
0001:000e369c  _sqlite3_bind_value
0001:000e377f  _sqlite3_vsnprintf
0001:000e37dc  _sqlite3_snprintf
0001:000e71b1  _sqlite3_value_text16le
0001:000e71c5  _sqlite3_value_text16be
0001:000e71ed  _sqlite3_errmsg16
0001:000e72b0  _sqlite3_column_text16
0001:000e731b  _sqlite3_errmsg
0001:000e858e  _sqlite3_column_text
0001:000e85bd  _sqlite3_value_blob
0001:000e8603  _sqlite3_column_blob
0001:000e8632  _sqlite3_value_bytes16
0001:000e8678  _sqlite3_column_bytes16
0001:000e86a7  _sqlite3_value_bytes
0001:000e95c1  _sqlite3_column_bytes
0001:000ee420  _sqlite3_complete16
0001:000ee492  _sqlite3_vmprintf
0001:000ee500  _sqlite3_mprintf
0001:000eed90  _sqlite3_load_extension
0001:000ef083  _sqlite3_soft_heap_limit64
0001:000ef124  _sqlite3_soft_heap_limit
0001:000ef145  _sqlite3_mutex_alloc
0001:000ef5e1  _sqlite3_vfs_register
0001:000ef69a  _sqlite3_vfs_find
0001:000ef71c  _sqlite3_sleep
0001:000efd97  _sqlite3_randomness
0001:000eff38  _sqlite3_test_control
0001:000ffc6c  _sqlite3_backup_init
0001:001022af  _sqlite3_close
0001:00102a3b  _sqlite3_backup_finish
0001:001073fa  _sqlite3_backup_step
0001:001088e9  _sqlite3_blob_write
0001:0010890b  _sqlite3_blob_read
0001:00108969  _sqlite3_finalize
0001:00108ac2  _sqlite3_blob_close
0001:00109865  _sqlite3_reset
0001:001159d5  _sqlite3_exec
0001:00113481  _sqlite3_step
0001:00129caf  _sqlite3_prepare
0001:001164e7  _sqlite3_table_column_metadata
0001:00125851  _sqlite3_declare_vtab
0001:00129a89  _sqlite3_prepare16_v2
0001:00129ab6  _sqlite3_prepare16
0001:00129ae3  _sqlite3_prepare_v2
0001:0012a584  _sqlite3_get_table
0001:0012c7a3  _sqlite3_blob_reopen
0001:0012c902  _sqlite3_blob_open
0001:001331cc  _sqlite3_open_v2
0001:001331e7  _sqlite3_open
0001:00133205  _sqlite3_open16
0001:001332b9  _sqlite3_wal_checkpoint_v2
0001:001333a5  _sqlite3_wal_checkpoint
0001:00133411  _sqlite3_global_recover
0001:00133418  _sqlite3_uri_parameter
0002:00009210  _sqlite3_temp_directory
Module: U:\dev\php-5.3.8\ext\zlib\zlib.o(zlib.o)
0002:00020260  _zlib_globals_id
0001:0013a3ca  _php_ob_gzhandler_check
0002:00001070  _php_zlib_module_entry
Module: U:\dev\php-5.3.8\ext\zlib\zlib_fopen_wrapper.o(zlib_fopen_wrapper.o)
0001:0013ae59  _php_stream_gzopen
0002:000010d0  _php_stream_gzip_wrapper
Module: U:\dev\php-5.3.8\ext\zlib\zlib_filter.o(zlib_filter.o)
0002:00001150  _php_zlib_filter_factory
Module: U:\dev\php-5.3.8\ext\ctype\ctype.o(ctype.o)
0002:00001170  _ctype_module_entry
Module: U:\dev\php-5.3.8\ext\dom\php_dom.o(php_dom.o)
0002:00020270  _dom_xpath_class_entry
0002:00020280  _dom_object_handlers
0002:000202f0  _dom_domexception_class_entry
0002:00020300  _dom_domstringlist_class_entry
0002:00020310  _dom_namelist_class_entry
0002:00020320  _dom_domimplementationlist_class_entry
0002:00020330  _dom_domimplementationsource_class_entry
0002:00020340  _dom_domimplementation_class_entry
0002:00020350  _dom_node_class_entry
0002:00020360  _dom_namespace_node_class_entry
0002:00020370  _dom_documentfragment_class_entry
0002:00020380  _dom_document_class_entry
0002:00020390  _dom_nodelist_class_entry
0002:000203a0  _dom_namednodemap_class_entry
0002:000203b0  _dom_characterdata_class_entry
0002:000203c0  _dom_attr_class_entry
0002:000203d0  _dom_element_class_entry
0002:000203e0  _dom_text_class_entry
0002:000203f0  _dom_comment_class_entry
0002:00020400  _dom_typeinfo_class_entry
0002:00020410  _dom_userdatahandler_class_entry
0002:00020420  _dom_domerror_class_entry
0002:00020430  _dom_domerrorhandler_class_entry
0002:00020440  _dom_domlocator_class_entry
0002:00020450  _dom_domconfiguration_class_entry
0002:00020460  _dom_cdatasection_class_entry
0002:00020470  _dom_documenttype_class_entry
0002:00020480  _dom_notation_class_entry
0002:00020490  _dom_entity_class_entry
0002:000204a0  _dom_entityreference_class_entry
0002:000204b0  _dom_processinginstruction_class_entry
0002:000204c0  _dom_string_extend_class_entry
0001:0013d4e7  _dom_nnodemap_objects_new
0001:00142841  _dom_objects_clone
0001:0013d61a  _dom_nnodemap_objects_free_storage
0001:0013d56e  _dom_objects_new
0001:0013d6e9  _dom_objects_free_storage
0001:0013d64e  _dom_xpath_objects_new
0001:0013d758  _dom_xpath_objects_free_storage
0001:0013d7d6  _zm_shutdown_dom
0001:0013d969  _zm_info_dom
0001:0013da8e  _dom_objects_store_clone_obj
0001:0013db59  _php_dom_export_node
0001:0013e432  _zm_startup_dom
0001:001422a5  _dom_read_property
0001:00142621  _dom_write_property
0001:00142715  _dom_node_is_read_only
0001:00142776  _dom_node_children_valid
0001:00142792  _dom_get_doc_props
0001:001429b9  _dom_set_doc_classmap
0001:00142a9c  _dom_get_doc_classmap
0001:00142af4  _dom_get_strict_error
0001:00142b28  _dom_object_get_node
0001:00142b41  _php_dom_object_get_data
0001:00142b5a  _node_list_unlink
0001:00142c14  _dom_namednode_iter
0001:00142c89  _php_dom_create_interator
0001:00142cdf  _php_dom_create_object
0001:00142f31  _zif_dom_import_simplexml
0001:00143015  _php_dom_create_implementation
0001:0014303a  _dom_hierarchy
0001:00143090  _dom_has_feature
0001:0014311c  _dom_get_elements_by_tag_name_ns_raw
0001:00143258  _dom_normalize
0001:00143361  _dom_set_old_ns
0001:001433e2  _dom_check_qname
0001:0014348f  _dom_get_ns
0001:00143570  _dom_get_nsdecl
0002:000011d0  _dom_module_entry
Module: U:\dev\php-5.3.8\ext\dom\attr.o(attr.o)
0001:00143714  _zif_dom_attr_is_id
0001:001437cd  _zim_domattr___construct
0001:0014394b  _dom_attr_name_read
0001:001439d5  _dom_attr_specified_read
0001:00143a02  _dom_attr_value_read
0001:00143ada  _dom_attr_value_write
0001:00143c02  _dom_attr_owner_element_read
0001:00143cdf  _dom_attr_schema_type_info_read
0001:00143d40  _php_dom_attr_class_functions
Module: U:\dev\php-5.3.8\ext\dom\document.o(document.o)
0001:00143e14  _zif_dom_document_rename_node
0001:00143e3b  _zif_dom_document_adopt_node
0001:00143efd  _zim_domdocument_registerNodeClass
0001:001441c9  _zif_dom_document_save_html
0001:0014448e  _zif_dom_document_save_html_file
0001:001445bf  _zif_dom_document_validate
0001:00144739  _zif_dom_document_xinclude
0001:00144840  _zif_dom_document_savexml
0001:00144b71  _zif_dom_document_save
0001:00144cfd  _zim_domdocument___construct
0001:00144e98  _zif_dom_document_normalize_document
0001:00144f5e  _zif_dom_document_get_element_by_id
0001:00145086  _zif_dom_document_get_elements_by_tag_name_ns
0001:001451bd  _zif_dom_document_get_elements_by_tag_name
0001:001452c8  _zif_dom_document_create_attribute
0001:00145461  _zif_dom_document_create_attribute_ns
0001:0014571f  _zif_dom_document_create_element
0001:001458b8  _zif_dom_document_create_element_ns
0001:00145ba7  _zif_dom_document_import_node
0001:00145e38  _zif_dom_document_create_entity_reference
0001:00145f9e  _zif_dom_document_create_processing_instruction
0001:0014612e  _zif_dom_document_create_cdatasection
0001:00146250  _zif_dom_document_create_comment
0001:0014636b  _zif_dom_document_create_text_node
0001:00146486  _zif_dom_document_create_document_fragment
0001:00146824  _zim_domdocument_loadHTML
0001:00146846  _zim_domdocument_loadHTMLFile
0001:00146868  _dom_document_doctype_read
0001:0014693a  _dom_document_implementation_read
0001:00146970  _dom_document_document_element_read
0001:00146a42  _dom_document_encoding_read
0001:00146af9  _dom_document_encoding_write
0001:00146c0e  _dom_document_standalone_read
0001:00146c79  _dom_document_standalone_write
0001:00146d43  _dom_document_version_read
0001:00146de0  _dom_document_version_write
0001:00146ec4  _dom_document_strict_error_checking_read
0001:00146f24  _dom_document_strict_error_checking_write
0001:00146f9b  _dom_document_format_output_read
0001:00146ffa  _dom_document_format_output_write
0001:00147070  _dom_document_validate_on_parse_read
0001:001470d0  _dom_document_validate_on_parse_write
0001:00147147  _dom_document_resolve_externals_read
0001:001471a7  _dom_document_resolve_externals_write
0001:0014721e  _dom_document_preserve_whitespace_read
0001:0014727e  _dom_document_preserve_whitespace_write
0001:001472f5  _dom_document_recover_read
0001:00147355  _dom_document_recover_write
0001:001473cc  _dom_document_substitue_entities_read
0001:0014742c  _dom_document_substitue_entities_write
0001:001474a3  _dom_document_document_uri_read
0001:0014753f  _dom_document_document_uri_write
0001:00147623  _dom_document_config_read
0001:00147666  __dom_get_valid_file_path
0001:00147a57  _zif_dom_document_relaxNG_validate_xml
0001:00147a84  _zif_dom_document_relaxNG_validate_file
0001:00147db6  _zif_dom_document_schema_validate_xml
0001:00147de3  _zif_dom_document_schema_validate_file
0001:001482f1  _zim_domdocument_loadXML
0001:00148313  _zim_domdocument_load
0001:00148520  _php_dom_document_class_functions
Module: U:\dev\php-5.3.8\ext\dom\domerrorhandler.o(domerrorhandler.o)
0001:00149044  _zif_dom_domerrorhandler_handle_error
0001:00149080  _php_dom_domerrorhandler_class_functions
Module: U:\dev\php-5.3.8\ext\dom\domstringlist.o(domstringlist.o)
0001:00149104  _zif_dom_domstringlist_item
0001:00149130  _dom_domstringlist_length_read
0001:00149190  _php_dom_domstringlist_class_functions
Module: U:\dev\php-5.3.8\ext\dom\domexception.o(domexception.o)
0001:001491f0  _php_dom_throw_error_with_message
0001:00149239  _php_dom_throw_error
0001:00149280  _php_dom_domexception_class_functions
Module: U:\dev\php-5.3.8\ext\dom\namelist.o(namelist.o)
0001:00149434  _zif_dom_namelist_get_namespace_uri
0001:0014945b  _zif_dom_namelist_get_name
0001:00149487  _dom_namelist_length_read
0001:001494f0  _php_dom_namelist_class_functions
Module: U:\dev\php-5.3.8\ext\dom\processinginstruction.o(processinginstruction.o)
0001:001495a5  _zim_domprocessinginstruction___construct
0001:0014971c  _dom_processinginstruction_target_read
0001:001497a7  _dom_processinginstruction_data_read
0001:0014987f  _dom_processinginstruction_data_write
0001:00149980  _php_dom_processinginstruction_class_functions
Module: U:\dev\php-5.3.8\ext\dom\cdatasection.o(cdatasection.o)
0001:00149a13  _zim_domcdatasection___construct
0001:00149b50  _php_dom_cdatasection_class_functions
Module: U:\dev\php-5.3.8\ext\dom\documentfragment.o(documentfragment.o)
0001:00149c2f  _zim_domdocumentfragment_appendXML
0001:00149da5  _zim_domdocumentfragment___construct
0001:00149ec0  _php_dom_documentfragment_class_functions
Module: U:\dev\php-5.3.8\ext\dom\domimplementation.o(domimplementation.o)
0001:00149f64  _zim_domimplementation_getFeature
0001:00149ff2  _zim_domimplementation_createDocument
0001:0014a3af  _zim_domimplementation_createDocumentType
0001:0014a5a8  _zim_domimplementation_hasFeature
0001:0014a660  _php_dom_domimplementation_class_functions
Module: U:\dev\php-5.3.8\ext\dom\element.o(element.o)
0001:0014a900  _zif_dom_element_set_id_attribute_node
0001:0014aa62  _zif_dom_element_set_id_attribute_ns
0001:0014abbb  _zif_dom_element_set_id_attribute
0001:0014ad26  _zif_dom_element_has_attribute_ns
0001:0014afb8  _zif_dom_element_has_attribute
0001:0014b086  _zif_dom_element_get_elements_by_tag_name_ns
0001:0014b1bd  _zif_dom_element_get_elements_by_tag_name
0001:0014b30a  _zif_dom_element_set_attribute_node_ns
0001:0014b609  _zif_dom_element_get_attribute_node_ns
0001:0014b73b  _zif_dom_element_remove_attribute_node
0001:0014b90c  _zif_dom_element_set_attribute_node
0001:0014bbbc  _zif_dom_element_remove_attribute_ns
0001:0014bd8c  _zif_dom_element_remove_attribute
0001:0014bf2b  _zif_dom_element_set_attribute
0001:0014c1e7  _zif_dom_element_set_attribute_ns
0001:0014c87e  _zif_dom_element_get_attribute_ns
0001:0014ca0a  _zif_dom_element_get_attribute
0001:0014cb7a  _zif_dom_element_get_attribute_node
0001:0014cd34  _zim_domelement___construct
0001:0014d049  _dom_element_tag_name_read
0001:0014d154  _dom_element_schema_type_info_read
0001:0014d2c0  _php_dom_element_class_functions
Module: U:\dev\php-5.3.8\ext\dom\node.o(node.o)
0001:0014da04  _zif_dom_node_get_user_data
0001:0014da2b  _zif_dom_node_set_user_data
0001:0014da52  _zif_dom_node_get_feature
0001:0014da79  _zif_dom_node_is_equal_node
0001:0014daa0  _zif_dom_node_compare_document_position
0001:0014daf4  _zim_domnode_getLineNo
0001:0014dbb6  _zim_domnode_getNodePath
0001:0014dca3  _zif_dom_node_is_same_node
0001:0014dd81  _zif_dom_node_has_attributes
0001:0014de40  _zif_dom_node_lookup_namespace_uri
0001:0014df63  _zif_dom_node_is_default_namespace
0001:0014e079  _zif_dom_node_lookup_prefix
0001:0014e1f2  _zif_dom_node_is_supported
0001:0014e284  _zif_dom_node_normalize
0001:0014e34e  _zif_dom_node_clone_node
0001:0014e55f  _zif_dom_node_has_child_nodes
0001:0014e62a  _zif_dom_node_remove_child
0001:0014efdb  _zim_domnode_C14NFile
0001:0014effd  _zim_domnode_C14N
0001:0014f105  _zif_dom_node_append_child
0001:0014f535  _zif_dom_node_replace_child
0001:0014f950  _zif_dom_node_insert_before
0001:00150099  _dom_node_node_name_read
0001:001502be  _dom_node_node_value_read
0001:001503dd  _dom_node_node_value_write
0001:00150521  _dom_node_node_type_read
0001:0015059c  _dom_node_parent_node_read
0001:00150665  _dom_node_child_nodes_read
0001:0015073b  _dom_node_first_child_read
0001:0015082b  _dom_node_last_child_read
0001:0015091b  _dom_node_previous_sibling_read
0001:001509e4  _dom_node_next_sibling_read
0001:00150aa2  _dom_node_attributes_read
0001:00150b70  _dom_node_owner_document_read
0001:00150c65  _dom_node_namespace_uri_read
0001:00150d40  _dom_node_prefix_read
0001:00150e73  _dom_node_prefix_write
0001:00151109  _dom_node_local_name_read
0001:001511b6  _dom_node_base_uri_read
0001:00151270  _dom_node_text_content_read
0001:00151343  _dom_node_text_content_write
0001:00151470  _php_dom_node_class_functions
Module: U:\dev\php-5.3.8\ext\dom\string_extend.o(string_extend.o)
0001:00151c34  _zif_dom_string_extend_find_offset32
0001:00151c5b  _zif_dom_string_extend_find_offset16
0001:00151ca0  _php_dom_string_extend_class_functions
Module: U:\dev\php-5.3.8\ext\dom\characterdata.o(characterdata.o)
0001:00151d77  _zif_dom_characterdata_replace_data
0001:00151fde  _zif_dom_characterdata_delete_data
0001:001521da  _zif_dom_characterdata_insert_data
0001:00152390  _zif_dom_characterdata_append_data
0001:00152457  _zif_dom_characterdata_substring_data
0001:0015261d  _dom_characterdata_data_read
0001:001526f5  _dom_characterdata_data_write
0001:001527e7  _dom_characterdata_length_read
0001:001528b0  _php_dom_characterdata_class_functions
Module: U:\dev\php-5.3.8\ext\dom\documenttype.o(documenttype.o)
0001:00152ac0  _dom_documenttype_name_read
0001:00152b4a  _dom_documenttype_entities_read
0001:00152c0b  _dom_documenttype_notations_read
0001:00152ccd  _dom_documenttype_public_id_read
0001:00152d73  _dom_documenttype_system_id_read
0001:00152e19  _dom_documenttype_internal_subset_read
0001:00152f30  _php_dom_documenttype_class_functions
Module: U:\dev\php-5.3.8\ext\dom\domimplementationlist.o(domimplementationlist.o)
0001:00152f64  _zif_dom_domimplementationlist_item
0001:00152f90  _dom_domimplementationlist_length_read
0001:00152ff0  _php_dom_domimplementationlist_class_functions
Module: U:\dev\php-5.3.8\ext\dom\entity.o(entity.o)
0001:00153050  _dom_entity_public_id_read
0001:001530ee  _dom_entity_system_id_read
0001:0015318c  _dom_entity_notation_name_read
0001:0015323f  _dom_entity_actual_encoding_read
0001:00153265  _dom_entity_actual_encoding_write
0001:0015326c  _dom_entity_encoding_read
0001:00153292  _dom_entity_encoding_write
0001:00153299  _dom_entity_version_read
0001:001532bf  _dom_entity_version_write
0001:001532d0  _php_dom_entity_class_functions
Module: U:\dev\php-5.3.8\ext\dom\nodelist.o(nodelist.o)
0001:00153316  _zif_dom_nodelist_item
0001:0015354a  _dom_nodelist_length_read
0001:00153690  _php_dom_nodelist_class_functions
Module: U:\dev\php-5.3.8\ext\dom\text.o(text.o)
0001:00153704  _zif_dom_text_replace_whole_text
0001:0015373f  _zif_dom_text_is_whitespace_in_element_content
0001:00153801  _zif_dom_text_split_text
0001:001539ef  _zim_domtext___construct
0001:00153b05  _dom_text_whole_text_read
0001:00153ca0  _php_dom_text_class_functions
Module: U:\dev\php-5.3.8\ext\dom\comment.o(comment.o)
0001:00153de4  _zim_domcomment___construct
0001:00153f10  _php_dom_comment_class_functions
Module: U:\dev\php-5.3.8\ext\dom\domconfiguration.o(domconfiguration.o)
0001:00153f84  _zif_dom_domconfiguration_can_set_parameter
0001:00153fab  _zif_dom_domconfiguration_get_parameter
0001:00153fd2  _zif_dom_domconfiguration_set_parameter
0001:00154030  _php_dom_domconfiguration_class_functions
Module: U:\dev\php-5.3.8\ext\dom\domimplementationsource.o(domimplementationsource.o)
0001:00154174  _zif_dom_domimplementationsource_get_domimplementations
0001:0015419b  _zif_dom_domimplementationsource_get_domimplementation
0001:001541f0  _php_dom_domimplementationsource_class_functions
Module: U:\dev\php-5.3.8\ext\dom\entityreference.o(entityreference.o)
0001:001542a3  _zim_domentityreference___construct
0001:00154420  _php_dom_entityreference_class_functions
Module: U:\dev\php-5.3.8\ext\dom\notation.o(notation.o)
0001:00154481  _dom_notation_public_id_read
0001:00154527  _dom_notation_system_id_read
0001:001545d0  _php_dom_notation_class_functions
Module: U:\dev\php-5.3.8\ext\dom\xpath.o(xpath.o)
0001:0015460a  _zif_dom_xpath_register_ns
0001:00154727  _zim_domxpath___construct
0001:00155852  _zif_dom_xpath_evaluate
0001:00155874  _zif_dom_xpath_query
0001:001558b4  _zif_dom_xpath_register_php_functions
0001:00155c02  _dom_xpath_document_read
0001:00155ce0  _php_dom_xpath_class_functions
Module: U:\dev\php-5.3.8\ext\dom\dom_iterators.o(dom_iterators.o)
0001:00156019  _create_notation
0001:001560ba  _php_dom_libxml_hash_iter
0001:00156128  _php_dom_libxml_notation_iter
0001:001563e9  _php_dom_get_iterator
0002:00001230  _php_dom_iterator_funcs
Module: U:\dev\php-5.3.8\ext\dom\typeinfo.o(typeinfo.o)
0001:00156600  _dom_typeinfo_type_name_read
0001:00156626  _dom_typeinfo_type_namespace_read
0001:00156650  _php_dom_typeinfo_class_functions
Module: U:\dev\php-5.3.8\ext\dom\domerror.o(domerror.o)
0001:00156675  _dom_domerror_severity_read
0001:001566c3  _dom_domerror_message_read
0001:00156711  _dom_domerror_type_read
0001:0015675f  _dom_domerror_related_exception_read
0001:001567ad  _dom_domerror_related_data_read
0001:001567fb  _dom_domerror_location_read
0001:00156850  _php_dom_domerror_class_functions
Module: U:\dev\php-5.3.8\ext\dom\domlocator.o(domlocator.o)
0001:00156875  _dom_domlocator_line_number_read
0001:001568c3  _dom_domlocator_column_number_read
0001:00156911  _dom_domlocator_offset_read
0001:0015695f  _dom_domlocator_related_node_read
0001:001569ad  _dom_domlocator_uri_read
0001:00156a00  _php_dom_domlocator_class_functions
Module: U:\dev\php-5.3.8\ext\dom\namednodemap.o(namednodemap.o)
0001:00156a34  _zif_dom_namednodemap_remove_named_item_ns
0001:00156a5b  _zif_dom_namednodemap_set_named_item_ns
0001:00156a82  _zif_dom_namednodemap_remove_named_item
0001:00156aa9  _zif_dom_namednodemap_set_named_item
0001:00156afa  _zif_dom_namednodemap_get_named_item_ns
0001:00156c79  _zif_dom_namednodemap_item
0001:00156dd8  _zif_dom_namednodemap_get_named_item
0001:00156f38  _dom_namednodemap_length_read
0001:00157040  _php_dom_namednodemap_class_functions
Module: U:\dev\php-5.3.8\ext\dom\userdatahandler.o(userdatahandler.o)
0001:001572d4  _zif_dom_userdatahandler_handle
0001:00157310  _php_dom_userdatahandler_class_functions
Module: U:\dev\php-5.3.8\ext\fileinfo\fileinfo.o(fileinfo.o)
0002:000204d0  _finfo_class_entry
0001:0015738d  _zif_finfo_set_flags
0001:0015750b  _zif_finfo_close
0001:001575ab  _finfo_resource_destructor
0001:0015761b  _zif_finfo_open
0001:0015785d  _zm_info_fileinfo
0001:0015794b  _zm_startup_finfo
0001:00157c47  _finfo_objects_new
0001:0015843c  _zif_mime_content_type
0001:00158465  _zif_finfo_buffer
0001:0015848e  _zif_finfo_file
0002:00001250  _finfo_class_functions
0002:000012c0  _fileinfo_functions
0002:00001350  _fileinfo_module_entry
Module: U:\dev\php-5.3.8\ext\fileinfo\libmagic\apprentice.o(apprentice.o)
0002:000204e0  _file_formats
0002:00020590  _file_names
0001:00159508  _file_delmagic
0001:0015955b  _file_signextend
0001:0015c7b0  _php_magic_database
0001:0015c4e4  _file_apprentice
0001:0015c646  _file_showstr
0001:0015c79c  _file_nformats
0001:0015c7a0  _file_nnames
Module: U:\dev\php-5.3.8\ext\fileinfo\libmagic\ascmagic.o(ascmagic.o)
0001:003087fe  _file_ascmagic_with_encoding
0001:0030907e  _file_ascmagic
Module: U:\dev\php-5.3.8\ext\fileinfo\libmagic\cdf.o(cdf.o)
0001:00309973  _cdf_tole2
0001:00309994  _cdf_tole4
0001:003099bb  _cdf_tole8
0001:00309a0d  _cdf_swap_header
0001:00309ba9  _cdf_unpack_header
0001:00309c6a  _cdf_swap_dir
0001:00309d64  _cdf_swap_class
0001:00309dd6  _cdf_unpack_dir
0001:00309e6b  _cdf_read_header
0001:00309f00  _cdf_read_sector
0001:00309f37  _cdf_read_short_sector
0001:00309f70  _cdf_read_sat
0001:0030a1f5  _cdf_count_chain
0001:0030a27e  _cdf_read_long_sector_chain
0001:0030a3ed  _cdf_read_short_sector_chain
0001:0030a528  _cdf_read_sector_chain
0001:0030a596  _cdf_read_dir
0001:0030a79a  _cdf_read_ssat
0001:0030a8ae  _cdf_read_short_stream
0001:0030a94a  _cdf_read_summary_info
0001:0030aa77  _cdf_read_property_info
0001:0030b0d2  _cdf_unpack_summary_info
0001:0030b301  _cdf_print_classid
0001:0030b384  _cdf_print_property_name
0001:0030b3fa  _cdf_print_elapsed_time
Module: U:\dev\php-5.3.8\ext\fileinfo\libmagic\cdf_time.o(cdf_time.o)
0001:0030b7d0  _cdf_timestamp_to_timespec
0001:0030ba9b  _cdf_timespec_to_timestamp
Module: U:\dev\php-5.3.8\ext\fileinfo\libmagic\compress.o(compress.o)
0001:0030bb6d  _sread
0001:0030bc7f  _file_pipe2file
Module: U:\dev\php-5.3.8\ext\fileinfo\libmagic\encoding.o(encoding.o)
0001:0030be40  _file_looks_utf8
0001:0030c0a5  _file_encoding
Module: U:\dev\php-5.3.8\ext\fileinfo\libmagic\fsmagic.o(fsmagic.o)
0001:0030c89d  _file_fsmagic
Module: U:\dev\php-5.3.8\ext\fileinfo\libmagic\funcs.o(funcs.o)
0001:0030cc16  _file_printf
0001:0030cdaf  _file_error
0001:0030cdd3  _file_magerror
0001:0030ce0f  _file_oomem
0001:0030ce4a  _file_badseek
0001:0030ce7e  _file_badread
0001:0030cf45  _file_buffer
0001:0030d393  _file_reset
0001:0030d401  _file_getbuffer
0001:0030d4ce  _file_check_mem
Module: U:\dev\php-5.3.8\ext\fileinfo\libmagic\is_tar.o(is_tar.o)
0001:0030d5a3  _file_is_tar
Module: U:\dev\php-5.3.8\ext\fileinfo\libmagic\magic.o(magic.o)
0001:0030dc42  _magic_open
0001:0030dcb3  _magic_close
0001:0030dd02  _magic_load
0001:0030dd41  _magic_compile
0001:0030dd74  _magic_descriptor
0001:0030dd87  _magic_file
0001:0030dd9b  _magic_stream
0001:0030ddaf  _magic_buffer
0001:0030de0c  _magic_error
0001:0030de1f  _magic_errno
0001:0030de32  _magic_setflags
Module: U:\dev\php-5.3.8\ext\fileinfo\libmagic\print.o(print.o)
0001:0030de9c  _file_magwarn
0001:0030df1b  _file_fmttime
Module: U:\dev\php-5.3.8\ext\fileinfo\libmagic\readcdf.o(readcdf.o)
0001:0030e517  _file_trycdf
Module: U:\dev\php-5.3.8\ext\fileinfo\libmagic\softmagic.o(softmagic.o)
0001:00310aa4  _file_softmagic
Module: U:\dev\php-5.3.8\ext\filter\filter.o(filter.o)
0002:00020640  _filter_globals_id
0001:0031258b  _zif_filter_id
0001:0031261f  _zif_filter_list
0001:00312834  _zif_filter_has_var
0001:00312960  _zm_info_filter
0001:003129b9  _zm_deactivate_filter
0001:00312ab0  _zm_shutdown_filter
0001:00312f60  _zm_startup_filter
0001:00314bf7  _zif_filter_var_array
0001:00314caa  _zif_filter_var
0001:00314d8d  _zif_filter_input_array
0001:00314f3b  _zif_filter_input
0002:000013b0  _filter_module_entry
Module: U:\dev\php-5.3.8\ext\filter\sanitizing_filters.o(sanitizing_filters.o)
0001:00315d5c  _php_filter_string
0001:00315f07  _php_filter_encoded
0001:0031601b  _php_filter_special_chars
0001:003160ba  _php_filter_full_special_chars
0001:00316139  _php_filter_unsafe_raw
0001:00316265  _php_filter_email
0001:00316353  _php_filter_url
0001:003163e1  _php_filter_number_int
0001:00316441  _php_filter_number_float
0001:003164ee  _php_filter_magic_quotes
Module: U:\dev\php-5.3.8\ext\filter\logical_filters.o(logical_filters.o)
0001:0031666f  _php_filter_int
0001:00316b8c  _php_filter_boolean
0001:00316d99  _php_filter_float
0001:0031739e  _php_filter_validate_regexp
0001:003175f0  _php_filter_validate_url
0001:00317bf3  _php_filter_validate_email
0001:00317d55  _php_filter_validate_ip
Module: U:\dev\php-5.3.8\ext\filter\callback_filter.o(callback_filter.o)
0001:00318392  _php_filter_callback
Module: U:\dev\php-5.3.8\ext\ftp\php_ftp.o(php_ftp.o)
0001:00318573  _zif_ftp_get_option
0001:003186f0  _zif_ftp_set_option
0001:00318879  _zif_ftp_close
0001:0031892b  _zif_ftp_site
0001:00318a07  _zif_ftp_delete
0001:00318ae7  _zif_ftp_rename
0001:00318bd8  _zif_ftp_mdtm
0001:00318c80  _zif_ftp_size
0001:00318d5d  _zif_ftp_nb_put
0001:00318fc6  _zif_ftp_put
0001:0031924d  _zif_ftp_nb_fput
0001:003194ba  _zif_ftp_fput
0001:00319732  _zif_ftp_nb_continue
0001:003198a7  _zif_ftp_nb_fget
0001:00319b2c  _zif_ftp_nb_get
0001:00319ea2  _zif_ftp_get
0001:0031a20c  _zif_ftp_fget
0001:0031a449  _zif_ftp_pasv
0001:0031a4f8  _zif_ftp_systype
0001:0031a5e1  _zif_ftp_rawlist
0001:0031a6e1  _zif_ftp_nlist
0001:0031a7d3  _zif_ftp_alloc
0001:0031a8e8  _zif_ftp_chmod
0001:0031a9dc  _zif_ftp_rmdir
0001:0031aab8  _zif_ftp_mkdir
0001:0031aba5  _zif_ftp_raw
0001:0031ac4b  _zif_ftp_exec
0001:0031ad27  _zif_ftp_chdir
0001:0031ae03  _zif_ftp_cdup
0001:0031aeca  _zif_ftp_pwd
0001:0031afae  _zif_ftp_login
0001:0031b0a8  _zif_ftp_ssl_connect
0001:0031b195  _zif_ftp_connect
0001:0031b296  _zm_info_ftp
0001:0031b33c  _zm_startup_ftp
0001:0031b6b0  _php_ftp_functions
0002:00001410  _php_ftp_module_entry
Module: U:\dev\php-5.3.8\ext\ftp\ftp.o(ftp.o)
0001:0031d026  _ftp_open
0001:0031d1d0  _ftp_gc
0001:0031d21c  _ftp_close
0001:0031d283  _ftp_quit
0001:0031d36d  _ftp_login
0001:0031d613  _ftp_reinit
0001:0031d67b  _ftp_syst
0001:0031d720  _ftp_pwd
0001:0031d7c2  _ftp_exec
0001:0031d80b  _ftp_raw
0001:0031d8f9  _ftp_chdir
0001:0031d96e  _ftp_cdup
0001:0031d9e1  _ftp_mkdir
0001:0031da81  _ftp_rmdir
0001:0031dadb  _ftp_chmod
0001:0031db7e  _ftp_alloc
0001:0031dc2b  _ftp_pasv
0001:0031e5c1  _ftp_list
0001:0031e5f3  _ftp_nlist
0001:0031e61d  _ftp_get
0001:0031e861  _ftp_put
0001:0031ea80  _ftp_size
0001:0031eafa  _ftp_mdtm
0001:0031ec38  _ftp_delete
0001:0031ec8b  _ftp_rename
0001:0031ecfa  _ftp_site
0001:0031ed4c  _data_available
0001:0031edb2  _data_writeable
0001:0031ee18  _ftp_nb_continue_read
0001:0031effb  _ftp_nb_get
0001:0031f113  _ftp_nb_continue_write
0001:0031f25d  _ftp_nb_put
Module: U:\dev\php-5.3.8\ext\hash\hash.o(hash.o)
0002:00020650  _php_hash_hashtable
0001:0031f3a9  _zm_info_hash
0001:0031f486  _zm_shutdown_hash
0001:0031f51a  _zif_hash_algos
0001:0031f5c9  _zif_hash_update
0001:0031f681  _zif_hash_copy
0001:0031f7c7  _zif_hash_final
0001:0031fa23  _zif_hash_update_file
0001:0031fbf6  _zif_hash_update_stream
0001:0031fda6  _php_hash_fetch_ops
0001:0031fe49  _zif_hash_init
0001:003202ed  _zif_hash
0001:00320309  _zif_hash_file
0001:0032071a  _zif_hash_hmac
0001:00320736  _zif_hash_hmac_file
0001:00320752  _php_hash_register_algo
0001:0032095e  _zm_startup_hash
0001:00320d38  _php_hash_copy
0001:00320de0  _hash_functions
0002:00001470  _hash_module_entry
Module: U:\dev\php-5.3.8\ext\hash\hash_md.o(hash_md.o)
0001:0032182c  _PHP_MD4Init
0001:003218d0  _PHP_MD2Init
0001:00321917  _PHP_MD2Final
0001:00321978  _PHP_MD2Update
0001:00321a7c  _PHP_MD4Update
0001:00321b38  _PHP_MD4Final
0001:00321bc0  _php_hash_md5_ops
0001:00321be0  _php_hash_md4_ops
0001:00321c00  _php_hash_md2_ops
Module: U:\dev\php-5.3.8\ext\hash\hash_sha.o(hash_sha.o)
0001:00321d9b  _PHP_SHA256Init
0001:00321de8  _PHP_SHA224Init
0001:00321ec6  _PHP_SHA384Init
0001:00321f59  _PHP_SHA512Init
0001:003229e5  _PHP_SHA512Update
0001:00322acb  _PHP_SHA512Final
0001:00322bf5  _PHP_SHA384Update
0001:00322cdb  _PHP_SHA384Final
0001:00322e05  _PHP_SHA256Update
0001:00322ec1  _PHP_SHA256Final
0001:00322f6d  _PHP_SHA224Update
0001:00323029  _PHP_SHA224Final
0001:003230e0  _php_hash_sha1_ops
0001:00323100  _php_hash_sha256_ops
0001:00323120  _php_hash_sha224_ops
0001:00323140  _php_hash_sha384_ops
0001:00323160  _php_hash_sha512_ops
Module: U:\dev\php-5.3.8\ext\hash\hash_ripemd.o(hash_ripemd.o)
0001:00323700  _PHP_RIPEMD128Init
0001:00323731  _PHP_RIPEMD256Init
0001:0032377e  _PHP_RIPEMD160Init
0001:003237b6  _PHP_RIPEMD320Init
0001:00323b07  _PHP_RIPEMD128Update
0001:00323bc3  _PHP_RIPEMD128Final
0001:00323f58  _PHP_RIPEMD256Update
0001:00324014  _PHP_RIPEMD256Final
0001:003244b2  _PHP_RIPEMD160Update
0001:0032456e  _PHP_RIPEMD160Final
0001:00324a88  _PHP_RIPEMD320Update
0001:00324b44  _PHP_RIPEMD320Final
0001:00324bf0  _php_hash_ripemd128_ops
0001:00324c10  _php_hash_ripemd160_ops
0001:00324c30  _php_hash_ripemd256_ops
0001:00324c50  _php_hash_ripemd320_ops
Module: U:\dev\php-5.3.8\ext\hash\hash_haval.o(hash_haval.o)
0001:00324e2a  _PHP_3HAVAL128Init
0001:00324e91  _PHP_3HAVAL160Init
0001:00324ef8  _PHP_3HAVAL192Init
0001:00324f5f  _PHP_3HAVAL224Init
0001:00324fc6  _PHP_3HAVAL256Init
0001:0032502d  _PHP_4HAVAL128Init
0001:00325094  _PHP_4HAVAL160Init
0001:003250fb  _PHP_4HAVAL192Init
0001:00325162  _PHP_4HAVAL224Init
0001:003251c9  _PHP_4HAVAL256Init
0001:00325230  _PHP_5HAVAL128Init
0001:00325297  _PHP_5HAVAL160Init
0001:003252fe  _PHP_5HAVAL192Init
0001:00325365  _PHP_5HAVAL224Init
0001:003253cc  _PHP_5HAVAL256Init
0001:00325433  _PHP_HAVALUpdate
0001:003254ff  _PHP_HAVAL256Final
0001:0032559f  _PHP_HAVAL224Final
0001:00325686  _PHP_HAVAL192Final
0001:003257ae  _PHP_HAVAL160Final
0001:003258ed  _PHP_HAVAL128Final
0001:003266d0  _php_hash_3haval128_ops
0001:003266f0  _php_hash_3haval160_ops
0001:00326710  _php_hash_3haval192_ops
0001:00326730  _php_hash_3haval224_ops
0001:00326750  _php_hash_3haval256_ops
0001:00326770  _php_hash_4haval128_ops
0001:00326790  _php_hash_4haval160_ops
0001:003267b0  _php_hash_4haval192_ops
0001:003267d0  _php_hash_4haval224_ops
0001:003267f0  _php_hash_4haval256_ops
0001:00326810  _php_hash_5haval128_ops
0001:00326830  _php_hash_5haval160_ops
0001:00326850  _php_hash_5haval192_ops
0001:00326870  _php_hash_5haval224_ops
0001:00326890  _php_hash_5haval256_ops
Module: U:\dev\php-5.3.8\ext\hash\hash_tiger.o(hash_tiger.o)
0001:00326e30  _PHP_4TIGERInit
0001:00326e72  _PHP_3TIGERInit
0001:0032c2ec  _PHP_TIGER192Final
0001:0032c409  _PHP_TIGER160Final
0001:0032c4f0  _PHP_TIGER128Final
0001:0032c5ba  _PHP_TIGERUpdate
0001:00332500  _php_hash_3tiger128_ops
0001:00332520  _php_hash_3tiger160_ops
0001:00332540  _php_hash_3tiger192_ops
0001:00332560  _php_hash_4tiger128_ops
0001:00332580  _php_hash_4tiger160_ops
0001:003325a0  _php_hash_4tiger192_ops
Module: U:\dev\php-5.3.8\ext\hash\hash_gost.o(hash_gost.o)
0001:0033563b  _PHP_GOSTInit
0001:00335650  _PHP_GOSTUpdate
0001:0033586b  _PHP_GOSTFinal
0001:00335980  _php_hash_gost_ops
Module: U:\dev\php-5.3.8\ext\hash\hash_snefru.o(hash_snefru.o)
0001:003369a0  _PHP_SNEFRUInit
0001:003369b5  _PHP_SNEFRUUpdate
0001:0033740c  _PHP_SNEFRUFinal
0001:00337c80  _php_hash_snefru_ops
Module: U:\dev\php-5.3.8\ext\hash\hash_whirlpool.o(hash_whirlpool.o)
0001:0033d5d9  _PHP_WHIRLPOOLUpdate
0001:0033d82e  _PHP_WHIRLPOOLInit
0001:0033d843  _PHP_WHIRLPOOLFinal
0001:0033d990  _php_hash_whirlpool_ops
Module: U:\dev\php-5.3.8\ext\hash\hash_adler32.o(hash_adler32.o)
0001:00341a10  _PHP_ADLER32Init
0001:00341a1e  _PHP_ADLER32Update
0001:00341a9b  _PHP_ADLER32Final
0001:00341ac6  _PHP_ADLER32Copy
0001:00341ae0  _php_hash_adler32_ops
Module: U:\dev\php-5.3.8\ext\hash\hash_crc32.o(hash_crc32.o)
0001:00341b00  _PHP_CRC32Init
0001:00341b0e  _PHP_CRC32Update
0001:00341b4b  _PHP_CRC32BUpdate
0001:00341b84  _PHP_CRC32Final
0001:00341bb4  _PHP_CRC32BFinal
0001:00341be4  _PHP_CRC32Copy
0001:00341c00  _php_hash_crc32_ops
0001:00341c20  _php_hash_crc32b_ops
Module: U:\dev\php-5.3.8\ext\hash\hash_salsa.o(hash_salsa.o)
0001:003429b2  _PHP_SALSA20Init
0001:003429d1  _PHP_SALSA10Init
0001:003429f0  _PHP_SALSAUpdate
0001:00342c18  _PHP_SALSAFinal
0001:00342ce0  _php_hash_salsa10_ops
0001:00342d00  _php_hash_salsa20_ops
Module: U:\dev\php-5.3.8\ext\json\json.o(json.o)
0002:00020680  _json_globals_id
0001:00344a29  _php_json_encode
0001:00345bc8  _php_json_decode
0002:000014d0  _json_module_entry
Module: U:\dev\php-5.3.8\ext\json\utf8_to_utf16.o(utf8_to_utf16.o)
0001:00346350  _utf8_to_utf16
Module: U:\dev\php-5.3.8\ext\json\utf8_decode.o(utf8_decode.o)
0001:003463e0  _utf8_decode_init
0001:00346408  _utf8_decode_at_byte
0001:00346413  _utf8_decode_at_character
0001:00346427  _utf8_decode_next
Module: U:\dev\php-5.3.8\ext\json\JSON_parser.o(JSON_parser.o)
0001:00346e83  _new_JSON_parser
0001:00346f22  _free_JSON_parser
0001:00346f59  _parse_JSON
Module: U:\dev\php-5.3.8\ext\pdo\pdo.o(pdo.o)
0002:00020690  _pdo_driver_hash
0002:000206c0  _pdo_dbh_ce
0002:000206d0  _pdo_exception_ce
0002:000206e0  _pdo_globals_id
0002:000206f0  _pdo_dbstmt_ce
0002:00020700  _pdo_row_ce
0001:00348df6  _zm_info_pdo
0001:00348f02  _zm_shutdown_pdo
0001:00348f1d  _zif_pdo_drivers
0001:00348fc2  _php_pdo_list_entry
0001:00348fcc  _php_pdo_get_dbh_ce
0001:00348fd6  _php_pdo_get_exception
0001:00348fe0  _php_pdo_str_tolower_dup
0001:00349025  _php_pdo_get_exception_base
0001:003490c3  _zm_startup_pdo
0001:00349309  _php_pdo_register_driver
0001:003493c2  _php_pdo_unregister_driver
0001:0034941b  _pdo_find_driver
0001:00349456  _php_pdo_parse_data_source
0001:0034965d  _php_pdo_int64_to_str
0001:00349830  _pdo_functions
0002:00001530  _pdo_module_entry
Module: U:\dev\php-5.3.8\ext\pdo\pdo_dbh.o(pdo_dbh.o)
0001:003499fc  _pdo_dbh_new
0001:00349ec0  _pdo_raise_impl_error
0001:0034a494  _pdo_handle_error
0001:0034d3ec  _pdo_hash_methods
0001:0034dbf7  _pdo_dbh_init
0001:0034e970  _pdo_dbh_functions
0001:0034e87c  _php_pdo_dbh_addref
0001:0034e888  _php_pdo_dbh_delref
0001:0034e89a  _php_pdo_pdbh_dtor
Module: U:\dev\php-5.3.8\ext\pdo\pdo_stmt.o(pdo_stmt.o)
0002:00020710  _pdo_dbstmt_object_handlers
0001:0034ff93  _pdo_row_new
0001:00351116  _pdo_row_free_storage
0001:00350c26  _pdo_dbstmt_new
0001:00354df1  _pdo_dbstmt_free_storage
0001:00351be5  _pdo_stmt_describe_columns
0001:00353839  _pdo_stmt_iter_get
0001:00354657  _pdo_stmt_setup_fetch_mode
0001:00354afc  _pdo_stmt_init
0001:00354ee0  _pdo_dbstmt_functions
0001:003550a0  _pdo_row_functions
0001:00354dc4  _php_pdo_stmt_addref
0001:00354dd0  _php_pdo_stmt_delref
0002:00001590  _pdo_row_object_handlers
Module: U:\dev\php-5.3.8\ext\pdo\pdo_sql_parser.o(pdo_sql_parser.o)
0001:00355663  _pdo_parse_params
Module: U:\dev\php-5.3.8\ext\pdo\pdo_sqlstate.o(pdo_sqlstate.o)
0001:003565d0  _pdo_sqlstate_fini_error_table
0001:003565e4  _pdo_sqlstate_init_error_table
0001:00356685  _pdo_sqlstate_state_to_description
Module: U:\dev\php-5.3.8\ext\phar\util.o(util.o)
0001:00359444  _phar_get_link_source
0001:0035957b  _phar_mount_entry
0001:0035983e  _phar_open_archive_fp
0001:0035997b  _phar_get_efp
0001:00359b74  _phar_seek_efp
0001:00359ed5  _phar_open_entry_fp
0001:0035a6da  _phar_copy_entry_fp
0001:0035a8a4  _phar_create_writeable_entry
0001:0035a9eb  _phar_separate_entry_fp
0001:0035ab9b  _phar_open_jit
0001:0035ac57  _phar_free_alias
0001:0035ad37  _phar_get_archive
0001:0035ba0a  _phar_find_in_include_path
0001:0035bebf  _phar_compress_filter
0001:0035bef8  _phar_decompress_filter
0001:0035c18d  _phar_get_entry_info_dir
0001:0035c72e  _phar_get_entry_info
0001:0035c818  _phar_verify_signature
0001:0035cf1b  _phar_create_signature
0001:0035d2fd  _phar_add_virtual_dirs
0001:0035d356  _phar_copy_on_write
0001:0035d925  _phar_get_entry_data
0001:0035e0e6  _phar_get_or_create_entry_data
Module: U:\dev\php-5.3.8\ext\phar\tar.o(tar.o)
0001:0035ee61  _phar_is_tar
0001:0035efaa  _phar_open_or_create_tar
0001:0035f4d7  _phar_parse_tarfile
0001:00360c55  _phar_tar_setmetadata
0001:0036146b  _phar_tar_flush
Module: U:\dev\php-5.3.8\ext\phar\zip.o(zip.o)
0001:003646b3  _phar_parse_zipfile
0001:00367e97  _phar_open_or_create_zip
0001:0036839c  _phar_zip_flush
Module: U:\dev\php-5.3.8\ext\phar\stream.o(stream.o)
0001:0036a180  _phar_parse_url
0001:0036c4b5  _phar_dostat
0002:00001620  _phar_ops
0002:00001650  _phar_stream_wops
0002:00001680  _php_stream_phar_wrapper
Module: U:\dev\php-5.3.8\ext\phar\func_interceptors.o(func_interceptors.o)
0001:0036fa9a  _phar_stat
0001:0036fb64  _phar_lstat
0001:0036fc2e  _phar_is_dir
0001:0036fcf8  _phar_file_exists
0001:0036fdc2  _phar_is_executable
0001:0036fe8c  _phar_is_readable
0001:0036ff56  _phar_is_writable
0001:00370020  _phar_filetype
0001:003700ea  _phar_filectime
0001:003701b4  _phar_filemtime
0001:0037027e  _phar_fileatime
0001:00370348  _phar_filegroup
0001:00370412  _phar_fileowner
0001:003704dc  _phar_filesize
0001:003705a6  _phar_fileinode
0001:00370670  _phar_fileperms
0001:00370737  _phar_intercept_functions
0001:00370770  _phar_release_functions
0001:00370860  _phar_intercept_functions_init
0001:003711cb  _phar_intercept_functions_shutdown
0001:00371bf0  _phar_save_orig_functions
0001:00371d0b  _phar_restore_orig_functions
Module: U:\dev\php-5.3.8\ext\phar\dirstream.o(dirstream.o)
0001:00372555  _phar_wrapper_open_dir
0001:00372bb9  _phar_wrapper_mkdir
0001:003733d8  _phar_wrapper_rmdir
0002:000016a0  _phar_dir_ops
Module: U:\dev\php-5.3.8\ext\phar\phar.o(phar.o)
0002:00020780  _phar_globals_id
0002:00020790  _cached_phars
0002:000207c0  _cached_alias
0002:000207f0  _phar_orig_compile_file
0002:00020800  _phar_save_resolve_path
0001:00373b0e  _zm_globals_dtor_phar
0001:00373b6d  _zm_deactivate_phar
0001:00373d3a  _zm_shutdown_phar
0001:00373e09  _zm_startup_phar
0001:00374055  _zm_globals_ctor_phar
0001:00374fc7  _destroy_phar_manifest_entry
0001:00375121  _phar_ini_modify_handler
0001:003752cb  _phar_destroy_phar_data
0001:00375588  _phar_archive_delref
0001:003756f3  _phar_entry_delref
0001:00375806  _phar_open_parsed_phar
0001:00375983  _phar_parse_metadata
0001:00375afa  _phar_fix_filepath
0001:00375faf  _phar_postprocess_file
0001:00376597  _phar_create_default_stub
0001:00376c45  _phar_flush
0001:00378cb1  _phar_entry_remove
0001:00378d96  _phar_request_initialize
0001:003791f9  _zm_info_phar
0001:0037d51d  _phar_open_executed_filename
0001:0037d7ee  _phar_open_from_filename
0001:0037dd46  _phar_ini_cache_list
0001:0037e264  _phar_detect_phar_fname_ext
0001:0037e866  _phar_split_fname
0001:0037ea7e  _phar_create_or_parse_filename
0001:0037f16d  _phar_open_or_create_filename
0002:000016d0  _phar_module_entry
0002:00009c70  _phar_functions
Module: U:\dev\php-5.3.8\ext\phar\phar_object.o(phar_object.o)
0001:00381677  _zim_Phar_hasMetadata
0001:0038171c  _zim_PharFileInfo_hasMetadata
0001:003817a6  _zim_PharFileInfo_getPharFlags
0001:0038182d  _zim_PharFileInfo_isCRCChecked
0001:00381903  _zim_PharFileInfo_getCRC32
0001:003819cf  _zim_PharFileInfo_isCompressed
0001:00381ac3  _zim_PharFileInfo_getCompressedSize
0001:00381b45  _zim_Phar_getModified
0001:00381bd1  _zim_Phar_isBuffering
0001:00381c5d  _zim_Phar_startBuffering
0001:00381cd4  _zim_Phar_isCompressed
0001:00381daf  _zim_Phar_isFileFormat
0001:00381ed1  _zim_Phar_canWrite
0001:003820b7  _zim_PharFileInfo_decompress
0001:0038242e  _zim_PharFileInfo_chmod
0001:003826be  _zim_PharFileInfo___destruct
0001:00382749  _zim_Phar_stopBuffering
0001:00382b95  _zim_PharFileInfo_compress
0001:00383052  _zim_PharFileInfo_getContent
0001:00383274  _zim_Phar_getPath
0001:00383307  _zim_Phar_getAlias
0001:003833a9  _zim_Phar_apiVersion
0001:0038349d  _zim_PharFileInfo_delMetadata
0001:0038369b  _zim_Phar_delMetadata
0001:003838d7  _zim_PharFileInfo___construct
0001:00383c06  _zim_Phar_isWritable
0001:00383cfb  _zim_Phar_count
0001:00384939  _zim_Phar_extractTo
0001:00384f03  _zim_Phar_getStub
0001:00385688  _zim_Phar_addFromString
0001:003857de  _zim_Phar_addEmptyDir
0001:00385b08  _zim_Phar_addFile
0001:00385d17  _zim_Phar_offsetUnset
0001:00385f26  _zim_Phar_offsetExists
0001:0038607e  _zim_Phar_delete
0001:0038638f  _zim_Phar_offsetSet
0001:0038660a  _zim_Phar_setSignatureAlgorithm
0001:003868c9  _zim_Phar_setStub
0001:00386ca5  _zim_Phar_offsetGet
0001:00386fce  _zim_Phar_getVersion
0001:0038721c  _zim_Phar_copy
0001:00387899  _zim_Phar_decompressFiles
0001:00387c53  _zim_Phar_compressFiles
0001:00387eb4  _zim_Phar_isValidPharFilename
0001:00387f86  _zim_Phar_getSignature
0001:0038828c  _zim_Phar_setDefaultStub
0001:003885ad  _zim_Phar_createDefaultStub
0001:00388684  _zim_Phar___destruct
0001:003887cb  _zim_Phar_setAlias
0001:00388e21  _zim_Phar_buildFromIterator
0001:00389118  _zim_Phar_buildFromDirectory
0001:0038a3e0  _zim_Phar_running
0001:0038a695  _zim_Phar_unlinkArchive
0001:0038a98b  _zim_Phar_canCompress
0001:0038aa5b  _zim_Phar_loadPhar
0001:0038ab4b  _zim_Phar_getSupportedCompression
0001:0038ac17  _zim_Phar_getSupportedSignatures
0001:0038adea  _zim_Phar___construct
0001:0038b2f4  _zim_Phar_mapPhar
0001:0038b3b9  _zim_Phar_interceptFileFuncs
0001:0038b604  _zim_Phar_mungServer
0001:0038c7bf  _zim_Phar_mount
0001:0038cfe6  _zim_Phar_webPhar
0001:0038f516  _zim_Phar_setMetadata
0001:0038f7ca  _zim_PharFileInfo_setMetadata
0001:0038fa37  _zim_PharFileInfo_getMetadata
0001:0038fb73  _zim_Phar_getMetadata
0001:0038fd38  _zim_Phar_decompress
0001:0038ffdf  _zim_Phar_compress
0001:0039033b  _zim_Phar_convertToExecutable
0001:003906a1  _zim_Phar_convertToData
0001:003909dc  _phar_object_init
0002:00001730  _php_archive_methods
0002:00001bb0  _php_entry_methods
0002:00009c90  _phar_exception_methods
Module: U:\dev\php-5.3.8\ext\phar\phar_path_check.o(phar_path_check.o)
0001:00391e95  _phar_path_check
Module: U:\dev\php-5.3.8\ext\posix\posix.o(posix.o)
0002:00020810  _posix_globals_id
0001:003922ef  _zif_posix_get_last_error
0001:00392337  _zif_posix_initgroups
0001:003923b4  _zif_posix_strerror
0001:00392433  _zif_posix_access
0001:00392642  _zif_posix_mknod
0001:003927dc  _zif_posix_mkfifo
0001:003928cd  _zif_posix_getcwd
0001:00392b34  _zif_posix_isatty
0001:00392c46  _zif_posix_ttyname
0001:00392db1  _zif_posix_times
0001:00392ef6  _zif_posix_uname
0001:00393037  _zif_posix_getsid
0001:003930ad  _zif_posix_getpgid
0001:00393126  _zif_posix_setpgid
0001:003931ab  _zif_posix_setsid
0001:003931e5  _zif_posix_getpgrp
0001:0039321f  _zif_posix_getlogin
0001:003932a3  _zif_posix_getgroups
0001:00393354  _zif_posix_setegid
0001:003933cb  _zif_posix_seteuid
0001:00393442  _zif_posix_setgid
0001:003934b9  _zif_posix_setuid
0001:00393530  _zif_posix_getegid
0001:0039356a  _zif_posix_geteuid
0001:003935a4  _zif_posix_getgid
0001:003935de  _zif_posix_getuid
0001:00393618  _zif_posix_getppid
0001:00393652  _zif_posix_getpid
0001:0039368c  _zif_posix_kill
0001:0039372b  _zif_posix_getrlimit
0001:00393976  _php_posix_group_to_array
0001:00393ae2  _zif_posix_getgrgid
0001:00393c33  _zif_posix_getgrnam
0001:00393d7b  _php_posix_passwd_to_array
0001:00393edb  _zif_posix_getpwuid
0001:00394002  _zif_posix_getpwnam
0001:00394320  _posix_functions
0002:00001d60  _limits
0002:00001d00  _posix_module_entry
Module: U:\dev\php-5.3.8\ext\reflection\php_reflection.o(php_reflection.o)
0002:00020820  _reflection_exception_ptr
0002:00020830  _reflection_function_ptr
0002:00020840  _reflection_method_ptr
0002:00020850  _reflection_property_ptr
0002:00020860  _reflection_extension_ptr
0002:00020870  _reflection_class_ptr
0002:00020880  _reflection_function_abstract_ptr
0002:00020890  _reflection_ptr
0002:000208a0  _reflector_ptr
0002:000208b0  _reflection_parameter_ptr
0002:000208c0  _reflection_object_ptr
0001:00394d45  _zm_info_reflection
0001:00394f4b  _zim_reflection_property_setAccessible
0001:00394fe1  _zim_reflection_property_getModifiers
0001:00395088  _zim_reflection_class_getModifiers
0001:0039512f  _zim_reflection_class_isInstantiable
0001:0039521f  _zim_reflection_class_getEndLine
0001:003952e5  _zim_reflection_class_getStartLine
0001:003953ab  _zim_reflection_class_isUserDefined
0001:00395458  _zim_reflection_class_isInternal
0001:00395505  _zim_reflection_method_getModifiers
0001:003955ac  _zim_reflection_method_isDestructor
0001:0039565a  _zim_reflection_method_isConstructor
0001:0039572b  _zim_reflection_parameter_isDefaultValueAvailable
0001:00395846  _zim_reflection_parameter_isOptional
0001:003958f5  _zim_reflection_parameter_getPosition
0001:0039599b  _zim_reflection_parameter_isPassedByReference
0001:00395a4c  _zim_reflection_parameter_allowsNull
0001:00395afd  _zim_reflection_parameter_isArray
0001:00395bae  _zim_reflection_function_getEndLine
0001:00395c71  _zim_reflection_function_getStartLine
0001:00395d34  _zim_reflection_function_isUserDefined
0001:00395de1  _zim_reflection_function_isInternal
0001:00395e8e  _zim_reflection_function_isClosure
0001:00395f3c  _zim_reflection_extension_info
0001:00395ff9  _zim_reflection_extension_getDependencies
0001:0039618d  _zim_reflection_extension_getClassNames
0001:00396282  _zim_reflection_extension_getClasses
0001:00396377  _zim_reflection_extension_getINIEntries
0001:00396469  _zim_reflection_extension_getConstants
0001:00396589  _zim_reflection_class_getInterfaceNames
0001:003966b1  _zim_reflection_getModifierNames
0001:003968f6  _zim_reflection_class_inNamespace
0001:003969a6  _zim_reflection_function_inNamespace
0001:00396a56  _zim_reflection_extension_getVersion
0001:00396b37  _zim_reflection_property_getDocComment
0001:00396c11  _zim_reflection_class_getNamespaceName
0001:00396cf9  _zim_reflection_class_getDocComment
0001:00396ddf  _zim_reflection_class_getFileName
0001:00396ebc  _zim_reflection_function_getNamespaceName
0001:00396fa6  _zim_reflection_function_getDocComment
0001:00397083  _zim_reflection_function_getFileName
0001:003972f7  _zim_reflection_extension_getFunctions
0001:00397640  _zim_reflection_class_getConstructor
0001:003979f7  _zim_reflection_class_getConstants
0001:00397afd  _zim_reflection_function_getStaticVariables
0001:00397e5e  _zim_reflection_extension___construct
0001:003981e4  _zim_reflection___clone
0001:0039822d  _zim_reflection_class_getExtensionName
0001:00398375  _zim_reflection_class_getExtension
0001:00398493  _zim_reflection_class_isIterateable
0001:00398653  _zim_reflection_class_newInstance
0001:00398934  _zim_reflection_class_isInstance
0001:00398a7a  _zim_reflection_class_hasConstant
0001:00398bcc  _zim_reflection_class_getProperties
0001:00398d99  _zim_reflection_class_hasProperty
0001:00398fac  _zim_reflection_class_getMethod
0001:003992ba  _zim_reflection_class_hasMethod
0001:00399494  _zim_reflection_method_getPrototype
0001:003995ec  _zim_reflection_function_getExtensionName
0001:00399710  _zim_reflection_function_getExtension
0001:00399814  _zim_reflection_function_getNumberOfRequiredParameters
0001:003998fe  _zim_reflection_function_getNumberOfParameters
0001:003999e8  _zim_reflection_function_returnsReference
0001:00399ad9  _zim_reflection_function_isDisabled
0001:00399c58  _zim_reflection_property___construct
0001:0039a20a  _zim_reflection_class_implementsInterface
0001:0039a44f  _zim_reflection_class_isSubclassOf
0001:0039a68d  _zim_reflection_class_newInstanceArgs
0001:0039ac48  _zim_reflection_class_getProperty
0001:0039aff2  _zim_reflection_function___construct
0001:0039b367  _zm_startup_reflection
0001:0039c3c5  _zim_reflection_class_getMethods
0001:0039c68a  _zim_reflection_property_isDefault
0001:0039c6b7  _zim_reflection_property_isStatic
0001:0039c6e4  _zim_reflection_property_isProtected
0001:0039c711  _zim_reflection_property_isPrivate
0001:0039c73e  _zim_reflection_property_isPublic
0001:0039c824  _zim_reflection_class_isAbstract
0001:0039c851  _zim_reflection_class_isFinal
0001:0039c87e  _zim_reflection_class_isInterface
0001:0039c964  _zim_reflection_function_isDeprecated
0001:0039c991  _zim_reflection_method_isStatic
0001:0039c9be  _zim_reflection_method_isProtected
0001:0039c9eb  _zim_reflection_method_isPrivate
0001:0039ca18  _zim_reflection_method_isPublic
0001:0039ca45  _zim_reflection_method_isAbstract
0001:0039ca72  _zim_reflection_method_isFinal
0001:0039cc6e  _zim_reflection_property___toString
0001:0039cda7  _zim_reflection_parameter_getDeclaringFunction
0001:0039cea5  _zim_reflection_function_getParameters
0001:0039d219  _zim_reflection_class_getDefaultProperties
0001:0039d495  _zim_reflection_class_getStaticProperties
0001:0039d777  _zim_reflection_class_setStaticPropertyValue
0001:0039d974  _zim_reflection_function_getName
0001:0039d9bc  _zim_reflection_parameter_getName
0001:0039da04  _zim_reflection_class_getName
0001:0039da4c  _zim_reflection_property_getName
0001:0039da94  _zim_reflection_extension_getName
0001:0039dadc  _zim_reflection_class_getShortName
0001:0039dbe4  _zim_reflection_function_getShortName
0001:0039dd53  _zim_reflection_export
0001:0039dfd2  _zim_reflection_class_getStaticPropertyValue
0001:0039e155  _zim_reflection_class_getConstant
0001:0039e5f5  _zim_reflection_object___construct
0001:0039e611  _zim_reflection_class___construct
0001:0039e653  _zim_reflection_function_invoke
0001:0039e8d9  _zim_reflection_function_invokeArgs
0001:0039ef58  _zim_reflection_extension_export
0001:0039ef7d  _zim_reflection_property_export
0001:0039efa2  _zim_reflection_object_export
0001:0039efc7  _zim_reflection_class_export
0001:0039efec  _zim_reflection_method_export
0001:0039f011  _zim_reflection_parameter_export
0001:0039f036  _zim_reflection_function_export
0001:0039f171  _zim_reflection_method_invokeArgs
0001:0039f5d3  _zim_reflection_parameter_getDefaultValue
0001:0039f7b8  _zim_reflection_method_invoke
0001:0039fbcb  _zim_reflection_property_getValue
0001:0039ff32  _zim_reflection_property_setValue
0001:003a0473  _zim_reflection_parameter___construct
0001:003a1710  _zim_reflection_method___toString
0001:003a17f5  _zim_reflection_function___toString
0001:003a2647  _zim_reflection_class___toString
0001:003a2826  _zim_reflection_extension___toString
0001:003a2e5b  _zim_reflection_parameter___toString
0001:003a2f57  _zim_reflection_method___construct
0001:003a33d8  _zend_reflection_class_factory
0001:003a3565  _zim_reflection_property_getDeclaringClass
0001:003a36e2  _zim_reflection_class_getParentClass
0001:003a37ad  _zim_reflection_class_getInterfaces
0001:003a38f0  _zim_reflection_method_getDeclaringClass
0001:003a3afc  _zim_reflection_parameter_getClass
0001:003a3cd0  _zim_reflection_parameter_getDeclaringClass
0001:003a3d97  _zim_reflection_method_setAccessible
0001:003a3df0  _reflection_ext_functions
0002:00001dc0  _reflection_module_entry
Module: U:\dev\php-5.3.8\ext\session\session.o(session.o)
0002:000208d0  _ps_globals_id
0001:003a9399  _php_add_session_var
0001:003a9904  _php_set_session_var
0001:003a9b9f  _ps_srlzr_decode_php
0001:003a9d6e  _ps_srlzr_decode_php_binary
0001:003a9f2e  _php_get_session_var
0001:003aa003  _ps_srlzr_encode_php
0001:003aa502  _ps_srlzr_encode_php_binary
0001:003aa9ed  _php_session_create_id
0001:003ab00e  _php_session_register_serializer
0001:003ab06c  _php_session_register_module
0001:003ab099  __php_find_ps_module
0001:003ab357  __php_find_ps_serializer
0001:003ab691  _php_session_start
0001:003ac8a9  _session_adapt_url
0002:00001e20  _session_module_entry
Module: U:\dev\php-5.3.8\ext\session\mod_files.o(mod_files.o)
0001:003adb93  _ps_gc_files
0001:003adc25  _ps_open_files
0001:003ade45  _ps_close_files
0001:003ae332  _ps_write_files
0001:003ae464  _ps_read_files
0001:003ae5b5  _ps_delete_files
0002:00001f70  _ps_mod_files
Module: U:\dev\php-5.3.8\ext\session\mod_user.o(mod_user.o)
0001:003ae6f3  _ps_gc_user
0001:003ae77d  _ps_close_user
0001:003ae7d7  _ps_delete_user
0001:003ae890  _ps_write_user
0001:003ae98a  _ps_read_user
0001:003aea63  _ps_open_user
0002:00001f90  _ps_mod_user
Module: U:\dev\php-5.3.8\ext\simplexml\simplexml.o(simplexml.o)
0001:003aeb94  _zm_shutdown_simplexml
0001:003aecf4  _sxe_object_new
0001:003aee3d  _php_sxe_get_iterator
0001:003aefe7  _zm_info_simplexml
0001:003af05d  _zm_startup_simplexml
0001:003b0165  _simplexml_export_node
0001:003af25b  _zif_simplexml_import_dom
0001:003af3a5  _zif_simplexml_load_file
0001:003af4e3  _zif_simplexml_load_string
0001:003af65a  _zim_simplexml_element___construct
0001:003af803  _zim_simplexml_element_registerXPathNamespace
0001:003afbc0  _zim_simplexml_element_getDocNamespaces
0001:003b01cb  _zim_simplexml_element_getName
0001:003b0286  _zim_simplexml_element_attributes
0001:003b0367  _zim_simplexml_element_children
0001:003b04cb  _zim_simplexml_element_addChild
0001:003b07d1  _zim_simplexml_element_addAttribute
0001:003b0a5b  _zim_simplexml_element_getNamespaces
0001:003b0ba8  _zim_simplexml_element_asXML
0001:003b0e35  _zim_simplexml_element_xpath
0001:003b12ac  _zim_simplexml_element_count
0001:003b2e4a  _zim_simplexml_element___toString
0001:003b4003  _sxe_get_element_class_entry
0001:003b400d  _php_sxe_move_forward_iterator
0001:003b4100  _simplexml_functions
0002:00001fb0  _php_sxe_iterator_funcs
0002:00001fd0  _simplexml_module_entry
0002:00009d80  _sxe_class_entry
Module: U:\dev\php-5.3.8\ext\simplexml\sxe.o(sxe.o)
0002:000208e0  _ce_SimpleXMLElement
0001:003b47c1  _zim_ce_SimpleXMLIterator_next
0001:003b4817  _zim_ce_SimpleXMLIterator_valid
0001:003b486a  _zim_ce_SimpleXMLIterator_rewind
0001:003b48c0  _zim_ce_SimpleXMLIterator_getChildren
0001:003b4949  _zim_ce_SimpleXMLIterator_current
0001:003b49e2  _zim_ce_SimpleXMLIterator_hasChildren
0001:003b4ab2  _zim_ce_SimpleXMLIterator_key
0001:003b4b6b  _zm_startup_sxe
0002:00009d90  _ce_SimpleXMLIterator
Module: U:\dev\php-5.3.8\ext\soap\soap.o(soap.o)
0002:000208f0  _soap_globals_id
0002:00020900  _soap_var_class_entry
0001:003b4ebc  _zm_activate_soap
0001:003b5405  _zif_use_soap_error_handler
0001:003b548b  _zim_SoapClient___getLastResponseHeaders
0001:003b5533  _zim_SoapClient___getLastRequestHeaders
0001:003b55d4  _zim_SoapClient___getLastResponse
0001:003b5674  _zim_SoapClient___getLastRequest
0001:003b5711  _zim_SoapClient___setLocation
0001:003b5837  _zif_is_soap_fault
0001:003b58e5  _zim_SoapParam_SoapParam
0001:003b5a82  _zim_SoapClient___setSoapHeaders
0001:003b5c80  _zim_SoapClient___setCookie
0001:003b5e8c  _zim_SoapClient___doRequest
0001:003b6078  _zim_SoapServer_setPersistence
0001:003b6210  _zim_SoapClient___getFunctions
0001:003b71e0  _zim_SoapFault_SoapFault
0001:003b770f  _zim_SoapHeader_SoapHeader
0001:003b80c2  _zim_SoapServer_SoapServer
0001:003b876f  _zim_SoapServer_addFunction
0001:003b8ca5  _zim_SoapServer_getFunctions
0001:003b8f47  _zim_SoapServer_setClass
0001:003b91c2  _zim_SoapVar_SoapVar
0001:003b948b  _zim_SoapFault___toString
0001:003b967c  _zm_info_soap
0001:003b9d8d  _zm_startup_soap
0001:003bb5b3  _zm_shutdown_soap
0001:003bb658  _OnUpdateCacheMode
0001:003bb6c3  _OnUpdateCacheEnabled
0001:003bdfcf  _zim_SoapClient___getTypes
0001:003bf657  _zim_SoapServer_addSoapHeader
0001:003bf83a  _zim_SoapServer_setObject
0001:003c13f9  _zim_SoapServer_fault
0001:003c1bac  _zim_SoapClient_SoapClient
0001:003c30f9  _zim_SoapServer_handle
0001:003c768d  _zim_SoapClient___call
0001:003c5dc5  _add_soap_fault
0002:000020a0  _soap_module_entry
0002:00009da0  _le_url
Module: U:\dev\php-5.3.8\ext\soap\php_encoding.o(php_encoding.o)
0001:003ca82a  _whiteSpace_replace
0001:003caa41  _whiteSpace_collapse
0001:003cb8be  _to_zval_user
0001:003cbaa1  _encode_add_ns
0001:003cd7a8  _to_xml_user
0001:003cd920  _encode_reset_ns
0001:003cd9c2  _encode_finish
0001:003cda6f  _get_conversion
0001:003ceef2  _master_to_xml
0001:003d29a1  _sdl_guess_convert_xml
0001:003d2ea0  _master_to_zval
0001:003d4f97  _sdl_guess_convert_zval
0001:003d5058  _delete_encoder
0001:003d50c0  _delete_encoder_persistent
0002:00002100  _defaultEncoding
0002:00002950  _numDefaultEncodings
Module: U:\dev\php-5.3.8\ext\soap\php_http.o(php_http.o)
0001:003d5aa9  _proxy_authentication
0001:003d5f42  _basic_authentication
0001:003d69d8  _make_http_soap_request
Module: U:\dev\php-5.3.8\ext\soap\php_packet_soap.o(php_packet_soap.o)
0001:003de463  _parse_packet_soap
Module: U:\dev\php-5.3.8\ext\soap\php_schema.o(php_schema.o)
0001:003df460  _delete_restriction_var_char
0001:003df491  _delete_extra_attribute
0001:003df4c7  _delete_attribute
0001:003df544  _delete_model
0001:003e0512  _schema_min_max
0001:003e062f  _schema_pass2
0001:003e0845  _delete_model_persistent
0001:003e089d  _delete_extra_attribute_persistent
0001:003e08d3  _delete_attribute_persistent
0001:003e0950  _delete_restriction_var_int
0001:003e096a  _delete_type
0001:003e6e26  _load_schema
0001:003e7887  _delete_restriction_var_int_persistent
0001:003e78a1  _delete_restriction_var_char_persistent
0001:003e78d2  _delete_type_persistent
Module: U:\dev\php-5.3.8\ext\soap\php_sdl.o(php_sdl.o)
0001:003ef463  _get_encoder_ex
0001:003f033c  _get_encoder
0001:003f0691  _get_encoder_from_prefix
0001:003f1a91  _get_binding_from_type
0001:003f1b08  _get_binding_from_name
0001:003f1d70  _sdl_set_uri_credentials
0001:003f1fb3  _sdl_restore_uri_credentials
0001:003f4726  _delete_sdl_impl
0001:003f4880  _get_sdl
0001:003f8a2a  _delete_sdl
Module: U:\dev\php-5.3.8\ext\soap\php_xml.o(php_xml.o)
0001:003f8b04  _soap_xmlParseFile
0001:003f8bed  _soap_xmlParseMemory
0001:003f8c8c  _attr_find_ns
0001:003f8cc1  _node_find_ns
0001:003f8cec  _attr_is_equal_ex
0001:003f8d4f  _node_is_equal_ex
0001:003f8db2  _get_attribute_ex
0001:003f8def  _get_node_ex
0001:003f8e2c  _get_node_recurisve_ex
0001:003f8e90  _get_node_with_attribute_ex
0001:003f8f11  _get_node_with_attribute_recursive_ex
0001:003f8fc7  _parse_namespace
Module: U:\dev\php-5.3.8\ext\sockets\sockets.o(sockets.o)
0002:00020910  _sockets_globals_id
0001:003f905f  _zif_socket_clear_error
0001:003f910d  _zif_socket_last_error
0001:003f91bf  _zm_deactivate_sockets
0001:003f9201  _zif_socket_close
0001:003f92d2  _zm_info_sockets
0001:003f98a2  _zm_startup_sockets
0001:003faaba  _zif_socket_shutdown
0001:003fac17  _zif_socket_get_option
0001:003faef0  _zif_socket_strerror
0001:003faf76  _zif_socket_send
0001:003fb16d  _zif_socket_create
0001:003fb304  _zif_socket_write
0001:003fb46f  _zif_socket_listen
0001:003fb5a7  _zif_socket_set_block
0001:003fb6e3  _zif_socket_set_nonblock
0001:003fb825  _zif_socket_accept
0001:003fb9ec  _zif_socket_create_listen
0001:003fbe25  _zif_socket_sendto
0001:003fc12b  _zif_socket_bind
0001:003fc398  _zif_socket_connect
0001:003fc94a  _zif_socket_read
0001:003fcce7  _zif_socket_select
0001:003fd02a  _zif_socket_create_pair
0001:003fd2f2  _zif_socket_getpeername
0001:003fd5ab  _zif_socket_getsockname
0001:003fd846  _zif_socket_recv
0001:003fda2c  _zif_socket_recvfrom
0001:003fde19  _zif_socket_set_option
0001:003fe5a3  _php_sockets_le_socket
0001:003fe760  _sockets_functions
0002:00002960  _sockets_module_entry
0002:00009ed0  _inet_ntoa_lock
Module: U:\dev\php-5.3.8\ext\spl\php_spl.o(php_spl.o)
0002:00020920  _spl_globals_id
0001:003ff3c3  _zm_activate_spl
0001:003ff3f4  _zm_deactivate_spl
0001:003ff480  _zm_startup_spl
0001:003ff51c  _zif_spl_classes
0001:003ffee1  _zm_info_spl
0001:00401325  _spl_build_class_list_string
0001:0040138f  _zif_spl_autoload_functions
0001:00401668  _zif_spl_autoload_unregister
0001:00401adf  _zif_spl_autoload_register
0001:004021d5  _zif_spl_autoload_call
0001:00402447  _zif_spl_autoload_extensions
0001:004026b9  _zif_class_implements
0001:0040279f  _zif_class_parents
0001:004028c1  _zif_spl_autoload
0001:00402d74  _php_spl_object_hash
0001:00402ea5  _zif_spl_object_hash
0001:00402ff0  _spl_functions
0002:000029c0  _spl_module_entry
Module: U:\dev\php-5.3.8\ext\spl\spl_functions.o(spl_functions.o)
0001:004034c0  _spl_register_interface
0001:004035ce  _spl_register_std_class
0001:004036f9  _spl_register_sub_class
0001:0040384a  _spl_register_property
0001:00403856  _spl_add_class_name
0001:00403939  _spl_add_interfaces
0001:00403996  _spl_add_classes
0001:00403a36  _spl_gen_private_prop_name
Module: U:\dev\php-5.3.8\ext\spl\spl_engine.o(spl_engine.o)
0001:00403a80  _spl_instantiate
0001:00403ad1  _spl_offset_convert_to_long
Module: U:\dev\php-5.3.8\ext\spl\spl_iterators.o(spl_iterators.o)
0002:00020930  _spl_ce_RecursiveIterator
0002:00020940  _spl_ce_RecursiveIteratorIterator
0002:00020950  _spl_ce_AppendIterator
0002:00020960  _spl_ce_InfiniteIterator
0002:00020970  _spl_ce_NoRewindIterator
0002:00020980  _spl_ce_IteratorIterator
0002:00020990  _spl_ce_RecursiveCachingIterator
0002:000209a0  _spl_ce_CachingIterator
0002:000209b0  _spl_ce_LimitIterator
0002:000209c0  _spl_ce_RecursiveRegexIterator
0002:000209d0  _spl_ce_RegexIterator
0002:000209e0  _spl_ce_ParentIterator
0002:000209f0  _spl_ce_RecursiveFilterIterator
0002:00020a00  _spl_ce_FilterIterator
0002:00020a10  _spl_ce_RecursiveTreeIterator
0002:00020a20  _spl_ce_SeekableIterator
0002:00020a30  _spl_ce_OuterIterator
0002:00020a40  _spl_ce_Countable
0002:00020a50  _spl_ce_EmptyIterator
0001:0040576b  _zim_spl_EmptyIterator_next
0001:004057ac  _zim_spl_EmptyIterator_current
0001:00405822  _zim_spl_EmptyIterator_key
0001:00405871  _zim_spl_EmptyIterator_valid
0001:004058aa  _zim_spl_EmptyIterator_rewind
0001:004058c3  _zim_spl_NoRewindIterator_rewind
0001:004058dc  _zim_spl_RecursiveTreeIterator_getPrefix
0001:00405938  _zim_spl_RecursiveIteratorIterator_getMaxDepth
0001:004059c2  _zim_spl_RecursiveIteratorIterator_setMaxDepth
0001:00405a3d  _zim_spl_RecursiveIteratorIterator_nextElement
0001:00405a56  _zim_spl_RecursiveIteratorIterator_endChildren
0001:00405a6f  _zim_spl_RecursiveIteratorIterator_beginChildren
0001:00405a88  _zim_spl_RecursiveIteratorIterator_callGetChildren
0001:00405b80  _zim_spl_RecursiveIteratorIterator_callHasChildren
0001:00405c8a  _zim_spl_RecursiveIteratorIterator_endIteration
0001:00405ca3  _zim_spl_RecursiveIteratorIterator_beginIteration
0001:00405cbc  _zim_spl_RecursiveIteratorIterator_getDepth
0001:00405d09  _zim_spl_RecursiveIteratorIterator_next
0001:00405d62  _zim_spl_RecursiveIteratorIterator_key
0001:00405e10  _zim_spl_RecursiveIteratorIterator_valid
0001:00405e71  _zim_spl_RecursiveIteratorIterator_rewind
0001:004060f3  _zim_spl_AppendIterator_valid
0001:00406171  _zim_spl_NoRewindIterator_next
0001:004061ef  _zim_spl_NoRewindIterator_key
0001:004062ba  _zim_spl_NoRewindIterator_valid
0001:00406345  _zim_spl_RecursiveCachingIterator_hasChildren
0001:004063c3  _zim_spl_CachingIterator_getFlags
0001:00406439  _zim_spl_CachingIterator_hasNext
0001:004064c9  _zim_spl_CachingIterator_valid
0001:00406546  _zim_spl_LimitIterator_getPosition
0001:0040659d  _zim_spl_LimitIterator_valid
0001:0040660e  _zim_spl_RegexIterator_setPregFlags
0001:00406686  _zim_spl_RegexIterator_getPregFlags
0001:00406703  _zim_spl_RegexIterator_setFlags
0001:00406774  _zim_spl_RegexIterator_getFlags
0001:004067fb  _zim_spl_RegexIterator_setMode
0001:0040689f  _zim_spl_RegexIterator_getMode
0001:00406915  _zim_spl_RecursiveFilterIterator_hasChildren
0001:00406a2a  _zim_spl_dual_it_valid
0001:00406ad9  _zim_spl_RecursiveTreeIterator_setPrefixPart
0001:00406c7a  _zim_spl_AppendIterator_getIteratorIndex
0001:00406cff  _zim_spl_dual_it_key
0001:00406da8  _zim_spl_RecursiveTreeIterator_getPostfix
0001:00406e4c  _zim_spl_CachingIterator_count
0001:00406ffd  _zim_spl_CachingIterator_setFlags
0001:004071da  _zim_spl_CachingIterator_offsetExists
0001:004073ea  _zim_spl_CachingIterator_offsetUnset
0001:00407612  _zim_spl_RecursiveFilterIterator_getChildren
0001:004077a8  _zim_spl_RegexIterator_accept
0001:00408523  _zim_spl_AppendIterator___construct
0001:00408554  _zim_spl_InfiniteIterator___construct
0001:00408585  _zim_spl_NoRewindIterator___construct
0001:004085b6  _zim_spl_IteratorIterator___construct
0001:004085e7  _zim_spl_RecursiveCachingIterator___construct
0001:00408618  _zim_spl_CachingIterator___construct
0001:00408649  _zim_spl_LimitIterator___construct
0001:0040867a  _zim_spl_RecursiveRegexIterator___construct
0001:004086ab  _zim_spl_RegexIterator___construct
0001:004086dc  _zim_spl_ParentIterator___construct
0001:0040870d  _zim_spl_RecursiveFilterIterator___construct
0001:0040873e  _zim_spl_FilterIterator___construct
0001:0040876f  _zim_spl_RecursiveIteratorIterator_getInnerIterator
0001:004088ef  _zim_spl_RecursiveTreeIterator_getEntry
0001:00408950  _zim_spl_AppendIterator_getArrayIterator
0001:004089f6  _zim_spl_RecursiveIteratorIterator_current
0001:00408a9a  _zim_spl_NoRewindIterator_current
0001:00408b62  _zim_spl_RecursiveCachingIterator_getChildren
0001:00408c18  _zim_spl_CachingIterator_getCache
0001:00408cfb  _zim_spl_dual_it_current
0001:00408db1  _zim_spl_dual_it_getInnerIterator
0001:00408e7c  _zim_spl_CachingIterator_offsetGet
0001:00409132  _zim_spl_RecursiveIteratorIterator_getSubIterator
0001:004091dc  _zim_spl_RecursiveTreeIterator_current
0001:00409398  _zim_spl_RecursiveTreeIterator_key
0001:00409626  _zim_spl_CachingIterator___toString
0001:00409f07  _zim_spl_RecursiveTreeIterator___construct
0001:00409f2c  _zim_spl_RecursiveIteratorIterator___construct
0001:00409f54  _zim_spl_CachingIterator_offsetSet
0001:0040a28f  _zim_spl_FilterIterator_next
0001:0040ad8e  _zim_spl_CachingIterator_next
0001:0040ae02  _zim_spl_CachingIterator_rewind
0001:0040af6a  _zim_spl_RecursiveRegexIterator_getChildren
0001:0040b155  _zim_spl_LimitIterator_next
0001:0040b38e  _zim_spl_dual_it_next
0001:0040b5c4  _zim_spl_dual_it_rewind
0001:0040b87a  _zim_spl_LimitIterator_seek
0001:0040bf4e  _zim_spl_InfiniteIterator_next
0001:0040c261  _zim_spl_FilterIterator_rewind
0001:0040c60f  _zim_spl_LimitIterator_rewind
0001:0040cd50  _spl_append_it_next_iterator
0001:0040cf7b  _spl_append_it_fetch
0001:0040d0c6  _zim_spl_AppendIterator_rewind
0001:0040d160  _zim_spl_AppendIterator_append
0001:0040d25d  _spl_append_it_next
0001:0040d330  _zim_spl_AppendIterator_next
0001:0040d3a8  _spl_iterator_apply
0001:0040d4ee  _zif_iterator_to_array
0001:0040d5a1  _zif_iterator_count
0001:0040d62b  _zif_iterator_apply
0001:0040d971  _zm_startup_spl_iterators
0001:0040e310  _spl_funcs_RecursiveIterator
0002:00002a20  _spl_recursive_it_iterator_funcs
Module: U:\dev\php-5.3.8\ext\spl\spl_array.o(spl_array.o)
0002:00020a60  _spl_handler_ArrayIterator
0002:00020ad0  _spl_ce_ArrayObject
0002:00020ae0  _spl_ce_ArrayIterator
0002:00020af0  _spl_ce_RecursiveArrayIterator
0002:00020b00  _spl_handler_ArrayObject
0001:0040f7e5  _spl_array_get_iterator
0001:0040f8ac  _zim_spl_Array_setFlags
0001:0040f909  _zim_spl_Array_getFlags
0001:0040f959  _zim_spl_Array_setIteratorClass
0001:0040f9ad  _zim_spl_Array_getIteratorClass
0001:00410843  _zim_spl_Array_offsetGet
0001:004112ce  _zim_spl_Array_rewind
0001:00411649  _zim_spl_Array___construct
0001:0041182f  _zim_spl_Array_getArrayCopy
0001:00411988  _zim_spl_Array_getIterator
0001:00411acc  _zim_spl_Array_exchangeArray
0001:00411ec2  _zim_spl_Array_natcasesort
0001:00411eff  _zim_spl_Array_natsort
0001:00411f3b  _zim_spl_Array_uksort
0001:00411f77  _zim_spl_Array_uasort
0001:00411fb2  _zim_spl_Array_ksort
0001:00411fed  _zim_spl_Array_asort
0001:004127c9  _zim_spl_Array_offsetExists
0001:00412f88  _zim_spl_Array_offsetSet
0001:00412fd9  _spl_hash_verify_pos_ex
0001:004136d3  _zim_spl_Array_getChildren
0001:004139b6  _zim_spl_Array_hasChildren
0001:00413b92  _zim_spl_Array_valid
0001:00413d8a  _zim_spl_Array_next
0001:00414099  _zim_spl_Array_count
0001:004140f2  _spl_array_object_count_elements
0001:00414252  _zim_spl_Array_seek
0001:004143ee  _zim_spl_Array_current
0001:004145ad  _spl_hash_verify_pos
0001:00414c12  _zim_spl_Array_offsetUnset
0001:00414c99  _spl_array_iterator_append
0001:00414e0b  _zim_spl_Array_append
0001:00414e54  _spl_array_iterator_key
0001:00414fe6  _zim_spl_Array_key
0001:00415031  _spl_array_serialize_helper
0001:004153d0  _spl_array_serialize
0001:0041547a  _zim_spl_Array_serialize
0001:004155b4  _spl_array_unserialize_helper
0001:00415830  _spl_array_unserialize
0001:00415988  _zim_spl_Array_unserialize
0001:00415aef  _zm_startup_spl_array
0002:00002a40  _spl_array_it_funcs
Module: U:\dev\php-5.3.8\ext\spl\spl_directory.o(spl_directory.o)
0002:00020b70  _spl_ce_SplFileObject
0002:00020b80  _spl_ce_SplFileInfo
0002:00020b90  _spl_ce_DirectoryIterator
0002:00020ba0  _spl_ce_RecursiveDirectoryIterator
0002:00020bb0  _spl_ce_FilesystemIterator
0002:00020bc0  _spl_ce_GlobIterator
0002:00020bd0  _spl_ce_SplTempFileObject
0001:0041679a  _zim_spl_SplFileInfo__bad_state_ex
0001:004167c3  _zim_spl_SplFileObject_getChildren
0001:004167dc  _zim_spl_SplFileObject_hasChildren
0001:00416953  _zim_spl_SplFileObject_setCsvControl
0001:00416aa1  _zim_spl_SplFileObject_getMaxLineLen
0001:00416b27  _zim_spl_SplFileObject_setMaxLineLen
0001:00416b9a  _zim_spl_SplFileObject_getFlags
0001:00416bea  _zim_spl_SplFileObject_setFlags
0001:00416c25  _zim_spl_SplFileObject_key
0001:00416c79  _zim_spl_RecursiveDirectoryIterator_getSubPathname
0001:00416d4b  _zim_spl_RecursiveDirectoryIterator_getSubPath
0001:00416ddd  _zim_spl_FilesystemIterator_setFlags
0001:00416e39  _zim_spl_FilesystemIterator_getFlags
0001:00416e8e  _zim_spl_SplFileInfo_setInfoClass
0001:00416f0f  _zim_spl_SplFileInfo_setFileClass
0001:00416f90  _zim_spl_DirectoryIterator_getFilename
0001:00416ffc  _zim_spl_DirectoryIterator_valid
0001:0041704f  _zim_spl_DirectoryIterator_key
0001:004170b8  _zim_spl_DirectoryIterator_rewind
0001:0041714c  _spl_filesystem_object_get_method_check
0001:004171ad  _zim_spl_SplFileObject_valid
0001:00417231  _zim_spl_SplFileObject_eof
0001:004172a9  _zim_spl_SplFileObject_ftruncate
0001:00417381  _zim_spl_SplFileObject_fwrite
0001:004174b7  _zim_spl_SplFileObject_fpassthru
0001:004174f0  _zim_spl_SplFileObject_ftell
0001:0041753f  _zim_spl_SplFileObject_fflush
0001:00417588  _zim_spl_SplFileObject_getCsvControl
0001:00417639  _spl_filesystem_tree_get_iterator
0001:00417696  _spl_filesystem_dir_get_iterator
0001:0041770c  _zim_spl_GlobIterator_count
0001:004177b7  _zim_spl_DirectoryIterator_seek
0001:00417a0a  _zim_spl_SplFileInfo_getLinkTarget
0001:00417bf4  _zim_spl_DirectoryIterator_getBasename
0001:00417ca2  _zim_spl_DirectoryIterator_getExtension
0001:00417f0d  _zim_spl_SplFileObject_fseek
0001:00418162  _zim_spl_SplFileObject_fgets
0001:004181e3  _zim_spl_SplFileObject_fgetc
0001:004184de  _zim_spl_SplTempFileObject___construct
0001:004185ff  _zim_spl_SplFileObject___construct
0001:0041877d  _zim_spl_DirectoryIterator_current
0001:004189b7  _zim_spl_SplFileObject_fstat
0001:00418a65  _zim_spl_SplFileObject_fscanf
0001:00418b1c  _zim_spl_SplFileObject_fgetss
0001:00418c22  _zim_spl_SplFileObject_flock
0001:00418e2f  _zim_spl_SplFileObject_fgetcsv
0001:004191ea  _zim_spl_SplFileObject_current
0001:004192d6  _zim_spl_SplFileObject_next
0001:00419408  _zim_spl_SplFileObject_seek
0001:004194bd  _zim_spl_SplFileObject_rewind
0001:0041976e  _zim_spl_FilesystemIterator_rewind
0001:0041983e  _zim_spl_DirectoryIterator_next
0001:004198ee  _zim_spl_DirectoryIterator_isDot
0001:00419d0a  _spl_filesystem_object_get_path
0001:00419d52  _zim_spl_SplFileInfo_getRealPath
0001:00419ef3  _zim_spl_SplFileInfo_getBasename
0001:00419fce  _zim_spl_SplFileInfo_getExtension
0001:0041a111  _zim_spl_SplFileInfo_getFilename
0001:0041a1b5  _zim_spl_SplFileInfo_getPath
0001:0041a373  _zim_spl_FilesystemIterator_key
0001:0041a4b7  _zim_spl_SplFileInfo_getInode
0001:0041a5e8  _zim_spl_SplFileInfo_getATime
0001:0041a719  _zim_spl_SplFileInfo_getOwner
0001:0041a84a  _zim_spl_SplFileInfo_getPerms
0001:0041a97b  _zim_spl_SplFileInfo_getSize
0001:0041aaac  _zim_spl_RecursiveDirectoryIterator_getChildren
0001:0041ad45  _zim_spl_SplFileInfo_getMTime
0001:0041ae78  _zim_spl_SplFileInfo_getCTime
0001:0041afa9  _zim_spl_SplFileInfo_getGroup
0001:0041b0da  _zim_spl_SplFileInfo_isWritable
0001:0041b20b  _zim_spl_SplFileInfo_isExecutable
0001:0041b33c  _zim_spl_SplFileInfo_isFile
0001:0041b46d  _zim_spl_SplFileInfo_getType
0001:0041b59e  _zim_spl_SplFileInfo_isLink
0001:0041b6cf  _zim_spl_SplFileInfo_isDir
0001:0041b800  _zim_spl_SplFileInfo_isReadable
0001:0041b934  _zim_spl_RecursiveDirectoryIterator_hasChildren
0001:0041bbbb  _zim_spl_SplFileInfo_getPathname
0001:0041c717  _zim_spl_SplFileInfo_getFileInfo
0001:0041c7ad  _zim_spl_SplFileInfo_openFile
0001:0041c7f0  _zim_spl_FilesystemIterator_current
0001:0041cc7e  _spl_filesystem_info_set_filename
0001:0041cd3e  _zim_spl_SplFileInfo___construct
0001:0041cdd7  _zim_spl_SplFileInfo_getPathInfo
0001:0041d03c  _spl_filesystem_object_construct
0001:0041d204  _zim_spl_GlobIterator___construct
0001:0041d242  _zim_spl_RecursiveDirectoryIterator___construct
0001:0041d280  _zim_spl_FilesystemIterator___construct
0001:0041d2be  _zim_spl_DirectoryIterator___construct
0001:0041d453  _zm_startup_spl_directory
0002:00002a80  _spl_filesystem_tree_it_funcs
0002:00002a60  _spl_filesystem_dir_it_funcs
Module: U:\dev\php-5.3.8\ext\spl\spl_exceptions.o(spl_exceptions.o)
0002:00020be0  _spl_ce_LogicException
0002:00020bf0  _spl_ce_BadFunctionCallException
0002:00020c00  _spl_ce_BadMethodCallException
0002:00020c10  _spl_ce_DomainException
0002:00020c20  _spl_ce_InvalidArgumentException
0002:00020c30  _spl_ce_LengthException
0002:00020c40  _spl_ce_OutOfRangeException
0002:00020c50  _spl_ce_RuntimeException
0002:00020c60  _spl_ce_OutOfBoundsException
0002:00020c70  _spl_ce_OverflowException
0002:00020c80  _spl_ce_RangeException
0002:00020c90  _spl_ce_UnderflowException
0002:00020ca0  _spl_ce_UnexpectedValueException
0001:0041ea3f  _zm_startup_spl_exceptions
Module: U:\dev\php-5.3.8\ext\spl\spl_observer.o(spl_observer.o)
0002:00020cb0  _spl_ce_SplObjectStorage
0002:00020cc0  _spl_handler_SplObjectStorage
0002:00020d30  _spl_ce_SplObserver
0002:00020d40  _spl_ce_SplSubject
0002:00020d50  _spl_ce_MultipleIterator
0001:0041f352  _zim_spl_MultipleIterator_setFlags
0001:0041f38e  _zim_spl_MultipleIterator_getFlags
0001:0041f3db  _zim_spl_SplObjectStorage_next
0001:0041f432  _zim_spl_SplObjectStorage_setInfo
0001:0041f4b1  _zim_spl_SplObjectStorage_key
0001:0041f4fe  _zim_spl_SplObjectStorage_rewind
0001:0041f556  _zim_spl_SplObjectStorage_count
0001:0041f5b1  _zim_spl_MultipleIterator_valid
0001:0041f739  _zim_spl_MultipleIterator_next
0001:0041f853  _zim_spl_MultipleIterator_rewind
0001:0041fdc7  _zim_spl_MultipleIterator_key
0001:0041fe27  _zim_spl_MultipleIterator_current
0001:0041fe8a  _zim_spl_MultipleIterator___construct
0001:0041ff07  _zim_spl_SplObjectStorage_serialize
0001:00420512  _zim_spl_SplObjectStorage_valid
0001:00420577  _zim_spl_SplObjectStorage_current
0001:00420616  _zim_spl_SplObjectStorage_contains
0001:00420689  _spl_SplOjectStorage_free_storage
0001:004206d4  _zim_spl_SplObjectStorage_getInfo
0001:00420772  _spl_object_storage_get
0001:004207ba  _zim_spl_SplObjectStorage_offsetGet
0001:0042087a  _spl_object_storage_attach
0001:00420987  _zim_spl_MultipleIterator_attachIterator
0001:00420b34  _zim_spl_SplObjectStorage_unserialize
0001:00420f8f  _zim_spl_SplObjectStorage_attach
0001:00420ffd  _spl_object_storage_detach
0001:00421034  _zim_spl_SplObjectStorage_removeAll
0001:00421121  _zim_spl_SplObjectStorage_detach
0001:00421193  _zim_spl_SplObjectStorage_removeAllExcept
0001:004212b0  _spl_object_storage_addall
0001:004214ad  _zim_spl_SplObjectStorage_addAll
0001:00421531  _spl_object_storage_contains
0001:004215c0  _zm_startup_spl_observer
Module: U:\dev\php-5.3.8\ext\spl\spl_dllist.o(spl_dllist.o)
0002:00020d60  _spl_ce_SplDoublyLinkedList
0002:00020d70  _spl_ce_SplStack
0002:00020d80  _spl_ce_SplQueue
0002:00020d90  _spl_handler_SplDoublyLinkedList
0001:00422a5d  _spl_dllist_get_iterator
0001:00422afb  _zim_spl_SplDoublyLinkedList_rewind
0001:00422b96  _zim_spl_SplDoublyLinkedList_valid
0001:00422be9  _zim_spl_SplDoublyLinkedList_next
0001:00422c4a  _zim_spl_SplDoublyLinkedList_prev
0001:00422cae  _zim_spl_SplDoublyLinkedList_key
0001:00422cfb  _zim_spl_SplDoublyLinkedList_getIteratorMode
0001:00422d8c  _zim_spl_SplDoublyLinkedList_setIteratorMode
0001:00422e1a  _zim_spl_SplDoublyLinkedList_count
0001:00422e8f  _zim_spl_SplDoublyLinkedList_offsetUnset
0001:00423033  _zim_spl_SplDoublyLinkedList_offsetSet
0001:004231fd  _zim_spl_SplDoublyLinkedList_offsetExists
0001:004233ae  _zim_spl_SplDoublyLinkedList_isEmpty
0001:00423404  _zim_spl_SplDoublyLinkedList_current
0001:004234bd  _zim_spl_SplDoublyLinkedList_bottom
0001:0042356c  _zim_spl_SplDoublyLinkedList_top
0001:00423644  _zim_spl_SplDoublyLinkedList_shift
0001:00423722  _zim_spl_SplDoublyLinkedList_pop
0001:004237d9  _zim_spl_SplDoublyLinkedList_offsetGet
0001:004238fb  _zim_spl_SplDoublyLinkedList_unshift
0001:004239f2  _zim_spl_SplDoublyLinkedList_push
0001:00423afc  _zm_startup_spl_dllist
0002:00002aa0  _spl_dllist_it_funcs
Module: U:\dev\php-5.3.8\ext\spl\spl_heap.o(spl_heap.o)
0002:00020e00  _spl_ce_SplPriorityQueue
0002:00020e10  _spl_ce_SplHeap
0002:00020e20  _spl_ce_SplMinHeap
0002:00020e30  _spl_ce_SplMaxHeap
0002:00020e40  _spl_handler_SplHeap
0002:00020eb0  _spl_handler_SplPriorityQueue
0001:00424501  _spl_pqueue_get_iterator
0001:00424587  _spl_heap_get_iterator
0001:00425204  _zim_spl_SplHeap_rewind
0001:0042521d  _zim_spl_SplHeap_valid
0001:00425275  _zim_spl_SplHeap_next
0001:004252d3  _zim_spl_SplHeap_key
0001:00425329  _zim_spl_SplMaxHeap_compare
0001:0042538c  _zim_spl_SplMinHeap_compare
0001:004253ef  _zim_spl_SplPriorityQueue_compare
0001:00425452  _zim_spl_SplHeap_recoverFromCorruption
0001:004254a5  _zim_spl_SplPriorityQueue_setExtractFlags
0001:004254fe  _zim_spl_SplHeap_isEmpty
0001:00425556  _zim_spl_SplHeap_count
0001:00425683  _zim_spl_SplHeap_insert
0001:004258d9  _zim_spl_SplHeap_top
0001:004259a1  _zim_spl_SplPriorityQueue_current
0001:00425a66  _zim_spl_SplPriorityQueue_top
0001:00425b99  _zim_spl_SplHeap_extract
0001:00425c7c  _zim_spl_SplHeap_current
0001:00425d25  _zim_spl_SplPriorityQueue_extract
0001:00425e5c  _zim_spl_SplPriorityQueue_insert
0001:004260b6  _zm_startup_spl_heap
0002:00002ae0  _spl_pqueue_it_funcs
0002:00002ac0  _spl_heap_it_funcs
Module: U:\dev\php-5.3.8\ext\spl\spl_fixedarray.o(spl_fixedarray.o)
0002:00020f20  _spl_ce_SplFixedArray
0002:00020f30  _spl_handler_SplFixedArray
0001:0042686d  _spl_fixedarray_get_iterator
0001:00426aec  _zim_spl_SplFixedArray_rewind
0001:00426b32  _zim_spl_SplFixedArray_valid
0001:00426b93  _zim_spl_SplFixedArray_next
0001:00426bd6  _zim_spl_SplFixedArray_key
0001:00426c23  _zim_spl_SplFixedArray_getSize
0001:00426c86  _zim_spl_SplFixedArray_count
0001:004272fc  _zim_spl_SplFixedArray___construct
0001:00427397  _zim_spl_SplFixedArray_setSize
0001:0042757d  _zim_spl_SplFixedArray_toArray
0001:00427840  _zim_spl_SplFixedArray_fromArray
0001:00428347  _zim_spl_SplFixedArray_offsetExists
0001:004283ce  _zim_spl_SplFixedArray_offsetUnset
0001:0042848c  _zim_spl_SplFixedArray_offsetGet
0001:00428570  _zim_spl_SplFixedArray_current
0001:00428784  _zim_spl_SplFixedArray_offsetSet
0001:004288a3  _zm_startup_spl_fixedarray
0002:00002b00  _spl_fixedarray_it_funcs
Module: U:\dev\php-5.3.8\ext\standard\crypt_freesec.o(crypt_freesec.o)
0001:004291fd  __crypt_extended_init
0001:004296c9  __crypt_extended_r
Module: U:\dev\php-5.3.8\ext\standard\crypt_blowfish.o(crypt_blowfish.o)
0001:0042bd9e  _php_crypt_blowfish_rn
Module: U:\dev\php-5.3.8\ext\standard\crypt_sha512.o(crypt_sha512.o)
0001:0042dd57  _php_sha512_crypt_r
0001:0042f430  _php_sha512_crypt
Module: U:\dev\php-5.3.8\ext\standard\crypt_sha256.o(crypt_sha256.o)
0001:0042fd7b  ___php_stpncpy
0001:0042fdbd  ___php_mempcpy
0001:0042fdee  _php_sha256_crypt_r
0001:00430ddc  _php_sha256_crypt
Module: U:\dev\php-5.3.8\ext\standard\php_crypt_r.o(php_crypt_r.o)
0002:00020fa0  _php_crypt_extended_init_lock
0001:00430fe0  _php_init_crypt_r
0001:00430ff2  _php_shutdown_crypt_r
0001:00431007  __crypt_extended_init_r
0001:00431043  _php_md5_crypt_r
Module: U:\dev\php-5.3.8\ext\standard\array.o(array.o)
0002:00020fb0  _array_globals_id
0001:004318d5  _php_multisort_compare
0001:00434fef  _zm_startup_array
0001:00435342  _zm_shutdown_array
0001:0043535d  _zif_krsort
0001:004353f6  _zif_ksort
0001:00435499  _zif_count
0001:0043566e  _zif_natsort
0001:00435695  _zif_natcasesort
0001:004356bc  _zif_asort
0001:00435755  _zif_arsort
0001:004357ee  _zif_sort
0001:00435887  _zif_rsort
0001:00435957  _zif_usort
0001:00435b5a  _zif_uasort
0001:00435d5d  _zif_uksort
0001:00435f62  _zif_end
0001:00436021  _zif_prev
0001:004360e0  _zif_next
0001:0043619f  _zif_reset
0001:0043625e  _zif_current
0001:00436301  _zif_key
0001:00436404  _zif_min
0001:004365e7  _zif_max
0001:004367c6  _zif_array_walk
0001:00436973  _zif_array_walk_recursive
0001:00436b23  _zif_in_array
0001:00436b3f  _zif_array_search
0001:00436b5b  _php_prefix_varname
0001:00436c7a  _zif_extract
0001:0043744c  _zif_compact
0001:00437584  _zif_array_fill
0001:00437690  _zif_array_fill_keys
0001:004379a5  _zif_range
0001:004385b4  _zif_shuffle
0001:0043874b  _php_splice
0001:00438b40  _zif_array_push
0001:00438c5f  _zif_array_pop
0001:00438c7b  _zif_array_shift
0001:00438c97  _zif_array_unshift
0001:00438daa  _zif_array_splice
0001:00438fda  _zif_array_slice
0001:00439328  _php_array_merge
0001:00439904  _php_array_replace_recursive
0001:00439e39  _zif_array_merge
0001:00439e5c  _zif_array_merge_recursive
0001:00439e7f  _zif_array_replace
0001:00439ea2  _zif_array_replace_recursive
0001:00439eca  _zif_array_keys
0001:0043a0d6  _zif_array_values
0001:0043a1d6  _zif_array_count_values
0001:0043a638  _zif_array_reverse
0001:0043a816  _zif_array_pad
0001:0043aa6d  _zif_array_flip
0001:0043ad92  _zif_array_change_key_case
0001:0043af40  _zif_array_unique
0001:0043b208  _zif_array_intersect_key
0001:0043b224  _zif_array_intersect_ukey
0001:0043b24e  _zif_array_intersect
0001:0043b278  _zif_array_uintersect
0001:0043b2a2  _zif_array_intersect_assoc
0001:0043b2be  _zif_array_intersect_uassoc
0001:0043b2e8  _zif_array_uintersect_assoc
0001:0043b304  _zif_array_uintersect_uassoc
0001:0043b32e  _zif_array_diff_key
0001:0043b34a  _zif_array_diff_ukey
0001:0043b374  _zif_array_diff
0001:0043b39e  _zif_array_udiff
0001:0043b3c8  _zif_array_diff_assoc
0001:0043b3e4  _zif_array_diff_uassoc
0001:0043b40e  _zif_array_udiff_assoc
0001:0043b42a  _zif_array_udiff_uassoc
0001:0043b52c  _zif_array_multisort
0001:0043bca8  _zif_array_rand
0001:0043be87  _zif_array_sum
0001:0043bfba  _zif_array_product
0001:0043c140  _zif_array_reduce
0001:0043c3ed  _zif_array_filter
0001:0043c6ba  _zif_array_map
0001:0043cd77  _zif_array_key_exists
0001:0043cf95  _zif_array_chunk
0001:0043d227  _zif_array_combine
Module: U:\dev\php-5.3.8\ext\standard\base64.o(base64.o)
0001:0043d460  _php_base64_encode
0001:0043d5e1  _php_base64_decode_ex
0001:0043d786  _php_base64_decode
0001:0043d7b1  _zif_base64_encode
0001:0043d82b  _zif_base64_decode
Module: U:\dev\php-5.3.8\ext\standard\basic_functions.o(basic_functions.o)
0002:00020fc0  _basic_globals_id
0001:0043db10  _zif_get_magic_quotes_runtime
0001:0043db31  _zif_get_magic_quotes_gpc
0001:0043db51  _zif_connection_aborted
0001:0043db78  _zif_connection_status
0001:0043db9c  _zif_sys_getloadavg
0001:0043dc2b  _zif_set_magic_quotes_runtime
0001:0043dcb8  _zif_import_request_variables
0001:0043e048  _zif_parse_ini_string
0001:0043e207  _zif_parse_ini_file
0001:0043e37a  _zif_is_uploaded_file
0001:0043e447  _zif_move_uploaded_file
0001:0043e6b7  _zif_unregister_tick_function
0001:0043e8ea  _zif_getprotobynumber
0001:0043e969  _zif_getprotobyname
0001:0043e9cd  _zif_getservbyport
0001:0043ea67  _zif_getservbyname
0001:0043eaf7  _zif_ignore_user_abort
0001:0043eba5  _zif_print_r
0001:0043ec80  _zif_restore_include_path
0001:0043ecc2  _zif_ini_restore
0001:0043ed14  _zif_get_include_path
0001:0043ed9d  _zif_ini_get
0001:0043ee8c  _zif_ini_get_all
0001:0043f1b4  _zif_php_strip_whitespace
0001:0043f356  _zif_register_shutdown_function
0001:0043f615  _zif_error_get_last
0001:0043f74a  _zif_get_cfg_var
0001:0043f928  _zif_get_current_user
0001:0043f9b6  _zif_time_sleep_until
0001:0043fb4a  _zif_time_nanosleep
0001:0043fc8e  _zif_usleep
0001:0043fd3d  _zif_sleep
0001:0043fdbb  _zif_flush
0001:0043fe8f  _zif_putenv
0001:004402de  _zif_getenv
0001:0044039e  _zif_long2ip
0001:00440490  _php_inet_ntop
0001:00440561  _zif_ip2long
0001:004405fc  _php_inet_pton
0001:0044070c  _zif_constant
0001:004407ab  _zm_info_basic
0001:004407ee  _zm_deactivate_basic
0001:004409b8  _zm_activate_basic
0001:00440bda  _zm_shutdown_basic
0001:00440e9f  _zm_startup_basic
0001:004419f0  _zif_forward_static_call
0001:00441bb3  _zif_call_user_method_array
0001:00441e0f  _zif_call_user_method
0001:00441fe7  _zif_call_user_func
0001:00442100  _zif_forward_static_call_array
0001:0044225d  _zif_call_user_func_array
0001:0044239a  _zif_register_tick_function
0001:00442ff4  _zif_ini_set
0001:004432dd  _zif_set_include_path
0001:00443c86  _zif_getopt
0001:00444875  _php_get_nan
0001:00444880  _php_get_inf
0001:004448c0  __php_error_log_ex
0001:004449f4  __php_error_log
0001:00444a4b  _zif_error_log
0001:00444b4e  _php_free_shutdown_functions
0001:00444bfc  _php_call_shutdown_functions
0001:00444ce9  _php_get_highlight_struct
0001:00444dd0  _zif_highlight_string
0001:00445003  _zif_highlight_file
0001:004469c0  _basic_functions
0002:00002cf0  _basic_functions_module
Module: U:\dev\php-5.3.8\ext\standard\browscap.o(browscap.o)
0002:00020fd0  _browscap_globals_id
0001:00453708  _OnChangeBrowscap
0001:0045376a  _zm_startup_browscap
0001:004537f1  _zm_deactivate_browscap
0001:0045381a  _zm_shutdown_browscap
0001:004538e0  _zif_get_browser
Module: U:\dev\php-5.3.8\ext\standard\crc32.o(crc32.o)
0001:00453d22  _php_if_crc32
Module: U:\dev\php-5.3.8\ext\standard\crypt.o(crypt.o)
0001:00454211  _zm_startup_crypt
0001:00454361  _zm_shutdown_crypt
0001:00454380  _zif_crypt
Module: U:\dev\php-5.3.8\ext\standard\cyr_convert.o(cyr_convert.o)
0001:00454910  _zif_convert_cyr_string
Module: U:\dev\php-5.3.8\ext\standard\datetime.o(datetime.o)
0001:004553e8  _php_std_date
0001:00455563  _zif_strptime
0002:00002d80  _mon_short_names
0002:00002db0  _day_full_names
0002:00002dd0  _day_short_names
0002:00002d50  _mon_full_names
Module: U:\dev\php-5.3.8\ext\standard\dir.o(dir.o)
0002:00020fe0  _dir_globals_id
0001:0045585d  _php_if_readdir
0001:00455aa4  _zif_rewinddir
0001:00455ce5  _zif_closedir
0001:00456082  _zm_activate_dir
0001:00456128  _zm_startup_dir
0001:0045642f  _zif_opendir
0001:0045644b  _zif_getdir
0001:00456477  _zif_chdir
0001:00456652  _zif_getcwd
0001:00456779  _zif_glob
0001:00456bc6  _zif_scandir
Module: U:\dev\php-5.3.8\ext\standard\dl.o(dl.o)
0001:00457059  _php_load_extension
0001:0045744c  _php_dl
0001:004575b2  _zif_dl
0001:00457750  _zm_info_dl
Module: U:\dev\php-5.3.8\ext\standard\dns.o(dns.o)
0001:0045779f  _zif_gethostname
0001:0045788f  _zif_gethostbyaddr
0001:0045796c  _zif_gethostbyname
0001:004579fe  _zif_gethostbynamel
Module: U:\dev\php-5.3.8\ext\standard\exec.o(exec.o)
0001:00457ac0  _php_escape_shell_cmd
0001:00457ec1  _php_exec
0001:0045851e  _zif_passthru
0001:0045853a  _zif_system
0001:00458556  _zif_exec
0001:00458572  _php_escape_shell_arg
0001:004586b5  _zif_escapeshellcmd
0001:00458749  _zif_escapeshellarg
0001:004587fa  _zif_shell_exec
0001:00458984  _zif_proc_nice
Module: U:\dev\php-5.3.8\ext\standard\file.o(file.o)
0002:00020ff0  _file_globals_id
0001:00458b17  _php_le_stream_context
0001:00459054  _zm_startup_file
0001:00459bf4  _zm_shutdown_file
0001:00459c22  _zif_flock
0001:00459e1e  _zif_file_get_contents
0001:0045a1df  _zif_file_put_contents
0001:0045a995  _zif_file
0001:0045ae7f  _zif_tempnam
0001:0045aff2  _php_if_tmpfile
0001:0045b057  _php_if_fopen
0001:0045b1b6  _zif_fclose
0001:0045b2bf  _zif_popen
0001:0045b5c2  _zif_pclose
0001:0045b679  _zif_feof
0001:0045b754  _zif_fgets
0001:0045b972  _zif_fgetc
0001:0045ba47  _zif_fgetss
0001:0045bbff  _zif_fscanf
0001:0045bd51  _zif_fwrite
0001:0045bedf  _zif_fflush
0001:0045bf95  _zif_rewind
0001:0045c060  _zif_ftell
0001:0045c110  _zif_fseek
0001:0045c1e2  _php_mkdir_ex
0001:0045c297  _php_mkdir
0001:0045c2c6  _zif_mkdir
0001:0045c3f6  _zif_rmdir
0001:0045c503  _zif_readfile
0001:0045c652  _zif_umask
0001:0045c6f9  _zif_fpassthru
0001:0045c81e  _zif_rename
0001:0045ca60  _zif_unlink
0001:0045cc36  _php_if_ftruncate
0001:0045cd86  _php_if_fstat
0001:0045db48  _php_copy_file_ctx
0001:0045de2f  _php_copy_file_ex
0001:0045de60  _php_copy_file
0001:0045de91  _zif_copy
0001:0045e03d  _zif_fread
0001:0045e1fd  _zif_fputcsv
0001:0045ea8d  _php_fgetcsv
0001:0045f0f5  _zif_fgetcsv
0001:0045f4ad  _zif_realpath
0001:0045f5db  _php_next_meta_token
0001:0045fa5a  _zif_get_meta_tags
0001:004600f8  _zif_fnmatch
0001:00460250  _zif_sys_get_temp_dir
Module: U:\dev\php-5.3.8\ext\standard\filestat.o(filestat.o)
0001:0046093c  _zm_activate_filestat
0001:00460966  _zm_deactivate_filestat
0001:004609d6  _zif_disk_total_space
0001:00460a9d  _zif_disk_free_space
0001:00460b76  _zif_chgrp
0001:00460b9d  _zif_lchgrp
0001:00460bc4  _zif_chown
0001:00460bf5  _zif_lchown
0001:00460c3c  _zif_chmod
0001:00460e19  _zif_touch
0001:00461015  _php_clear_stat_cache
0001:004610c4  _zif_clearstatcache
0001:004611ff  _php_stat
0001:0046277e  _zif_fileperms
0001:004627dd  _zif_fileinode
0001:0046283c  _zif_filesize
0001:0046289b  _zif_fileowner
0001:004628fa  _zif_filegroup
0001:00462959  _zif_fileatime
0001:004629b8  _zif_filemtime
0001:00462a17  _zif_filectime
0001:00462a76  _zif_filetype
0001:00462ad5  _zif_is_writable
0001:00462b34  _zif_is_readable
0001:00462b93  _zif_is_executable
0001:00462bf2  _zif_is_file
0001:00462c51  _zif_is_dir
0001:00462cb0  _zif_is_link
0001:00462d0f  _zif_file_exists
0001:00462d6e  _php_if_lstat
0001:00462dcd  _php_if_stat
0001:00462e2c  _zif_realpath_cache_size
0001:00462e87  _zif_realpath_cache_get
Module: U:\dev\php-5.3.8\ext\standard\flock_compat.o(flock_compat.o)
0001:00463030  _php_flock
Module: U:\dev\php-5.3.8\ext\standard\formatted_print.o(formatted_print.o)
0001:00465003  _zif_user_sprintf
0001:0046504e  _zif_vsprintf
0001:0046509c  _zif_user_printf
0001:00465106  _zif_vprintf
0001:0046517c  _zif_fprintf
0001:0046527d  _zif_vfprintf
Module: U:\dev\php-5.3.8\ext\standard\fsock.o(fsock.o)
0001:0046571b  _zif_fsockopen
0001:00465742  _zif_pfsockopen
Module: U:\dev\php-5.3.8\ext\standard\head.o(head.o)
0001:004657a0  _zif_header
0001:0046581f  _zif_header_remove
0001:0046588c  _php_header
0001:00465a0f  _php_setcookie
0001:00465de9  _zif_setcookie
0001:00465f1e  _zif_setrawcookie
0001:00466057  _zif_headers_sent
0001:004661b5  _zif_headers_list
Module: U:\dev\php-5.3.8\ext\standard\html.o(html.o)
0001:00466540  _php_utf32_utf8
0001:004666a6  _php_unescape_html_entities
0001:00466d88  _php_escape_html_entities_ex
0001:004676a5  _php_escape_html_entities
0001:00467738  _register_html_constants
0001:00467855  _zif_htmlspecialchars
0001:00467875  _zif_htmlspecialchars_decode
0001:00467afd  _zif_html_entity_decode
0001:00467bba  _zif_htmlentities
0001:00467be3  _zif_get_html_translation_table
Module: U:\dev\php-5.3.8\ext\standard\image.o(image.o)
0001:0046b0d3  _zm_startup_imagetypes
0001:0046b473  _php_image_type_to_mime_type
0001:0046b491  _zif_image_type_to_mime_type
0001:0046b55f  _zif_image_type_to_extension
0001:0046b8ef  _php_getimagetype
0001:0046cad5  _php_sig_gif
0001:0046cae4  _php_sig_jpg
0001:0046cae7  _php_sig_png
0001:0046cade  _php_sig_swf
0001:0046cae1  _php_sig_swc
0001:0046cad8  _php_sig_psd
0001:0046cadc  _php_sig_bmp
0001:0046caf7  _php_sig_jpc
0001:0046caef  _php_sig_tif_ii
0001:0046caf3  _php_sig_tif_mm
0001:0046cb06  _php_sig_iff
0001:0046cb0a  _php_sig_ico
0001:0046cafa  _php_sig_jp2
0001:0046bc3a  _zif_getimagesize
0001:0046cb10  _php_tiff_bytes_per_format
Module: U:\dev\php-5.3.8\ext\standard\info.o(info.o)
0001:0046cd08  _php_info_print_style
0001:0046cd37  _php_info_html_esc_write
0001:0046d23e  _php_info_html_esc
0001:0046d4d7  _php_get_uname
0001:0046d669  _php_print_info_htmlhead
0001:0046d75c  _php_info_print_table_start
0001:0046d797  _php_info_print_table_end
0001:0046d7df  _php_info_print_box_start
0001:0046d83f  _php_info_print_box_end
0001:0046d8b5  _php_info_print_hr
0001:0046d91b  _php_info_print_table_colspan_header
0001:0046d9ac  _php_info_print_table_header
0001:0046db14  _php_info_print_table_row
0001:0046db73  _php_info_print_module
0001:0046dcac  _php_info_print_table_row_ex
0001:0046dda2  _register_phpinfo_constants
0001:0046e07f  _zif_phpversion
0001:0046e1df  _zif_phpcredits
0001:0046e288  _php_logo_guid
0001:0046f01d  _php_print_info
0001:0047038d  _zif_phpinfo
0001:0047041e  _zif_php_logo_guid
0001:0047046f  _zif_php_real_logo_guid
0001:004704bf  _zif_php_egg_logo_guid
0001:00470538  _zif_zend_logo_guid
0001:00470588  _zif_php_sapi_name
0001:004705fe  _zif_php_uname
0001:00470674  _zif_php_ini_scanned_files
0001:004706ad  _zif_php_ini_loaded_file
Module: U:\dev\php-5.3.8\ext\standard\iptc.o(iptc.o)
0001:0047085a  _zif_iptcembed
0001:00470d3b  _zif_iptcparse
Module: U:\dev\php-5.3.8\ext\standard\lcg.o(lcg.o)
0002:00021000  _lcg_globals_id
0001:00470feb  _php_combined_lcg
0001:00471163  _zm_startup_lcg
0001:00471191  _zif_lcg_value
Module: U:\dev\php-5.3.8\ext\standard\link.o(link.o)
0001:004711c5  _zif_readlink
0001:00471307  _zif_linkinfo
0001:004713e7  _zif_symlink
0001:00471703  _zif_link
Module: U:\dev\php-5.3.8\ext\standard\mail.o(mail.o)
0001:00471952  _zif_ezmlm_hash
0001:00471b41  _php_mail
0001:00471fbe  _zif_mail
0001:004724b8  _zm_info_mail
Module: U:\dev\php-5.3.8\ext\standard\math.o(math.o)
0001:00472508  __php_math_round
0001:00472a99  _zif_abs
0001:00472bc7  _zif_ceil
0001:00472d55  _zif_floor
0001:00472ee8  _zif_round
0001:00473046  _zif_sin
0001:0047308d  _zif_cos
0001:004730d4  _zif_tan
0001:0047311b  _zif_asin
0001:00473162  _zif_acos
0001:004731a9  _zif_atan
0001:004731f3  _zif_atan2
0001:00473248  _zif_sinh
0001:0047328f  _zif_cosh
0001:004732d6  _zif_tanh
0001:0047331d  _zif_asinh
0001:00473364  _zif_acosh
0001:004733ab  _zif_atanh
0001:004733f2  _zif_pi
0001:00473406  _zif_is_finite
0001:00473458  _zif_is_infinite
0001:004734ac  _zif_is_nan
0001:004734fb  _zif_pow
0001:00473668  _zif_exp
0001:004736af  _zif_expm1
0001:004736f6  _zif_log1p
0001:0047375d  _zif_log
0001:0047384d  _zif_log10
0001:00473894  _zif_sqrt
0001:004738ec  _zif_hypot
0001:00473941  _zif_deg2rad
0001:0047398c  _zif_rad2deg
0001:004739fe  __php_math_basetolong
0001:00473ad2  __php_math_basetozval
0001:00473c04  __php_math_longtobase
0001:00473c8e  __php_math_zvaltobase
0001:00473eb3  _zif_bindec
0001:00473fac  _zif_hexdec
0001:004740a5  _zif_octdec
0001:0047419e  _zif_decbin
0001:00474288  _zif_decoct
0001:00474372  _zif_dechex
0001:00474492  _zif_base_convert
0001:00474625  __php_math_number_format
0001:0047486a  _zif_number_format
0001:004749a4  _zif_fmod
Module: U:\dev\php-5.3.8\ext\standard\md5.o(md5.o)
0001:004753bf  _make_digest_ex
0001:00475408  _make_digest
0001:0047542a  _PHP_MD5Init
0001:0047545b  _PHP_MD5Update
0001:0047551f  _PHP_MD5Final
0001:00475673  _php_if_md5_file
0001:00475851  _php_if_md5
Module: U:\dev\php-5.3.8\ext\standard\metaphone.o(metaphone.o)
0001:004759a4  _zif_metaphone
0002:00002e60  __codes
Module: U:\dev\php-5.3.8\ext\standard\microtime.o(microtime.o)
0001:00476bb0  _zif_microtime
0001:00476bcc  _zif_gettimeofday
Module: U:\dev\php-5.3.8\ext\standard\pack.o(pack.o)
0002:00021010  _machine_little_endian
0001:00476dbf  _zif_pack
0001:0047810c  _zif_unpack
0001:00478e42  _zm_startup_pack
Module: U:\dev\php-5.3.8\ext\standard\pageinfo.o(pageinfo.o)
0001:00479030  _php_statpage
0001:004790bb  _php_getuid
0001:004790f8  _php_getgid
0001:00479135  _zif_getmyuid
0001:00479164  _zif_getmygid
0001:00479193  _zif_getmypid
0001:004791c2  _zif_getmyinode
0001:0047921a  _php_getlastmod
0001:00479244  _zif_getlastmod
Module: U:\dev\php-5.3.8\ext\standard\quot_print.o(quot_print.o)
0001:004792c6  _php_quot_print_decode
0001:004794e5  _php_quot_print_encode
0001:0047964c  _zif_quoted_printable_decode
0001:00479848  _zif_quoted_printable_encode
Module: U:\dev\php-5.3.8\ext\standard\rand.o(rand.o)
0001:00479ce0  _php_srand
0001:00479d04  _php_rand
0001:00479d92  _php_mt_srand
0001:00479ef5  _php_mt_rand
0001:0047a06b  _zif_srand
0001:0047a102  _zif_mt_srand
0001:0047a19c  _zif_rand
0001:0047a26a  _zif_mt_rand
0001:0047a3c7  _zif_getrandmax
0001:0047a400  _zif_mt_getrandmax
Module: U:\dev\php-5.3.8\ext\standard\soundex.o(soundex.o)
0001:0047a452  _zif_soundex
Module: U:\dev\php-5.3.8\ext\standard\string.o(string.o)
0001:0047aadb  _register_string_constants
0001:0047ad84  _localeconv_r
0001:0047adc4  _zm_startup_localeconv
0001:0047add8  _zm_shutdown_localeconv
0001:0047adfb  _zif_bin2hex
0001:0047aeb2  _zif_strspn
0001:0047aed9  _zif_strcspn
0001:0047b0ab  _zm_startup_nl_langinfo
0001:0047baa8  _zif_nl_langinfo
0001:0047bb72  _zif_strcoll
0001:0047bc9a  _php_trim
0001:0047c11d  _zif_trim
0001:0047c139  _zif_rtrim
0001:0047c155  _zif_ltrim
0001:0047c1bb  _zif_wordwrap
0001:0047c71f  _php_explode
0001:0047c93f  _php_explode_negative_limit
0001:0047cbd9  _zif_explode
0001:0047cd51  _php_implode
0001:0047d4e8  _zif_implode
0001:0047d7fa  _zif_strtok
0001:0047da89  _php_strtoupper
0001:0047dab1  _zif_strtoupper
0001:0047db21  _php_strtolower
0001:0047db49  _zif_strtolower
0001:0047dbb9  _php_basename
0001:0047dd1f  _zif_basename
0001:0047ddbb  _php_dirname
0001:0047ddc7  _zif_dirname
0001:0047de5a  _zif_pathinfo
0001:0047e23f  _php_stristr
0001:0047e311  _php_strspn
0001:0047e34c  _php_strcspn
0001:0047e390  _zif_stristr
0001:0047e537  _zif_strstr
0001:0047e753  _zif_strpos
0001:0047e90d  _zif_stripos
0001:0047ebf9  _zif_strrpos
0001:0047edd3  _zif_strripos
0001:0047f12a  _zif_strrchr
0001:0047f239  _zif_chunk_split
0001:0047f4b3  _zif_substr
0001:0047f6b3  _zif_substr_replace
0001:0048057b  _zif_quotemeta
0001:0048075c  _zif_ord
0001:004807a5  _zif_chr
0001:0048082e  _zif_ucfirst
0001:004808bd  _zif_lcfirst
0001:0048094c  _zif_ucwords
0001:00480a07  _php_strtr
0001:00480ab4  _zif_strtr
0001:004812a0  _zif_strrev
0001:0048132c  _zif_similar_text
0001:00481477  _php_stripslashes
0001:004815de  _zif_stripslashes
0001:0048164b  _php_stripcslashes
0001:0048190d  _zif_stripcslashes
0001:00481979  _php_addcslashes
0001:00481cfa  _zif_addcslashes
0001:00481dcf  _php_addslashes_ex
0001:00481f4d  _php_addslashes
0001:00481f84  _zif_addslashes
0001:00482032  _php_char_to_str_ex
0001:0048232b  _php_char_to_str
0001:00482ae7  _php_str_to_str_ex
0001:00483e7f  _php_str_to_str
0001:00483ecc  _zif_str_replace
0001:00483ee8  _zif_str_ireplace
0001:00483f04  _zif_hebrev
0001:00483f20  _zif_hebrevc
0001:00483f40  _zif_nl2br
0001:004841d2  _zif_setlocale
0001:00484688  _zif_parse_str
0001:0048479a  _php_tag_find
0001:004848ae  _php_strip_tags_ex
0001:004853c8  _php_strip_tags
0001:00485403  _zif_strip_tags
0001:00485549  _zif_str_getcsv
0001:00485681  _zif_str_repeat
0001:004857ec  _zif_count_chars
0001:004859a2  _zif_strnatcmp
0001:00485ac9  _zif_localeconv
0001:00485ea5  _zif_strnatcasecmp
0001:00485f77  _zif_substr_count
0001:00486287  _zif_str_pad
0001:004864ec  _zif_sscanf
0001:004865aa  _zif_str_rot13
0001:00486629  _zif_str_shuffle
0001:004866fd  _zif_str_word_count
0001:00486b65  _zif_str_split
0001:00486cbf  _zif_strpbrk
0001:00486deb  _zif_substr_compare
Module: U:\dev\php-5.3.8\ext\standard\scanf.o(scanf.o)
0001:004870e9  _ValidateFormat
0001:00487709  _php_sscanf_internal
Module: U:\dev\php-5.3.8\ext\standard\syslog.o(syslog.o)
0001:0048b1e9  _zm_startup_syslog
0001:0048b7da  _zm_activate_syslog
0001:0048b841  _zm_shutdown_syslog
0001:0048b888  _zif_define_syslog_variables
0001:0048b8da  _zif_openlog
0001:0048b99d  _zif_closelog
0001:0048ba17  _zif_syslog
Module: U:\dev\php-5.3.8\ext\standard\type.o(type.o)
0001:0048bb96  _zif_gettype
0001:0048bdad  _zif_settype
0001:0048bfc4  _zif_intval
0001:0048c0a3  _zif_floatval
0001:0048c120  _zif_strval
0001:0048c1e2  _zif_is_null
0001:0048c209  _zif_is_resource
0001:0048c230  _zif_is_bool
0001:0048c257  _zif_is_long
0001:0048c27e  _zif_is_float
0001:0048c2a5  _zif_is_string
0001:0048c2cc  _zif_is_array
0001:0048c2f3  _zif_is_object
0001:0048c31a  _zif_is_numeric
0001:0048c53c  _zif_is_scalar
0001:0048c5a6  _zif_is_callable
Module: U:\dev\php-5.3.8\ext\standard\uniqid.o(uniqid.o)
0001:0048c6ff  _zif_uniqid
Module: U:\dev\php-5.3.8\ext\standard\url.o(url.o)
0001:0048c88f  _php_url_free
0001:0048c90e  _php_replace_controlchars_ex
0001:0048c93e  _php_replace_controlchars
0001:0048c96f  _php_url_parse_ex
0001:0048d1ae  _php_url_parse
0001:0048d234  _zif_parse_url
0001:0048d548  _php_url_encode
0001:0048d603  _zif_urlencode
0001:0048d665  _php_url_decode
0001:0048d729  _zif_urldecode
0001:0048d794  _php_raw_url_encode
0001:0048d86a  _zif_rawurlencode
0001:0048d8cc  _php_raw_url_decode
0001:0048d983  _zif_rawurldecode
0001:0048d9f8  _zif_get_headers
Module: U:\dev\php-5.3.8\ext\standard\var.o(var.o)
0001:00492805  _php_var_dump
0001:00492e6a  _zif_var_dump
0001:00492ff3  _php_debug_zval_dump
0001:00493695  _zif_debug_zval_dump
0001:0049373b  _php_var_export_ex
0001:00495340  _php_var_export
0001:004953bb  _zif_var_export
0001:00495485  _php_var_serialize
0001:004954b9  _zif_serialize
0001:004955a8  _zif_unserialize
0001:0049569c  _zif_memory_get_usage
0001:004956ff  _zif_memory_get_peak_usage
Module: U:\dev\php-5.3.8\ext\standard\versioning.o(versioning.o)
0001:00495855  _php_canonicalize_version
0001:00495a44  _php_version_compare
0001:00495d31  _zif_version_compare
Module: U:\dev\php-5.3.8\ext\standard\assert.o(assert.o)
0002:00021018  _assert_globals_id
0001:0049634b  _zm_startup_assert
0001:00496476  _zm_shutdown_assert
0001:004964b6  _zm_deactivate_assert
0001:004964f9  _zm_info_assert
0001:00496582  _zif_assert
0001:00496b0c  _zif_assert_options
Module: U:\dev\php-5.3.8\ext\standard\strnatcmp.o(strnatcmp.o)
0001:00497210  _strnatcmp_ex
Module: U:\dev\php-5.3.8\ext\standard\levenshtein.o(levenshtein.o)
0001:00497845  _zif_levenshtein
Module: U:\dev\php-5.3.8\ext\standard\incomplete_class.o(incomplete_class.o)
0001:00497a98  _php_create_incomplete_class
0001:00497c06  _php_lookup_class_name
0001:00497f11  _php_store_class_name
Module: U:\dev\php-5.3.8\ext\standard\url_scanner_ex.o(url_scanner_ex.o)
0001:0049a97d  _php_url_scanner_adapt_single_url
0001:0049b023  _php_url_scanner_add_var
0001:0049b96c  _php_url_scanner_reset_vars
0001:0049b996  _zm_startup_url_scanner_ex
0001:0049b9f8  _zm_shutdown_url_scanner_ex
0001:0049ba14  _zm_activate_url_scanner_ex
0001:0049ba34  _zm_deactivate_url_scanner_ex
Module: U:\dev\php-5.3.8\ext\standard\ftp_fopen_wrapper.o(ftp_fopen_wrapper.o)
0001:0049e2bc  _php_stream_ftp_opendir
0001:0049efb5  _php_stream_url_wrap_ftp
0002:00002f00  _php_stream_ftp_wrapper
Module: U:\dev\php-5.3.8\ext\standard\http_fopen_wrapper.o(http_fopen_wrapper.o)
0001:004a03d4  _php_stream_url_wrap_http_ex
0001:004a3eae  _php_stream_url_wrap_http
0002:00002f80  _php_stream_http_wrapper
Module: U:\dev\php-5.3.8\ext\standard\php_fopen_wrapper.o(php_fopen_wrapper.o)
0001:004a43e3  _php_stream_url_wrap_php
0002:00003000  _php_stream_input_ops
0002:00002fd0  _php_stream_output_ops
0002:00003030  _php_stream_php_wrapper
Module: U:\dev\php-5.3.8\ext\standard\credits.o(credits.o)
0001:004a6586  _php_print_credits
Module: U:\dev\php-5.3.8\ext\standard\css.o(css.o)
0001:004a7831  _php_info_print_css
Module: U:\dev\php-5.3.8\ext\standard\var_unserializer.o(var_unserializer.o)
0001:004a7abc  _var_push_dtor
0001:004a7b64  _var_replace
0001:004a7bae  _var_destroy
0001:004a7dc2  _php_var_unserialize
Module: U:\dev\php-5.3.8\ext\standard\ftok.o(ftok.o)
0001:004a9fb8  _zif_ftok
Module: U:\dev\php-5.3.8\ext\standard\sha1.o(sha1.o)
0001:004ab63c  _make_sha1_digest
0001:004ab65e  _PHP_SHA1Init
0001:004ab696  _PHP_SHA1Update
0001:004ab752  _PHP_SHA1Final
0001:004ab825  _zif_sha1_file
0001:004aba0d  _zif_sha1
Module: U:\dev\php-5.3.8\ext\standard\user_filters.o(user_filters.o)
0001:004abb50  _zif_user_filter_nop
0001:004ac1ae  _userfilter_filter
0001:004ac938  _zm_startup_user_filters
0001:004acc84  _zm_deactivate_user_filters
0001:004accee  _zif_stream_bucket_make_writeable
0001:004ace7d  _zif_stream_bucket_prepend
0001:004ace9d  _zif_stream_bucket_append
0001:004acec3  _zif_stream_bucket_new
0001:004ad102  _zif_stream_get_filters
0001:004ad217  _zif_stream_filter_register
Module: U:\dev\php-5.3.8\ext\standard\uuencode.o(uuencode.o)
0001:004ad560  _php_uuencode
0001:004ad84f  _php_uudecode
0001:004ada38  _zif_convert_uuencode
0001:004adae4  _zif_convert_uudecode
Module: U:\dev\php-5.3.8\ext\standard\filters.o(filters.o)
0001:004b0c55  _zm_startup_standard_filters
0001:004b0ca2  _zm_shutdown_standard_filters
0002:000030d0  _consumed_filter_factory
Module: U:\dev\php-5.3.8\ext\standard\proc_open.o(proc_open.o)
0001:004b13df  _zm_startup_proc_open
0001:004b1415  _zif_proc_terminate
0001:004b14c9  _zif_proc_close
0001:004b15b1  _zif_proc_get_status
0001:004b1adb  _zif_proc_open
Module: U:\dev\php-5.3.8\ext\standard\streamsfuncs.o(streamsfuncs.o)
0001:004b3947  _zif_stream_socket_pair
0001:004b3ae0  _zif_stream_socket_client
0001:004b3ee6  _zif_stream_socket_server
0001:004b41d9  _zif_stream_socket_accept
0001:004b4403  _zif_stream_socket_get_name
0001:004b4526  _zif_stream_socket_sendto
0001:004b46d8  _zif_stream_socket_recvfrom
0001:004b4915  _zif_stream_get_contents
0001:004b4b66  _zif_stream_copy_to_stream
0001:004b4d59  _zif_stream_get_meta_data
0001:004b5010  _zif_stream_get_transports
0001:004b50ea  _zif_stream_get_wrappers
0001:004b5282  _zif_stream_select
0001:004b583c  _zif_stream_context_get_options
0001:004b5933  _zif_stream_context_set_option
0001:004b5a72  _zif_stream_context_set_params
0001:004b5b08  _zif_stream_context_get_params
0001:004b5c73  _zif_stream_context_get_default
0001:004b5d22  _zif_stream_context_set_default
0001:004b5dbf  _zif_stream_context_create
0001:004b5e4e  _zif_stream_filter_prepend
0001:004b5e6e  _zif_stream_filter_append
0001:004b5f12  _zif_stream_filter_remove
0001:004b608d  _zif_stream_get_line
0001:004b61cd  _zif_stream_set_blocking
0001:004b62a9  _zif_stream_set_timeout
0001:004b63c7  _zif_stream_set_write_buffer
0001:004b64c6  _zif_stream_set_read_buffer
0001:004b6606  _zif_stream_socket_enable_crypto
0001:004b67bd  _zif_stream_resolve_include_path
0001:004b6848  _zif_stream_is_local
0001:004b69ba  _zif_stream_supports_lock
0001:004b6a84  _zif_stream_socket_shutdown
Module: U:\dev\php-5.3.8\ext\standard\http.o(http.o)
0001:004b6b96  _php_url_encode_hash_ex
0001:004b77fc  _zif_http_build_query
Module: U:\dev\php-5.3.8\ext\tokenizer\tokenizer.o(tokenizer.o)
0001:004b79c2  _zif_token_name
0001:004b7a2f  _zif_token_get_all
0001:004b7d6f  _zm_info_tokenizer
0001:004b7d9c  _zm_startup_tokenizer
0001:004b7de0  _tokenizer_functions
0002:00003200  _tokenizer_module_entry
Module: U:\dev\php-5.3.8\ext\tokenizer\tokenizer_data.o(tokenizer_data.o)
0001:004b8430  _tokenizer_register_constants
0001:004b999d  _get_token_type_name
Module: U:\dev\php-5.3.8\ext\xml\xml.o(xml.o)
0002:00021028  _xml_globals_id
0001:004b9c20  _zif_xml_parser_get_option
0001:004b9df4  _zif_xml_parser_free
0001:004b9ebf  _zif_xml_get_current_byte_index
0001:004b9f55  _zif_xml_get_current_column_number
0001:004b9feb  _zif_xml_get_current_line_number
0001:004ba083  _zif_xml_error_string
0001:004ba0f1  _zif_xml_get_error_code
0001:004ba18c  _zif_xml_parse
0001:004ba26f  _zif_xml_parse_into_struct
0001:004bc947  __xml_defaultHandler
0001:004bd2cc  __xml_endElementHandler
0001:004bce48  __xml_startElementHandler
0001:004bca2b  __xml_characterDataHandler
0001:004ba50d  _zm_info_xml
0001:004ba83d  _zm_startup_xml
0001:004bb0db  _zif_xml_parser_create_ns
0001:004bb0f7  _zif_xml_parser_create
0001:004bb49b  _zif_xml_set_object
0001:004bb661  _zif_xml_set_end_namespace_decl_handler
0001:004bc6ad  __xml_endNamespaceDeclHandler
0001:004bb717  _zif_xml_set_default_handler
0001:004bb7cd  _zif_xml_set_character_data_handler
0001:004bb887  _zif_xml_set_element_handler
0001:004bb957  _zif_xml_set_start_namespace_decl_handler
0001:004bc709  __xml_startNamespaceDeclHandler
0001:004bba0d  _zif_xml_set_external_entity_ref_handler
0001:004bc775  __xml_externalEntityRefHandler
0001:004bbac3  _zif_xml_set_notation_decl_handler
0001:004bc817  __xml_notationDeclHandler
0001:004bbb79  _zif_xml_set_unparsed_entity_decl_handler
0001:004bc8a3  __xml_unparsedEntityDeclHandler
0001:004bbc2f  _zif_xml_set_processing_instruction_handler
0001:004bc9a4  __xml_processingInstructionHandler
0001:004bbd0d  _zif_xml_parser_set_option
0001:004bc0b8  _xml_utf8_encode
0001:004bc206  _zif_utf8_encode
0001:004bc280  _xml_utf8_decode
0001:004bc5af  _zif_utf8_decode
0001:004bd4e3  __xml_zval_strdup
0001:004bd790  _xml_functions
0002:000032c0  _xml_encodings
0002:00003260  _xml_module_entry
Module: U:\dev\php-5.3.8\ext\xml\compat.o(compat.o)
0001:004beb75  _php_XML_ParserCreate_MM
0001:004bec32  _php_XML_ParserCreateNS
0001:004bec5e  _php_XML_ParserCreate
0001:004bec81  _php_XML_SetUserData
0001:004bec8f  _XML_GetUserData
0001:004bec9a  _php_XML_SetElementHandler
0001:004becae  _php_XML_SetCharacterDataHandler
0001:004becbc  _php_XML_SetProcessingInstructionHandler
0001:004becca  _php_XML_SetCommentHandler
0001:004becd8  _php_XML_SetDefaultHandler
0001:004bece6  _php_XML_SetUnparsedEntityDeclHandler
0001:004becf4  _php_XML_SetNotationDeclHandler
0001:004bed02  _php_XML_SetExternalEntityRefHandler
0001:004bed10  _php_XML_SetStartNamespaceDeclHandler
0001:004bed1e  _php_XML_SetEndNamespaceDeclHandler
0001:004bed2c  _php_XML_Parse
0001:004bed77  _php_XML_GetErrorCode
0001:004bed8d  _php_XML_ErrorString
0001:004beda8  _php_XML_GetCurrentLineNumber
0001:004bedb9  _php_XML_GetCurrentColumnNumber
0001:004bedca  _php_XML_GetCurrentByteIndex
0001:004bede1  _php_XML_GetCurrentByteCount
0001:004bedfc  _php_XML_ExpatVersion
0001:004bee06  _php_XML_ParserFree
Module: U:\dev\php-5.3.8\ext\xmlreader\php_xmlreader.o(php_xmlreader.o)
0002:00021038  _xmlreader_class_entry
0001:004bfaa0  _xmlreader_objects_clone
0001:004bfab7  _zm_info_xmlreader
0001:004bfae4  _zm_shutdown_xmlreader
0001:004bfb9a  _zim_xmlreader_expand
0001:004bfde6  _zim_xmlreader_XML
0001:004c0053  _zim_xmlreader_close
0001:004c009f  _zim_xmlreader_setParserProperty
0001:004c01c3  _zim_xmlreader_setSchema
0001:004c02cc  _zim_xmlreader_next
0001:004c03f8  _zim_xmlreader_read
0001:004c04b1  _zim_xmlreader_moveToAttributeNs
0001:004c0598  _zim_xmlreader_moveToAttributeNo
0001:004c0631  _zim_xmlreader_moveToAttribute
0001:004c06f3  _zim_xmlreader_getParserProperty
0001:004c0794  _zim_xmlreader_getAttributeNs
0001:004c08bb  _zim_xmlreader_getAttributeNo
0001:004c097b  _xmlreader_objects_new
0001:004c0a35  _xmlreader_objects_free_storage
0001:004c0ab3  _zim_xmlreader_moveToNextAttribute
0001:004c0ad2  _zim_xmlreader_moveToFirstAttribute
0001:004c0af4  _zim_xmlreader_moveToElement
0001:004c0b16  _zim_xmlreader_isValid
0001:004c0bc7  _zim_xmlreader_readString
0001:004c0be3  _zim_xmlreader_readOuterXml
0001:004c0bff  _zim_xmlreader_readInnerXml
0001:004c0d26  _zim_xmlreader_lookupNamespace
0001:004c0d48  _zim_xmlreader_getAttribute
0001:004c0f26  _zm_startup_xmlreader
0001:004c1663  _xmlreader_read_property
0001:004c18bb  _xmlreader_write_property
0001:004c1573  _xmlreader_get_property_ptr_ptr
0001:004c19d0  __xmlreader_get_valid_file_path
0001:004c1abf  _zim_xmlreader_open
0001:004c1e29  _zim_xmlreader_setRelaxNGSchemaSource
0001:004c1e56  _zim_xmlreader_setRelaxNGSchema
0002:00003370  _xmlreader_module_entry
Module: U:\dev\php-5.3.8\ext\xmlrpc\xmlrpc-epi-php.o(xmlrpc-epi-php.o)
0001:004c285a  _zif_xmlrpc_is_fault
0001:004c31f8  _zif_xmlrpc_server_register_method
0001:004c32f8  _zif_xmlrpc_server_destroy
0001:004c3379  _zif_xmlrpc_server_create
0001:004c34ec  _zm_info_xmlrpc
0001:004c3598  _zm_startup_xmlrpc
0001:004c3a4b  _zif_xmlrpc_server_register_introspection_callback
0001:004c3b1c  _xmlrpc_type_as_str
0001:004c3b3c  _xmlrpc_str_as_type
0001:004c3b86  _xmlrpc_str_as_vector_type
0001:004c3bea  _set_zval_xmlrpc_type
0001:004c3e56  _zif_xmlrpc_set_type
0001:004c4167  _zif_xmlrpc_parse_method_descriptions
0001:004c4297  _decode_request_worker
0001:004c4382  _zif_xmlrpc_decode
0001:004c4452  _zif_xmlrpc_decode_request
0001:004c452c  _get_zval_xmlrpc_type
0001:004c4693  _zif_xmlrpc_get_type
0001:004c4b79  _zif_xmlrpc_server_add_introspection_data
0001:004c4c1f  _zif_xmlrpc_server_call_method
0001:004c50c2  _zif_xmlrpc_encode
0001:004c5171  _zif_xmlrpc_encode_request
0001:004c5430  _xmlrpc_functions
0002:000033d0  _xmlrpc_module_entry
Module: U:\dev\php-5.3.8\ext\xmlwriter\php_xmlwriter.o(php_xmlwriter.o)
0002:00003430  _xmlwriter_module_entry
Module: U:\dev\php-5.3.8\ext\zip\php_zip.o(php_zip.o)
0001:004cefe5  _php_zip_glob
0001:004cf376  _php_zip_pcre
0002:00003490  _zip_module_entry
Module: U:\dev\php-5.3.8\ext\zip\zip_stream.o(zip_stream.o)
0001:004d12cb  _php_stream_zip_opener
0001:004d14c4  _php_stream_zip_open
0002:000034f0  _php_stream_zipio_ops
0002:00003520  _php_stream_zip_wrapper
Module: U:\dev\php-5.3.8\ext\zip\lib\zip_add.o(zip_add.o)
0001:004d1600  _zip_add
Module: U:\dev\php-5.3.8\ext\zip\lib\zip_error.o(zip_error.o)
0001:004d1660  __zip_error_clear
0001:004d1675  __zip_error_copy
0001:004d168a  __zip_error_fini
0001:004d16ac  __zip_error_get
0001:004d16f0  __zip_error_init
0001:004d170c  __zip_error_set
Module: U:\dev\php-5.3.8\ext\zip\lib\zip_fclose.o(zip_fclose.o)
0001:004d1730  _zip_fclose
Module: U:\dev\php-5.3.8\ext\zip\lib\zip_fread.o(zip_fread.o)
0001:004d17e0  _zip_fread
Module: U:\dev\php-5.3.8\ext\zip\lib\zip_open.o(zip_open.o)
0001:004d1d27  _zip_open
Module: U:\dev\php-5.3.8\ext\zip\lib\zip_source_filep.o(zip_source_filep.o)
0001:004d2907  __zip_source_file_or_p
0001:004d2a34  _zip_source_filep
Module: U:\dev\php-5.3.8\ext\zip\lib\zip_strerror.o(zip_strerror.o)
0001:004d2ac0  _zip_strerror
Module: U:\dev\php-5.3.8\ext\zip\lib\zip_close.o(zip_close.o)
0001:004d330d  _zip_close
Module: U:\dev\php-5.3.8\ext\zip\lib\zip_error_get.o(zip_error_get.o)
0001:004d3fd0  _zip_error_get
Module: U:\dev\php-5.3.8\ext\zip\lib\zip_file_error_get.o(zip_file_error_get.o)
0001:004d3ff0  _zip_file_error_get
Module: U:\dev\php-5.3.8\ext\zip\lib\zip_free.o(zip_free.o)
0001:004d4010  __zip_free
Module: U:\dev\php-5.3.8\ext\zip\lib\zip_rename.o(zip_rename.o)
0001:004d4100  _zip_rename
Module: U:\dev\php-5.3.8\ext\zip\lib\zip_source_free.o(zip_source_free.o)
0001:004d41d0  _zip_source_free
Module: U:\dev\php-5.3.8\ext\zip\lib\zip_unchange_all.o(zip_unchange_all.o)
0001:004d4220  _zip_unchange_all
Module: U:\dev\php-5.3.8\ext\zip\lib\zip_delete.o(zip_delete.o)
0001:004d4270  _zip_delete
Module: U:\dev\php-5.3.8\ext\zip\lib\zip_error_get_sys_type.o(zip_error_get_sys_type.o)
0001:004d42f0  _zip_error_get_sys_type
Module: U:\dev\php-5.3.8\ext\zip\lib\zip_file_get_offset.o(zip_file_get_offset.o)
0001:004d4310  __zip_file_get_offset
Module: U:\dev\php-5.3.8\ext\zip\lib\zip_get_name.o(zip_get_name.o)
0001:004d43e0  __zip_get_name
0001:004d4472  _zip_get_name
Module: U:\dev\php-5.3.8\ext\zip\lib\zip_replace.o(zip_replace.o)
0001:004d44a0  __zip_replace
0001:004d452d  _zip_replace
Module: U:\dev\php-5.3.8\ext\zip\lib\zip_source_function.o(zip_source_function.o)
0001:004d45a0  _zip_source_function
Module: U:\dev\php-5.3.8\ext\zip\lib\zip_unchange.o(zip_unchange.o)
0001:004d4600  __zip_unchange
0001:004d4710  _zip_unchange
Module: U:\dev\php-5.3.8\ext\zip\lib\zip_dirent.o(zip_dirent.o)
0001:004d4907  __zip_cdir_grow
0001:004d4989  __zip_cdir_new
0001:004d4a2a  __zip_dirent_finalize
0001:004d4a70  __zip_cdir_free
0001:004d4ace  __zip_dirent_init
0001:004d4b4a  __zip_dirent_torrent_normalize
0001:004d4c3c  __zip_dirent_write
0001:004d4e62  __zip_cdir_write
0001:004d4f88  __zip_read2
0001:004d4fa5  __zip_read4
0001:004d4fd4  __zip_dirent_read
Module: U:\dev\php-5.3.8\ext\zip\lib\zip_error_strerror.o(zip_error_strerror.o)
0001:004d54ac  __zip_error_strerror
Module: U:\dev\php-5.3.8\ext\zip\lib\zip_filerange_crc.o(zip_filerange_crc.o)
0001:004d5600  __zip_filerange_crc
Module: U:\dev\php-5.3.8\ext\zip\lib\zip_file_strerror.o(zip_file_strerror.o)
0001:004d5730  _zip_file_strerror
Module: U:\dev\php-5.3.8\ext\zip\lib\zip_get_num_files.o(zip_get_num_files.o)
0001:004d5740  _zip_get_num_files
Module: U:\dev\php-5.3.8\ext\zip\lib\zip_get_archive_flag.o(zip_get_archive_flag.o)
0001:004d5760  _zip_get_archive_flag
Module: U:\dev\php-5.3.8\ext\zip\lib\zip_set_archive_flag.o(zip_set_archive_flag.o)
0001:004d5790  _zip_set_archive_flag
Module: U:\dev\php-5.3.8\ext\zip\lib\zip_set_name.o(zip_set_name.o)
0001:004d57b0  __zip_set_name
Module: U:\dev\php-5.3.8\ext\zip\lib\zip_source_zip.o(zip_source_zip.o)
0001:004d5afa  _zip_source_zip
Module: U:\dev\php-5.3.8\ext\zip\lib\zip_unchange_data.o(zip_unchange_data.o)
0001:004d5d50  __zip_unchange_data
Module: U:\dev\php-5.3.8\ext\zip\lib\zip_entry_free.o(zip_entry_free.o)
0001:004d5db0  __zip_entry_free
Module: U:\dev\php-5.3.8\ext\zip\lib\zip_error_to_str.o(zip_error_to_str.o)
0001:004d5e1c  _zip_error_to_str
Module: U:\dev\php-5.3.8\ext\zip\lib\zip_fopen.o(zip_fopen.o)
0001:004d5ed0  _zip_fopen
Module: U:\dev\php-5.3.8\ext\zip\lib\zip_name_locate.o(zip_name_locate.o)
0001:004d5f20  __zip_name_locate
0001:004d6054  _zip_name_locate
Module: U:\dev\php-5.3.8\ext\zip\lib\zip_source_buffer.o(zip_source_buffer.o)
0001:004d617b  _zip_source_buffer
Module: U:\dev\php-5.3.8\ext\zip\lib\zip_stat.o(zip_stat.o)
0001:004d6260  _zip_stat
Module: U:\dev\php-5.3.8\ext\zip\lib\zip_entry_new.o(zip_entry_new.o)
0001:004d62b0  __zip_entry_new
Module: U:\dev\php-5.3.8\ext\zip\lib\zip_err_str.o(zip_err_str.o)
0001:004d65a0  __zip_err_str
0001:004d6600  __zip_nerr_str
0001:004d6610  __zip_err_type
Module: U:\dev\php-5.3.8\ext\zip\lib\zip_fopen_index.o(zip_fopen_index.o)
0001:004d6670  __zip_file_fillbuf
0001:004d6780  _zip_fopen_index
Module: U:\dev\php-5.3.8\ext\zip\lib\zip_get_archive_comment.o(zip_get_archive_comment.o)
0001:004d6b30  _zip_get_archive_comment
Module: U:\dev\php-5.3.8\ext\zip\lib\zip_get_file_comment.o(zip_get_file_comment.o)
0001:004d6b80  _zip_get_file_comment
Module: U:\dev\php-5.3.8\ext\zip\lib\zip_new.o(zip_new.o)
0001:004d6c20  __zip_new
Module: U:\dev\php-5.3.8\ext\zip\lib\zip_source_file.o(zip_source_file.o)
0001:004d6cd0  _zip_source_file
Module: U:\dev\php-5.3.8\ext\zip\lib\zip_stat_index.o(zip_stat_index.o)
0001:004d6d60  _zip_stat_index
Module: U:\dev\php-5.3.8\ext\zip\lib\zip_set_archive_comment.o(zip_set_archive_comment.o)
0001:004d6ec0  _zip_set_archive_comment
Module: U:\dev\php-5.3.8\ext\zip\lib\zip_set_file_comment.o(zip_set_file_comment.o)
0001:004d6f50  _zip_set_file_comment
Module: U:\dev\php-5.3.8\ext\zip\lib\zip_unchange_archive.o(zip_unchange_archive.o)
0001:004d7010  _zip_unchange_archive
Module: U:\dev\php-5.3.8\ext\zip\lib\zip_memdup.o(zip_memdup.o)
0001:004d7050  __zip_memdup
Module: U:\dev\php-5.3.8\ext\zip\lib\zip_stat_init.o(zip_stat_init.o)
0001:004d70b0  _zip_stat_init
Module: U:\dev\php-5.3.8\ext\zip\lib\zip_add_dir.o(zip_add_dir.o)
0001:004d7100  _zip_add_dir
Module: U:\dev\php-5.3.8\ext\zip\lib\zip_error_clear.o(zip_error_clear.o)
0001:004d7240  _zip_error_clear
Module: U:\dev\php-5.3.8\ext\zip\lib\zip_file_error_clear.o(zip_file_error_clear.o)
0001:004d7250  _zip_file_error_clear
Module: U:\dev\php-5.3.8\ext\mysqlnd\mysqlnd.o(mysqlnd.o)
0001:004d9c65  _php_mysqlnd_conn_list_fields_pub
0001:004da75e  _php_mysqlnd_conn_list_method_pub
0001:004dc6df  _mysqlnd_library_end
0001:004dc710  _mysqlnd_stream_array_check_for_readiness
0001:004dc8ba  __mysqlnd_poll
0001:004dcb06  _mysqlnd_old_escape_string
0001:004dcb73  _mysqlnd_get_client_info
0001:004dcb7d  _mysqlnd_get_client_version
0001:004dcbe1  _mysqlnd_field_type_name
0001:004dccbe  __mysqlnd_init
0001:004dcd74  _mysqlnd_connect
0001:004dce29  _mysqlnd_library_init
0001:004dce66  _mysqlnd_conn_get_methods
0001:004dce70  _mysqlnd_conn_set_methods
0001:004dce7d  _mysqlnd_plugin_register
0001:004dce90  _mysqlnd_plugin_count
0001:004dce9a  __mysqlnd_plugin_get_plugin_connection_data
0001:004dcebc  _mysqlnd_old_passwd
0001:004dcec0  _mysqlnd_server_gone
0001:004dcec4  _mysqlnd_out_of_sync
0001:004dcec8  _mysqlnd_out_of_memory
0002:0001b870  _mysqlnd_global_stats
Module: U:\dev\php-5.3.8\ext\mysqlnd\mysqlnd_charset.o(mysqlnd_charset.o)
0001:004dd47b  _mysqlnd_find_charset_nr
0001:004de1d0  _mysqlnd_charsets
0001:004dd49d  _mysqlnd_find_charset_name
0001:004dd4d4  _mysqlnd_cset_escape_quotes
0001:004dd59c  _mysqlnd_cset_escape_slashes
Module: U:\dev\php-5.3.8\ext\mysqlnd\mysqlnd_wireprotocol.o(mysqlnd_wireprotocol.o)
0001:004dfaa7  _php_mysqlnd_cmd_write
0001:004e29cf  _php_mysqlnd_net_field_length
0001:004e34ca  _php_mysqlnd_net_field_length_ll
0001:004e4400  _php_mysqlnd_net_store_length
0001:004e446b  _php_mysqlnd_scramble
0001:004e470d  _php_mysqlnd_rowp_read_binary_protocol
0001:004e5097  _php_mysqlnd_rowp_read_text_protocol
0001:004e5bed  _mysqlnd_protocol_init
0001:004e5c46  _mysqlnd_protocol_free
0001:004e5c6d  __mysqlnd_plugin_get_plugin_protocol_data
0001:004e5ca3  _mysqlnd_protocol_get_methods
0001:004e5cb0  _mysqlnd_empty_string
0001:004e5cc0  _mysqlnd_read_header_name
0001:004e5ce0  _mysqlnd_read_body_name
0001:004e5e30  _mysqlnd_command_to_text
Module: U:\dev\php-5.3.8\ext\mysqlnd\mysqlnd_loaddata.o(mysqlnd_loaddata.o)
0001:004e61a1  _mysqlnd_local_infile_default
0001:004e61c5  _mysqlnd_set_local_infile_handler
0001:004e62af  _mysqlnd_handle_local_infile
Module: U:\dev\php-5.3.8\ext\mysqlnd\mysqlnd_net.o(mysqlnd_net.o)
0001:004e6932  _php_mysqlnd_net_consume_uneaten_data_pub
0001:004e75ec  _php_mysqlnd_net_send_pub
0001:004e7d1c  _mysqlnd_net_init
0001:004e7dad  _mysqlnd_net_free
0001:004e7e52  __mysqlnd_plugin_get_plugin_net_data
0001:004e7e8b  _mysqlnd_net_get_methods
Module: U:\dev\php-5.3.8\ext\mysqlnd\mysqlnd_statistics.o(mysqlnd_statistics.o)
0001:004e7ea5  _mysqlnd_fill_stats_hash
0001:004e7f6d  __mysqlnd_get_client_stats
0001:004e8ed0  _mysqlnd_stats_values_names
0001:004e7fc4  _mysqlnd_stats_init
0001:004e802d  _mysqlnd_stats_end
0001:004e8064  _mysqlnd_stats_set_trigger
0001:004e80a5  _mysqlnd_stats_reset_triggers
Module: U:\dev\php-5.3.8\ext\mysqlnd\mysqlnd_result.o(mysqlnd_result.o)
0001:004eb604  _php_mysqlnd_res_store_result_fetch_data_pub
0001:004ec4f6  _mysqlnd_query_read_result_set_header
0001:004ed1c6  __mysqlnd_fetch_lengths
0001:004ed1dd  _mysqlnd_result_init
0001:004ed242  __mysqlnd_plugin_get_plugin_result_data
0001:004ed27b  _mysqlnd_result_get_methods
Module: U:\dev\php-5.3.8\ext\mysqlnd\mysqlnd_result_meta.o(mysqlnd_result_meta.o)
0001:004eda62  _mysqlnd_result_meta_init
0001:004edb21  _mysqlnd_result_metadata_get_methods
0001:004edb2b  __mysqlnd_plugin_get_plugin_result_metadata_data
Module: U:\dev\php-5.3.8\ext\mysqlnd\mysqlnd_debug.o(mysqlnd_debug.o)
0001:004f0029  __mysqlnd_efree
0001:004f01af  __mysqlnd_erealloc
0001:004f038e  __mysqlnd_emalloc
0001:004f054b  __mysqlnd_malloc
0001:004f0715  __mysqlnd_pemalloc
0001:004f0992  __mysqlnd_free
0001:004f0b18  __mysqlnd_pefree
0001:004f0d33  __mysqlnd_realloc
0001:004f0f1e  __mysqlnd_perealloc
0001:004f11e3  __mysqlnd_calloc
0001:004f13a9  __mysqlnd_ecalloc
0001:004f15c3  __mysqlnd_pecalloc
0001:004f183d  __mysqlnd_pestrndup
0001:004f1a01  __mysqlnd_pestrdup
0001:004f1c5f  _mysqlnd_debug_init
0001:004f1d18  __mysqlnd_debug
0001:004f1db4  _mysqlnd_get_backtrace
0002:00003890  _mysqlnd_mysqlnd_debug_methods
0002:00003850  _mysqlnd_debug_std_no_trace_funcs
0002:000038b0  _mysqlnd_allocator
Module: U:\dev\php-5.3.8\ext\mysqlnd\mysqlnd_block_alloc.o(mysqlnd_block_alloc.o)
0001:004f225a  _mysqlnd_mempool_create
0001:004f22db  _mysqlnd_mempool_destroy
Module: U:\dev\php-5.3.8\ext\mysqlnd\php_mysqlnd.o(php_mysqlnd.o)
0002:00021048  _mysqlnd_globals_id
0001:004f24d0  _mysqlnd_minfo_print_hash
0001:004f263b  _zm_info_mysqlnd
0002:000038f0  _mysqlnd_module_entry
Module: U:\dev\php-5.3.8\ext\mysqlnd\mysqlnd_ps.o(mysqlnd_ps.o)
0001:004f30f5  _php_mysqlnd_stmt_free_parameter_bind_pub
0001:004f311f  _php_mysqlnd_stmt_free_result_bind_pub
0001:004f52e1  _mysqlnd_fetch_stmt_row_cursor
0001:004f6a3e  _mysqlnd_fetch_stmt_row_buffered
0001:004f7495  __mysqlnd_stmt_init
0001:004f7636  __mysqlnd_plugin_get_plugin_stmt_data
0001:004f766c  __mysqlnd_init_ps_subsystem
0001:004f7682  _mysqlnd_stmt_get_methods
0001:004f768c  _mysqlnd_stmt_set_methods
0001:004f769c  _mysqlnd_not_bound_as_blob
0001:004f76a0  _mysqlnd_stmt_not_prepared
0002:00003950  _mysqlnd_mysqlnd_stmt_methods
Module: U:\dev\php-5.3.8\ext\mysqlnd\mysqlnd_ps_codec.o(mysqlnd_ps_codec.o)
0002:00021058  _mysqlnd_ps_fetch_functions
0001:004f7b47  _ps_fetch_from_1_to_8_bytes
0001:004f8074  __mysqlnd_init_ps_fetch_subsystem
0001:004f846b  _mysqlnd_stmt_execute_generate_request
Module: U:\dev\php-5.3.8\TSRM\TSRM.o(TSRM.o)
0001:004f92e9  _tsrm_startup
0001:004f93d2  _ts_allocate_id
0001:004f956b  _tsrm_free_interpreter_context
0001:004f9612  _tsrm_set_interpreter_context
0001:004f9624  _ts_free_id
0001:004f9792  _tsrm_thread_id
0001:004f97a1  _ts_free_worker_threads
0001:004f98b9  _ts_free_thread
0001:004f99cd  _tsrm_new_interpreter_context
0001:004f9a0b  _ts_resource_ex
0001:004f9ab1  _tsrm_mutex_alloc
0001:004f9ab8  _tsrm_mutex_free
0001:004f9acd  _tsrm_shutdown
0001:004f9c7e  _tsrm_mutex_lock
0001:004f9c8a  _tsrm_mutex_unlock
0001:004f9c8f  _tsrm_set_new_thread_begin_handler
0001:004f9ca2  _tsrm_set_new_thread_end_handler
0001:004f9cb5  _tsrm_error_set
Module: U:\dev\php-5.3.8\TSRM\tsrm_strtok_r.o(tsrm_strtok_r.o)
0001:004f9cd0  _tsrm_strtok_r
Module: U:\dev\php-5.3.8\TSRM\tsrm_virtual_cwd.o(tsrm_virtual_cwd.o)
0002:00022058  _cwd_globals_id
0002:00022068  _main_cwd_state
0002:00022078  _cwd_mutex
0001:004fa849  _virtual_cwd_startup
0001:004fa8d2  _virtual_cwd_shutdown
0001:004fa8f4  _virtual_getcwd_ex
0001:004fa9b2  _virtual_getcwd
0001:004faa1f  _realpath_cache_clean
0001:004faaac  _realpath_cache_del
0001:004fab9d  _realpath_cache_lookup
0001:004fac8f  _realpath_cache_size
0001:004faca6  _realpath_cache_max_buckets
0001:004facb0  _realpath_cache_get_buckets
0001:004facc7  _virtual_file_ex
0001:004fb329  _virtual_chdir
0001:004fb366  _virtual_chdir_file
0001:004fb4a6  _virtual_realpath
0001:004fb616  _virtual_filepath_ex
0001:004fb683  _virtual_filepath
0001:004fb6ac  _virtual_fopen
0001:004fb750  _virtual_access
0001:004fb7ef  _virtual_utime
0001:004fb88e  _virtual_chmod
0001:004fb92d  _virtual_chown
0001:004fb9f4  _virtual_open
0001:004fbab5  _virtual_creat
0001:004fbb54  _virtual_rename
0001:004fbc7f  _virtual_stat
0001:004fbd1e  _virtual_lstat
0001:004fbdbd  _virtual_unlink
0001:004fbe55  _virtual_mkdir
0001:004fbef4  _virtual_rmdir
0001:004fbf8c  _virtual_opendir
0001:004fc026  _virtual_popen
0001:004fc0b6  _tsrm_realpath
Module: U:\dev\php-5.3.8\main\main.o(main.o)
0002:00022088  _core_globals_id
0001:004fc921  _zm_info_php_core
0001:004fca88  _php_on_timeout
0001:004fcb67  _php_printf
0001:004fcbea  _php_log_err
0001:004fd960  _php_write
0001:004fda17  _php_verror
0001:004fe0f2  _php_error_docref0
0001:004fe42e  _php_error_docref1
0001:004fe46e  _php_error_docref2
0001:004fe4e7  _php_html_puts
0001:004fe530  _zif_set_time_limit
0001:004fe631  _php_stream_open_for_zend_ex
0001:004fe7ab  _php_request_startup
0001:004fea59  _php_request_startup_for_hook
0001:004fea96  _php_request_shutdown_for_exec
0001:004feaca  _php_request_shutdown_for_hook
0001:004fed56  _php_request_shutdown
0001:004ff250  _php_com_initialize
0001:004ff255  _php_register_extensions
0001:004ff656  _php_module_startup
0001:00500356  _php_module_shutdown_for_exec
0001:0050035b  _php_module_shutdown
0001:005003e1  _php_module_shutdown_wrapper
0001:00500407  _php_execute_script
0001:00500743  _php_execute_simple_script
0001:00500891  _php_handle_aborted_connection
0001:00500912  _php_handle_auth_data
0001:00500a4d  _php_lint_script
0002:000039f0  _php_register_internal_extensions_func
Module: U:\dev\php-5.3.8\main\snprintf.o(snprintf.o)
0001:005027a8  _ap_php_conv_10
0001:00502844  _php_conv_fp
0001:00502bc2  _ap_php_conv_p2
0001:00502c25  _ap_php_snprintf
0001:00502c53  _php_gcvt
0001:005044ff  _ap_php_vslprintf
0001:0050453c  _ap_php_slprintf
0001:00504579  _ap_php_vsnprintf
0001:0050459f  _ap_php_vasprintf
0001:00504623  _ap_php_asprintf
Module: U:\dev\php-5.3.8\main\spprintf.o(spprintf.o)
0001:00505c40  _vspprintf
0001:00505ca0  _spprintf
Module: U:\dev\php-5.3.8\main\php_sprintf.o(php_sprintf.o)
0001:00505cd0  _php_sprintf
Module: U:\dev\php-5.3.8\main\safe_mode.o(safe_mode.o)
0001:00505e0b  _php_checkuid_ex
0001:0050636c  _php_checkuid
0001:00506396  _php_get_current_user
Module: U:\dev\php-5.3.8\main\fopen_wrappers.o(fopen_wrappers.o)
0001:005064ae  _php_fopen_primary_script
0001:005069a1  _php_resolve_path
0001:00506f70  _php_strip_url_passwd
0001:00507013  _expand_filepath_ex
0001:0050724d  _expand_filepath
0001:0050727e  _php_check_safe_mode_include_dir
0001:00507381  _php_check_specific_open_basedir
0001:00507761  _php_check_open_basedir_ex
0001:005078b8  _php_check_open_basedir
0001:005078da  _OnUpdateBaseDir
0001:00507a57  _php_fopen_with_path
Module: U:\dev\php-5.3.8\main\php_scandir.o(php_scandir.o)
0001:00507e60  _php_alphasort
0001:00507e82  _php_scandir
Module: U:\dev\php-5.3.8\main\php_ini.o(php_ini.o)
0001:0050809d  _config_zval_dtor
0001:0050895b  _display_ini_entries
0001:00508a87  _php_init_config
0001:005094e8  _php_shutdown_config
0001:00509534  _php_ini_register_extensions
0001:0050958b  _php_parse_user_ini_file
0001:0050969c  _php_ini_activate_config
0001:0050975e  _php_ini_has_per_dir_config
0001:00509768  _php_ini_activate_per_dir_config
0001:00509816  _php_ini_has_per_host_config
0001:00509820  _php_ini_activate_per_host_config
0001:00509885  _cfg_get_entry
0001:005098b9  _cfg_get_long
0001:0050993d  _cfg_get_double
0001:005099bf  _cfg_get_string
0001:00509a12  _php_ini_get_configuration_hash
0002:0001b9b0  _php_ini_opened_path
0002:0001b9b4  _php_ini_scanned_path
0002:0001b9b8  _php_ini_scanned_files
Module: U:\dev\php-5.3.8\main\SAPI.o(SAPI.o)
0002:00022098  _sapi_globals_id
0002:000220a8  _sapi_module
0001:00509ab2  _sapi_free_header
0001:00509b83  _sapi_startup
0001:00509bd3  _sapi_shutdown
0001:00509bdf  _sapi_handle_post
0001:00509cf0  _sapi_read_standard_form_data
0001:00509e81  _sapi_get_default_content_type
0001:00509f44  _sapi_get_default_content_type_header
0001:00509fdc  _sapi_apply_default_charset
0001:0050a0e8  _sapi_activate_headers_only
0001:0050a23c  _sapi_activate
0001:0050a558  _sapi_deactivate
0001:0050a74a  _sapi_initialize_empty_request
0001:0050a95b  _sapi_header_op
0001:0050b325  _sapi_add_header_ex
0001:0050b38f  _sapi_send_headers
0001:0050b5ca  _sapi_register_post_entry
0001:0050b646  _sapi_register_post_entries
0001:0050b68d  _sapi_unregister_post_entry
0001:0050b6f4  _sapi_register_default_post_reader
0001:0050b749  _sapi_register_treat_data
0001:0050b79e  _sapi_register_input_filter
0001:0050b7fb  _sapi_flush
0001:0050b82a  _sapi_get_stat
0001:0050b893  _sapi_getenv
0001:0050b91b  _sapi_get_fd
0001:0050b934  _sapi_force_http_10
0001:0050b94d  _sapi_get_target_uid
0001:0050b966  _sapi_get_target_gid
0001:0050b97f  _sapi_get_request_time
0001:0050b9e7  _sapi_terminate_process
Module: U:\dev\php-5.3.8\main\rfc1867.o(rfc1867.o)
0001:0050c40f  _php_rfc1867_register_constants
0001:0050c59f  _destroy_uploaded_files_hash
0001:0050c867  _rfc1867_post_handler
0002:0001ba70  _php_rfc1867_callback
Module: U:\dev\php-5.3.8\main\php_content_types.o(php_content_types.o)
0001:0050e168  _php_default_post_reader
0001:0050e3a8  _php_startup_sapi_content_types
0001:0050e3de  _php_setup_sapi_content_types
Module: U:\dev\php-5.3.8\main\mergesort.o(mergesort.o)
0001:0050e4ba  _php_mergesort
Module: U:\dev\php-5.3.8\main\php_variables.o(php_variables.o)
0001:0050f8e8  _php_register_variable_ex
0001:00510440  _php_register_variable_safe
0001:005104c0  _php_register_variable
0001:00510501  __php_import_environment_variables
0001:00510aee  _php_std_post_handler
0001:00510c17  _php_default_input_filter
0001:00510c31  _php_default_treat_data
0001:0051104f  _php_std_auto_global_callback
0001:00511098  _php_handle_special_queries
0001:00511145  _php_hash_environment
0001:0051199b  _php_startup_auto_globals
0002:00003a90  _php_import_environment_variables
Module: U:\dev\php-5.3.8\main\php_ticks.o(php_ticks.o)
0001:00511b80  _php_startup_ticks
0001:00511bbe  _php_deactivate_ticks
0001:00511be1  _php_shutdown_ticks
0001:00511c04  _php_add_tick_function
0001:00511c40  _php_remove_tick_function
0001:00511c84  _php_run_ticks
Module: U:\dev\php-5.3.8\main\network.o(network.o)
0001:00511e9e  _php_network_parse_network_address_with_port
0001:00512026  _php_network_populate_name_from_sockaddr
0001:0051213f  _php_network_get_peer_name
0001:005121c1  _php_network_get_sock_name
0001:00512243  _php_any_addr
0001:005122af  _php_sockaddr_size
0001:005122d1  _php_socket_strerror
0001:00512315  _php_network_accept_incoming
0001:00512463  _php_network_bind_socket_to_local_addr
0001:005125ac  _php_network_connect_socket
0001:005127df  _php_network_connect_socket_to_host
0001:00512ac8  __php_stream_sock_open_from_socket
0001:00512bcb  __php_stream_sock_open_host
0001:00512c5a  _php_set_sock_blocking
0001:00512df3  __php_emit_fd_setsize_warning
Module: U:\dev\php-5.3.8\main\php_open_temporary_file.o(php_open_temporary_file.o)
0001:00512fde  _php_shutdown_temporary_directory
0001:0051300a  _php_get_temporary_directory
0001:0051308f  _php_open_temporary_fd_ex
0001:00513130  _php_open_temporary_fd
0001:00513164  _php_open_temporary_file
Module: U:\dev\php-5.3.8\main\php_logos.o(php_logos.o)
0001:005131c0  _php_register_info_logo
0001:00513237  _php_unregister_info_logo
0001:00513300  _php_init_info_logos
0001:005133ae  _php_shutdown_info_logos
0001:005133c4  _php_info_logos
Module: U:\dev\php-5.3.8\main\output.o(output.o)
0002:00022148  _output_globals_id
0001:0051639e  _php_default_output_func
0001:0051600a  _php_ub_body_write_no_header
0001:0051608b  _php_ub_body_write
0001:00516846  _php_output_startup
0001:00516872  _php_output_activate
0001:0051690a  _php_output_register_constants
0001:005169aa  _php_output_set_status
0001:005169c6  _php_body_write
0001:005169e0  _php_header_write
0001:00516a58  _php_start_ob_buffer
0001:00516b26  _php_start_ob_buffer_named
0001:00516be2  _php_end_ob_buffer
0001:0051724f  _php_end_ob_buffers
0001:005172a2  _php_start_implicit_flush
0001:005172ba  _php_end_implicit_flush
0001:005172d2  _php_get_output_start_filename
0001:005172e9  _php_get_output_start_lineno
0001:00517300  _php_ob_set_internal_handler
0001:005173e6  _php_ob_handler_used
0001:00517488  _php_ob_init_conflict
0001:005174e1  _php_ob_get_buffer
0001:00517529  _php_ob_get_length
0001:0051756a  _zif_ob_start
0001:00517655  _zif_ob_flush
0001:00517774  _zif_ob_clean
0001:0051788c  _zif_ob_end_flush
0001:00517963  _zif_ob_end_clean
0001:00517a3a  _zif_ob_get_flush
0001:00517b23  _zif_ob_get_clean
0001:00517c0c  _zif_ob_get_contents
0001:00517c5f  _zif_ob_get_level
0001:00517ca5  _zif_ob_get_length
0001:00517cf8  _zif_ob_list_handlers
0001:00517d99  _zif_ob_get_status
0001:00517f6e  _zif_ob_implicit_flush
0001:00517fd5  _zif_output_reset_rewrite_vars
0001:00518011  _zif_output_add_rewrite_var
Module: U:\dev\php-5.3.8\main\getopt.o(getopt.o)
0001:0051820b  _php_getopt
0002:00003aa0  _php_optidx
Module: U:\dev\php-5.3.8\main\streams\streams.o(streams.o)
0001:00518e2c  _php_file_le_stream
0001:00518e36  _php_file_le_pstream
0001:00518e40  _php_file_le_stream_filter
0001:00518e4a  __php_stream_get_url_stream_wrappers_hash
0001:00518e6c  _php_stream_get_url_stream_wrappers_hash_global
0001:00518e76  _zm_deactivate_streams
0001:00518ea8  _php_stream_from_persistent_id
0001:0051905f  _php_stream_display_wrapper_errors
0001:005192ba  _php_stream_tidy_wrapper_error_log
0001:00519316  _php_stream_wrapper_log_error
0001:005193ca  __php_stream_alloc
0001:00519551  __php_stream_read
0001:0051969e  __php_stream_getc
0001:005196d6  __php_stream_stat
0001:0051973e  _php_stream_locate_eol
0001:00519829  __php_stream_get_line
0001:005199dc  _php_stream_get_record
0001:00519be3  __php_stream_flush
0001:00519c35  __php_stream_write
0001:00519c80  __php_stream_puts
0001:00519d04  __php_stream_putc
0001:00519d3b  __php_stream_printf
0001:00519d9b  __php_stream_tell
0001:00519dcc  __php_stream_seek
0001:0051a0f2  __php_stream_set_option
0001:0051a170  __php_stream_eof
0001:0051a1e9  __php_stream_truncate_set_size
0001:0051a21a  __php_stream_passthru
0001:0051a338  __php_stream_copy_to_mem
0001:0051a5b0  __php_stream_copy_to_stream_ex
0001:0051a807  __php_stream_copy_to_stream
0001:0051a855  _php_shutdown_stream_hashes
0001:0051a91b  _php_init_stream_wrappers
0001:0051aab3  _php_shutdown_stream_wrappers
0001:0051aae3  _php_register_url_stream_wrapper
0001:0051ab8a  _php_unregister_url_stream_wrapper
0001:0051abcb  _php_register_url_stream_wrapper_volatile
0001:0051aca0  _php_unregister_url_stream_wrapper_volatile
0001:0051aee5  _php_stream_locate_url_wrapper
0001:0051b3a3  __php_stream_mkdir
0001:0051b40b  __php_stream_rmdir
0001:0051b46c  __php_stream_stat_path
0001:0051b65f  __php_stream_opendir
0001:0051b75a  __php_stream_readdir
0001:0051b799  _php_stream_context_set
0001:0051b7fa  _php_stream_notification_notify
0001:0051b83b  _php_stream_context_alloc
0001:0051b8b3  _php_stream_notification_alloc
0001:0051b8cf  _php_stream_notification_free
0001:0051b8f2  _php_stream_context_free
0001:0051b94f  _php_stream_context_get_option
0001:0051b9c8  _php_stream_context_set_option
0001:0051bb58  _php_stream_context_get_link
0001:0051bbca  _php_stream_context_set_link
0001:0051bcb8  _php_stream_context_del_link
0001:0051bdd3  __php_stream_free
0001:0051c19b  __php_stream_open_wrapper_ex
0001:0051c6fb  _php_stream_dirent_alphasort
0001:0051c717  _php_stream_dirent_alphasortr
0001:0051c733  __php_stream_scandir
Module: U:\dev\php-5.3.8\main\streams\cast.o(cast.o)
0001:0051c880  _php_stream_mode_sanitize_fdopen_fopencookie
0001:0051c9a2  __php_stream_cast
0001:0051cd74  __php_stream_open_wrapper_as_file
0001:0051ce21  __php_stream_make_seekable
Module: U:\dev\php-5.3.8\main\streams\memory.o(memory.o)
0001:0051d6bc  __php_stream_memory_create
0001:0051d733  __php_stream_memory_open
0001:0051d7a9  __php_stream_memory_get_buffer
0001:0051d7be  __php_stream_temp_create
0001:0051deb8  __php_stream_temp_open
0002:00003ac0  _php_stream_memory_ops
0002:00003af0  _php_stream_temp_ops
0002:00003b20  _php_stream_rfc2397_ops
0002:00003b50  _php_stream_rfc2397_wops
0002:00003b80  _php_stream_rfc2397_wrapper
Module: U:\dev\php-5.3.8\main\streams\filter.o(filter.o)
0001:0051df60  _php_get_stream_filters_hash_global
0001:0051df6a  __php_get_stream_filters_hash
0001:0051df8c  _php_stream_filter_register_factory
0001:0051dfdc  _php_stream_filter_unregister_factory
0001:0051e01d  _php_stream_filter_register_factory_volatile
0001:0051e12a  _php_stream_bucket_new
0001:0051e20b  _php_stream_bucket_split
0001:0051e53f  _php_stream_bucket_delref
0001:0051e5aa  _php_stream_bucket_prepend
0001:0051e5d6  _php_stream_bucket_append
0001:0051e601  _php_stream_bucket_unlink
0001:0051e64d  _php_stream_bucket_make_writeable
0001:0051e7c7  _php_stream_filter_create
0001:0051e9b5  __php_stream_filter_alloc
0001:0051ea35  _php_stream_filter_free
0001:0051ea75  _php_stream_filter_prepend_ex
0001:0051eaa6  __php_stream_filter_prepend
0001:0051eaff  _php_stream_filter_append_ex
0001:0051ee65  __php_stream_filter_append
0001:0051eeb1  __php_stream_filter_flush
0001:0051f15d  _php_stream_filter_remove
Module: U:\dev\php-5.3.8\main\streams\plain_wrapper.o(plain_wrapper.o)
0001:0052020d  _php_stream_parse_fopen_modes
0001:0052033b  __php_stream_fopen_temporary_file
0001:005203ba  __php_stream_fopen_tmpfile
0001:00520463  __php_stream_fopen_from_fd
0001:00520526  __php_stream_fopen_from_file
0001:005205fb  __php_stream_fopen_from_pipe
0001:005206ab  __php_stream_fopen
0001:005209ff  __php_stream_fopen_with_path
0002:00003ba0  _php_stream_stdio_ops
0002:00003bd0  _php_plain_files_wrapper
Module: U:\dev\php-5.3.8\main\streams\userspace.o(userspace.o)
0001:00524771  _zm_startup_user_streams
0001:00524b6c  _zif_stream_wrapper_register
0001:00524d94  _zif_stream_wrapper_unregister
0001:00524ea9  _zif_stream_wrapper_restore
0002:00003c80  _php_stream_userspace_dir_ops
0002:00003c50  _php_stream_userspace_ops
Module: U:\dev\php-5.3.8\main\streams\transports.o(transports.o)
0001:00525010  _php_stream_xport_get_hash
0001:0052501a  _php_stream_xport_register
0001:0052506a  _php_stream_xport_unregister
0001:005250ab  _php_stream_xport_bind
0001:00525120  _php_stream_xport_connect
0001:005251b6  _php_stream_xport_listen
0001:0052530e  __php_stream_xport_create
0001:005258ad  _php_stream_xport_accept
0001:00525977  _php_stream_xport_get_name
0001:00525a53  _php_stream_xport_crypto_setup
0001:00525add  _php_stream_xport_crypto_enable
0001:00525b68  _php_stream_xport_recvfrom
0001:00525c6a  _php_stream_xport_sendto
0001:00525d37  _php_stream_xport_shutdown
Module: U:\dev\php-5.3.8\main\streams\xp_socket.o(xp_socket.o)
0001:005273ca  _php_stream_generic_socket_factory
0002:00003d70  _php_stream_unix_socket_ops
0002:00003da0  _php_stream_unixdg_socket_ops
0002:00003d40  _php_stream_udp_socket_ops
0002:00003d10  _php_stream_socket_ops
0002:00003ce0  _php_stream_generic_socket_ops
Module: U:\dev\php-5.3.8\main\streams\mmap.o(mmap.o)
0001:005275d0  __php_stream_mmap_range
0001:00527641  __php_stream_mmap_unmap
0001:0052767b  __php_stream_mmap_unmap_ex
Module: U:\dev\php-5.3.8\main\streams\glob_wrapper.o(glob_wrapper.o)
0001:00527a13  __php_glob_stream_get_path
0001:00527a5f  __php_glob_stream_get_pattern
0001:00527aab  __php_glob_stream_get_count
0002:00003dd0  _php_glob_stream_ops
0002:00003e00  _php_glob_stream_wrapper
Module: U:\dev\php-5.3.8\main\internal_functions.o(internal_functions.o)
0001:00527ae0  _php_register_internal_extensions
Module: U:\dev\php-5.3.8\Zend\zend_language_parser.o(zend_language_parser.o)
0001:00527e63  _zendparse
Module: U:\dev\php-5.3.8\Zend\zend_language_scanner.o(zend_language_scanner.o)
0002:00022158  _language_scanner_globals_id
0001:0053584c  _startup_scanner
0001:0053589d  _shutdown_scanner
0001:00535934  _zend_save_lexical_state
0001:005359d5  _zend_restore_lexical_state
0001:00535ab6  _zend_destroy_file_handle
0001:00535b1c  _open_file_for_scanning
0001:00535cea  _compile_file
0001:00535ec6  _compile_filename
0001:00536083  _zend_prepare_string_for_scanning
0001:00536174  _zend_get_scanned_file_offset
0001:0053618e  _compile_string
0001:00536377  _highlight_file
0001:00536428  _highlight_string
0001:00536557  _lex_scan
Module: U:\dev\php-5.3.8\Zend\zend_ini_parser.o(zend_ini_parser.o)
0001:0053e582  _ini_parse
0001:0053f12b  _zend_parse_ini_string
0001:0053f1b0  _zend_parse_ini_file
Module: U:\dev\php-5.3.8\Zend\zend_ini_scanner.o(zend_ini_scanner.o)
0002:00022168  _ini_scanner_globals_id
0001:0053f9db  _shutdown_ini_scanner
0001:0053fa22  _zend_ini_scanner_get_lineno
0001:0053fa41  _zend_ini_scanner_get_filename
0001:0053fa63  _zend_ini_open_file_for_scanning
0001:0053fac2  _zend_ini_prepare_string_for_scanning
0001:0053fb53  _ini_lex
Module: U:\dev\php-5.3.8\Zend\zend_alloc.o(zend_alloc.o)
0001:00546faf  _zend_mm_startup_ex
0001:005472e7  _zend_mm_startup
0001:005474ef  _zend_mm_shutdown
0001:00547627  __zend_mm_alloc
0001:00547639  __zend_mm_free
0001:0054764b  __zend_mm_realloc
0001:00547660  __zend_mm_block_size
0001:00547676  _is_zend_mm
0001:0054768e  __emalloc
0001:005476d9  __efree
0001:00547724  __erealloc
0001:0054777a  __zend_mem_block_size
0001:005477e9  __safe_emalloc
0001:00547843  __safe_malloc
0001:005478c4  __safe_erealloc
0001:0054791e  __safe_realloc
0001:005479a6  __ecalloc
0001:005479f0  __estrdup
0001:00547a33  __estrndup
0001:00547a6f  _zend_strndup
0001:00547ab1  _zend_set_memory_limit
0001:00547aec  _zend_memory_usage
0001:00547b22  _zend_memory_peak_usage
0001:00547b55  _shutdown_memory_manager
0001:00547bab  _start_memory_manager
0001:00547bd7  _zend_mm_set_heap
0001:00547bf2  _zend_mm_get_storage
0001:00547bfd  _zend_mm_set_custom_handlers
Module: U:\dev\php-5.3.8\Zend\zend_compile.o(zend_compile.o)
0002:00022178  _zend_compile_file
0002:00022188  _zend_compile_string
0001:00547c60  _zend_auto_global_arm
0001:00548c1c  _file_handle_dtor
0001:00548f64  _zend_auto_global_disable_jit
0001:00548fb6  _zend_init_compiler_data_structures
0001:00549180  _init_compiler
0001:00549233  _shutdown_compiler
0001:0054932d  _zend_set_compiled_filename
0001:0054940f  _zend_restore_compiled_filename
0001:0054942c  _zend_get_compiled_filename
0001:00549446  _zend_get_compiled_lineno
0001:00549460  _zend_is_compiling
0001:0054947b  _zend_do_binary_op
0001:0054955a  _zend_do_unary_op
0001:0054960f  _zend_do_binary_assign_op
0001:00549877  _fetch_array_dim
0001:0054997a  _fetch_string_offset
0001:00549986  _zend_do_print
0001:00549a32  _zend_do_echo
0001:00549b2b  _zend_do_abstract_method
0001:00549c9a  _zend_do_assign_ref
0001:00549eb3  _zend_do_while_cond
0001:00549f92  _zend_do_while_end
0001:0054a06f  _zend_do_for_cond
0001:0054a0ee  _zend_do_for_before_statement
0001:0054a1d0  _zend_do_for_end
0001:0054a2b8  _zend_do_pre_incdec
0001:0054a438  _zend_do_post_incdec
0001:0054a5aa  _zend_do_if_cond
0001:0054a645  _zend_do_if_after_statement
0001:0054a758  _zend_do_if_end
0001:0054a885  _zend_check_writable_variable
0001:0054a8d5  _zend_do_begin_variable_parse
0001:0054a95e  _zend_do_end_variable_parse
0001:0054acb2  _zend_do_assign
0001:0054b321  _zend_do_add_string
0001:0054b488  _zend_do_add_variable
0001:0054b57c  _zend_do_free
0001:0054b79e  _zend_do_verify_access_types
0001:0054b896  _zend_do_handle_exception
0001:0054b8d1  _zend_do_clone
0001:0054b998  _zend_do_label
0001:0054bb07  _zend_resolve_goto_label
0001:0054bcb3  _zend_do_goto
0001:0054bd4d  _zend_release_labels
0001:0054be12  _zend_do_build_full_name
0001:0054bf1c  _zend_do_end_function_call
0001:0054c21a  _zend_do_pass_param
0001:0054c679  _zend_do_return
0001:0054c895  _zend_do_first_catch
0001:0054c8c0  _zend_initialize_try_catch_element
0001:0054c9c8  _zend_do_mark_last_catch
0001:0054ca79  _zend_do_try
0001:0054cb1d  _zend_do_end_catch
0001:0054cbda  _zend_do_throw
0001:0054cc33  _function_add_ref
0001:0054ccce  _zend_visibility_string
0001:0054cd4d  _zend_do_inherit_interfaces
0001:0054cf85  _zend_do_inheritance
0001:0054d692  _zend_do_implement_interface
0001:0054d97b  _do_bind_function
0001:0054daf1  _do_bind_class
0001:0054dc19  _do_bind_inherited_class
0001:0054dd4a  _zend_do_early_binding
0001:0054e09b  _zend_do_delayed_early_binding
0001:0054e19a  _zend_do_boolean_or_begin
0001:0054e28a  _zend_do_boolean_or_end
0001:0054e35f  _zend_do_boolean_and_begin
0001:0054e44f  _zend_do_boolean_and_end
0001:0054e524  _zend_do_do_while_begin
0001:0054e598  _zend_do_do_while_end
0001:0054e65c  _zend_do_brk_cont
0001:0054e6fe  _zend_do_switch_cond
0001:0054e7c6  _zend_do_switch_end
0001:0054e996  _zend_do_case_before_statement
0001:0054eb73  _zend_do_case_after_statement
0001:0054ec28  _zend_do_default_before_statement
0001:0054ed7b  _zend_do_end_class_declaration
0001:0054ef95  _zend_mangle_property_name
0001:0054f584  _zend_unmangle_property_name
0001:0054f70b  _zend_do_declare_property
0001:0054f93a  _zend_do_declare_class_constant
0001:0054fa9f  _zend_do_fetch_property
0001:0054fcd8  _zend_do_declare_implicit_property
0001:0054fcdd  _zend_do_push_object
0001:0054fd0e  _zend_do_pop_object
0001:0054fd7b  _zend_do_begin_new_object
0001:0054fe58  _zend_do_end_new_object
0001:0054ff2c  _zend_do_shell_exec
0001:00550072  _zend_do_init_array
0001:0055017c  _zend_do_add_array_element
0001:0055024e  _zend_do_add_static_array_element
0001:00550707  _zend_do_add_list_element
0001:00550794  _zend_do_new_list_begin
0001:005507c4  _zend_do_new_list_end
0001:005507fe  _zend_do_list_init
0001:005508bf  _zend_do_list_end
0001:00550baa  _zend_do_cast
0001:00550c5c  _zend_do_unset
0001:00550d36  _zend_do_isset_or_isempty
0001:00550eb6  _zend_do_instanceof
0001:00551023  _zend_do_foreach_begin
0001:005513d9  _zend_do_foreach_cont
0001:00551732  _zend_do_foreach_end
0001:00551883  _zend_do_declare_begin
0001:005518df  _zend_do_declare_stmt
0001:005519cc  _zend_do_declare_end
0001:00551a5c  _zend_do_exit
0001:00551acb  _zend_do_begin_silence
0001:00551b5c  _zend_do_end_silence
0001:00551bb5  _zend_do_jmp_set
0001:00551cb5  _zend_do_jmp_set_else
0001:00551db4  _zend_do_begin_qm_op
0001:00551e73  _zend_do_qm_true
0001:00551fc7  _zend_do_qm_false
0001:005520c4  _zend_do_extended_info
0001:0055213a  _zend_do_end_function_declaration
0001:005522b0  _zend_do_extended_fcall_begin
0001:00552320  _zend_do_begin_dynamic_function_call
0001:00552593  _zend_do_begin_method_call
0001:00552772  _zend_do_extended_fcall_end
0001:005527b8  _zend_do_include_or_eval
0001:0055288b  _zend_do_ticks
0001:005528fb  _zend_auto_global_dtor
0001:0055290f  _zend_is_auto_global
0001:0055298b  _fetch_simple_variable_ex
0001:00552bd3  _fetch_simple_variable
0001:00552c03  _zend_do_fetch_global_variable
0001:00552d62  _zend_do_fetch_static_variable
0001:00553045  _zend_do_fetch_lexical_variable
0001:005530d9  _fetch_array_begin
0001:0055311e  _zend_do_indirect_references
0001:0055322d  _zend_register_auto_global
0001:005532a1  _zendlex
0001:005533ab  _zend_initialize_class_data
0001:005536f6  _zend_get_class_fetch_type
0001:00553764  _zend_get_compiled_variable_name
0001:0055379e  _zend_do_build_namespace_name
0001:005539d8  _zend_do_begin_class_declaration
0001:00553e6b  _zend_resolve_class_name
0001:00554220  _zend_do_implements_interface
0001:0055435b  _zend_do_fetch_class
0001:0055453e  _zend_do_begin_catch
0001:0055465c  _zend_do_fetch_static_member
0001:005548e5  _zend_do_begin_class_member_function_call
0001:00554b4f  _zend_do_receive_arg
0001:00554f43  _zend_resolve_non_class_name
0001:005551f4  _zend_do_fetch_constant
0001:00555596  _zend_do_begin_function_call
0001:00555a17  _zend_do_begin_function_declaration
0001:005566fd  _zend_do_begin_lambda_function_declaration
0001:0055690d  _zend_do_begin_namespace
0001:00556dd0  _zend_do_use
0001:0055731b  _zend_do_declare_constant
0001:00557492  _zend_verify_namespace
0001:005574d1  _zend_do_end_namespace
0001:00557612  _zend_do_halt_compiler_register
0001:00557724  _zend_do_end_compilation
0001:00557749  _zend_dirname
Module: U:\dev\php-5.3.8\Zend\zend_constants.o(zend_constants.o)
0001:0055782d  _free_zend_constant
0001:0055786b  _copy_zend_constant
0001:005578ac  _zend_copy_constants
0001:005578dd  _clean_module_constants
0001:00557915  _zend_startup_constants
0001:00557987  _zend_shutdown_constants
0001:005579cd  _clean_non_persistent_constants
0001:00557a3c  _zend_get_constant
0001:00557d2e  _zend_get_constant_ex
0001:00558266  _zend_register_constant
0001:00558401  _zend_register_stringl_constant
0001:00558457  _zend_register_string_constant
0001:005584a6  _zend_register_double_constant
0001:005584f6  _zend_register_long_constant
0001:005586cd  _zend_register_standard_constants
Module: U:\dev\php-5.3.8\Zend\zend_dynamic_array.o(zend_dynamic_array.o)
0001:005589a0  _zend_dynamic_array_init
0001:005589d8  _zend_dynamic_array_push
0001:00558a26  _zend_dynamic_array_pop
0001:00558a3f  _zend_dynamic_array_get_element
Module: U:\dev\php-5.3.8\Zend\zend_execute_API.o(zend_execute_API.o)
0002:00022198  _zend_execute
0002:000221a8  _zend_execute_internal
0001:00558b7f  _zend_timeout
0001:00558c05  __zval_ptr_dtor
0001:00558d77  _init_executor
0001:00559121  _shutdown_destructors
0001:00559236  _shutdown_executor
0001:0055981c  _get_active_class_name
0001:00559885  _get_active_function_name
0001:005598de  _zend_get_executed_filename
0001:00559904  _zend_get_executed_lineno
0001:00559961  _zend_is_executing
0001:0055997c  __zval_internal_ptr_dtor
0001:005599c1  _zend_is_true
0001:00559bac  _zval_update_constant_ex
0001:0055a63d  _zval_update_constant_inline_change
0001:0055a666  _zval_update_constant_no_inline_change
0001:0055a68f  _zval_update_constant
0001:0055a7c7  _zend_call_function
0001:0055b56f  _call_user_function_ex
0001:0055b5d0  _call_user_function
0001:0055b711  _zend_lookup_class_ex
0001:0055bcd1  _zend_lookup_class
0001:0055bd01  _execute_new_code
0001:0055bf76  _zend_set_timeout
0001:0055c03e  _zend_unset_timeout
0001:0055c1a7  _zend_fetch_class
0001:0055c459  _zend_verify_abstract_class
0001:0055c6b0  _zend_reset_all_cv
0001:0055c70b  _zend_delete_global_variable
0001:0055c991  _zend_rebuild_symbol_table
0001:0055cb55  _zend_eval_stringl
0001:0055ce5c  _zend_eval_stringl_ex
0001:0055cec8  _zend_eval_string_ex
0001:0055cf10  _zend_eval_string
0001:0055cf60  _empty_fcall_info
0001:0055cf90  _empty_fcall_info_cache
Module: U:\dev\php-5.3.8\Zend\zend_highlight.o(zend_highlight.o)
0001:0055cff7  _zend_html_putc
0001:0055d18e  _zend_html_puts
0001:0055d22a  _zend_highlight
0001:0055d408  _zend_strip
Module: U:\dev\php-5.3.8\Zend\zend_llist.o(zend_llist.o)
0001:0055d560  _zend_llist_init
0001:0055d59d  _zend_llist_add_element
0001:0055d64a  _zend_llist_prepend_element
0001:0055d6f6  _zend_llist_del_element
0001:0055d781  _zend_llist_destroy
0001:0055d7d6  _zend_llist_clean
0001:0055d7fb  _zend_llist_remove_tail
0001:0055d85d  _zend_llist_copy
0001:0055d8b4  _zend_llist_apply_with_del
0001:0055d938  _zend_llist_apply
0001:0055d96a  _zend_llist_sort
0001:0055da26  _zend_llist_apply_with_argument
0001:0055da5d  _zend_llist_apply_with_arguments
0001:0055da9b  _zend_llist_count
0001:0055daa6  _zend_llist_get_first_ex
0001:0055dac7  _zend_llist_get_last_ex
0001:0055dae9  _zend_llist_get_next_ex
0001:0055db12  _zend_llist_get_prev_ex
Module: U:\dev\php-5.3.8\Zend\zend_opcode.o(zend_opcode.o)
0001:0055db91  _pass_two
0001:0055ddb5  _zend_cleanup_function_data_full
0001:0055ddda  _init_op_array
0001:0055df78  _zend_cleanup_function_data
0001:0055dfa6  _zend_cleanup_class_data
0001:0055e07b  _destroy_zend_class
0001:0055e1ad  _zend_class_add_ref
0001:0055e1bb  _destroy_op_array
0001:0055e373  _destroy_zend_function
0001:0055e389  _zend_function_dtor
0001:0055e3b4  _init_op
0001:0055e46c  _get_next_op
0001:0055e50a  _get_next_op_number
0001:0055e515  _get_next_brk_cont_element
0001:0055e574  _print_class
0001:0055e5c6  _get_unary_op
0001:0055e5e1  _get_binary_op
Module: U:\dev\php-5.3.8\Zend\zend_operators.o(zend_operators.o)
0001:0055e868  _zend_atoi
0001:0055e975  _zend_atol
0001:0055ea81  _zend_string_to_double
0001:0055ec4c  _convert_to_long_base
0001:0055ef1c  _convert_to_long
0001:0055ef3d  _convert_scalar_to_number
0001:0055f29b  _convert_to_double
0001:0055f518  _convert_to_null
0001:0055f610  _convert_to_boolean
0001:0055f8d7  __convert_to_string
0001:0055fc1a  _convert_to_array
0001:0055fe88  _convert_to_object
0001:0055fefe  _multi_convert_to_long_ex
0001:0055ff9d  _multi_convert_to_double_ex
0001:0056003c  _multi_convert_to_string_ex
0001:0056010c  _add_function
0001:00560905  _sub_function
0001:00561075  _mul_function
0001:005617f6  _div_function
0001:00562025  _mod_function
0001:00562342  _boolean_xor_function
0001:00562585  _boolean_not_function
0001:0056269a  _bitwise_not_function
0001:005627b6  _bitwise_or_function
0001:00562b47  _bitwise_and_function
0001:00562eae  _bitwise_xor_function
0001:00563212  _shift_left_function
0001:005634d4  _shift_right_function
0001:00563798  _add_char_to_string
0001:005637ea  _add_string_to_string
0001:00563867  _concat_function
0001:00563a47  _string_locale_compare_function
0001:00563b09  _numeric_compare_function
0001:00563bbf  _is_identical_function
0001:00563d16  _is_not_identical_function
0001:00563d5b  _instanceof_function
0001:00563d84  _instanceof_function_ex
0001:00563e10  _increment_function
0001:005642b7  _decrement_function
0001:005645e9  _zval_is_true
0001:00564609  _zend_str_tolower_copy
0001:00564647  _zend_str_tolower_dup
0001:00564675  _zend_str_tolower
0001:00564699  _zend_binary_strcmp
0001:005646cf  _zend_binary_strncmp
0001:00564732  _zend_binary_strcasecmp
0001:0056477f  _zend_binary_strncasecmp
0001:005647f5  _zend_binary_zval_strcmp
0001:00564821  _string_compare_function
0001:005648e5  _zend_binary_zval_strncmp
0001:0056491a  _zend_binary_zval_strcasecmp
0001:00564946  _zend_binary_zval_strncasecmp
0001:0056497b  _zendi_smart_strcmp
0001:0056502c  _zend_compare_symbol_tables_i
0001:0056505d  _zend_compare_symbol_tables
0001:0056509c  _compare_function
0001:00566389  _is_smaller_or_equal_function
0001:005663d2  _is_smaller_function
0001:00566414  _is_not_equal_function
0001:0056645d  _is_equal_function
0001:005664a6  _zend_compare_arrays
0001:005664c2  _zend_compare_objects
0001:0056651a  _zend_locale_sprintf_double
Module: U:\dev\php-5.3.8\Zend\zend_ptr_stack.o(zend_ptr_stack.o)
0001:005665bf  _zend_ptr_stack_init_ex
0001:0056664a  _zend_ptr_stack_init
0001:00566665  _zend_ptr_stack_n_push
0001:00566737  _zend_ptr_stack_n_pop
0001:0056677e  _zend_ptr_stack_destroy
0001:005667a8  _zend_ptr_stack_apply
0001:005667dc  _zend_ptr_stack_clean
0001:00566863  _zend_ptr_stack_num_elements
Module: U:\dev\php-5.3.8\Zend\zend_stack.o(zend_stack.o)
0001:00566870  _zend_stack_init
0001:005668a9  _zend_stack_push
0001:00566932  _zend_stack_top
0001:0056695b  _zend_stack_del_top
0001:00566981  _zend_stack_int_top
0001:005669a3  _zend_stack_is_empty
0001:005669b5  _zend_stack_destroy
0001:00566a01  _zend_stack_base
0001:00566a0c  _zend_stack_count
0001:00566a16  _zend_stack_apply
0001:00566aa0  _zend_stack_apply_with_argument
Module: U:\dev\php-5.3.8\Zend\zend_variables.o(zend_variables.o)
0001:00566b40  _zval_add_ref
0001:00566b4e  __zval_dtor_func
0001:00566c66  __zval_internal_dtor
0001:00566cc1  __zval_copy_ctor_func
0001:00566dfb  _zend_print_variable
0001:00566e16  __zval_dtor_wrapper
0001:00566e64  _zval_property_ctor
Module: U:\dev\php-5.3.8\Zend\zend.o(zend.o)
0002:000221b8  _compiler_globals_id
0002:000221c8  _executor_globals_id
0002:000221d8  _zend_write
0002:000221e8  _zend_printf
0002:000221f8  _zend_error_cb
0002:00022208  _zend_fopen
0002:00022218  _zend_stream_open_function
0002:00022228  _zend_block_interruptions
0002:00022238  _zend_unblock_interruptions
0002:00022248  _zend_ticks_function
0002:00022258  _zend_on_timeout
0002:00022268  _zend_vspprintf
0002:00022278  _zend_getenv
0002:00022288  _zend_resolve_path
0002:00022298  _zval_used_for_init
0002:000222a8  _zend_uv
0001:00567507  _zend_print_flat_zval_r
0001:00567803  _zend_startup
0001:00567c10  _zend_register_standard_ini_entries
0001:00567c33  _zend_post_startup
0001:00567d8a  _zend_shutdown
0001:00567e71  _zend_set_utility_values
0001:00567ea8  __zend_bailout
0001:00567f5d  _zend_append_version_info
0001:0056802f  _get_zend_version
0001:00568039  _zend_activate
0001:00568068  _zend_activate_modules
0001:0056808b  _zend_deactivate_modules
0001:00568105  _zend_call_destructors
0001:00568165  _zend_deactivate
0001:005682f1  _zend_post_deactivate_modules
0001:00568331  _zend_message_dispatcher
0001:0056834e  _zend_get_configuration_directive
0001:00568378  _zend_error
0001:00568e10  _zenderror
0001:00568e84  _zend_make_printable_zval
0001:00569156  _zend_print_zval_ex
0001:005691ea  _zend_print_zval_r_ex
0001:00569696  _zend_print_zval_r
0001:005696c0  _zend_print_zval
0001:005696e3  _zend_output_debug_string
0001:005696e8  _zend_execute_scripts
0001:005699cf  _zend_make_compiled_string_description
0001:00569a55  _free_estring
0001:00568378  _zend_error_noreturn
0002:0001bb90  _zend_standard_class_def
Module: U:\dev\php-5.3.8\Zend\zend_API.o(zend_API.o)
0002:000222b8  _module_registry
0001:00569ce3  _zif_display_disabled_function
0001:00569e3d  _zend_startup_module_ex
0001:00569fe1  _zend_get_parameters
0001:0056a0c7  __zend_get_parameters_array
0001:0056a192  _zend_get_parameters_ex
0001:0056a202  __zend_get_parameters_array_ex
0001:0056a277  _zend_wrong_param_count
0001:0056a2cd  _zend_get_type_by_const
0001:0056a2e6  _zend_zval_type_name
0001:0056a33a  _zend_get_class_entry
0001:0056b53f  _zend_get_object_classname
0001:0056b5a5  __array_init
0001:0056b5f0  _zend_merge_properties
0001:0056b6a2  _zend_update_class_constants
0001:0056bb7c  __object_and_properties_init
0001:0056bcad  __object_init_ex
0001:0056bcd6  __object_init
0001:0056bd28  _add_assoc_function
0001:0056bd49  _add_assoc_long_ex
0001:0056beba  _add_assoc_null_ex
0001:0056c024  _add_assoc_bool_ex
0001:0056c19a  _add_assoc_resource_ex
0001:0056c30a  _add_assoc_double_ex
0001:0056c482  _add_assoc_string_ex
0001:0056c615  _add_assoc_stringl_ex
0001:0056c7ad  _add_assoc_zval_ex
0001:0056c904  _add_index_long
0001:0056c969  _add_index_null
0001:0056c9c9  _add_index_bool
0001:0056ca34  _add_index_resource
0001:0056ca99  _add_index_double
0001:0056cb04  _add_index_string
0001:0056cb9f  _add_index_stringl
0001:0056cc29  _add_index_zval
0001:0056cc64  _add_next_index_long
0001:0056ccca  _add_next_index_null
0001:0056cd2b  _add_next_index_bool
0001:0056cd97  _add_next_index_resource
0001:0056cdfd  _add_next_index_double
0001:0056ce69  _add_next_index_string
0001:0056cf05  _add_next_index_stringl
0001:0056cf90  _add_next_index_zval
0001:0056cfcc  _zend_copy_parameters_array
0001:0056d033  _add_get_assoc_string_ex
0001:0056d1c4  _add_get_assoc_stringl_ex
0001:0056d35a  _add_get_index_long
0001:0056d3be  _add_get_index_double
0001:0056d428  _add_get_index_string
0001:0056d4c2  _add_get_index_stringl
0001:0056d54b  _add_property_long_ex
0001:0056d5fe  _add_property_bool_ex
0001:0056d6b7  _add_property_null_ex
0001:0056d765  _add_property_resource_ex
0001:0056d818  _add_property_double_ex
0001:0056d8d1  _add_property_string_ex
0001:0056d9b2  _add_property_stringl_ex
0001:0056da85  _add_property_zval_ex
0001:0056db03  _zend_startup_modules
0001:0056dcba  _zend_check_magic_method_implementation
0001:0056e0f5  _zend_unregister_functions
0001:0056e35b  _zend_register_functions
0001:0056f281  _zend_register_module_ex
0001:0056f47f  _zend_register_internal_module
0001:0056f4a7  _zend_startup_module
0001:0056f4f7  _zend_get_module_started
0001:0056f543  _module_destructor
0001:0056f65f  _module_registry_request_startup
0001:0056f6bb  _module_registry_cleanup
0001:0056f6e6  _module_registry_unload_temp
0001:0056f6fb  _zend_next_free_module
0001:0056f70d  _zend_class_implements
0001:0056f74a  _zend_register_internal_class
0001:0056f75e  _zend_register_internal_class_ex
0001:0056f7ef  _zend_register_internal_interface
0001:0056f806  _zend_register_class_alias_ex
0001:0056f889  _zend_set_hash_symbol
0001:0056f90b  _zend_disable_function
0001:0056f9a0  _zend_disable_class
0001:0056fba7  _zend_is_callable_ex
0001:0057021e  _zend_is_callable
0001:00570266  _zend_make_callable
0001:0057035e  _zend_fcall_info_init
0001:0057210d  _zend_parse_method_parameters_ex
0001:0057227d  _zend_parse_method_parameters
0001:005723db  _zend_parse_parameters
0001:00572460  _zend_parse_parameters_ex
0001:005724e8  _zend_fcall_info_args_clear
0001:0057251c  _zend_fcall_info_args_save
0001:00572542  _zend_fcall_info_args_restore
0001:0057256e  _zend_fcall_info_args
0001:0057261f  _zend_fcall_info_argp
0001:00572696  _zend_fcall_info_argv
0001:00572714  _zend_fcall_info_argn
0001:00572742  _zend_fcall_info_call
0001:0057280f  _zend_get_module_version
0001:005728b8  _zend_declare_property_ex
0001:00572be6  _zend_declare_property
0001:00572c2c  _zend_declare_property_null
0001:00572cb4  _zend_declare_property_bool
0001:00572d51  _zend_declare_property_long
0001:00572de6  _zend_declare_property_double
0001:00572e81  _zend_declare_property_string
0001:00572f5d  _zend_declare_property_stringl
0001:00573029  _zend_declare_class_constant
0001:00573071  _zend_declare_class_constant_null
0001:005730de  _zend_declare_class_constant_long
0001:00573167  _zend_declare_class_constant_bool
0001:005731fb  _zend_declare_class_constant_double
0001:00573284  _zend_declare_class_constant_stringl
0001:00573344  _zend_declare_class_constant_string
0001:005733b6  _zend_update_property
0001:005734b3  _zend_update_property_null
0001:00573508  _zend_update_property_bool
0001:0057357f  _zend_update_property_long
0001:005735ee  _zend_update_property_double
0001:0057365d  _zend_update_property_string
0001:005736f9  _zend_update_property_stringl
0001:00573788  _zend_update_static_property
0001:005738cc  _zend_update_static_property_null
0001:0057391a  _zend_update_static_property_bool
0001:00573985  _zend_update_static_property_long
0001:005739e8  _zend_update_static_property_double
0001:00573a4b  _zend_update_static_property_string
0001:00573adb  _zend_update_static_property_stringl
0001:00573b87  _zend_read_property
0001:00573c9b  _zend_read_static_property
0001:00573d06  _zend_save_error_handling
0001:00573d3f  _zend_replace_error_handling
0001:00573df9  _zend_restore_error_handling
Module: U:\dev\php-5.3.8\Zend\zend_extensions.o(zend_extensions.o)
0002:000222e8  _zend_extensions
0001:00573f4e  _zend_extension_dtor
0001:00573fa2  _zend_startup_extensions_mechanism
0001:00573fda  _zend_startup_extensions
0001:00573ff8  _zend_shutdown_extensions
0001:00574026  _zend_extension_dispatch_message
0001:00574070  _zend_register_extension
0001:005742c3  _zend_load_extension
0001:005744e7  _zend_get_resource_handle
0001:0057450c  _zend_get_extension
0001:00574558  _zend_os2_load_module
0001:00574592  _zend_os2_query_symbol
0001:005745df  _zend_os2_module_error
Module: U:\dev\php-5.3.8\Zend\zend_hash.o(zend_hash.o)
0001:005748a0  _zend_hash_func
0001:005749f2  __zend_hash_init
0001:00574adb  __zend_hash_init_ex
0001:00574b1a  _zend_hash_set_apply_protection
0001:00574b28  _zend_hash_rehash
0001:00574c52  __zend_hash_index_update_or_next_insert
0001:00574fbb  __zend_hash_quick_add_or_update
0001:0057539f  __zend_hash_add_or_update
0001:0057588a  _zend_hash_add_empty_element
0001:005758d1  _zend_hash_del_key_or_index
0001:00575ba1  _zend_hash_destroy
0001:00575c34  _zend_hash_clean
0001:00575ce5  _zend_hash_graceful_destroy
0001:00575d29  _zend_hash_graceful_reverse_destroy
0001:00575d9f  _zend_hash_apply
0001:00575e2e  _zend_hash_apply_with_argument
0001:00575ec2  _zend_hash_apply_with_arguments
0001:00575f7c  _zend_hash_reverse_apply
0001:00576007  _zend_hash_copy
0001:005760e3  _zend_hash_merge_ex
0001:0057619c  _zend_get_hash_value
0001:005762ee  _zend_hash_find
0001:005764a6  _zend_hash_exists
0001:00576659  _zend_hash_index_find
0001:0057669b  _zend_hash_quick_find
0001:00576723  _zend_hash_index_exists
0001:0057675c  _zend_hash_quick_exists
0001:005767dd  __zend_hash_merge
0001:005768c2  _zend_hash_num_elements
0001:005768cd  _zend_hash_get_pointer
0001:005768f6  _zend_hash_set_pointer
0001:00576951  _zend_hash_internal_pointer_reset_ex
0001:0057696d  _zend_hash_internal_pointer_end_ex
0001:00576989  _zend_hash_move_forward_ex
0001:005769af  _zend_hash_move_backwards_ex
0001:005769d5  _zend_hash_get_current_key_ex
0001:00576a52  _zend_hash_get_current_key_type_ex
0001:00576a7c  _zend_hash_get_current_data_ex
0001:00576aa5  _zend_hash_update_current_key_ex
0001:00577327  _zend_hash_sort
0001:0057750b  _zend_hash_compare
0001:005777cb  _zend_hash_minmax
0001:0057786d  _zend_hash_next_free_element
Module: U:\dev\php-5.3.8\Zend\zend_list.o(zend_list.o)
0002:00022308  _le_index_ptr
0001:0057792b  _plist_entry_destructor
0001:00577a01  _list_entry_destructor
0001:00577aa3  _zend_list_insert
0001:00577b34  __zend_list_delete
0001:00577bc6  __zend_list_find
0001:00577c1c  __zend_list_addref
0001:00577c62  _zend_register_resource
0001:00577d4b  _zend_fetch_resource
0001:00577f42  _zend_init_rsrc_list
0001:00577fae  _zend_init_rsrc_plist
0001:00577ffa  _zend_destroy_rsrc_list
0001:00578006  _zend_clean_module_rsrc_dtors
0001:00578030  _zend_register_list_destructors
0001:005780b2  _zend_register_list_destructors_ex
0001:00578133  _zend_fetch_list_dtor_id
0001:005781ae  _zend_init_rsrc_list_dtors
0001:005781ec  _zend_destroy_rsrc_list_dtors
0001:00578200  _zend_rsrc_list_get_rsrc_type
Module: U:\dev\php-5.3.8\Zend\zend_indent.o(zend_indent.o)
0001:005782dd  _zend_indent
Module: U:\dev\php-5.3.8\Zend\zend_builtin_functions.o(zend_builtin_functions.o)
0001:0057a816  _zm_startup_core
0001:0057c3fa  _zend_startup_builtin_functions
0001:0057c445  _debug_print_backtrace_args
0001:0057c903  _zend_fetch_debug_backtrace
0002:00003f30  _zend_builtin_module
Module: U:\dev\php-5.3.8\Zend\zend_sprintf.o(zend_sprintf.o)
0001:0057de70  _zend_sprintf
Module: U:\dev\php-5.3.8\Zend\zend_ini.o(zend_ini.o)
0001:0057e09b  _zend_ini_startup
0001:0057e10f  _zend_ini_shutdown
0001:0057e155  _zend_ini_global_shutdown
0001:0057e179  _zend_ini_deactivate
0001:0057e1ff  _zend_copy_ini_directives
0001:0057e2c5  _zend_ini_sort_entries
0001:0057e306  _zend_unregister_ini_entries
0001:0057e331  _zend_register_ini_entries
0001:0057e49b  _zend_ini_refresh_caches
0001:0057e4d3  _zend_alter_ini_entry_ex
0001:0057e6f1  _zend_alter_ini_entry
0001:0057e747  _zend_restore_ini_entry
0001:0057e822  _zend_ini_register_displayer
0001:0057e863  _zend_ini_long
0001:0057e8f4  _zend_ini_double
0001:0057e979  _zend_ini_string_ex
0001:0057ea05  _zend_ini_string
0001:0057ea5b  _zend_ini_boolean_displayer_cb
0001:0057eb6b  _zend_ini_color_displayer_cb
0001:0057ec0c  _display_link_numbers
0001:0057ec74  _OnUpdateBool
0001:0057ed0e  _OnUpdateLong
0001:0057ed4c  _OnUpdateLongGEZero
0001:0057ed95  _OnUpdateReal
0001:0057edd4  _OnUpdateString
0001:0057edfc  _OnUpdateStringUnempty
Module: U:\dev\php-5.3.8\Zend\zend_qsort.o(zend_qsort.o)
0001:0057ee9e  _zend_qsort
Module: U:\dev\php-5.3.8\Zend\zend_ts_hash.o(zend_ts_hash.o)
0001:0057f0ed  __zend_ts_hash_init
0001:0057f145  __zend_ts_hash_init_ex
0001:0057f1ab  _zend_ts_hash_destroy
0001:0057f1e8  _zend_ts_hash_clean
0001:0057f216  __zend_ts_hash_add_or_update
0001:0057f26e  __zend_ts_hash_quick_add_or_update
0001:0057f2cd  __zend_ts_hash_index_update_or_next_insert
0001:0057f31e  _zend_ts_hash_add_empty_element
0001:0057f35a  _zend_ts_hash_graceful_destroy
0001:0057f397  _zend_ts_hash_apply
0001:0057f3d0  _zend_ts_hash_apply_with_argument
0001:0057f416  _zend_ts_hash_apply_with_arguments
0001:0057f45c  _zend_ts_hash_reverse_apply
0001:0057f495  _zend_ts_hash_del_key_or_index
0001:0057f4df  _zend_ts_get_hash_value
0001:0057f515  _zend_ts_hash_find
0001:0057f556  _zend_ts_hash_quick_find
0001:0057f59e  _zend_ts_hash_index_find
0001:0057f5d8  _zend_ts_hash_exists
0001:0057f612  _zend_ts_hash_index_exists
0001:0057f645  _zend_ts_hash_copy
0001:0057f6a6  _zend_ts_hash_copy_to_hash
0001:0057f6f7  _zend_ts_hash_merge
0001:0057f765  _zend_ts_hash_merge_ex
0001:0057f7d3  _zend_ts_hash_sort
0001:0057f81d  _zend_ts_hash_compare
0001:0057f87c  _zend_ts_hash_minmax
0001:0057f8c4  _zend_ts_hash_num_elements
0001:0057f8f0  _zend_ts_hash_rehash
Module: U:\dev\php-5.3.8\Zend\zend_stream.o(zend_stream.o)
0001:0057fabb  _zend_stream_open
0001:0057fb2c  _zend_stream_fixup
0001:0057fece  _zend_file_handle_dtor
0001:0057ff4e  _zend_compare_file_handles
Module: U:\dev\php-5.3.8\Zend\zend_iterators.o(zend_iterators.o)
0001:0058000a  _zend_register_iterator_wrapper
0001:00580132  _zend_iterator_wrap
0001:00580198  _zend_iterator_unwrap
Module: U:\dev\php-5.3.8\Zend\zend_interfaces.o(zend_interfaces.o)
0002:00022318  _zend_ce_serializable
0002:00022328  _zend_ce_aggregate
0002:00022338  _zend_ce_iterator
0002:00022348  _zend_ce_traversable
0002:00022358  _zend_ce_arrayaccess
0001:00580207  _zend_user_it_invalidate_current
0001:00580b4d  _zend_user_serialize
0001:00580a33  _zend_user_unserialize
0001:00581242  _zend_user_it_get_new_iterator
0001:005806e7  _zend_call_method
0001:00580c61  _zend_user_it_rewind
0001:00580cdc  _zend_user_it_move_forward
0001:00580d9d  _zend_user_it_get_current_key
0001:00580f4a  _zend_user_it_get_current_data
0001:00580fce  _zend_user_it_valid
0001:0058118c  _zend_user_it_new_iterator
0001:00581359  _zend_class_serialize_deny
0001:005813cb  _zend_class_unserialize_deny
0001:00581445  _zend_register_interfaces
0001:00581980  _zend_funcs_aggregate
0001:005819b0  _zend_funcs_iterator
0001:00581a60  _zend_funcs_arrayaccess
0001:00581ad0  _zend_funcs_serializable
0002:00004000  _zend_interface_iterator_funcs_iterator
0002:0001c330  _zend_funcs_traversable
Module: U:\dev\php-5.3.8\Zend\zend_exceptions.o(zend_exceptions.o)
0002:00022368  _default_exception_ce
0002:00022378  _error_exception_ce
0002:00022388  _zend_throw_exception_hook
0001:00581e84  _zim_error_exception_getSeverity
0001:00581ed8  _zim_exception_getTrace
0001:00581f31  _zim_exception_getCode
0001:00581f8d  _zim_exception_getMessage
0001:00581fe1  _zim_exception_getLine
0001:00582035  _zim_exception_getFile
0001:00582092  _zim_exception_getPrevious
0001:00582136  _zim_exception_getTraceAsString
0001:00582c79  _zim_error_exception___construct
0001:00582eda  _zim_exception___construct
0001:0058302b  _zend_exception_set_previous
0001:00583115  _zend_exception_save
0001:00583177  _zend_exception_restore
0001:005831d5  _zend_clear_exception
0001:00583259  _zend_spprintf
0001:0058331c  _zim_exception___toString
0001:0058375c  _zend_register_default_exception
0001:00583b1d  _zend_exception_get_default
0001:00583b27  _zend_get_error_exception
0001:00583bd3  _zend_exception_error
0001:00583f4b  _zend_throw_exception_internal
0001:0058406d  _zend_throw_exception
0001:00584177  _zend_throw_error_exception
0001:005841d7  _zend_throw_exception_ex
0001:00584258  _zim_exception___clone
0001:005842fb  _zend_throw_exception_object
Module: U:\dev\php-5.3.8\Zend\zend_strtod.o(zend_strtod.o)
0001:00585280  _zend_startup_strtod
0001:005852a1  _zend_shutdown_strtod
0001:00585336  _zend_freedtoa
0001:00585367  _zend_dtoa
0001:00586306  _zend_strtod
0001:005872f9  _zend_hex_strtod
0001:005873bc  _zend_oct_strtod
Module: U:\dev\php-5.3.8\Zend\zend_gc.o(zend_gc.o)
0002:00022398  _gc_globals_id
0001:00587b40  _gc_globals_ctor
0001:00587b6c  _gc_globals_dtor
0001:00587b71  _gc_reset
0001:00587bcb  _gc_init
0001:00587c1a  _gc_remove_zval_from_buffer
0001:00587c78  _gc_collect_cycles
0001:0058832d  _gc_zobj_possible_root
0001:00588430  _gc_zval_possible_root
Module: U:\dev\php-5.3.8\Zend\zend_closures.o(zend_closures.o)
0002:000223a8  _zend_ce_closure
0001:00588584  _zend_closure_get_closure
0001:005886ec  _zim_Closure___construct
0001:00588865  _zim_Closure___invoke
0001:00588ff3  _zend_get_closure_invoke_method
0001:00589114  _zend_get_closure_method_def
0001:00589139  _zend_register_closure_ce
0001:005892e6  _zend_create_closure
Module: U:\dev\php-5.3.8\Zend\zend_float.o(zend_float.o)
0001:00589400  _zend_init_fpu
0001:00589464  _zend_shutdown_fpu
0001:005894aa  _zend_ensure_fpu_mode
Module: U:\dev\php-5.3.8\Zend\zend_objects.o(zend_objects.o)
0001:0058958d  _zend_objects_destroy_object
0001:0058986e  _zend_object_std_init
0001:005898c1  _zend_object_std_dtor
0001:0058990a  _zend_objects_free_object_storage
0001:00589930  _zend_objects_new
0001:00589988  _zend_objects_get_address
0001:0058999c  _zend_objects_clone_members
0001:00589a91  _zend_objects_clone_obj
Module: U:\dev\php-5.3.8\Zend\zend_object_handlers.o(zend_object_handlers.o)
0001:00589b50  _zend_std_object_get_class
0001:00589b6c  _zend_std_get_properties
0001:00589ca0  _zend_std_get_constructor
0001:00589e10  _zend_std_object_get_class_name
0001:00589e6d  _zend_std_get_closure
0001:0058a0db  _zend_std_callstatic_user_call
0001:0058a307  _zend_std_call_user_call
0001:0058a66a  _zend_std_read_dimension
0001:0058ab80  _zend_std_cast_object_tostring
0001:0058b87e  _zend_std_get_debug_info
0001:0058b936  _zend_get_property_info
0001:0058cb17  _zend_std_read_property
0001:0058ce9c  _zend_check_property_access
0001:0058cf6d  _zend_check_private
0001:0058d031  _zend_check_protected
0001:0058d080  _zend_std_get_static_method
0001:0058d4e6  _zend_std_get_static_property
0001:0058d68d  _zend_std_unset_static_property
0002:00004020  _std_object_handlers
Module: U:\dev\php-5.3.8\Zend\zend_objects_API.o(zend_objects_API.o)
0001:0058d6c0  _zend_objects_store_add_ref
0001:0058d721  _zend_object_proxy_get
0001:0058d7cb  _zend_object_proxy_set
0001:0058d83c  _zend_objects_proxy_clone
0001:0058d87d  _zend_objects_proxy_free_storage
0001:0058d8a7  _zend_objects_store_init
0001:0058d8ed  _zend_objects_store_destroy
0001:0058d90d  _zend_objects_store_call_destructors
0001:0058d978  _zend_objects_store_mark_destructed
0001:0058d9b2  _zend_objects_store_free_object_storage
0001:0058da70  _zend_objects_store_put
0001:0058dbab  _zend_objects_store_clone_obj
0001:0058dc7c  _zend_objects_store_get_refcount
0001:0058dca1  _zend_objects_store_add_ref_by_handle
0001:0058dcf1  _zend_objects_store_del_ref_by_handle_ex
0001:0058df9b  _zend_objects_store_del_ref
0001:0058e002  _zend_object_store_get_object
0001:0058e027  _zend_object_store_get_object_by_handle
0001:0058e04a  _zend_object_store_set_object
0001:0058e072  _zend_object_store_ctor_failed
0001:0058e09d  _zend_object_create_proxy
0001:0058e12e  _zend_get_std_object_handlers
Module: U:\dev\php-5.3.8\Zend\zend_default_classes.o(zend_default_classes.o)
0001:0058e140  _zend_register_default_classes
Module: U:\dev\php-5.3.8\Zend\zend_execute.o(zend_execute.o)
0002:000223b8  _zend_opcode_handlers
0001:0058f431  _execute
0001:005f72ca  _zend_get_compiled_variable_value
0001:005f72db  _execute_internal
0001:005f7330  _zend_init_opcodes_handlers
0001:005f733f  _zend_vm_set_opcode_handler
0001:005f7380  _zend_do_fcall
0001:005f7392  _zend_set_user_opcode_handler
0001:005f73bb  _zend_get_user_opcode_handler
0001:005f73cb  _zend_get_zval_ptr
0001:005f7539  _zend_get_zval_ptr_ptr
Module: U:\tmp\ldconv_libgcc_eh_a_3ed14e78ff52199cf0.lib(emx-dllinit.obj)
0001:005fb2c0  _DLL_InitTerm
Module: U:\usr\lib\libend.lib(src/libend/386/endlink386.asm)
0002:00022440  _end
0002:00008e70  _edata
Module: U:\usr\lib\libend.lib(src/libend/386/end.asm)
0001:00814a80* _etext
0001:00814a80* __etext
0000:00000000* WEAK$ZERO
0002:00022440  __end
0002:00008e70  __edata
Module: U:\tmp\ldconv_libgcc_a_3ed14e78ff521a1dd8.lib(_moddi3.obj)
0001:005fb310  ___moddi3
Module: U:\tmp\ldconv_libgcc_a_3ed14e78ff521a1dd8.lib(_divdi3.obj)
0001:005fb4d0  ___divdi3
Module: U:\tmp\ldconv_libgcc_a_3ed14e78ff521a1dd8.lib(_umoddi3.obj)
0001:005fb620  ___umoddi3
Module: U:\extras\lib\xml2.lib(xmlIO.obj)
0001:005fb767* _xmlFileMatch
0001:005fb8af* _xmlIOFTPMatch
0001:005fb8e2* _xmlIOHTTPMatch
0001:005fba4c* _xmlIOHTTPClose
0001:005fba94* _xmlIOFTPClose
0001:005fbaa0* _xmlIOFTPRead
0001:005fbacd* _xmlIOFTPOpen
0001:005fbad9* _xmlIOHTTPRead
0001:005fbb06* _xmlIOHTTPOpen
0001:005fbb21  ___xmlIOErr
0001:005fc7a9* _xmlFileClose
0001:005fc828* _xmlFileRead
0001:005fc879  ___xmlLoaderErr
0001:005fc989* _xmlNormalizeWindowsPath
0001:005fc995  _xmlCleanupInputCallbacks
0001:005fc9ee* _xmlPopInputCallbacks
0001:005fca40  _xmlCleanupOutputCallbacks
0001:005fca9a* _xmlCheckFilename
0001:005fce39* _xmlFileOpen
0001:005fce8a* _xmlRegisterInputCallbacks
0001:005fcedc* _xmlRegisterOutputCallbacks
0001:005fcf2e  _xmlRegisterDefaultInputCallbacks
0001:005fcfdc  _xmlRegisterDefaultOutputCallbacks
0001:005fd041* _xmlRegisterHTTPPostCallbacks
0001:005fd092  _xmlAllocParserInputBuffer
0001:005fd152  ___xmlParserInputBufferCreateFilename
0001:005fd26d  _xmlAllocOutputBuffer
0001:005fd32f  _xmlAllocOutputBufferInternal
0001:005fd3ee  _xmlFreeParserInputBuffer
0001:005fd45a  _xmlParserInputBufferCreateFilename
0001:005fd490* _xmlParserInputBufferCreateFile
0001:005fd4d6  _xmlOutputBufferCreateFile
0001:005fd51c  _xmlParserInputBufferCreateFd
0001:005fd551  _xmlParserInputBufferCreateMem
0001:005fd5b9  _xmlParserInputBufferCreateStatic
0001:005fd685  _xmlOutputBufferCreateFd
0001:005fd6ba  _xmlParserInputBufferCreateIO
0001:005fd6ed  _xmlOutputBufferCreateIO
0001:005fd720  _xmlOutputBufferCreateBuffer
0001:005fd750  _xmlParserInputBufferCreateFilenameDefault
0001:005fd77b  _xmlOutputBufferCreateFilenameDefault
0001:005fe86c  ___xmlOutputBufferCreateFilename
0001:005fd7a6  _xmlParserInputBufferPush
0001:005fd88e  _xmlParserInputBufferGrow
0001:005fda1a  _xmlParserInputBufferRead
0001:005fda57  _xmlOutputBufferWrite
0001:005fde83  _xmlOutputBufferWriteEscape
0001:005fe159  _xmlOutputBufferWriteString
0001:005fe1a7  _xmlOutputBufferFlush
0001:005fe2a0  _xmlOutputBufferClose
0001:005fe7bc* _xmlIOHTTPOpenW
0001:005feb2c  _xmlOutputBufferCreateFilename
0001:005feb92  _xmlParserGetDirectory
0001:005feca7  _xmlCheckHTTPInput
0001:005fee36* _xmlSetExternalEntityLoader
0001:005fee43* _xmlGetExternalEntityLoader
0001:005fee66  _xmlLoadExternalEntity
0001:005feee2* _xmlNoNetExternalEntityLoader
Module: U:\extras\lib\xml2.lib(uri.obj)
0001:005ff9b8  _xmlCreateURI
0001:005ffa2e  _xmlSaveUri
0001:00600825* _xmlPrintURI
0001:00600864  _xmlFreeURI
0001:0060091a* _xmlNormalizeURIPath
0001:00600b91  _xmlURIUnescapeString
0001:00601cae  _xmlParseURIReference
0001:00601cc0  _xmlParseURIRaw
0001:00601d0b  _xmlParseURI
0001:00601d68  _xmlURIEscapeStr
0001:00601f7f  _xmlURIEscape
0001:006022fd  _xmlBuildURI
0001:006027d0  _xmlBuildRelativeURI
0001:00602be4  _xmlCanonicPath
0001:00602caa  _xmlPathToURI
Module: U:\extras\lib\xml2.lib(xmlstring.obj)
0001:00602d20  _xmlStrndup
0001:00602d8c  _xmlStrdup
0001:00602dba  _xmlCharStrndup
0001:00602e36  _xmlCharStrdup
0001:00602e64  _xmlStrcmp
0001:00602eb6  _xmlStrEqual
0001:00602ef2  _xmlStrQEqual
0001:00602f5f  _xmlStrncmp
0001:00602fa7  _xmlStrcasecmp
0001:00603007  _xmlStrncasecmp
0001:00603072  _xmlStrchr
0001:00603094  _xmlStrstr
0001:006030fb  _xmlStrcasestr
0001:00603173* _xmlStrsub
0001:006031ca  _xmlStrlen
0001:006031e6  _xmlStrncat
0001:00603295  _xmlStrncatNew
0001:0060338f  _xmlStrcat
0001:006033d5  _xmlStrPrintf
0001:0060341d* _xmlStrVPrintf
0001:00603465* _xmlUTF8Size
0001:006034a8* _xmlUTF8Charcmp
0001:006034e7  _xmlUTF8Strlen
0001:0060358d  _xmlGetUTF8Char
0001:006036d1  _xmlCheckUTF8
0001:006037ab  _xmlUTF8Strsize
0001:0060380b  _xmlUTF8Strndup
0001:0060389f  _xmlUTF8Strpos
0001:006038f7  _xmlUTF8Strloc
0001:00603998  _xmlUTF8Strsub
Module: U:\extras\lib\xml2.lib(globals.obj)
0002:000223d0+ _xmlLastError
0001:00603b30  _xmlInitGlobals
0001:00603b4d  _xmlCleanupGlobals
0001:00603b7a  _xmlInitializeGlobalState
0001:00603d3f* _xmlThrDefSetGenericErrorFunc
0001:00603d89* _xmlThrDefSetStructuredErrorFunc
0001:00603dc3* _xmlRegisterNodeDefault
0001:00603de0* _xmlThrDefRegisterNodeDefault
0001:00603e21* _xmlDeregisterNodeDefault
0001:00603e3e* _xmlThrDefDeregisterNodeDefault
0001:00603e7f* _xmlThrDefParserInputBufferCreateFilenameDefault
0001:00603ec1* _xmlThrDefOutputBufferCreateFilenameDefault
0001:00603f03  ___docbDefaultSAXHandler
0001:00603f27  ___htmlDefaultSAXHandler
0001:00603f4b  ___xmlLastError
0001:00603f71* ___oldXMLWDcompatibility
0001:00603f95  ___xmlBufferAllocScheme
0001:00603fb9* _xmlThrDefBufferAllocScheme
0001:00603ff0  ___xmlDefaultBufferSize
0001:00604014* _xmlThrDefDefaultBufferSize
0001:0060404b  ___xmlDefaultSAXHandler
0001:00604071  ___xmlDefaultSAXLocator
0001:00604093  ___xmlDoValidityCheckingDefaultValue
0001:006040b7* _xmlThrDefDoValidityCheckingDefaultValue
0001:006040ee  ___xmlGenericError
0001:00604112  ___xmlStructuredError
0001:00604136  ___xmlGenericErrorContext
0001:0060415a  ___xmlStructuredErrorContext
0001:0060417e  ___xmlGetWarningsDefaultValue
0001:006041a2* _xmlThrDefGetWarningsDefaultValue
0001:006041d9  ___xmlIndentTreeOutput
0001:006041fd* _xmlThrDefIndentTreeOutput
0001:00604234  ___xmlTreeIndentString
0001:00604258* _xmlThrDefTreeIndentString
0001:0060428f  ___xmlKeepBlanksDefaultValue
0001:006042b3* _xmlThrDefKeepBlanksDefaultValue
0001:006042ea  ___xmlLineNumbersDefaultValue
0001:0060430e* _xmlThrDefLineNumbersDefaultValue
0001:00604345  ___xmlLoadExtDtdDefaultValue
0001:00604369* _xmlThrDefLoadExtDtdDefaultValue
0001:006043a0  ___xmlParserDebugEntities
0001:006043c4* _xmlThrDefParserDebugEntities
0001:006043fb  ___xmlParserVersion
0001:00604421  ___xmlPedanticParserDefaultValue
0001:00604445* _xmlThrDefPedanticParserDefaultValue
0001:0060447c  ___xmlSaveNoEmptyTags
0001:006044a1* _xmlThrDefSaveNoEmptyTags
0001:006044d8  ___xmlSubstituteEntitiesDefaultValue
0001:006044fc* _xmlThrDefSubstituteEntitiesDefaultValue
0001:00604533  ___xmlRegisterNodeDefaultValue
0001:00604557  ___xmlDeregisterNodeDefaultValue
0001:0060457b  ___xmlParserInputBufferCreateFilenameValue
0001:006045a1  ___xmlOutputBufferCreateFilenameValue
0002:000045f0* _docbDefaultSAXHandler
0002:00004580* _htmlDefaultSAXHandler
0002:000044d8* _xmlBufferAllocScheme
0002:000044dc* _xmlDefaultBufferSize
0002:00004500* _xmlDefaultSAXHandler
0002:00004570* _xmlDefaultSAXLocator
0002:000044e8* _xmlGenericError
0002:000044e0* _xmlGetWarningsDefaultValue
0002:000044ec* _xmlIndentTreeOutput
0002:000044f0* _xmlTreeIndentString
0002:000044e4* _xmlKeepBlanksDefaultValue
0002:000044d4* _xmlParserVersion
0002:000044c0  _xmlFree
0002:000044c4  _xmlMalloc
0002:000044c8  _xmlMallocAtomic
0002:000044cc  _xmlRealloc
0002:000044d0  _xmlMemStrdup
0002:0001cacc* _xmlRegisterNodeDefaultValue
0002:0001cad0* _xmlDeregisterNodeDefaultValue
0002:0001cab0* _oldXMLWDcompatibility
0002:0001cab8* _xmlDoValidityCheckingDefaultValue
0002:0001cadc* _xmlStructuredError
0002:0001cae0* _xmlGenericErrorContext
0002:0001cae4* _xmlStructuredErrorContext
0002:0001cac4* _xmlLineNumbersDefaultValue
0002:0001cabc* _xmlLoadExtDtdDefaultValue
0002:0001cab4* _xmlParserDebugEntities
0002:0001cac0* _xmlPedanticParserDefaultValue
0002:0001cae8* _xmlSaveNoEmptyTags
0002:0001cac8* _xmlSubstituteEntitiesDefaultValue
0002:0001cad4* _xmlParserInputBufferCreateFilenameValue
0002:0001cad8* _xmlOutputBufferCreateFilenameValue
Module: U:\extras\lib\xml2.lib(error.obj)
0001:00604f40  _xmlGenericErrorDefaultFunc
0001:00604f84  _initGenericErrorDefaultFunc
0001:00604fb2  _xmlSetGenericErrorFunc
0001:00604fe8  _xmlSetStructuredErrorFunc
0001:00605004* _xmlParserPrintFileInfo
0001:00605076* _xmlParserPrintFileContext
0001:006050ab  _xmlParserValidityWarning
0001:0060526c  _xmlParserValidityError
0001:0060545d  _xmlParserWarning
0001:00605649  _xmlParserError
0001:00605829  _xmlGetLastError
0001:00605845  _xmlResetError
0001:006058bd  _xmlResetLastError
0001:006058e1* _xmlCtxtGetLastError
0001:00605901* _xmlCtxtResetLastError
0001:0060592f  _xmlCopyError
0001:00605a60  ___xmlRaiseError
0001:006060bd  ___xmlSimpleError
Module: U:\extras\lib\xml2.lib(tree.obj)
0001:006067b7  _xmlBuildQName
0001:00606891  _xmlSplitQName2
0001:0060694a  _xmlSplitQName3
0001:006069aa  _xmlValidateNCName
0001:00606d10  _xmlValidateQName
0001:006072cc  _xmlValidateName
0001:00607648  _xmlValidateNMToken
0001:00607a69* _xmlSetBufferAllocationScheme
0001:00607a8b* _xmlGetBufferAllocationScheme
0001:00607a9a  _xmlSetNs
0001:00607aac  _xmlFreeNs
0001:00607b02  _xmlNewNs
0001:0060807a  _xmlFreeNsList
0001:006080ad  _xmlNewDtd
0001:00608182  _xmlGetIntSubset
0001:006081c4  _xmlCreateIntSubset
0001:006083c9  _xmlNewDoc
0001:0060849b  _xmlNodeListGetString
0001:0060863a* _xmlNodeListGetRawString
0001:0060876b  _xmlNewDocPI
0001:00608835  _xmlNewPI
0001:00608865  _xmlNewNode
0001:006088ec* _xmlNewNodeEatName
0001:0060897d  _xmlNewDocFragment
0001:006089fb  _xmlNewText
0001:00610f73  _xmlStringText
0001:00608a9e  _xmlNewCharRef
0001:00608b77  _xmlNewReference
0001:00608c60  _xmlNewDocText
0001:00608ec7  _xmlNewNsPropEatName
0001:00608efa  _xmlNewNsProp
0001:00608f2d  _xmlNewProp
0001:00608f56  _xmlNewTextLen
0001:00608fe3* _xmlNewDocTextLen
0001:00609018  _xmlNewComment
0001:00610f82  _xmlStringComment
0001:006090ad  _xmlNewCDataBlock
0001:00609139  _xmlNewDocComment
0001:00609156* _xmlSetListDoc
0001:00609187  _xmlSetTreeDoc
0001:006091e5  _xmlGetLastChild
0001:006091f6* _xmlChildElementCount
0001:0060923f* _xmlFirstElementChild
0001:00609284* _xmlLastElementChild
0001:006092ca* _xmlPreviousElementSibling
0001:0060934f* _xmlNextElementSibling
0001:006093d3  _xmlUnlinkNode
0001:006095b0  _xmlFreeDoc
0001:00609c85  _xmlFreeDtd
0001:00609785  _xmlFreeNodeList
0001:00609a5c  _xmlFreePropList
0001:00609930  _xmlFreeProp
0001:006099d8* _xmlRemoveProp
0001:00609a83  _xmlFreeNode
0001:00609e04  _xmlReplaceNode
0001:00609ee5* _xmlCopyNamespace
0001:00609f18  _xmlCopyNamespaceList
0001:00609f64  _xmlGetLineNo
0001:0060a027  _xmlGetNodePath
0001:0060a81f  _xmlDocGetRootElement
0001:0060a844  _xmlNodeSetName
0001:0060a948  _xmlGetNsList
0001:0060ad1e  _xmlSearchNs
0001:0060aedf  _xmlSearchNsByHref
0001:0060b270  _xmlReconciliateNs
0001:0060b5b7  _xmlHasProp
0001:0060b670  _xmlHasNsProp
0001:0060b68c  _xmlAddChild
0001:0060b959  _xmlNodeAddContent
0001:0060b823  _xmlNodeAddContentLen
0001:0060b98e* _xmlTextMerge
0001:0060b9eb  _xmlAddChildList
0001:0060bb8d  _xmlAddSibling
0001:0060bc84  _xmlDocSetRootElement
0001:0060bd0a  _xmlAddNextSibling
0001:0060c24b  _xmlNodeSetContent
0001:0060be28  _xmlStringGetNodeList
0001:0060c37d  _xmlNewDocNodeEatName
0001:0060c41f  _xmlNewDocNode
0001:0060c4c1  _xmlNewChild
0001:0060c5ab* _xmlNewDocRawNode
0001:0060c62a  _xmlNewTextChild
0001:0060c714  _xmlNewDocProp
0001:0060ca5d* _xmlCopyProp
0001:0060ca71  _xmlCopyPropList
0001:00610f78  _xmlStringTextNoenc
0001:0060d17f  _xmlCopyDoc
0001:0060cf04  _xmlDocCopyNode
0001:0060cf1e  _xmlCopyNode
0001:0060cf37  _xmlCopyDtd
0001:0060d27a  _xmlCopyNodeList
0001:0060d28d  _xmlDocCopyNodeList
0001:0060d2a1  _xmlStringLenGetNodeList
0001:0060d72a  _xmlNodeSetContentLen
0001:0060d86f  _xmlAddPrevSibling
0001:0060d984  _xmlGetProp
0001:0060d9aa  _xmlGetNoNsProp
0001:0060d9d2  _xmlGetNsProp
0001:0060da23  _xmlNodeGetBase
0001:0060dc61  _xmlNodeGetSpacePreserve
0001:0060dd05  _xmlNodeGetLang
0001:0060dd40  _xmlUnsetProp
0001:0060dd7e* _xmlUnsetNsProp
0001:0060ddc6  _xmlSetNsProp
0001:0060df23  _xmlSetProp
0001:0060dfdc  _xmlNodeSetBase
0001:0060e0ff* _xmlNodeSetSpacePreserve
0001:0060e186* _xmlNodeSetLang
0001:0060e1db  _xmlNodeIsText
0001:0060e1f2  _xmlIsBlankNode
0001:0060e244  _xmlTextConcat
0001:0060e308  _xmlBufferCreate
0001:0060e384  _xmlBufferCreateSize
0001:0060e415  _xmlBufferCreateStatic
0001:0060e470* _xmlBufferSetAllocationScheme
0001:0060e492  _xmlBufferFree
0001:0060e4e3  _xmlBufferEmpty
0001:0060e527  _xmlBufferShrink
0001:0060e5fb  _xmlBufferGrow
0001:0060e6a6* _xmlBufferDump
0001:0060e6ec  _xmlBufferContent
0001:0060e6fc  _xmlBufferLength
0001:0060e70d  _xmlBufferResize
0001:0060e850  _xmlBufferAdd
0001:0060e906  _xmlBufferAddHead
0001:0060ea01  _xmlBufferCat
0001:0060ea38  _xmlNodeBufGetContent
0001:0060ec33  _xmlNodeGetContent
0001:0060ed5f  _xmlBufferCCat
0001:0060ede3  _xmlBufferWriteCHAR
0001:0060edfe  _xmlBufferWriteChar
0001:0060ee24  _xmlBufferWriteQuotedString
0001:0060ef48* _xmlGetDocCompressMode
0001:0060ef5c  _xmlSetDocCompressMode
0001:0060ef89  _xmlGetCompressMode
0001:0060ef93* _xmlSetCompressMode
0001:0060efe3* _xmlDOMWrapNewCtxt
0001:0060f02c* _xmlDOMWrapFreeCtxt
0001:0060f05b* _xmlDOMWrapRemoveNode
0001:0060f22f* _xmlDOMWrapReconcileNamespaces
0001:0060f75c* _xmlDOMWrapCloneNode
0001:00610143* _xmlDOMWrapAdoptNode
0002:0001cbf0  ___xmlRegisterCallbacks
Module: U:\extras\lib\xml2.lib(parser.obj)
0001:00613678* _xmlHasFeature
0001:00613691  _xmlCheckLanguageID
0001:00613942  _inputPush
0001:00613aee  _inputPop
0001:00613b73  _nodePush
0001:00613c16  _nodePop
0001:00613c5d* _namePush
0001:00613d03* _namePop
0001:00613d6e  _xmlPopInput
0001:00613ebf  _xmlPushInput
0001:00613fcc  _xmlSplitQName
0001:006144a8* _xmlParsePubidLiteral
0001:0061472e* _xmlParseVersionNum
0001:0061487b* _xmlParseEncName
0001:00614a94* _xmlParseEncodingDecl
0001:0061ad8c* _xmlSkipBlankChars
0001:0061500b  _xmlParserHandlePEReference
0001:00614d4a* _xmlParseTextDecl
0001:0061de3d* _xmlParseVersionInfo
0001:00617663* _xmlParseName
0001:006155c6* _xmlParseCDSect
0001:00615b8f* _xmlParseComment
0001:00616bc5* _xmlParseCharData
0001:00616fab* _xmlParseSystemLiteral
0001:00617343* _xmlParseNmtoken
0001:0061827c* _xmlParseEntityRef
0001:006185a4* _xmlParsePITarget
0001:00618859  _xmlStringLenDecodeEntities
0001:00619763  _xmlStringDecodeEntities
0001:0061981c* _xmlParseEntityValue
0001:00619c93* _xmlParseCharRef
0001:0061ad63* _xmlParseAttValue
0001:0061c47d* _xmlParseAttribute
0001:0061c62c* _xmlParseStartTag
0001:0061d3d4* _xmlParseElementChildrenContentDecl
0001:0061d429* _xmlParseEnumerationType
0001:0061d66a* _xmlParseNotationType
0001:0061de2c* _xmlParseEndTag
0001:0061dfc9* _xmlParseElementMixedContentDecl
0001:0061e43e* _xmlParseElementContentDecl
0001:0061e657* _xmlParseElementDecl
0001:0061e9f9* _xmlParseEnumeratedType
0001:0061eaf3* _xmlParseAttributeType
0001:0061ef0b* _xmlParseDefaultDecl
0001:0061f2a2* _xmlParseAttributeListDecl
0001:0061fb24* _xmlParsePI
0001:006202ac* _xmlParseExternalID
0001:006205bd* _xmlParseDocTypeDecl
0001:006208c6* _xmlParseEntityDecl
0001:0062120c* _xmlParseNotationDecl
0001:006214bf* _xmlParsePEReference
0001:00621e51* _xmlParseMarkupDecl
0001:00622097  _xmlParseExternalSubset
0001:00622369* _xmlParseSDDecl
0001:006226bc* _xmlParseXMLDecl
0001:00622a63* _xmlParseMisc
0001:00622b04  _xmlCreatePushParserCtxt
0001:00622dc3  _xmlStopParser
0001:00622df8* _xmlCreateIOParserCtxt
0001:00622f22* _xmlIOParseDTD
0001:00623180* _xmlSAXParseDTD
0001:006233f9  _xmlParseDTD
0001:0062341b* _xmlCreateEntityParserCtxt
0001:00623457* _xmlCreateURLParserCtxt
0001:0062350e  _xmlCreateFileParserCtxt
0001:0062354f* _xmlSetupParserForBuffer
0001:006235e7  _xmlCreateMemoryParserCtxt
0001:00626292* _xmlParseContent
0001:00623b7a* _xmlParseReference
0001:00625ec8  _xmlParseChunk
0001:0062722d* _xmlParseElement
0001:0062694a* _xmlParseExternalEntity
0001:006269b6  _xmlParseCtxtExternalEntity
0001:00626ee0* _xmlParseExtParsedEnt
0001:0062713b* _xmlSAXParseEntity
0001:006271ba* _xmlParseEntity
0001:00627685* _xmlParseBalancedChunkMemoryRecover
0001:00627a5b  _xmlParseBalancedChunkMemory
0001:00627a99  _xmlParseInNodeContext
0001:00627ef5* _xmlCreateDocParserCtxt
0001:00627f1f* _xmlSetEntityReferenceFunc
0001:00627f2c  _xmlInitParser
0001:00627fe7  _xmlParseDocument
0001:00628516* _xmlSAXParseDoc
0001:006285a7* _xmlParseDoc
0001:006285ca* _xmlRecoverDoc
0001:006285ed* _xmlSAXUserParseFile
0001:00628697* _xmlSAXUserParseMemory
0001:0062874d* _xmlSAXParseMemoryWithData
0001:006287f3* _xmlSAXParseMemory
0001:00628823* _xmlRecoverMemory
0001:0062884d* _xmlParseMemory
0001:00628877* _xmlSAXParseFileWithData
0001:0062894f* _xmlSAXParseFile
0001:00628978* _xmlRecoverFile
0001:0062899b* _xmlParseFile
0001:006289be  _xmlCleanupParser
0001:00628a16  _xmlCtxtReset
0001:00628d43* _xmlCtxtResetPush
0001:00628fb8  _xmlCtxtUseOptions
0001:00628fcc* _xmlReadDoc
0001:00629015  _xmlReadFile
0001:00629058  _xmlReadMemory
0001:006290a4* _xmlReadFd
0001:00629166* _xmlReadIO
0001:0062922a* _xmlCtxtReadDoc
0001:006292a0  _xmlCtxtReadFile
0001:00629315  _xmlCtxtReadMemory
0001:006293cd* _xmlCtxtReadFd
0001:0062947f* _xmlCtxtReadIO
0002:00004680* _xmlParserMaxDepth
Module: U:\extras\lib\xml2.lib(relaxng.obj)
0001:00638e8c  _xmlRelaxNGFree
0001:00638f7d* _xmlRelaxParserSetFlag
0001:00638fe8* _xmlRelaxNGInitTypes
0001:006390a4  _xmlRelaxNGCleanupTypes
0001:006390ed  _xmlRelaxNGNewParserCtxt
0001:00639153  _xmlRelaxNGNewMemParserCtxt
0001:006391c8* _xmlRelaxNGNewDocParserCtxt
0001:00639246  _xmlRelaxNGFreeParserCtxt
0001:006393bb  _xmlRelaxNGParse
0001:00639668  _xmlRelaxNGSetParserErrors
0001:0063968c* _xmlRelaxNGGetParserErrors
0001:006396c6* _xmlRelaxNGSetParserStructuredErrors
0001:00639806* _xmlRelaxNGDump
0001:00639a81* _xmlRelaxNGDumpTree
0001:00639aec  _xmlRelaxNGValidatePushElement
0001:00639c23  _xmlRelaxNGValidatePushCData
0001:00639cc6  _xmlRelaxNGValidatePopElement
0001:00639d5c  _xmlRelaxNGValidateFullElement
0001:00639df2  _xmlRelaxNGNewValidCtxt
0001:00639e8c  _xmlRelaxNGFreeValidCtxt
0001:00639f69  _xmlRelaxNGSetValidErrors
0001:00639f8d  _xmlRelaxNGSetValidStructuredErrors
0001:00639fb2* _xmlRelaxNGGetValidErrors
0001:00639fec  _xmlRelaxNGValidateDoc
Module: U:\extras\lib\xml2.lib(valid.obj)
0001:0063bb5d  _xmlNewValidCtxt
0001:0063bb9a  _xmlFreeValidCtxt
0001:0063bc23  _xmlNewDocElementContent
0001:0063bdb5* _xmlNewElementContent
0001:0063bdd7* _xmlCopyDocElementContent
0001:0063bfec* _xmlCopyElementContent
0001:0063c0a6  _xmlFreeDocElementContent
0001:0063c20e* _xmlFreeElementContent
0001:0063c229* _xmlSprintfElementContent
0001:0063c22e  _xmlSnprintfElementContent
0001:0063c598* _xmlValidBuildContentModel
0001:0063cf6f  _xmlAddElementDecl
0001:0063d3eb  _xmlFreeElementTable
0001:0063d406  _xmlCopyElementTable
0001:0063d475  _xmlDumpElementDecl
0001:0063d609* _xmlDumpElementTable
0001:0063d635  _xmlCreateEnumeration
0001:0063d686  _xmlFreeEnumeration
0001:0063d807* _xmlCopyEnumeration
0001:0063da11  _xmlAddAttributeDecl
0001:0063dfdc  _xmlFreeAttributeTable
0001:0063dff7  _xmlCopyAttributeTable
0001:0063e0ba  _xmlDumpAttributeDecl
0001:0063e332* _xmlDumpAttributeTable
0001:0063e3b4  _xmlAddNotationDecl
0001:0063e4ee  _xmlFreeNotationTable
0001:0063e509  _xmlCopyNotationTable
0001:0063e546* _xmlDumpNotationDecl
0001:0063e604  _xmlDumpNotationTable
0001:0063e669  _xmlAddID
0001:0063e7ea  _xmlFreeIDTable
0001:0063e805  _xmlRemoveID
0001:0063e8a9  _xmlGetID
0001:0063ecad  _xmlAddRef
0001:0063ee70  _xmlFreeRefTable
0001:0063ee8b* _xmlRemoveRef
0001:0063ef5d* _xmlGetRefs
0001:0063ef85* _xmlGetDtdElementDesc
0001:0063f00b  _xmlGetDtdQElementDesc
0001:0063f172  _xmlGetDtdAttrDesc
0001:0063f219  _xmlIsRef
0001:0063f2d1  _xmlIsID
0001:0063f583  _xmlGetDtdQAttrDesc
0001:0063f5bf* _xmlGetDtdNotationDesc
0001:0063fbfe  _xmlValidateNotationUse
0001:0063fceb  _xmlIsMixedElement
0001:0063fd53* _xmlValidateNameValue
0001:0063fd64* _xmlValidateNamesValue
0001:0063fd75* _xmlValidateNmtokenValue
0001:0063fd86* _xmlValidateNmtokensValue
0001:0063fd97  _xmlValidateNotationDecl
0001:0063fda1* _xmlValidateAttributeValue
0001:0063fe0e  _xmlValidCtxtNormalizeAttributeValue
0001:00640034  _xmlValidNormalizeAttributeValue
0001:0064032f  _xmlValidateAttributeDecl
0001:00640680  _xmlValidateElementDecl
0001:00640b73  _xmlValidateOneAttribute
0001:006414c2  _xmlValidateOneNamespace
0001:00641dac  _xmlValidatePushElement
0001:00642252  _xmlValidatePushCData
0001:00642376  _xmlValidatePopElement
0001:0064271d  _xmlValidateOneElement
0001:006431da  _xmlValidateRoot
0001:0064334c  _xmlValidateElement
0001:006434e3  _xmlValidateDocumentFinal
0001:00643542  _xmlValidateDtd
0001:006435f0  _xmlValidateDtdFinal
0001:00643729  _xmlValidateDocument
0001:006438c1* _xmlValidGetPotentialChildren
0001:006439e3* _xmlValidGetValidElements
Module: U:\tmp\ldconv_libgcc_a_3ed14e78ff521a1dd8.lib(_alloca.obj)
0001:00643cf0  __alloca
Module: U:\tmp\ldconv_libgcc_a_3ed14e78ff521a1dd8.lib(_udivdi3.obj)
0001:00643d20  ___udivdi3
Module: U:\extras\lib\libz.lib(deflate.obj)
0001:00643e30* _deflateSetHeader
0001:00643e5c* _deflatePrime
0001:00643e94* _deflateTune
0001:00643ed4* _deflateBound
0001:00644004  _deflateEnd
0001:006440d4* _deflateCopy
0001:006442e0* _deflateSetDictionary
0001:0064467c  _deflateReset
0001:006447f4  _deflateInit2_
0001:00644a54  _deflateInit_
0001:00645b6c  _deflate
0001:00646b9c  _deflateParams
0001:00646c90* _deflate_copyright
Module: U:\extras\lib\libz.lib(crc32.obj)
0001:00646d60* _get_crc_table
0001:00646d6c  _crc32
0001:006472b0* _crc32_combine
0001:006472bc* _crc32_combine64
Module: U:\extras\lib\libz.lib(zutil.obj)
0001:006492d8  _zlibVersion
0001:006492e4* _zlibCompileFlags
0001:006492f0  _zError
0001:006493b0  _z_errmsg
0001:00649304  _zcfree
0001:00649318  _zcalloc
Module: U:\extras\lib\libz.lib(inflate.obj)
0001:006493e0  _inflateReset
0001:0064948c* _inflatePrime
0001:006494f0  _inflateEnd
0001:0064954c* _inflateGetHeader
0001:0064957c* _inflateSync
0001:00649728* _inflateSyncPoint
0001:0064975c* _inflateUndermine
0001:00649788* _inflateMark
0001:006497d4* _inflateCopy
0001:00649a84* _inflateSetDictionary
0001:00649d40  _inflate
0001:0064bc0c* _inflateReset2
0001:0064bd3c  _inflateInit2_
0001:0064be04  _inflateInit_
Module: U:\extras\lib\libz.lib(uncompr.obj)
0001:0064c788  _uncompress
Module: U:\extras\lib\libz.lib(compress.obj)
0001:0064c840* _compressBound
0001:0064c864  _compress2
0001:0064c918  _compress
Module: U:\extras\lib\libz.lib(gzlib.obj)
0001:0064c9d0* _gzbuffer
0001:0064ca0c* _gztell64
0001:0064ca60* _gztell
0001:0064cab4  _gzeof
0001:0064cae8* _gzerror
0001:0064cb38  _gz_error
0001:0064cc04* _gzoffset64
0001:0064d03c  _gzdopen
0001:0064d0a4* _gzopen64
0001:0064d0c8  _gzopen
0001:0064d0ec* _gzrewind
0001:0064d194* _gzseek64
0001:0064d360  _gzseek
0001:0064d36c* _gzclearerr
0001:0064d3a0* _gzoffset
Module: U:\extras\lib\libz.lib(gzclose.obj)
0001:0064d410  _gzclose
Module: U:\extras\lib\libz.lib(gzwrite.obj)
0001:0064d8a4  _gzclose_w
0001:0064d974  _gzflush
0001:0064d9f0* _gzsetparams
0001:0064daa4* _gzprintf
0001:0064dbc8  _gzwrite
0001:0064dd68* _gzputs
0001:0064ddb0* _gzputc
Module: U:\extras\lib\libz.lib(gzread.obj)
0001:0064de60  _gzclose_r
0001:0064e5b4  _gzdirect
0001:0064ec00* _gzgets
0001:0064ed3c* _gzungetc
0001:0064ee5c  _gzread
0001:0064efe0* _gzgetc
Module: U:\extras\lib\xml2.lib(xpath.obj)
0001:0064f657* _xmlXPathNextSelf
0001:0064f678* _xmlXPathNextChild
0001:0064f721* _xmlXPathNextDescendant
0001:0064f7ab* _xmlXPathNextDescendantOrSelf
0001:0064f7ee* _xmlXPathNextFollowingSibling
0001:0064f832* _xmlXPathNextPrecedingSibling
0001:0064f883* _xmlXPathNextFollowing
0001:0064f997* _xmlXPathNextAttribute
0001:0064fff6* _xmlXPathNodeSetAddUnique
0001:006502cd* _xmlXPathNextAncestor
0001:006504c0* _xmlXPathNextAncestorOrSelf
0001:006504f9* _xmlXPathNextParent
0001:006511a7* _xmlXPathNextNamespace
0001:006513ac  _xmlXPathInit
0001:006514b3  _xmlXPathIsNaN
0001:0065151c* _xmlXPathIsInf
0001:00651558  _xmlXPathErr
0001:00651e3d* _xmlXPatherror
0001:0065208f  _xmlXPathDebugDumpObject
0001:006536b7* _xmlXPathDebugDumpCompExpr
0001:0065376f* _xmlXPathContextSetCache
0001:00653855  _valuePop
0001:006538ae  _valuePush
0001:00653933* _xmlXPathOrderDocElems
0001:0065398c  _xmlXPathCmpNodes
0001:00653c18* _xmlXPathNodeSetSort
0001:00653cfe* _xmlXPathNodeSetFreeNs
0001:00653e21* _xmlXPathNodeSetCreate
0001:006542bf  _xmlXPathNodeSetContains
0001:00654362* _xmlXPathNodeSetAddNs
0001:006544af* _xmlXPathNodeSetAdd
0001:00654695* _xmlXPathNodeSetMerge
0001:0065483b* _xmlXPathNodeSetDel
0001:006548b8* _xmlXPathNodeSetRemove
0001:00654914* _xmlXPathFreeNodeSet
0001:00654985  _xmlXPathFreeObject
0001:00654a18* _xmlXPathFreeCompExpr
0001:00654dab* _xmlXPathPopExternal
0001:00654e40* _xmlXPathPopNodeSet
0001:00654ec2  _xmlXPathNewNodeSet
0001:00655399* _xmlXPathNewValueTree
0001:006553fa* _xmlXPathNewNodeSetList
0001:00655492* _xmlXPathWrapNodeSet
0001:0065552a* _xmlXPathFreeNodeSetList
0001:00655541* _xmlXPathDifference
0001:006555fc* _xmlXPathIntersection
0001:006556b4* _xmlXPathHasSameNodes
0001:0065573c* _xmlXPathNodeLeadingSorted
0001:006557e8* _xmlXPathNodeLeading
0001:0065580f* _xmlXPathLeadingSorted
0001:0065584d* _xmlXPathLeading
0001:006558c6* _xmlXPathNodeTrailingSorted
0001:0065597f* _xmlXPathNodeTrailing
0001:006559a6* _xmlXPathTrailingSorted
0001:006559e2* _xmlXPathTrailing
0001:00655a5b  _xmlXPathRegisterFuncNS
0001:00655ae1  _xmlXPathRegisterFunc
0001:00655b0a* _xmlXPathRegisterFuncLookup
0001:00655b22* _xmlXPathFunctionLookupNS
0001:00655b81* _xmlXPathFunctionLookup
0001:00655bd6* _xmlXPathRegisteredFuncsCleanup
0001:00655c04* _xmlXPathRegisterVariableNS
0001:00655c98* _xmlXPathRegisterVariable
0001:00655cc1* _xmlXPathRegisterVariableLookup
0001:00655cd9* _xmlXPathRegisteredVariablesCleanup
0001:00655d07  _xmlXPathRegisterNs
0001:00655dc9* _xmlXPathNsLookup
0001:00655e76* _xmlXPathRegisteredNsCleanup
0001:00655ebc* _xmlXPathNewFloat
0001:00655f77* _xmlXPathCountFunction
0001:00656074* _xmlXPathPositionFunction
0001:006560dc* _xmlXPathLastFunction
0001:0065615d  _xmlXPathNewBoolean
0001:0065621e* _xmlXPathFalseFunction
0001:00656264* _xmlXPathTrueFunction
0001:006562c5  _xmlXPathNewString
0001:006563c9* _xmlXPathWrapString
0001:00656489* _xmlXPathNewCString
0001:00656575* _xmlXPathLocalNameFunction
0001:00656817* _xmlXPathNamespaceURIFunction
0001:006568fc* _xmlXPathWrapCString
0001:0065691e* _xmlXPathWrapExternal
0001:006569a5  _xmlXPathObjectCopy
0001:00656b7f* _xmlXPathVariableLookupNS
0001:00656bef* _xmlXPathVariableLookup
0001:00656c3f* _xmlXPathCastBooleanToString
0001:00656c8b* _xmlXPathCastNumberToString
0001:0065706e* _xmlXPathCastNodeToString
0001:00657092* _xmlXPathDistinctSorted
0001:00657192* _xmlXPathDistinct
0001:006571ca* _xmlXPathCastNodeSetToString
0001:00657337* _xmlXPathStringFunction
0001:006573c2* _xmlXPathLangFunction
0001:0065751c* _xmlXPathTranslateFunction
0001:00657734* _xmlXPathNormalizeFunction
0001:006578c8* _xmlXPathSubstringAfterFunction
0001:006579fb* _xmlXPathSubstringBeforeFunction
0001:00657afe* _xmlXPathStartsWithFunction
0001:00657c41* _xmlXPathContainsFunction
0001:00657d75* _xmlXPathConcatFunction
0001:00657e84* _xmlXPathStringLengthFunction
0001:00657fbe  _xmlXPathIdFunction
0001:00658110  _xmlXPathCastToString
0001:006581dd* _xmlXPathPopString
0001:00658242* _xmlXPathConvertString
0001:0065832a* _xmlXPathCastBooleanToNumber
0001:0065833c* _xmlXPathCastNumberToBoolean
0001:00658383* _xmlXPathCastStringToBoolean
0001:006583a4* _xmlXPathCastNodeSetToBoolean
0001:006583ba* _xmlXPathCastToBoolean
0001:0065847c* _xmlXPathBooleanFunction
0001:00658503* _xmlXPathNotFunction
0001:00658578* _xmlXPathPopBoolean
0001:00658862* _xmlXPathConvertBoolean
0001:006588ad  _xmlXPathFreeContext
0001:0065891e  _xmlXPathNewParserContext
0001:006589af  _xmlXPathFreeParserContext
0001:00658a00* _xmlXPathNextPreceding
0001:00658a9b  _xmlXPathRoot
0001:00658acc  _xmlXPathParseNCName
0001:00658bdc  _xmlXPathParseName
0001:00658c7b* _xmlXPathStringEvalNumber
0001:00658eb0* _xmlXPathCastStringToNumber
0001:00658ebc* _xmlXPathCastNodeSetToNumber
0001:00658efd* _xmlXPathCastToNumber
0001:00658fbb* _xmlXPathConvertNumber
0001:00659002* _xmlXPathPopNumber
0001:00659067* _xmlXPathNumberFunction
0001:00659157* _xmlXPathRoundFunction
0001:006592f1* _xmlXPathCeilingFunction
0001:0065943b* _xmlXPathFloorFunction
0001:00659541* _xmlXPathSubstringFunction
0001:00659820* _xmlXPathValueFlipSign
0001:00659e0e* _xmlXPathNotEqualValues
0001:00659fda* _xmlXPathEqualValues
0001:0065a1a2* _xmlXPathModValues
0001:0065a281* _xmlXPathDivValues
0001:0065a40b* _xmlXPathMultValues
0001:0065a49f* _xmlXPathSubValues
0001:0065a533* _xmlXPathAddValues
0001:0065a5c7* _xmlXPathCastNodeToNumber
0001:0065a60c* _xmlXPathSumFunction
0001:0065a964* _xmlXPathCompareValues
0001:0065afc7* _xmlXPathIsNodeType
0001:0065d8e1* _xmlXPathEvalPredicate
0001:0065d9c8  _xmlXPathEvaluatePredicateResult
0001:00661a3f* _xmlXPathCtxtCompile
0001:00661b12* _xmlXPathCompile
0001:00661b2d* _xmlXPathCompiledEval
0001:00661b54* _xmlXPathCompiledEvalToBoolean
0001:00661b6f  _xmlXPathEvalExpr
0001:00661c7b  _xmlXPathEval
0001:00661e79  _xmlXPathEvalExpression
0001:006620f2* _xmlXPathRegisterAllFunctions
0001:006623bc  _xmlXPathNewContext
0002:000047a0  _xmlXPathPINF
0002:000047a8  _xmlXPathNINF
0002:0001cc50  _xmlXPathNAN
Module: U:\extras\lib\xml2.lib(HTMLtree.obj)
0001:00662828  _htmlGetMetaEncoding
0001:00662aeb  _htmlSetMetaEncoding
0001:00662e7a  _htmlIsBooleanAttr
0001:006630a7* _htmlDocContentDumpOutput
0001:006636ff  _htmlDocContentDumpFormatOutput
0001:006630ff  _htmlNodeDumpFormatOutput
0001:00663849  _htmlDocDumpMemoryFormat
0001:00663979* _htmlDocDumpMemory
0001:006639a2  _htmlNodeDumpOutput
0001:006639d2* _htmlNodeDumpFileFormat
0001:00663a80  _htmlNodeDumpFile
0001:00663acf  _htmlNodeDump
0001:00663bb5  _htmlDocDump
0001:00663c6d  _htmlSaveFile
0001:00663d34  _htmlSaveFileFormat
0001:00663e3b* _htmlSaveFileEnc
Module: U:\extras\lib\xml2.lib(xinclude.obj)
0001:0066537d  _xmlXIncludeNewContext
0001:006653c9  _xmlXIncludeFreeContext
0001:006671db  _xmlXIncludeSetFlags
0001:006671f4* _xmlXIncludeProcessTreeFlagsData
0001:0066726d* _xmlXIncludeProcessFlagsData
0001:006672ae  _xmlXIncludeProcessFlags
0001:006672d0* _xmlXIncludeProcess
0001:006672eb* _xmlXIncludeProcessTreeFlags
0001:0066735f* _xmlXIncludeProcessTree
0001:0066737a  _xmlXIncludeProcessNode
Module: U:\extras\lib\xml2.lib(xmlsave.obj)
0001:00667dd8* _xmlIsXHTML
0001:00667ea3  _xmlNsListDumpOutput
0001:00667ec7* _xmlSaveToFd
0001:00667f0b* _xmlSaveToFilename
0001:00667f57* _xmlSaveToBuffer
0001:00667fcd* _xmlSaveToIO
0001:0066801f* _xmlSaveFlush
0001:00668043* _xmlSaveClose
0001:00668071* _xmlSaveSetEscape
0001:0066808a* _xmlSaveSetAttrEscape
0001:006680d6  _xmlAttrSerializeTxtContent
0001:0066a6fe* _xmlSaveTree
0001:0066a722* _xmlSaveDoc
0001:0066a747  _xmlNodeDumpOutput
0001:0066a814  _xmlElemDump
0001:0066a8b8  _xmlNodeDump
0001:0066a992* _xmlDocDumpFormatMemoryEnc
0001:0066ab1c  _xmlDocDumpMemory
0001:0066ab4d  _xmlDocDumpFormatMemory
0001:0066ab7d  _xmlDocDumpMemoryEnc
0001:0066abad* _xmlDocFormatDump
0001:0066aca1  _xmlDocDump
0001:0066acc3* _xmlSaveFileTo
0001:0066ad41  _xmlSaveFormatFileTo
0001:0066add8  _xmlSaveFormatFileEnc
0001:0066aecc* _xmlSaveFileEnc
0001:0066aef5* _xmlSaveFormatFile
0001:0066af1e  _xmlSaveFile
Module: U:\extras\lib\xml2.lib(HTMLparser.obj)
0001:0066de98  _htmlInitAutoClose
0001:0066e42f  _htmlTagLookup
0001:0066e834* _htmlAutoCloseTag
0001:0066e8b0* _htmlIsAutoClosed
0001:0066e8fe* _htmlIsScriptAttribute
0001:0066e94b* _htmlEntityLookup
0001:0066e99f* _htmlEntityValueLookup
0001:0066e9e5  _UTF8ToHtml
0001:0066ec64* _htmlEncodeEntities
0001:0066eef7  _htmlNewDocNoDtD
0001:0066efde* _htmlNewDoc
0001:0066f053* _htmlParseEntityRef
0001:0066f1f8* _htmlParseCharRef
0001:00670a51* _htmlParseElement
0001:006710d6  ___htmlParseContent
0001:00671121  _htmlParseDocument
0001:00671470  _htmlFreeParserCtxt
0001:006714bf* _htmlNewParserCtxt
0001:0067173e  _htmlCreateMemoryParserCtxt
0001:00671aa2* _htmlParseChunk
0001:00672d3e* _htmlCreatePushParserCtxt
0001:00672f34* _htmlSAXParseDoc
0001:00672fba* _htmlParseDoc
0001:00672ff3  _htmlCreateFileParserCtxt
0001:00673102* _htmlSAXParseFile
0001:00673172  _htmlParseFile
0001:0067319c* _htmlHandleOmittedElem
0001:006731af* _htmlElementAllowedHere
0001:00673204* _htmlElementStatusHere
0001:0067324f* _htmlAttrAllowed
0001:00673310* _htmlNodeStatus
0001:006733d5* _htmlCtxtReset
0001:006736d5* _htmlCtxtUseOptions
0001:006738e0* _htmlReadDoc
0001:00673933* _htmlReadFile
0001:0067397e* _htmlReadMemory
0001:006739fe* _htmlReadFd
0001:00673ac5* _htmlReadIO
0001:00673b9a* _htmlCtxtReadDoc
0001:00673c10* _htmlCtxtReadFile
0001:00673c85* _htmlCtxtReadMemory
0001:00673d3d* _htmlCtxtReadFd
0001:00673de8* _htmlCtxtReadIO
Module: U:\extras\lib\xml2.lib(encoding.obj)
0001:0067b493* _isolat1ToUTF8
0001:0067b58f* _UTF8Toisolat1
0001:0067c2c3  _xmlDetectCharEncoding
0001:0067c454* _xmlCleanupEncodingAliases
0001:0067c4e3* _xmlGetEncodingAlias
0001:0067c595* _xmlAddEncodingAlias
0001:0067c779* _xmlDelEncodingAlias
0001:0067c938  _xmlParseCharEncoding
0001:0067cc81  _xmlGetCharEncodingName
0001:0067cc9a  _xmlCleanupCharEncodingHandlers
0001:0067cdb1* _xmlRegisterCharEncodingHandler
0001:0067cfed  _xmlInitCharEncodingHandlers
0001:0067ce79* _xmlNewCharEncodingHandler
0001:0067d188  _xmlFindCharEncodingHandler
0001:0067d457  _xmlGetCharEncodingHandler
0001:0067d695  _xmlCharEncFirstLineInt
0001:0067d7f3* _xmlCharEncFirstLine
0001:0067d86e  _xmlCharEncInFunc
0001:0067da5a  _xmlCharEncOutFunc
0001:0067dd0a  _xmlCharEncCloseFunc
0001:0067dd9b  _xmlByteConsumed
Module: U:\extras\lib\xml2.lib(xmlschemas.obj)
0001:0068e0f1  _xmlSchemaNewFacet
0001:0068e11b  _xmlSchemaFreeWildcard
0001:0068e17a  _xmlSchemaFreeFacet
0001:00694cb6  _xmlSchemaFreeType
0001:0069501a  _xmlSchemaFree
0001:00696135* _xmlSchemaDump
0001:00696269  _xmlSchemaNewParserCtxt
0001:006962b6  _xmlSchemaNewMemParserCtxt
0001:006962f4* _xmlSchemaNewDocParserCtxt
0001:0069632b* _xmlSchemaGetParserErrors
0001:00696384  _xmlSchemaNewValidCtxt
0001:006963e3  _xmlSchemaFreeValidCtxt
0001:00696602  _xmlSchemaFreeParserCtxt
0001:006968be  _xmlSchemaCheckFacet
0001:00696d20  _xmlSchemaIsValid
0001:00696d3a  _xmlSchemaSetValidErrors
0001:00696d71  _xmlSchemaSetParserErrors
0001:00696da8  _xmlSchemaSetValidStructuredErrors
0001:0069e784* _xmlSchemaSetParserStructuredErrors
0001:006a36eb  _xmlSchemaParse
0001:006a38d7* _xmlSchemaGetValidErrors
0001:006a3912* _xmlSchemaSetValidOptions
0001:006a394c* _xmlSchemaValidCtxtGetOptions
0001:006a3960* _xmlSchemaValidateOneElement
0001:006a3999  _xmlSchemaValidateDoc
0001:006a3a0f  _xmlSchemaSAXPlug
0001:006a3cae  _xmlSchemaSAXUnplug
0001:006a3d29* _xmlSchemaValidateStream
0001:006a3e5d* _xmlSchemaValidateFile
0001:006a3ebe* _xmlSchemaValidCtxtGetParserCtxt
Module: U:\extras\lib\xml2.lib(parserInternals.obj)
0001:006a44f0* _xmlCheckVersion
0001:006a45e9  _xmlErrMemory
0001:006a473d  ___xmlErrEncoding
0001:006a4890* _xmlIsLetter
0001:006a4931* _xmlParserInputRead
0001:006a49bc  _xmlParserInputGrow
0001:006a4a3e  _xmlParserInputShrink
0001:006a4b8a  _xmlNextChar
0001:006a4f7b  _xmlCurrentChar
0001:006a534a  _xmlStringCurrentChar
0001:006a55c4  _xmlCopyCharMultiByte
0001:006a566d  _xmlCopyChar
0001:006a5728  _xmlSwitchEncoding
0001:006a5a60  _xmlSwitchInputEncoding
0001:006a5a7c  _xmlSwitchToEncoding
0001:006a5a93  _xmlFreeInputStream
0001:006a5b3e  _xmlNewInputStream
0001:006a5bbb  _xmlNewIOInputStream
0001:006a5d24  _xmlNewEntityInputStream
0001:006a5eaf  _xmlNewStringInputStream
0001:006a5fb1  _xmlNewInputFromFile
0001:006a614e* _xmlInitParserCtxt
0001:006a660d  _xmlFreeParserCtxt
0001:006a688c  _xmlNewParserCtxt
0001:006a68e9  _xmlClearParserCtxt
0001:006a692f  _xmlInitNodeInfoSeq
0001:006a694f* _xmlClearNodeInfoSeq
0001:006a6987* _xmlParserFindNodeInfoIndex
0001:006a6a16* _xmlParserFindNodeInfo
0001:006a6a7f  _xmlParserAddNodeInfo
0001:006a6c03* _xmlPedanticParserDefault
0001:006a6c23* _xmlLineNumbersDefault
0001:006a6c43* _xmlSubstituteEntitiesDefault
0001:006a6c63* _xmlKeepBlanksDefault
Module: U:\extras\lib\xml2.lib(c14n.obj)
0001:006a9517* _xmlC14NExecute
0001:006a970e  _xmlC14NDocSaveTo
0001:006a97b3* _xmlC14NDocDumpMemory
0001:006a98eb* _xmlC14NDocSave
Module: U:\extras\lib\xml2.lib(hash.obj)
0001:006a9a7a  _xmlHashCreate
0001:006a9af6  _xmlHashCreateDict
0001:006a9b26  _xmlHashFree
0001:006a9c6d  _xmlHashAddEntry3
0001:006aa144  _xmlHashAddEntry2
0001:006aa174  _xmlHashAddEntry
0001:006aa1a5* _xmlHashUpdateEntry3
0001:006aa507  _xmlHashUpdateEntry2
0001:006aa53e  _xmlHashUpdateEntry
0001:006aa576  _xmlHashLookup3
0001:006aa63a  _xmlHashLookup2
0001:006aa663  _xmlHashLookup
0001:006aa68d* _xmlHashQLookup3
0001:006aa8be  _xmlHashQLookup2
0001:006aa8fd* _xmlHashQLookup
0001:006aa93e  _xmlHashScanFull
0001:006aaa02  _xmlHashScan
0001:006aaa30* _xmlHashScanFull3
0001:006aab32  _xmlHashScan3
0001:006aab3e  _xmlHashCopy
0001:006aac00  _xmlHashSize
0001:006aac14* _xmlHashRemoveEntry3
0001:006aad9d  _xmlHashRemoveEntry2
0001:006aadcd  _xmlHashRemoveEntry
Module: U:\extras\lib\libssl.lib(ssl_lib.obj)
0001:006af09b  _ssl_undefined_function
0001:006aae24  _SSL_clear
0001:006af688* _ssl_clear_cipher_ctx
0001:006b0055* _ssl_clear_hash_ctx
0001:006ab048* _SSL_CTX_set_ssl_version
0001:006ab10f  _SSL_new
0001:006ade91  _SSL_CTX_free
0001:006ab586* _SSL_CTX_set_session_id_context
0001:006ab5f7* _SSL_set_session_id_context
0001:006ab668* _SSL_CTX_set_generate_session_id
0001:006ab6c9* _SSL_set_generate_session_id
0001:006ab72a  _SSL_has_matching_session_id
0001:006ab830* _SSL_CTX_set_purpose
0001:006ab850* _SSL_set_purpose
0001:006ab86d* _SSL_CTX_set_trust
0001:006ab88d* _SSL_set_trust
0001:006ab8aa* _SSL_CTX_set1_param
0001:006ab8ca* _SSL_set1_param
0001:006ab8e7* _SSL_free
0001:006abc20* _SSL_set_bio
0001:006abcc6  _SSL_get_rbio
0001:006abcd1* _SSL_get_wbio
0001:006abcdc* _SSL_get_fd
0001:006abcef* _SSL_get_rfd
0001:006abd4d* _SSL_get_wfd
0001:006abdab  _SSL_set_fd
0001:006abe4a* _SSL_set_wfd
0001:006abf71* _SSL_set_rfd
0001:006ac098* _SSL_get_finished
0001:006ac0f3* _SSL_get_peer_finished
0001:006ac14e* _SSL_get_verify_mode
0001:006ac15c* _SSL_get_verify_depth
0001:006ac172* _SSL_get_verify_callback
0001:006ac180* _SSL_CTX_get_verify_mode
0001:006ac18e* _SSL_CTX_get_verify_depth
0001:006ac1a7* _SSL_CTX_get_verify_callback
0001:006ac1b5* _SSL_set_verify
0001:006ac1d8* _SSL_set_verify_depth
0001:006ac1f5* _SSL_set_read_ahead
0001:006ac203* _SSL_get_read_ahead
0001:006ac20e* _SSL_pending
0001:006ac227* _SSL_get_peer_certificate
0001:006ac299* _SSL_get_peer_cert_chain
0001:006ac2e7  _SSL_copy_session_id
0001:006ac3eb* _SSL_CTX_check_private_key
0001:006ac4b6* _SSL_check_private_key
0001:006ac5ed* _SSL_accept
0001:006aefdb* _SSL_set_accept_state
0001:006ac61b  _SSL_connect
0001:006af03b* _SSL_set_connect_state
0001:006ac649  _SSL_get_default_timeout
0001:006ac65c  _SSL_read
0001:006ac6de  _SSL_peek
0001:006ac756  _SSL_write
0001:006ac804  _SSL_shutdown
0001:006afb46  _SSL_state
0001:006ac87b* _SSL_renegotiate
0001:006ac8a8* _SSL_renegotiate_pending
0001:006ac8bb  _SSL_ctrl
0001:006afa06  _SSL_version
0001:006acb88* _SSL_callback_ctrl
0001:006acbc7* _SSL_CTX_sessions
0001:006acbd2  _SSL_CTX_ctrl
0001:006acf19* _SSL_CTX_callback_ctrl
0001:006acf5a* _ssl_cipher_id_cmp
0001:006acf96  _ssl_cipher_ptr_id_cmp
0001:006acfd6  _SSL_get_ciphers
0001:006ad023  _ssl_get_ciphers_by_id
0001:006ad070* _SSL_get_cipher_list
0001:006ad0d8* _SSL_CTX_set_cipher_list
0001:006ad164* _SSL_set_cipher_list
0001:006ad1f6* _SSL_get_shared_ciphers
0001:006ad2e1  _ssl_cipher_list_to_bytes
0001:006ad402  _ssl_bytes_to_cipher_list
0001:006ad60f* _SSL_get_servername
0001:006ad655* _SSL_get_servername_type
0001:006ad79a  _SSL_CTX_new
0001:006ae098* _SSL_CTX_set_default_passwd_cb
0001:006ae0a6* _SSL_CTX_set_default_passwd_cb_userdata
0001:006ae0b4* _SSL_CTX_set_cert_verify_callback
0001:006ae0cb* _SSL_CTX_set_verify
0001:006ae0e8* _SSL_CTX_set_verify_depth
0001:006ae118  _ssl_set_cert_masks
0001:006ae670  _ssl_check_srvr_ecc_cert_and_alg
0001:006ae8bd* _ssl_get_server_send_cert
0001:006aea38* _ssl_get_sign_pkey
0001:006aeaf6  _ssl_update_cache
0001:006aec68* _SSL_get_ssl_method
0001:006aec73  _SSL_set_ssl_method
0001:006aed2f* _SSL_get_error
0001:006afcaa* _SSL_want
0001:006aef42* _SSL_do_handshake
0001:006af0d4  _ssl_undefined_void_function
0001:006af10d  _ssl_undefined_const_function
0001:006af146* _ssl_bad_method
0001:006af18b* _SSL_get_version
0001:006af1cc* _SSL_dup
0001:006afa10* _SSL_get_SSL_CTX
0001:006afb38* _SSL_get_info_callback
0001:006afb27* _SSL_set_info_callback
0001:006af75e* _SSL_get_certificate
0001:006af784* _SSL_get_privatekey
0001:006af7ab* _SSL_get_current_cipher
0001:006af7e6* _SSL_get_current_compression
0001:006af80a* _SSL_get_current_expansion
0001:006af82e  _ssl_init_wbio_buffer
0001:006af964  _ssl_free_wbio_buffer
0001:006af9b5* _SSL_CTX_set_quiet_shutdown
0001:006af9c6* _SSL_CTX_get_quiet_shutdown
0001:006af9d4* _SSL_set_quiet_shutdown
0001:006af9e2* _SSL_get_quiet_shutdown
0001:006af9ed* _SSL_set_shutdown
0001:006af9fb* _SSL_get_shutdown
0001:006afa1e* _SSL_set_SSL_CTX
0001:006afaed* _SSL_CTX_set_default_verify_paths
0001:006afb03* _SSL_CTX_load_verify_locations
0001:006afb51* _SSL_set_verify_result
0001:006afb62* _SSL_get_verify_result
0001:006afb70* _SSL_get_ex_new_index
0001:006afba7* _SSL_set_ex_data
0001:006afbce* _SSL_get_ex_data
0001:006afbee* _SSL_CTX_get_ex_new_index
0001:006afc25* _SSL_CTX_set_ex_data
0001:006afc4c* _SSL_CTX_get_ex_data
0001:006afc6c  _ssl_ok
0001:006afc76* _SSL_CTX_get_cert_store
0001:006afc81* _SSL_CTX_set_cert_store
0001:006afcb5* _SSL_CTX_set_tmp_rsa_callback
0001:006afcd7* _SSL_set_tmp_rsa_callback
0001:006afcf9* _SSL_CTX_set_tmp_dh_callback
0001:006afd1b* _SSL_set_tmp_dh_callback
0001:006afd3d* _SSL_CTX_set_tmp_ecdh_callback
0001:006afd5f* _SSL_set_tmp_ecdh_callback
0001:006afd81* _SSL_CTX_use_psk_identity_hint
0001:006afe32* _SSL_use_psk_identity_hint
0001:006aff2d* _SSL_get_psk_identity_hint
0001:006aff5b* _SSL_get_psk_identity
0001:006aff89* _SSL_set_psk_client_callback
0001:006aff9a* _SSL_CTX_set_psk_client_callback
0001:006affab* _SSL_set_psk_server_callback
0001:006affbc* _SSL_CTX_set_psk_server_callback
0001:006affcd* _SSL_CTX_set_msg_callback
0001:006affef* _SSL_set_msg_callback
0001:006b0011  _ssl_replace_hash
0001:006b00a2  _OBJ_bsearch_ssl_cipher_id
0002:000047f0* _SSL_version_str
0002:00004800  _ssl3_undef_enc_method
Module: U:\extras\lib\libssl.lib(s23_clnt.obj)
0001:006b011a  _SSLv23_client_method
0001:006b012f* _ssl23_connect
Module: U:\extras\lib\poll.lib(poll.obj)
0001:006b13d0  _poll
Module: U:\usr\lib\libc_dll.lib(accept.obj)
0001:006b17e0  _accept
Module: U:\usr\lib\libc_dll.lib(send.obj)
0001:006b18c0  _send
Module: U:\usr\lib\libc_dll.lib(recv.obj)
0001:006b1970  _recv
Module: U:\usr\lib\libc_dll.lib(getsockname.obj)
0001:006b1a20  _getsockname
Module: U:\usr\lib\libc_dll.lib(socket.obj)
0001:006b1ac0  _socket
Module: U:\usr\lib\libc_dll.lib(bind.obj)
0001:006b1b40  _bind
Module: U:\usr\lib\libc_dll.lib(listen.obj)
0001:006b1be0  _listen
Module: U:\extras\lib\xml2.lib(entities.obj)
0001:006b2352  _xmlGetPredefinedEntity
0001:006b248a  _xmlAddDtdEntity
0001:006b256a  _xmlAddDocEntity
0001:006b25f4* _xmlNewEntity
0001:006b265d  _xmlGetParameterEntity
0001:006b26be* _xmlGetDtdEntity
0001:006b26e6  _xmlGetDocEntity
0001:006b281f  _xmlEncodeEntitiesReentrant
0001:006b2c61  _xmlEncodeSpecialChars
0001:006b2dc1* _xmlCreateEntitiesTable
0001:006b2dd5  _xmlFreeEntitiesTable
0001:006b2df0  _xmlCopyEntitiesTable
0001:006b2e78  _xmlDumpEntityDecl
0001:006b30eb* _xmlDumpEntitiesTable
Module: U:\usr\lib\libc_dll.lib(shutdown.obj)
0001:006b3120  _shutdown
Module: U:\usr\lib\libc_dll.lib(getsockopt.obj)
0001:006b31c0  _getsockopt
Module: U:\usr\lib\libc_dll.lib(sendto.obj)
0001:006b32a0  _sendto
Module: U:\usr\lib\libc_dll.lib(connect.obj)
0001:006b3350  _connect
Module: U:\usr\lib\libc_dll.lib(socketpair.obj)
0001:006b33f0  _socketpair
Module: U:\usr\lib\libc_dll.lib(getpeername.obj)
0001:006b34b0  _getpeername
Module: U:\usr\lib\libc_dll.lib(recvfrom.obj)
0001:006b3550  _recvfrom
Module: U:\usr\lib\libc_dll.lib(setsockopt.obj)
0001:006b3620  _setsockopt
Module: U:\usr\lib\libc_dll.lib(syslog.obj)
0001:006b376c  _syslog
0001:006b37d4* _vsyslog
0001:006b3c31  _openlog
0001:006b3c80  _closelog
0001:006b3cb4* _setlogmask
Module: U:\tmp\ldconv_libgcc_a_3ed14e78ff521a1dd8.lib(_fixunsdfdi.obj)
0001:006b3ce0  ___fixunsdfdi
Module: U:\extras\lib\xml2.lib(xmlreader.obj)
0001:006b519a* _xmlTextReaderReadState
0001:006b51ad  _xmlTextReaderExpand
0001:006b5351  _xmlTextReaderReadInnerXml
0001:006b5440  _xmlTextReaderReadOuterXml
0001:006b551a  _xmlTextReaderReadString
0001:006b55ce  _xmlNewTextReader
0001:006b5888* _xmlNewTextReaderFilename
0001:006b5929  _xmlFreeTextReader
0001:006b5b39* _xmlTextReaderClose
0001:006b5bc1  _xmlTextReaderGetAttributeNo
0001:006b5c7a  _xmlTextReaderGetAttribute
0001:006b5e07  _xmlTextReaderGetAttributeNs
0001:006b5ecb* _xmlTextReaderGetRemainder
0001:006b5f7f  _xmlTextReaderLookupNamespace
0001:006b5fbd  _xmlTextReaderMoveToAttributeNo
0001:006b6049  _xmlTextReaderMoveToAttribute
0001:006b6202  _xmlTextReaderMoveToAttributeNs
0001:006b6322  _xmlTextReaderMoveToFirstAttribute
0001:006b6363  _xmlTextReaderMoveToNextAttribute
0001:006b63cd  _xmlTextReaderMoveToElement
0001:006b63ff* _xmlTextReaderReadAttributeValue
0001:006b64ab* _xmlTextReaderConstEncoding
0001:006b64f5  _xmlTextReaderAttributeCount
0001:006b655a  _xmlTextReaderNodeType
0001:006b66ac  _xmlTextReaderIsEmptyElement
0001:006b6733* _xmlTextReaderName
0001:006b68a9* _xmlTextReaderLocalName
0001:006b6905  _xmlTextReaderConstName
0001:006b6ab0  _xmlTextReaderConstLocalName
0001:006b6b15* _xmlTextReaderPrefix
0001:006b6b73  _xmlTextReaderConstPrefix
0001:006b6bfa* _xmlTextReaderNamespaceUri
0001:006b6c4d  _xmlTextReaderConstNamespaceUri
0001:006b6ccb* _xmlTextReaderBaseUri
0001:006b6cf5  _xmlTextReaderConstBaseUri
0001:006b6d52  _xmlTextReaderDepth
0001:006b6d93  _xmlTextReaderHasAttributes
0001:006b6dd4  _xmlTextReaderHasValue
0001:006b6e0d* _xmlTextReaderValue
0001:006b6f18  _xmlTextReaderConstValue
0001:006b702d  _xmlTextReaderIsDefault
0001:006b7038* _xmlTextReaderQuoteChar
0001:006b7046* _xmlTextReaderXmlLang
0001:006b7067  _xmlTextReaderConstXmlLang
0001:006b70bc* _xmlTextReaderConstString
0001:006b70e7* _xmlTextReaderNormalization
0001:006b70f5  _xmlTextReaderSetParserProp
0001:006b71dd  _xmlTextReaderGetParserProp
0001:006b724a* _xmlTextReaderGetParserLineNumber
0001:006b7269* _xmlTextReaderGetParserColumnNumber
0001:006b7288* _xmlTextReaderCurrentNode
0001:006b72a2* _xmlTextReaderPreserve
0001:006b7338  _xmlTextReaderRead
0001:006b7da7* _xmlTextReaderNextSibling
0001:006b7df2  _xmlTextReaderNext
0001:006b7e6d* _xmlTextReaderPreservePattern
0001:006b7f95* _xmlTextReaderCurrentDoc
0001:006b7fc1  _xmlTextReaderRelaxNGSetSchema
0001:006b80be* _xmlTextReaderSetSchema
0001:006b82c3* _xmlTextReaderRelaxNGValidate
0001:006b8434* _xmlTextReaderSchemaValidateCtxt
0001:006b8448  _xmlTextReaderSchemaValidate
0001:006b845c* _xmlTextReaderIsNamespaceDecl
0001:006b848b* _xmlTextReaderConstXmlVersion
0001:006b84d5* _xmlTextReaderStandalone
0001:006b8502* _xmlTextReaderLocatorLineNumber
0001:006b854f* _xmlTextReaderLocatorBaseURI
0001:006b85a4* _xmlTextReaderSetErrorHandler
0001:006b8714* _xmlTextReaderSetStructuredErrorHandler
0001:006b889d  _xmlTextReaderIsValid
0001:006b88ea* _xmlTextReaderGetErrorHandler
0001:006b8914  _xmlTextReaderSetup
0001:006b8e31* _xmlTextReaderByteConsumed
0001:006b8e55* _xmlReaderWalker
0001:006b8ebe  _xmlReaderForFile
0001:006b8f04* _xmlReaderForMemory
0001:006b8f7e* _xmlReaderForDoc
0001:006b8fbd* _xmlReaderForFd
0001:006b9042* _xmlReaderForIO
0001:006b90d1* _xmlReaderNewWalker
0001:006b9183* _xmlReaderNewFile
0001:006b91df* _xmlReaderNewMemory
0001:006b9248* _xmlReaderNewDoc
0001:006b929e* _xmlReaderNewFd
0001:006b9307* _xmlReaderNewIO
Module: U:\extras\lib\xmlrpc.lib(xmlrpc.obj)
0001:006b93d0  _XMLRPC_RequestGetMethodName
0001:006b93e1  _XMLRPC_RequestSetRequestType
0001:006b93f7  _XMLRPC_RequestGetRequestType
0001:006b9408  _XMLRPC_RequestGetData
0001:006b9418  _XMLRPC_RequestGetError
0001:006b9429  _XMLRPC_RequestGetOutputOptions
0001:006b943a  _XMLRPC_SetValueInt
0001:006b9452  _XMLRPC_SetValueBoolean
0001:006b9470  _XMLRPC_CopyValue
0001:006b9480  _XMLRPC_SetValueDouble
0001:006b949c  _XMLRPC_GetValueString
0001:006b94b4  _XMLRPC_GetValueStringLen
0001:006b94c5  _XMLRPC_GetValueInt
0001:006b94e1  _XMLRPC_GetValueBoolean
0001:006b94f9  _XMLRPC_GetValueDouble
0001:006b9511  _XMLRPC_GetValueBase64
0001:006b9529  _XMLRPC_GetValueDateTime
0001:006b9541  _XMLRPC_GetValueDateTime_ISO8601
0001:006b9559  _XMLRPC_GetValueID
0001:006b9573  _XMLRPC_GetValueType
0001:006b9586  _XMLRPC_GetVectorType
0001:006b95a1  _XMLRPC_GetValueTypeEasy
0001:006b9632  _type_to_str
0001:006b96d3  _XMLRPC_GetDefaultIdCase
0001:006b96dd* _XMLRPC_SetDefaultIdCase
0001:006b96ea  _XMLRPC_GetDefaultIdCaseComparison
0001:006b96f4* _XMLRPC_SetDefaultIdCaseComparison
0001:006b9714  _XMLRPC_GetVersionString
0001:006b971e* _XMLRPC_Free
0001:006b9733* _XMLRPC_ServerFindMethod
0001:006b9780  _find_method
0001:006b97cc  _XMLRPC_ServerRegisterMethod
0001:006b9832  _XMLRPC_VectorRewind
0001:006b985e  _XMLRPC_VectorNext
0001:006b9887  _XMLRPC_CreateValueEmpty
0001:006b98cc  _XMLRPC_RequestNew
0001:006b98fd  _XMLRPC_ServerCreate
0001:006b9941* _XMLRPC_GetGlobalServer
0001:006b995e  _XMLRPC_VectorSize
0001:006b9987  _XMLRPC_SetIsVector
0001:006b9a24  _XMLRPC_RequestSetMethodName
0001:006b9a59  _XMLRPC_SetValueBase64
0001:006b9abc  _XMLRPC_SetValueString
0001:006b9b24  _XMLRPC_SetValueID_Case
0001:006b9c03  _XMLRPC_CreateValueDouble
0001:006b9c55  _XMLRPC_CreateValueBase64
0001:006b9cab  _XMLRPC_CreateValueBoolean
0001:006b9cfd  _XMLRPC_CreateValueInt
0001:006b9d49  _XMLRPC_CreateValueString
0001:006b9da7  _XMLRPC_CreateVector
0001:006b9e02  _XMLRPC_SetValueDateTime_ISO8601
0001:006b9f95  _XMLRPC_CreateValueDateTime_ISO8601
0001:006b9ff5* _XMLRPC_SetValueDateTime
0001:006ba063* _XMLRPC_CreateValueDateTime
0001:006ba0e5  _XMLRPC_CleanupValue
0001:006ba1f3  _XMLRPC_ServerDestroy
0001:006ba2b4  _XMLRPC_RequestSetError
0001:006ba2f3  _XMLRPC_RequestSetData
0001:006ba330  _XMLRPC_RequestFree
0001:006ba406  _XMLRPC_AddValueToVector
0001:006ba61b* _XMLRPC_UtilityCreateFault
0001:006ba7bd  _XMLRPC_ServerCallMethod
0001:006ba856  _XMLRPC_DupValueNew
0001:006ba99f  _XMLRPC_VectorRemoveValue
0001:006baa13  _XMLRPC_VectorGetValueWithID_Case
0001:006baa8d* _XMLRPC_GetValueFaultString
0001:006baac1* _XMLRPC_GetResponseFaultString
0001:006baad8* _XMLRPC_GetValueFaultCode
0001:006bab0c* _XMLRPC_GetResponseFaultCode
0001:006bab23* _XMLRPC_ValueIsFault
0001:006bab73* _XMLRPC_ResponseIsFault
0001:006bab8a  _XMLRPC_AddValuesToVector
0001:006bac9f  _XMLRPC_REQUEST_FromXML
0001:006badb5* _XMLRPC_VALUE_FromXML
0001:006badf5  _XMLRPC_REQUEST_ToXML
0001:006bae73  _XMLRPC_VALUE_ToXML
0001:006baeb8  _XMLRPC_RequestSetOutputOptions
Module: U:\extras\lib\xmlrpc.lib(xmlrpc_introspection.obj)
0001:006baf84* _XMLRPC_ServerSetValidationLevel
0001:006bafa2* _find_named_value
0001:006bb016* _validate_scalar
0001:006bb173* _validate_value
0001:006bb374* _validate_vector
0001:006bb267* _validate_method
0001:006bb2f2  _XMLRPC_ServerValidateRequest
0001:006bb489  _XMLRPC_ServerRegisterIntrospectionCallback
0001:006bb4f2* _describe_method
0001:006bb614* _xml_element_to_method_description
0001:006bbc01  _XMLRPC_IntrospectionCreateDescription
0001:006bbcb0  _xi_register_system_methods
0001:006bc10b  _XMLRPC_ServerAddIntrospectionData
Module: U:\extras\lib\xml2.lib(xmlwriter.obj)
0001:006bc9b1* _xmlNewTextWriter
0001:006bcb37  _xmlNewTextWriterFilename
0001:006bcbdd  _xmlNewTextWriterMemory
0001:006bccf1* _xmlNewTextWriterPushParser
0001:006bce30* _xmlNewTextWriterDoc
0001:006bcf8b* _xmlNewTextWriterTree
0001:006bd096  _xmlFreeTextWriter
0001:006bd200  _xmlTextWriterStartDocument
0001:006bd5a2  _xmlTextWriterEndComment
0001:006bd66a  _xmlTextWriterEndAttribute
0001:006bd6d5  _xmlTextWriterStartAttribute
0001:006bd81c  _xmlTextWriterStartAttributeNS
0001:006bd9d7  _xmlTextWriterWriteAttribute
0001:006be0ab  _xmlTextWriterWriteString
0001:006bdc34* _xmlTextWriterWriteBinHex
0001:006bdd6d* _xmlTextWriterWriteBase64
0001:006bdfb9* _xmlTextWriterWriteRawLen
0001:006be080  _xmlTextWriterWriteRaw
0001:006be164* _xmlTextWriterWriteVFormatString
0001:006be1b6* _xmlTextWriterWriteFormatString
0001:006be1e6* _xmlTextWriterWriteVFormatRaw
0001:006be22f* _xmlTextWriterWriteFormatRaw
0001:006be255  _xmlTextWriterFullEndElement
0001:006be3d0  _xmlTextWriterEndElement
0001:006be592  _xmlTextWriterStartElement
0001:006be7b6  _xmlTextWriterStartElementNS
0001:006be926  _xmlTextWriterStartComment
0001:006bea95  _xmlTextWriterWriteComment
0001:006beb20* _xmlTextWriterWriteVFormatComment
0001:006beb84* _xmlTextWriterWriteFormatComment
0001:006beba5* _xmlTextWriterWriteVFormatAttribute
0001:006bebf5* _xmlTextWriterWriteFormatAttribute
0001:006bec1d  _xmlTextWriterWriteAttributeNS
0001:006bec97* _xmlTextWriterWriteVFormatAttributeNS
0001:006becf5* _xmlTextWriterWriteFormatAttributeNS
0001:006bed2b  _xmlTextWriterWriteElement
0001:006bed8a* _xmlTextWriterWriteVFormatElement
0001:006bedda* _xmlTextWriterWriteFormatElement
0001:006bee02  _xmlTextWriterWriteElementNS
0001:006bee7e* _xmlTextWriterWriteVFormatElementNS
0001:006beedc* _xmlTextWriterWriteFormatElementNS
0001:006befbe  _xmlTextWriterStartPI
0001:006bf1f3  _xmlTextWriterEndPI
0001:006bf28b  _xmlTextWriterWritePI
0001:006bf2fe* _xmlTextWriterWriteVFormatPI
0001:006bf34e* _xmlTextWriterWriteFormatPI
0001:006bf3ec  _xmlTextWriterStartCDATA
0001:006bf55b  _xmlTextWriterEndCDATA
0001:006bf5c4  _xmlTextWriterWriteCDATA
0001:006bf630* _xmlTextWriterWriteVFormatCDATA
0001:006bf679* _xmlTextWriterWriteFormatCDATA
0001:006bf754  _xmlTextWriterStartDTD
0001:006bfae2  _xmlTextWriterStartDTDElement
0001:006bfc8b  _xmlTextWriterEndDTDElement
0001:006bfd1b  _xmlTextWriterWriteDTDElement
0001:006bfd7f* _xmlTextWriterWriteVFormatDTDElement
0001:006bfdcf* _xmlTextWriterWriteFormatDTDElement
0001:006bfe32  _xmlTextWriterStartDTDAttlist
0001:006bffdb  _xmlTextWriterEndDTDAttlist
0001:006c006b  _xmlTextWriterWriteDTDAttlist
0001:006c00cf* _xmlTextWriterWriteVFormatDTDAttlist
0001:006c011f* _xmlTextWriterWriteFormatDTDAttlist
0001:006c0154  _xmlTextWriterStartDTDEntity
0001:006c0337  _xmlTextWriterEndDTDEntity
0001:006c03fd  _xmlTextWriterEndDTD
0001:006c0512  _xmlTextWriterWriteDTD
0001:006c0593* _xmlTextWriterWriteVFormatDTD
0001:006c05f1* _xmlTextWriterWriteFormatDTD
0001:006c0627* _xmlTextWriterWriteDTDInternalEntity
0001:006c06aa* _xmlTextWriterWriteVFormatDTDInternalEntity
0001:006c0701* _xmlTextWriterWriteFormatDTDInternalEntity
0001:006c08b1* _xmlTextWriterWriteDTDExternalEntityContents
0001:006c0b52* _xmlTextWriterWriteDTDExternalEntity
0001:006c0bf0  _xmlTextWriterWriteDTDEntity
0001:006c0c90* _xmlTextWriterWriteDTDNotation
0001:006c0f40  _xmlTextWriterFlush
0001:006c0f94  _xmlTextWriterEndDocument
0001:006c10cf  _xmlTextWriterSetIndent
0001:006c10f8  _xmlTextWriterSetIndentString
Module: U:\usr\lib\libos2.lib(code2.obj)
0001:006c1194  DosGetMessage
0001:006c1180* __msgseg32
Module: U:\tmp\ldconv_libgcc_a_3ed14e78ff521a1dd8.lib(emx-ctordtor.obj)
0001:006c11b0  ___ctordtorInit
0001:006c11e2  ___ctordtorTerm
Module: U:\tmp\ldconv_libgcc_eh_a_3ed14e78ff52199cf0.lib(emx-eh.obj)
0001:006c1220  ___ehInit
0001:006c1255* ___ehTerm
Module: U:\extras\lib\xml2.lib(nanohttp.obj)
0001:006c1e7a* _xmlNanoHTTPCleanup
0001:006c1ebb* _xmlNanoHTTPScanProxy
0001:006c1fbd* _xmlNanoHTTPInit
0001:006c2035  _xmlNanoHTTPRead
0001:006c2131  _xmlNanoHTTPClose
0001:006c22c9* _xmlNanoHTTPMethodRedir
0001:006c2f9b* _xmlNanoHTTPOpenRedir
0001:006c2ff0  _xmlNanoHTTPMethod
0001:006c302e  _xmlNanoHTTPOpen
0001:006c3074* _xmlNanoHTTPFetch
0001:006c3164* _xmlNanoHTTPSave
0001:006c3226  _xmlNanoHTTPReturnCode
0001:006c323a* _xmlNanoHTTPAuthHeader
0001:006c324b* _xmlNanoHTTPContentLength
0001:006c325f  _xmlNanoHTTPRedir
0001:006c3270  _xmlNanoHTTPEncoding
0001:006c3281  _xmlNanoHTTPMimeType
Module: U:\extras\lib\xml2.lib(nanoftp.obj)
0001:006c362d* _xmlNanoFTPCleanup
0001:006c3693* _xmlNanoFTPProxy
0001:006c3747* _xmlNanoFTPUpdateURL
0001:006c383e* _xmlNanoFTPScanProxy
0001:006c3960* _xmlNanoFTPInit
0001:006c3a21* _xmlNanoFTPNewCtxt
0001:006c3ae3* _xmlNanoFTPFreeCtxt
0001:006c3b67* _xmlNanoFTPGetResponse
0001:006c3b7d* _xmlNanoFTPCheckResponse
0001:006c3c65* _xmlNanoFTPQuit
0001:006c3dfe* _xmlNanoFTPConnect
0001:006c4482* _xmlNanoFTPConnectTo
0001:006c44f9* _xmlNanoFTPCwd
0001:006c45e1* _xmlNanoFTPDele
0001:006c4762* _xmlNanoFTPGetConnection
0001:006c4b61* _xmlNanoFTPCloseConnection
0001:006c4cce* _xmlNanoFTPList
0001:006c5490* _xmlNanoFTPGetSocket
0001:006c5651* _xmlNanoFTPGet
0001:006c5807  _xmlNanoFTPRead
0001:006c5897  _xmlNanoFTPOpen
0001:006c5908  _xmlNanoFTPClose
Module: U:\extras\lib\xml2.lib(catalog.obj)
0001:006c7bae* _xmlFreeCatalog
0001:006c7c14* _xmlConvertSGMLCatalog
0001:006c7c89* _xmlParseCatalogFile
0001:006c90e2* _xmlLoadSGMLSuperCatalog
0001:006c9153* _xmlLoadACatalog
0001:006c9254* _xmlACatalogResolveSystem
0001:006c92f7* _xmlACatalogResolvePublic
0001:006c93ca* _xmlACatalogResolve
0001:006c94d5* _xmlACatalogResolveURI
0001:006c95e1* _xmlACatalogDump
0001:006c9792* _xmlACatalogAdd
0001:006c9cde* _xmlACatalogRemove
0001:006c9ded* _xmlNewCatalog
0001:006c9e46* _xmlCatalogIsEmpty
0001:006c9ed7* _xmlInitializeCatalog
0001:006ca014* _xmlLoadCatalog
0001:006ca0a0* _xmlLoadCatalogs
0001:006ca14c  _xmlCatalogCleanup
0001:006ca20c* _xmlCatalogResolveSystem
0001:006ca236* _xmlCatalogResolvePublic
0001:006ca261  _xmlCatalogResolve
0001:006ca293  _xmlCatalogResolveURI
0001:006ca2bd* _xmlCatalogDump
0001:006ca2f3* _xmlCatalogAdd
0001:006ca3c6* _xmlCatalogRemove
0001:006ca411* _xmlCatalogConvert
0001:006ca456  _xmlCatalogGetDefaults
0001:006ca4dd* _xmlCatalogSetDefaults
0001:006ca5fa* _xmlCatalogSetDefaultPrefer
0001:006ca66e* _xmlCatalogSetDebug
0001:006ca691  _xmlCatalogFreeLocal
0001:006ca6db  _xmlCatalogAddLocal
0001:006ca7cc  _xmlCatalogLocalResolve
0001:006ca8ab  _xmlCatalogLocalResolveURI
0001:006ca955* _xmlCatalogGetSystem
0001:006caa56* _xmlCatalogGetPublic
Module: U:\extras\lib\xml2.lib(threads.obj)
0001:006cab7b  _xmlNewMutex
0001:006cabb5  _xmlFreeMutex
0001:006cabf5  _xmlMutexLock
0001:006cac14  _xmlMutexUnlock
0001:006cac32  _xmlNewRMutex
0001:006cac8e  _xmlFreeRMutex
0001:006cacd9  _xmlRMutexLock
0001:006cad72  _xmlRMutexUnlock
0001:006cadcd  ___xmlGlobalInitMutexLock
0001:006cade1  ___xmlGlobalInitMutexUnlock
0001:006cadf5  ___xmlGlobalInitMutexDestroy
0001:006cae1e  _xmlGetGlobalState
0001:006caec8  _xmlGetThreadId
0001:006caee1* _xmlLockLibrary
0001:006caef5* _xmlUnlockLibrary
0001:006caf09  _xmlInitThreads
0001:006caf23  _xmlIsMainThread
0001:006caf78  _xmlCleanupThreads
Module: U:\extras\lib\xml2.lib(SAX.obj)
0001:006cafa0  _initxmlDefaultSAXHandler
0001:006cb07e  _inithtmlDefaultSAXHandler
0001:006cb153  _initdocbDefaultSAXHandler
Module: U:\extras\lib\xml2.lib(SAX2.obj)
0001:006cb230  _xmlSAX2IsStandalone
0001:006cb24e  _xmlSAX2HasInternalSubset
0001:006cb26c  _xmlSAX2HasExternalSubset
0001:006cb28a  _xmlSAX2SetDocumentLocator
0001:006cb28f  _xmlSAX2IgnorableWhitespace
0001:006cb294  _xmlSAX2CDataBlock
0001:006cb304  _xmlSAX2Comment
0001:006cb3cd  _xmlSAX2ProcessingInstruction
0001:006cb761  _xmlSAX2Characters
0001:006cba7a  _xmlSAX2Reference
0001:006cbadd* _xmlSAX2EndElementNs
0001:006cbb72  _xmlSAX2EndElement
0001:006cbf8e* _xmlSAX2StartElementNs
0001:006cd608  _xmlSAX2StartElement
0001:006cde5b  _xmlSAX2EndDocument
0001:006cdf33  _xmlSAX2StartDocument
0001:006ce078  _xmlSAX2GetParameterEntity
0001:006ce095  _xmlSAX2ResolveEntity
0001:006ce110  _xmlSAX2ExternalSubset
0001:006ce35d  _xmlSAX2InternalSubset
0001:006ce5e6  _xmlSAX2GetEntity
0001:006ce7c5  _xmlSAX2AttributeDecl
0001:006ce9c3  _xmlSAX2ElementDecl
0001:006ceb14  _xmlSAX2NotationDecl
0001:006ceca6  _xmlSAX2EntityDecl
0001:006ceebe  _xmlSAX2UnparsedEntityDecl
0001:006cefff  _xmlSAX2GetPublicId
0001:006cf006  _xmlSAX2GetSystemId
0001:006cf021  _xmlSAX2GetLineNumber
0001:006cf039  _xmlSAX2GetColumnNumber
0001:006cf051* _xmlSAXDefaultVersion
0001:006cf073  _xmlSAXVersion
0001:006cf18d  _xmlSAX2InitDefaultSAXHandler
0001:006cf2c2  _xmlDefaultSAXHandlerInit
0001:006cf39a* _xmlSAX2InitHtmlDefaultSAXHandler
0001:006cf478  _htmlDefaultSAXHandlerInit
0001:006cf55b* _xmlSAX2InitDocbDefaultSAXHandler
0001:006cf639* _docbDefaultSAXHandlerInit
Module: U:\extras\lib\xml2.lib(chvalid.obj)
0001:006cf720  _xmlCharInRange
0001:006cf7be* _xmlIsBaseChar
0001:006cfa90  _xmlIsBaseCharGroup
0001:006cf824* _xmlIsBlank
0001:006cf852* _xmlIsChar
0001:006cf8ac* _xmlIsCombining
0001:006cfab0  _xmlIsCombiningGroup
0001:006cf8d3* _xmlIsDigit
0001:006cfac0  _xmlIsDigitGroup
0001:006cf903* _xmlIsExtender
0001:006cfad0  _xmlIsExtenderGroup
0001:006cf932* _xmlIsIdeographic
0001:006cf96e* _xmlIsPubidChar
0001:006cf990  _xmlIsPubidChar_tab
0001:006cfaa0* _xmlIsCharGroup
0001:006cfae0* _xmlIsIdeographicGroup
Module: U:\extras\lib\xml2.lib(dict.obj)
0001:006d0685  _xmlDictCleanup
0001:006d06b0  _xmlDictCreate
0001:006d0742  _xmlDictReference
0001:006d0799* _xmlDictCreateSub
0001:006d07d0  _xmlDictFree
0001:006d08ea  _xmlDictLookup
0001:006d0c09  _xmlDictExists
0001:006d0e00  _xmlDictQLookup
0001:006d12bd  _xmlDictOwns
0001:006d1310* _xmlDictSize
Module: U:\extras\lib\xml2.lib(xmlmemory.obj)
0001:006d13bd* _xmlMallocBreakpoint
0001:006d1441* _xmlMemFree
0001:006d156f* _xmlMemUsed
0001:006d1579* _xmlMemBlocks
0001:006d15c7* _xmlMemDisplayLast
0001:006d1649* _xmlMemDisplay
0001:006d16ef  _xmlMemShow
0001:006d1722* _xmlMemoryDump
0001:006d174f  _xmlInitMemory
0001:006d17ed* _xmlMemStrdupLoc
0001:006d191c* _xmlMemoryStrdup
0001:006d1977* _xmlMallocAtomicLoc
0001:006d1aa0* _xmlMallocLoc
0001:006d1bbd* _xmlMemMalloc
0001:006d1bff* _xmlReallocLoc
0001:006d1d97* _xmlMemRealloc
0001:006d1dc1  _xmlCleanupMemory
0001:006d1df5* _xmlMemSetup
0001:006d1e44* _xmlMemGet
0001:006d1e8b* _xmlGcMemSetup
0001:006d1ee4* _xmlGcMemGet
Module: U:\extras\lib\xml2.lib(xmlschemastypes.obj)
0001:006d3477  _xmlSchemaInitTypes
0001:006d3a4b  _xmlSchemaCleanupTypes
0001:006d3ada  _xmlSchemaIsBuiltInTypeFacet
0001:006d3c68  _xmlSchemaGetBuiltInType
0001:006d3f27  _xmlSchemaValueAppend
0001:006d3f46  _xmlSchemaValueGetNext
0001:006d3f57  _xmlSchemaValueGetAsString
0001:006d403d  _xmlSchemaValueGetAsBoolean
0001:006d4055* _xmlSchemaNewStringValue
0001:006d4095  _xmlSchemaNewNOTATIONValue
0001:006d40c0  _xmlSchemaNewQNameValue
0001:006d40e2  _xmlSchemaFreeValue
0001:006d5aef  _xmlSchemaGetPredefinedType
0001:006d5b2d* _xmlSchemaGetBuiltInListSimpleTypeItemType
0001:006d5b67  _xmlSchemaWhiteSpaceReplace
0001:006d5bec  _xmlSchemaCollapseString
0001:006d5d91  _xmlSchemaValPredefTypeNode
0001:006d85e5  _xmlSchemaValPredefTypeNodeNoNorm
0001:006d861a  _xmlSchemaValidatePredefinedType
0001:006d8643  _xmlSchemaCopyValue
0001:006d87cc  _xmlSchemaCompareValues
0001:006d8cc0  _xmlSchemaCompareValuesWhtsp
0001:006d8d07  _xmlSchemaGetFacetValueAsULong
0001:006d8d1b* _xmlSchemaValidateLengthFacet
0001:006d8d54  _xmlSchemaValidateLengthFacetWhtsp
0001:006d8d80  _xmlSchemaValidateFacet
0001:006d8dd7  _xmlSchemaValidateListSimpleTypeFacet
0001:006d8e79  _xmlSchemaValidateFacetWhtsp
0001:006d8ff2  _xmlSchemaGetCanonValue
0001:006d9e48* _xmlSchemaGetCanonValueWhtsp
0001:006d9f44  _xmlSchemaGetValType
Module: U:\extras\lib\xml2.lib(xmlregexp.obj)
0001:006e03d2  _xmlRegNewExecCtxt
0001:006e050c  _xmlRegFreeExecCtxt
0001:006e05d3  _xmlRegExecPushString
0001:006e05ef  _xmlRegExecPushString2
0001:006e077b  _xmlRegExecNextValues
0001:006e07a6  _xmlRegExecErrInfo
0001:006e0999* _xmlRegexpPrint
0001:006e11c5  _xmlRegexpExec
0001:006e1769  _xmlRegFreeRegexp
0001:006e187b  _xmlFreeAutomata
0001:006e1890  _xmlNewAutomata
0001:006e18f0  _xmlRegexpIsDeterminist
0001:006e20ff  _xmlRegexpCompile
0001:006e21a7  _xmlAutomataSetFlags
0001:006e21b9  _xmlAutomataGetInitState
0001:006e21ca  _xmlAutomataSetFinalState
0001:006e21ec  _xmlAutomataNewTransition
0001:006e226f  _xmlAutomataNewTransition2
0001:006e23ad  _xmlAutomataNewNegTrans
0001:006e2568  _xmlAutomataNewCountTrans2
0001:006e277f* _xmlAutomataNewCountTrans
0001:006e28ca  _xmlAutomataNewOnceTrans2
0001:006e2a85* _xmlAutomataNewOnceTrans
0001:006e2b74  _xmlAutomataNewState
0001:006e2b9a  _xmlAutomataNewEpsilon
0001:006e2bca  _xmlAutomataNewAllTrans
0001:006e2c60  _xmlAutomataNewCounter
0001:006e2ca2  _xmlAutomataNewCountedTrans
0001:006e2ce2  _xmlAutomataNewCounterTrans
0001:006e2d22  _xmlAutomataCompile
0001:006e2d52* _xmlAutomataIsDeterminist
0001:006e2d6c* _xmlExpNewCtxt
0001:006e2e1b* _xmlExpFreeCtxt
0001:006e2e58* _xmlExpFree
0001:006e4650* _xmlExpRef
0001:006e4660* _xmlExpNewAtom
0001:006e46c5* _xmlExpNewOr
0001:006e472e* _xmlExpNewSeq
0001:006e4797* _xmlExpNewRange
0001:006e4803* _xmlExpGetLanguage
0001:006e4846* _xmlExpGetStart
0001:006e4888* _xmlExpIsNillable
0001:006e48a0* _xmlExpStringDerive
0001:006e48f7* _xmlExpExpDerive
0001:006e494c* _xmlExpSubsume
0001:006e49fb* _xmlExpParse
0001:006e4a51* _xmlExpDump
0001:006e4a75* _xmlExpMaxToken
0001:006e4a89* _xmlExpCtxtNbNodes
0001:006e4a9d* _xmlExpCtxtNbCons
0002:00004b40* _forbiddenExp
0002:00004b44* _emptyExp
Module: U:\extras\lib\xml2.lib(list.obj)
0001:006e4cd6  _xmlListCreate
0001:006e4d99  _xmlListSearch
0001:006e4dc8* _xmlListReverseSearch
0001:006e4e1e  _xmlListInsert
0001:006e4ea8  _xmlListAppend
0001:006e4f31  _xmlListRemoveFirst
0001:006e4f83* _xmlListRemoveLast
0001:006e4fd5* _xmlListRemoveAll
0001:006e5009* _xmlListClear
0001:006e5052  _xmlListDelete
0001:006e5088  _xmlListEmpty
0001:006e50a3  _xmlListFront
0001:006e50b5* _xmlListEnd
0001:006e50c8  _xmlListSize
0001:006e50ec  _xmlListPopFront
0001:006e512f* _xmlListPopBack
0001:006e5173  _xmlListPushFront
0001:006e51d6* _xmlListPushBack
0001:006e523c  _xmlLinkGetData
0001:006e524d* _xmlListReverse
0001:006e5285  _xmlListWalk
0001:006e52c7* _xmlListReverseWalk
0001:006e530b* _xmlListCopy
0001:006e5373* _xmlListDup
0001:006e53c0* _xmlListMerge
0001:006e53e6* _xmlListSort
Module: U:\extras\lib\libz.lib(adler32.obj)
0001:006e5440  _adler32
0001:006e56b0* _adler32_combine
0001:006e5758* _adler32_combine64
Module: U:\extras\lib\libz.lib(trees.obj)
0001:006e5800  __tr_init
0001:006e5ebc  __tr_stored_block
0001:006e6020  __tr_align
0001:006e639c* __tr_tally
0001:006e7f30  __length_code
0001:006e7d30  __dist_code
0001:006e724c  __tr_flush_block
Module: U:\extras\lib\libz.lib(inftrees.obj)
0001:006e87a0  _inflate_table
0001:006e9150* _inflate_copyright
Module: U:\extras\lib\libz.lib(inffast.obj)
0001:006e92d0  _inflate_fast
Module: U:\extras\lib\xml2.lib(pattern.obj)
0001:006eb255  _xmlFreePattern
0001:006eb336  _xmlFreePatternList
0001:006eb364  _xmlFreeStreamCtxt
0001:006eb39d  _xmlStreamPush
0001:006eb3b9  _xmlStreamPushNode
0001:006eb3d4  _xmlStreamPushAttr
0001:006eb3f0  _xmlStreamPop
0001:006eb453  _xmlStreamWantsAnyNode
0001:006eb48c  _xmlPatterncompile
0001:006ec11d  _xmlPatternMatch
0001:006ec6a2  _xmlPatternGetStreamCtxt
0001:006ec77b  _xmlPatternStreamable
0001:006ec7ae  _xmlPatternMaxDepth
0001:006ec818  _xmlPatternMinDepth
0001:006ec869  _xmlPatternFromRoot
Module: U:\extras\lib\xml2.lib(debugXML.obj)
0001:006ef75a  _xmlDebugDumpString
0001:006ef837  _xmlDebugDumpAttr
0001:006ef924* _xmlDebugDumpEntities
0001:006efab8* _xmlDebugDumpAttrList
0001:006efbac  _xmlDebugDumpOneNode
0001:006efc1c* _xmlDebugDumpNode
0001:006efc94* _xmlDebugDumpNodeList
0001:006efd0c* _xmlDebugDumpDocumentHead
0001:006efd85* _xmlDebugDumpDocument
0001:006efe1d* _xmlDebugDumpDTD
0001:006eff13* _xmlDebugCheckDocument
0001:006eff8f* _xmlLsCountNode
0001:006f005b* _xmlLsOneNode
0001:006f03a7* _xmlBoolToText
0001:006f0455* _xmlShellPrintXPathError
0001:006f05da* _xmlShellPrintNode
0001:006f05e9* _xmlShellPrintXPathResult
0001:006f05ee* _xmlShellList
0001:006f068d* _xmlShellBase
0001:006f072b* _xmlShellDir
0001:006f07bf* _xmlShellCat
0001:006f0873* _xmlShellLoad
0001:006f0943* _xmlShellWrite
0001:006f0a5f* _xmlShellSave
0001:006f0b19* _xmlShellValidate
0001:006f0bbe* _xmlShellDu
0001:006f0d40* _xmlShellPwd
0001:006f1565* _xmlShell
Module: U:\extras\lib\xml2.lib(xpointer.obj)
0001:006f3673  _xmlXPtrNewRange
0001:006f36fb* _xmlXPtrNewRangePoints
0001:006f3782* _xmlXPtrNewRangePointNode
0001:006f3802* _xmlXPtrNewRangeNodePoint
0001:006f3887* _xmlXPtrNewRangeNodes
0001:006f38fd* _xmlXPtrNewCollapsedRange
0001:006f3989  _xmlXPtrNewRangeNodeObject
0001:006f3ac1  _xmlXPtrLocationSetCreate
0001:006f3b73  _xmlXPtrLocationSetAdd
0001:006f3c98  _xmlXPtrLocationSetMerge
0001:006f3ce3* _xmlXPtrLocationSetDel
0001:006f3d3b* _xmlXPtrLocationSetRemove
0001:006f3d78  _xmlXPtrFreeLocationSet
0001:006f3dd8* _xmlXPtrNewLocationSetNodes
0001:006f3f2b* _xmlXPtrNewLocationSetNodeSet
0001:006f3fcd  _xmlXPtrWrapLocationSet
0001:006f4018* _xmlXPtrRangeToFunction
0001:006f4b25  _xmlXPtrNewContext
0001:006f4ce3  _xmlXPtrEval
0001:006f5364  _xmlXPtrAdvanceNode
0001:006f540c* _xmlXPtrBuildNodeList
0001:006f61ce* _xmlXPtrEvalRangePredicate
Module: U:\extras\lib\libcrypto.lib(err.obj)
0001:006f6951* _ERR_get_implementation
0001:006f6963* _ERR_set_implementation
0001:006f73b6* _ERR_load_ERR_strings
0001:006f745d* _ERR_load_strings
0001:006f747c* _ERR_unload_strings
0001:006f74c1* _ERR_free_strings
0001:006f74d8  _ERR_put_error
0001:006f7f43* _ERR_get_state
0001:006f7635  _ERR_clear_error
0001:006f771a* _ERR_get_error
0001:006f7756* _ERR_get_error_line
0001:006f7790  _ERR_get_error_line_data
0001:006f77c8  _ERR_peek_error
0001:006f7804* _ERR_peek_error_line
0001:006f783e* _ERR_peek_error_line_data
0001:006f7876  _ERR_peek_last_error
0001:006f78b2* _ERR_peek_last_error_line
0001:006f78ec* _ERR_peek_last_error_line_data
0001:006f7b6e  _ERR_error_string_n
0001:006f7da4* _ERR_lib_error_string
0001:006f7dee* _ERR_func_error_string
0001:006f7e55* _ERR_reason_error_string
0001:006f7d1a* _ERR_error_string
0001:006f7d4c* _ERR_get_string_table
0001:006f7d69* _ERR_get_err_state_table
0001:006f7d87* _ERR_release_err_state_table
0001:006f7ee1* _ERR_remove_thread_state
0001:006f7f2f* _ERR_remove_state
0001:006f8080* _ERR_get_next_error_library
0001:006f8097* _ERR_set_error_data
0001:006f813c  _ERR_add_error_data
0001:006f8249  _ERR_set_mark
0001:006f82a0  _ERR_pop_to_mark
Module: U:\extras\lib\libssl.lib(ssl_sess.obj)
0001:006f8430  _SSL_get_session
0001:006f8449* _SSL_get1_session
0001:006f84c3* _SSL_SESSION_get_ex_new_index
0001:006f84fa* _SSL_SESSION_set_ex_data
0001:006f8521* _SSL_SESSION_get_ex_data
0001:006f8541  _SSL_SESSION_new
0001:006f869f* _SSL_SESSION_get_id
0001:006f8723  _ssl_get_new_session
0001:006f954d  _SSL_SESSION_free
0001:006f8dba* _ssl_get_prev_session
0001:006f9255  _SSL_CTX_add_session
0001:006f9416  _SSL_CTX_remove_session
0001:006f9749  _SSL_set_session
0001:006f9921* _SSL_SESSION_set_timeout
0001:006f9944* _SSL_SESSION_get_timeout
0001:006f995f* _SSL_SESSION_get_time
0001:006f997a* _SSL_SESSION_set_time
0001:006f999b* _SSL_CTX_set_timeout
0001:006f99c5* _SSL_CTX_get_timeout
0001:006f99dd* _SSL_set_session_secret_cb
0001:006f9a0c* _SSL_set_session_ticket_ext_cb
0001:006f9a3b* _SSL_set_session_ticket_ext
0001:006f9c1f  _SSL_CTX_flush_sessions
0001:006f9cc8  _ssl_clear_bad_session
0001:006f9f05* _SSL_CTX_sess_set_new_cb
0001:006f9f13* _SSL_CTX_sess_get_new_cb
0001:006f9f1e* _SSL_CTX_sess_set_remove_cb
0001:006f9f2c* _SSL_CTX_sess_get_remove_cb
0001:006f9f37* _SSL_CTX_sess_set_get_cb
0001:006f9f45* _SSL_CTX_sess_get_get_cb
0001:006f9f50* _SSL_CTX_set_info_callback
0001:006f9f61* _SSL_CTX_get_info_callback
0001:006f9f6f* _SSL_CTX_set_client_cert_cb
0001:006f9f7d* _SSL_CTX_get_client_cert_cb
0001:006f9f88* _SSL_CTX_set_client_cert_engine
0001:006fa030* _SSL_CTX_set_cookie_generate_cb
0001:006fa03e* _SSL_CTX_set_cookie_verify_cb
0001:006fa063* _PEM_read_bio_SSL_SESSION
0001:006fa09c* _PEM_read_SSL_SESSION
0001:006fa0d5* _PEM_write_bio_SSL_SESSION
0001:006fa128* _PEM_write_SSL_SESSION
Module: U:\extras\lib\libcrypto.lib(buffer.obj)
0001:006fa189  _BUF_MEM_new
0001:006fa209  _BUF_MEM_free
0001:006fa25d  _BUF_MEM_grow
0001:006fa3b9  _BUF_MEM_grow_clean
0001:006fa548  _BUF_strdup
0001:006fa577  _BUF_strndup
0001:006fa686  _BUF_strlcpy
0001:006fa601  _BUF_memdup
0001:006fa6d6  _BUF_strlcat
0001:006fa71b* _BUF_reverse
Module: U:\extras\lib\libssl.lib(ssl_ciph.obj)
0001:006fb761* _ssl_load_ciphers
0001:006fbaf8  _ssl_cipher_get_evp
0001:006fbda6  _ssl_get_handshake_digest
0001:006fcf89  _ssl_create_cipher_list
0001:006fd88e* _SSL_CIPHER_description
0001:006fdd24* _SSL_CIPHER_get_version
0001:006fdd64* _SSL_CIPHER_get_name
0001:006fdd7c* _SSL_CIPHER_get_bits
0001:006fddae  _ssl3_comp_find
0001:006fde14  _SSL_COMP_get_compression_methods
0001:006fde26* _SSL_COMP_add_compression_method
0001:006fdfb7* _SSL_COMP_get_name
Module: U:\extras\lib\libcrypto.lib(stack.obj)
0001:006fe000* _STACK_version
0001:006fe028  _sk_set_cmp_func
0001:006fe062  _sk_dup
0001:006fe14f  _sk_new
0001:006fe685  _sk_free
0001:006fe13b  _sk_new_null
0001:006fe215  _sk_insert
0001:006fe32e  _sk_delete_ptr
0001:006fe37a  _sk_delete
0001:006fe739  _sk_sort
0001:006fe4e0  _sk_find
0001:006fe502* _sk_find_ex
0001:006fe524  _sk_push
0001:006fe547* _sk_unshift
0001:006fe569* _sk_shift
0001:006fe5a1  _sk_pop
0001:006fe5db  _sk_zero
0001:006fe627  _sk_pop_free
0001:006fe6b9  _sk_num
0001:006fe6d0  _sk_value
0001:006fe702  _sk_set
0001:006fe78c  _sk_is_sorted
Module: U:\extras\lib\libcrypto.lib(mem.obj)
0001:006fe7f9* _CRYPTO_set_mem_functions
0001:006fe872* _CRYPTO_set_mem_ex_functions
0001:006fe8eb* _CRYPTO_set_locked_mem_functions
0001:006fe932* _CRYPTO_set_locked_mem_ex_functions
0001:006fe979* _CRYPTO_set_mem_debug_functions
0001:006fe9bb* _CRYPTO_get_mem_functions
0001:006fea17* _CRYPTO_get_mem_ex_functions
0001:006fea73* _CRYPTO_get_locked_mem_functions
0001:006feaac* _CRYPTO_get_locked_mem_ex_functions
0001:006feae5* _CRYPTO_get_mem_debug_functions
0001:006feb3f  _CRYPTO_malloc_locked
0001:006fec17  _CRYPTO_free_locked
0001:006fec6b  _CRYPTO_malloc
0001:006fed43* _CRYPTO_strdup
0001:006fed85  _CRYPTO_realloc
0001:006fee68  _CRYPTO_realloc_clean
0001:006fef83  _CRYPTO_free
0001:006fefdd* _CRYPTO_remalloc
0001:006ff017* _CRYPTO_set_mem_debug_options
0001:006ff036* _CRYPTO_get_mem_debug_options
Module: U:\extras\lib\libssl.lib(ssl_cert.obj)
0001:006ff083  _SSL_get_ex_data_X509_STORE_CTX_idx
0001:006ff1a1  _ssl_cert_new
0001:006ff234  _ssl_cert_dup
0001:006ff6d9  _ssl_cert_free
0001:006ff7db  _ssl_cert_inst
0001:006ff870  _ssl_sess_cert_new
0001:006ff904  _ssl_sess_cert_free
0001:006ff9fb  _ssl_set_peer_cert_type
0001:006ffa24  _ssl_verify_cert_chain
0001:006ffbf9* _SSL_dup_CA_list
0001:006ffc7c* _SSL_set_client_CA_list
0001:006ffc9c* _SSL_CTX_set_client_CA_list
0001:006ffcbc* _SSL_CTX_get_client_CA_list
0001:006ffcca  _SSL_get_client_CA_list
0001:006ffdbb* _SSL_add_client_CA
0001:006ffddb* _SSL_CTX_add_client_CA
0001:006ffe19* _SSL_load_client_CA_file
0001:0070000a* _SSL_add_file_cert_subjects_to_stack
0001:007001a6* _SSL_add_dir_cert_subjects_to_stack
Module: U:\extras\lib\libcrypto.lib(cryptlib.obj)
0001:0070058f* _CRYPTO_get_new_lockid
0001:0070065e* _CRYPTO_num_locks
0001:00700668* _CRYPTO_get_new_dynlockid
0001:00700d2d  _CRYPTO_lock
0001:0070091d* _CRYPTO_destroy_dynlockid
0001:00700a5b* _CRYPTO_get_dynlock_value
0001:00700b13* _CRYPTO_get_dynlock_create_callback
0001:00700b1d* _CRYPTO_get_dynlock_lock_callback
0001:00700b27* _CRYPTO_get_dynlock_destroy_callback
0001:00700b31* _CRYPTO_set_dynlock_create_callback
0001:00700b3e* _CRYPTO_set_dynlock_lock_callback
0001:00700b4b* _CRYPTO_set_dynlock_destroy_callback
0001:00700b58* _CRYPTO_get_locking_callback
0001:00700b62* _CRYPTO_get_add_lock_callback
0001:00700b6c* _CRYPTO_set_locking_callback
0001:00700b79* _CRYPTO_set_add_lock_callback
0001:00700b86* _CRYPTO_THREADID_set_numeric
0001:00700bba* _CRYPTO_THREADID_set_pointer
0001:00700c06* _CRYPTO_THREADID_set_callback
0001:00700c28* _CRYPTO_THREADID_get_callback
0001:00700c32  _CRYPTO_THREADID_current
0001:00700c88  _CRYPTO_THREADID_cmp
0001:00700caa  _CRYPTO_THREADID_cpy
0001:00700ccc  _CRYPTO_THREADID_hash
0001:00700cd7* _CRYPTO_get_id_callback
0001:00700ce1* _CRYPTO_set_id_callback
0001:00700cee* _CRYPTO_thread_id
0001:00700f5a  _OpenSSLDie
0001:00700dd4  _CRYPTO_add_lock
0001:00700e81* _CRYPTO_get_lock_name
0001:00700ee2* _OPENSSL_ia32cap_loc
0001:00700eec* _OPENSSL_cpuid_setup
0001:00700ef1* _OPENSSL_showfatal
0001:00700f1a* _OPENSSL_isservice
0001:00700f86* _OPENSSL_stderr
0002:0001f3b0* _OPENSSL_ia32cap_P
0002:0001f3b4* _OPENSSL_NONPIC_relocated
Module: U:\extras\lib\libcrypto.lib(x509_vpm.obj)
0001:00701012  _X509_VERIFY_PARAM_new
0001:00701062  _X509_VERIFY_PARAM_free
0001:00701080  _X509_VERIFY_PARAM_inherit
0001:007013ca* _X509_VERIFY_PARAM_set1_policies
0001:00701228  _X509_VERIFY_PARAM_set1
0001:0070126b* _X509_VERIFY_PARAM_set1_name
0001:007012ae  _X509_VERIFY_PARAM_set_flags
0001:007012e6* _X509_VERIFY_PARAM_clear_flags
0001:00701303* _X509_VERIFY_PARAM_get_flags
0001:0070130e  _X509_VERIFY_PARAM_set_purpose
0001:0070132b  _X509_VERIFY_PARAM_set_trust
0001:00701348  _X509_VERIFY_PARAM_set_depth
0001:00701356  _X509_VERIFY_PARAM_set_time
0001:00701375* _X509_VERIFY_PARAM_add0_policy
0001:007014cb  _X509_VERIFY_PARAM_get_depth
0001:00701647* _X509_VERIFY_PARAM_add0_table
0001:007016f1  _X509_VERIFY_PARAM_lookup
0001:00701756* _X509_VERIFY_PARAM_table_cleanup
Module: U:\extras\lib\libcrypto.lib(ex_data.obj)
0001:007017fd* _CRYPTO_get_ex_data_implementation
0001:00701818* _CRYPTO_set_ex_data_implementation
0001:007025a1  _CRYPTO_get_ex_data
0001:007024bc  _CRYPTO_set_ex_data
0001:0070238b* _CRYPTO_ex_data_new_class
0001:007023aa* _CRYPTO_cleanup_all_ex_data
0001:007023ca  _CRYPTO_get_ex_new_index
0001:00702420  _CRYPTO_new_ex_data
0001:00702454  _CRYPTO_dup_ex_data
0001:00702488  _CRYPTO_free_ex_data
Module: U:\extras\lib\libcrypto.lib(lhash.obj)
0001:007025f0* _lh_version
0001:00702620  _lh_new
0001:00702f5a  _lh_strhash
0001:007027bd  _lh_free
0001:00702831  _lh_insert
0001:0070294f  _lh_delete
0001:00702a29  _lh_retrieve
0001:00702b0a  _lh_doall
0001:00702b3c  _lh_doall_arg
0001:00702fd1  _lh_num_items
Module: U:\extras\lib\libcrypto.lib(bio_lib.obj)
0001:00702ffa  _BIO_new
0001:0070308c  _BIO_set
0001:00703180  _BIO_free
0001:00703280  _BIO_vfree
0001:00703293  _BIO_clear_flags
0001:007032ab  _BIO_test_flags
0001:007032b9  _BIO_set_flags
0001:007032cf* _BIO_get_callback
0001:007032da* _BIO_set_callback
0001:007032e8* _BIO_set_callback_arg
0001:007032f6* _BIO_get_callback_arg
0001:00703301* _BIO_method_name
0001:0070330e  _BIO_method_type
0001:0070331a  _BIO_read
0001:00703475  _BIO_write
0001:007035da  _BIO_puts
0001:00703730  _BIO_gets
0001:00703876  _BIO_indent
0001:007038ce  _BIO_int_ctrl
0001:00703939  _BIO_ctrl
0001:007038fc* _BIO_ptr_ctrl
0001:00703a4c  _BIO_callback_ctrl
0001:00703b5a* _BIO_ctrl_pending
0001:00703b85* _BIO_ctrl_wpending
0001:00703bb0  _BIO_push
0001:00703c1b  _BIO_pop
0001:00703ca4* _BIO_get_retry_BIO
0001:00703cfe  _BIO_get_retry_reason
0001:00703d09  _BIO_find_type
0001:00703d74  _BIO_next
0001:00703d8c  _BIO_free_all
0001:00703dc8* _BIO_dup_chain
0001:00703f00  _BIO_copy_next_retry
0001:00703f3c* _BIO_get_ex_new_index
0001:00703f73* _BIO_set_ex_data
0001:00703f97* _BIO_get_ex_data
0001:00703fb4* _BIO_number_read
0001:00703fcc* _BIO_number_written
Module: U:\extras\lib\libcrypto.lib(x_exten.obj)
0001:00704060  _X509_EXTENSION_it
0001:007040c0  _X509_EXTENSIONS_it
0001:007040dc* _d2i_X509_EXTENSION
0001:00704105* _i2d_X509_EXTENSION
0001:00704127  _X509_EXTENSION_new
0001:0070413b  _X509_EXTENSION_free
0001:00704156  _d2i_X509_EXTENSIONS
0001:0070417f  _i2d_X509_EXTENSIONS
0001:007041a1  _X509_EXTENSION_dup
Module: U:\extras\lib\libcrypto.lib(ocsp_asn.obj)
0001:00704240* _OCSP_SIGNATURE_it
0001:0070425c* _d2i_OCSP_SIGNATURE
0001:00704285* _i2d_OCSP_SIGNATURE
0001:007042a7* _OCSP_SIGNATURE_new
0001:007042bb* _OCSP_SIGNATURE_free
0001:00704370* _OCSP_CERTID_it
0001:0070438c* _d2i_OCSP_CERTID
0001:007043b5* _i2d_OCSP_CERTID
0001:007043d7* _OCSP_CERTID_new
0001:007043eb* _OCSP_CERTID_free
0001:00704470* _OCSP_ONEREQ_it
0001:0070448c* _d2i_OCSP_ONEREQ
0001:007044b5* _i2d_OCSP_ONEREQ
0001:007044d7* _OCSP_ONEREQ_new
0001:007044eb* _OCSP_ONEREQ_free
0001:007045a0* _OCSP_REQINFO_it
0001:007045bc* _d2i_OCSP_REQINFO
0001:007045e5* _i2d_OCSP_REQINFO
0001:00704607* _OCSP_REQINFO_new
0001:0070461b* _OCSP_REQINFO_free
0001:007046a0* _OCSP_REQUEST_it
0001:007046bc* _d2i_OCSP_REQUEST
0001:007046e5* _i2d_OCSP_REQUEST
0001:00704707* _OCSP_REQUEST_new
0001:0070471b* _OCSP_REQUEST_free
0001:00704790* _OCSP_RESPBYTES_it
0001:007047ac* _d2i_OCSP_RESPBYTES
0001:007047d5* _i2d_OCSP_RESPBYTES
0001:007047f7* _OCSP_RESPBYTES_new
0001:0070480b* _OCSP_RESPBYTES_free
0001:00704890* _OCSP_RESPONSE_it
0001:007048ac* _d2i_OCSP_RESPONSE
0001:007048d5* _i2d_OCSP_RESPONSE
0001:007048f7* _OCSP_RESPONSE_new
0001:0070490b* _OCSP_RESPONSE_free
0001:00704980* _OCSP_RESPID_it
0001:0070499c  _d2i_OCSP_RESPID
0001:007049c5  _i2d_OCSP_RESPID
0001:007049e7* _OCSP_RESPID_new
0001:007049fb  _OCSP_RESPID_free
0001:00704a80* _OCSP_REVOKEDINFO_it
0001:00704a9c* _d2i_OCSP_REVOKEDINFO
0001:00704ac5* _i2d_OCSP_REVOKEDINFO
0001:00704ae7* _OCSP_REVOKEDINFO_new
0001:00704afb* _OCSP_REVOKEDINFO_free
0001:00704b90* _OCSP_CERTSTATUS_it
0001:00704bac* _d2i_OCSP_CERTSTATUS
0001:00704bd5* _i2d_OCSP_CERTSTATUS
0001:00704bf7* _OCSP_CERTSTATUS_new
0001:00704c0b* _OCSP_CERTSTATUS_free
0001:00704ce0* _OCSP_SINGLERESP_it
0001:00704cfc* _d2i_OCSP_SINGLERESP
0001:00704d25* _i2d_OCSP_SINGLERESP
0001:00704d47* _OCSP_SINGLERESP_new
0001:00704d5b* _OCSP_SINGLERESP_free
0001:00704e30* _OCSP_RESPDATA_it
0001:00704e4c* _d2i_OCSP_RESPDATA
0001:00704e75* _i2d_OCSP_RESPDATA
0001:00704e97* _OCSP_RESPDATA_new
0001:00704eab* _OCSP_RESPDATA_free
0001:00704f40* _OCSP_BASICRESP_it
0001:00704f5c* _d2i_OCSP_BASICRESP
0001:00704f85* _i2d_OCSP_BASICRESP
0001:00704fa7* _OCSP_BASICRESP_new
0001:00704fbb* _OCSP_BASICRESP_free
0001:00705040  _OCSP_CRLID_it
0001:0070505c* _d2i_OCSP_CRLID
0001:00705085* _i2d_OCSP_CRLID
0001:007050a7* _OCSP_CRLID_new
0001:007050bb* _OCSP_CRLID_free
0001:00705130  _OCSP_SERVICELOC_it
0001:0070514c* _d2i_OCSP_SERVICELOC
0001:00705175* _i2d_OCSP_SERVICELOC
0001:00705197* _OCSP_SERVICELOC_new
0001:007051ab* _OCSP_SERVICELOC_free
Module: U:\extras\lib\libcrypto.lib(x_name.obj)
0001:007052a0  _X509_NAME_ENTRY_it
0001:007052bc* _d2i_X509_NAME_ENTRY
0001:007052e5* _i2d_X509_NAME_ENTRY
0001:00705307  _X509_NAME_ENTRY_new
0001:0070531b  _X509_NAME_ENTRY_free
0001:00705336  _X509_NAME_ENTRY_dup
0001:00705390* _X509_NAME_ENTRIES_it
0001:007053f0* _X509_NAME_INTERNAL_it
0001:00705410* _x509_name_ff
0001:00705440  _X509_NAME_it
0001:0070545c  _d2i_X509_NAME
0001:00705485  _i2d_X509_NAME
0001:007054a7  _X509_NAME_new
0001:007054bb  _X509_NAME_free
0001:007054d6  _X509_NAME_dup
0001:00705f86  _X509_NAME_set
Module: U:\extras\lib\libcrypto.lib(bss_sock.obj)
0001:00705ff7  _BIO_s_socket
0001:00706001* _BIO_new_socket
0001:007062d7* _BIO_sock_should_retry
0001:00706307* _BIO_sock_non_fatal_error
Module: U:\extras\lib\libcrypto.lib(x509_cmp.obj)
0001:00706340* _X509_issuer_and_serial_cmp
0001:00706616  _X509_NAME_cmp
0001:00706396* _X509_issuer_and_serial_hash
0001:0070649d* _X509_issuer_name_cmp
0001:007064c1  _X509_subject_name_cmp
0001:007064e5  _X509_CRL_cmp
0001:00706509  _X509_CRL_match
0001:00706531  _X509_get_issuer_name
0001:0070653e* _X509_issuer_name_hash
0001:007066d0  _X509_NAME_hash
0001:00706556* _X509_issuer_name_hash_old
0001:00706759* _X509_NAME_hash_old
0001:0070656e  _X509_get_subject_name
0001:0070657b  _X509_get_serialNumber
0001:00706588* _X509_subject_name_hash
0001:007065a0* _X509_subject_name_hash_old
0001:007065b8  _X509_cmp
0001:007067e5  _X509_find_by_issuer_and_serial
0001:0070686d* _X509_find_by_subject
0001:007068ce  _X509_get_pubkey
0001:007068fc  _X509_get0_pubkey_bitstr
0001:00706924  _X509_check_private_key
Module: U:\extras\lib\libssl.lib(s3_pkt.obj)
0001:00706a39* _ssl3_read_n
0001:0070742a* _ssl3_do_uncompress
0001:00708ced  _ssl3_send_alert
0001:007074a8* _ssl3_do_compress
0001:00707526  _ssl3_write_bytes
0001:00707b22* _ssl3_write_pending
0001:00707cf5  _ssl3_read_bytes
0001:00708b75* _ssl3_do_change_cipher_spec
0001:00708dbc  _ssl3_dispatch_alert
Module: U:\extras\lib\libcrypto.lib(x509_lu.obj)
0001:00708f5a* _X509_LOOKUP_new
0001:00708fef* _X509_LOOKUP_free
0001:00709033* _X509_LOOKUP_init
0001:00709071* _X509_LOOKUP_shutdown
0001:007090af  _X509_LOOKUP_ctrl
0001:00709109* _X509_LOOKUP_by_subject
0001:00709166* _X509_LOOKUP_by_issuer_serial
0001:007091b9* _X509_LOOKUP_by_fingerprint
0001:0070920c* _X509_LOOKUP_by_alias
0001:007092e8  _X509_STORE_new
0001:0070946a  _X509_STORE_free
0001:00709531  _X509_STORE_add_lookup
0001:007095d5* _X509_STORE_get_by_subject
0001:00709ba6* _X509_OBJECT_retrieve_by_subject
0001:007099cd* _X509_OBJECT_up_ref_count
0001:00709717  _X509_STORE_add_cert
0001:0070a083* _X509_OBJECT_retrieve_match
0001:00709a4b* _X509_OBJECT_free_contents
0001:00709872  _X509_STORE_add_crl
0001:00709b7d* _X509_OBJECT_idx_by_subject
0001:00709be9  _X509_STORE_get1_certs
0001:00709e3b  _X509_STORE_get1_crls
0001:0070a18f  _X509_STORE_CTX_get1_issuer
0001:0070a3ae* _X509_STORE_set_flags
0001:0070a3cb* _X509_STORE_set_depth
0001:0070a3ed* _X509_STORE_set_purpose
0001:0070a40a* _X509_STORE_set_trust
0001:0070a427* _X509_STORE_set1_param
0001:0070a444* _X509_STORE_set_verify_cb
Module: U:\extras\lib\libcrypto.lib(names.obj)
0001:0070a460* _EVP_add_cipher
0001:0070a4d8* _EVP_add_digest
0001:0070a5ed  _EVP_get_cipherbyname
0001:0070a60e  _EVP_get_digestbyname
0001:0070a62f* _EVP_cleanup
0001:0070a6f5* _EVP_CIPHER_do_all
0001:0070a724* _EVP_CIPHER_do_all_sorted
0001:0070a7ca* _EVP_MD_do_all
0001:0070a7f9* _EVP_MD_do_all_sorted
Module: U:\extras\lib\libcrypto.lib(rand_lib.obj)
0001:0070a830  _RAND_set_rand_method
0001:0070a865* _RAND_get_rand_method
0001:0070a8ce* _RAND_set_rand_engine
0001:0070a937* _RAND_cleanup
0001:0070a96b  _RAND_seed
0001:0070a99e  _RAND_add
0001:0070a9ed  _RAND_bytes
0001:0070aa29  _RAND_pseudo_bytes
0001:0070aa65  _RAND_status
Module: U:\extras\lib\libcrypto.lib(x_x509.obj)
0001:0070ac00  _X509_CINF_it
0001:0070ac1c* _d2i_X509_CINF
0001:0070ac45* _i2d_X509_CINF
0001:0070ac67* _X509_CINF_new
0001:0070ac7b* _X509_CINF_free
0001:0070aea0  _X509_it
0001:0070aebc  _d2i_X509
0001:0070aee5  _i2d_X509
0001:0070af07* _X509_new
0001:0070af1b  _X509_free
0001:0070af36* _X509_dup
0001:0070af51* _X509_get_ex_new_index
0001:0070af88* _X509_set_ex_data
0001:0070afac* _X509_get_ex_data
0001:0070afc9  _d2i_X509_AUX
0001:0070b054  _i2d_X509_AUX
Module: U:\extras\lib\libcrypto.lib(eng_init.obj)
0001:0070b0a0  _engine_unlocked_init
0001:0070b106  _engine_unlocked_finish
0001:0070b1f7  _ENGINE_init
0001:0070b291  _ENGINE_finish
Module: U:\extras\lib\libcrypto.lib(rsa_lib.obj)
0001:0070b380* _RSA_version
0001:0070b3a6  _RSA_new
0001:0070b473* _RSA_new_method
0001:0070b3c0* _RSA_set_default_method
0001:0070b3cd* _RSA_get_default_method
0001:0070b3ed* _RSA_get_method
0001:0070b3f8* _RSA_set_method
0001:0070b733  _RSA_free
0001:0070b8ec  _RSA_up_ref
0001:0070b92f* _RSA_get_ex_new_index
0001:0070b966* _RSA_set_ex_data
0001:0070b98a* _RSA_get_ex_data
0001:0070b9a7  _RSA_size
0001:0070b9ca  _RSA_public_encrypt
0001:0070b9ff  _RSA_private_encrypt
0001:0070ba34  _RSA_private_decrypt
0001:0070ba69  _RSA_public_decrypt
0001:0070ba9e  _RSA_flags
0001:0070bab9* _RSA_blinding_off
0001:0070bb05* _RSA_blinding_on
0001:0070bc84  _RSA_setup_blinding
0001:0070bf09* _RSA_memory_lock
Module: U:\extras\lib\libcrypto.lib(dh_lib.obj)
0001:0070c100* _DH_version
0001:0070c131* _DH_set_default_method
0001:0070c13e* _DH_get_default_method
0001:0070c15e* _DH_set_method
0001:0070c1cf  _DH_new
0001:0070c1ec* _DH_new_method
0001:0070c460  _DH_free
0001:0070c5d1  _DH_up_ref
0001:0070c614* _DH_get_ex_new_index
0001:0070c64b* _DH_set_ex_data
0001:0070c66f* _DH_get_ex_data
0001:0070c68c  _DH_size
Module: U:\extras\lib\libcrypto.lib(p_lib.obj)
0001:0070c6b0  _EVP_PKEY_bits
0001:0070c6ed  _EVP_PKEY_size
0001:0070c72a* _EVP_PKEY_save_parameters
0001:0070c78f  _EVP_PKEY_copy_parameters
0001:0070c846  _EVP_PKEY_missing_parameters
0001:0070c87d  _EVP_PKEY_cmp_parameters
0001:0070c8d0  _EVP_PKEY_cmp
0001:0070c956  _EVP_PKEY_new
0001:0070cb30  _EVP_PKEY_set_type
0001:0070cb5a  _EVP_PKEY_set_type_str
0001:0070cb83  _EVP_PKEY_assign
0001:0070cbbb* _EVP_PKEY_get0
0001:0070cbc6  _EVP_PKEY_set1_RSA
0001:0070cbff  _EVP_PKEY_get1_RSA
0001:0070cc58  _EVP_PKEY_set1_DSA
0001:0070cc91  _EVP_PKEY_get1_DSA
0001:0070ccea  _EVP_PKEY_set1_EC_KEY
0001:0070cd23  _EVP_PKEY_get1_EC_KEY
0001:0070cd7e* _EVP_PKEY_set1_DH
0001:0070cdb7* _EVP_PKEY_get1_DH
0001:0070ce10  _EVP_PKEY_type
0001:0070ce59  _EVP_PKEY_id
0001:0070ce63* _EVP_PKEY_base_id
0001:0070ce78  _EVP_PKEY_free
0001:0070cfd4  _EVP_PKEY_print_public
0001:0070d048  _EVP_PKEY_print_private
0001:0070d0bb  _EVP_PKEY_print_params
0001:0070d123  _EVP_PKEY_get_default_digest_nid
Module: U:\extras\lib\libcrypto.lib(v3_purp.obj)
0001:0070d281  _X509_check_purpose
0001:0070d45a  _X509_PURPOSE_get_by_id
0001:0070d3bd  _X509_PURPOSE_get0
0001:0070d33d  _X509_PURPOSE_set
0001:0070d395* _X509_PURPOSE_get_count
0001:0070d40b* _X509_PURPOSE_get_by_sname
0001:0070d4b4* _X509_PURPOSE_add
0001:0070d72a* _X509_PURPOSE_cleanup
0001:0070d784* _X509_PURPOSE_get_id
0001:0070d78e* _X509_PURPOSE_get0_name
0001:0070d799* _X509_PURPOSE_get0_sname
0001:0070d7a4* _X509_PURPOSE_get_trust
0001:0070d81b* _X509_supported_extension
0001:0070e10b  _X509_check_ca
0001:0070e5b8  _X509_check_issued
0001:0070e692  _X509_check_akid
Module: U:\extras\lib\libcrypto.lib(obj_dat.obj)
0001:0071d921  _OBJ_bsearch_
0001:0071cb74  _check_defer
0001:0071cb95  _OBJ_cleanup
0001:0071cc20* _OBJ_new_nid
0001:0071cc4a* _OBJ_add_object
0001:0071ce62  _OBJ_nid2obj
0001:0071cf59  _OBJ_nid2sn
0001:0071d054  _OBJ_nid2ln
0001:0071d212  _OBJ_obj2nid
0001:0071d2bc  _OBJ_txt2obj
0001:0071d88e  _OBJ_sn2nid
0001:0071d7fb  _OBJ_ln2nid
0001:0071d419  _OBJ_obj2txt
0001:0071d7c1* _OBJ_txt2nid
0001:0071d958  _OBJ_bsearch_ex_
0001:0071da5a* _OBJ_create_objects
0001:0071dc27* _OBJ_create
0002:0001f4d0  _obj_cleanup_defer
Module: U:\extras\lib\libcrypto.lib(evp_enc.obj)
0001:0071dd60* _EVP_version
0001:0071dd86  _EVP_CIPHER_CTX_init
0001:0071ddb3* _EVP_CIPHER_CTX_new
0001:0071ddee* _EVP_CipherInit
0001:0071dece  _EVP_CipherInit_ex
0001:0071ec21  _EVP_CIPHER_CTX_cleanup
0001:0071eda8  _EVP_CIPHER_CTX_ctrl
0001:0071e2fa  _EVP_CipherUpdate
0001:0071e4d2  _EVP_EncryptUpdate
0001:0071e873  _EVP_DecryptUpdate
0001:0071e35c  _EVP_CipherFinal_ex
0001:0071e741  _EVP_EncryptFinal_ex
0001:0071ea06  _EVP_DecryptFinal_ex
0001:0071e3a2* _EVP_CipherFinal
0001:0071e705* _EVP_EncryptFinal
0001:0071e9df  _EVP_DecryptFinal
0001:0071e3e8* _EVP_EncryptInit
0001:0071e418  _EVP_EncryptInit_ex
0001:0071e44f* _EVP_DecryptInit
0001:0071e47f  _EVP_DecryptInit_ex
0001:0071ebfd* _EVP_CIPHER_CTX_free
0001:0071eccf  _EVP_CIPHER_CTX_set_key_length
0001:0071ed74* _EVP_CIPHER_CTX_set_padding
0001:0071ee92  _EVP_CIPHER_CTX_rand_key
0001:0071eef4  _EVP_CIPHER_CTX_copy
Module: U:\extras\lib\libcrypto.lib(comp_lib.obj)
0001:0071f0ab  _COMP_CTX_new
0001:0071f137  _COMP_CTX_free
0001:0071f16f  _COMP_compress_block
0001:0071f1e4  _COMP_expand_block
Module: U:\extras\lib\libcrypto.lib(bf_buff.obj)
0001:0071f267  _BIO_f_buffer
Module: U:\extras\lib\libcrypto.lib(x509_d2.obj)
0001:00720040  _X509_STORE_set_default_paths
0001:007200f3  _X509_STORE_load_locations
Module: U:\extras\lib\libcrypto.lib(digest.obj)
0001:007201e0  _EVP_MD_CTX_init
0001:0072020c  _EVP_MD_CTX_create
0001:00720247  _EVP_DigestInit
0001:00720274  _EVP_DigestInit_ex
0001:0072053d  _EVP_DigestUpdate
0001:00720561  _EVP_DigestFinal
0001:007205bc  _EVP_DigestFinal_ex
0001:00720971  _EVP_MD_CTX_cleanup
0001:00720672  _EVP_MD_CTX_copy
0001:00720697  _EVP_MD_CTX_copy_ex
0001:007208b9  _EVP_Digest
0001:00720953  _EVP_MD_CTX_destroy
Module: U:\extras\lib\libssl.lib(s2_clnt.obj)
0001:00720a8a  _SSLv2_client_method
0001:00720a9e* _ssl2_connect
0001:00722c36* _ssl2_set_certificate
Module: U:\extras\lib\libssl.lib(s3_clnt.obj)
0001:0072306d  _SSLv3_client_method
0001:00723081  _ssl3_connect
0001:00723cde* _ssl3_client_hello
0001:0072411f* _ssl3_get_server_hello
0001:00728de1* _ssl3_check_finished
0001:0072493d* _ssl3_get_server_certificate
0001:00725045* _ssl3_get_key_exchange
0001:00728945* _ssl3_check_cert_and_algorithm
0001:007263a9* _ssl3_get_certificate_request
0001:00726f15* _ssl3_get_server_done
0001:007286fc* _ssl3_send_client_certificate
0001:00726fc9* _ssl3_send_client_key_exchange
0001:00728252* _ssl3_send_client_verify
0001:007268da* _ssl3_get_new_session_ticket
0001:00726c55* _ssl3_get_cert_status
0001:00728e90* _ssl_do_client_cert_cb
Module: U:\extras\lib\libssl.lib(t1_clnt.obj)
0001:00728fed  _TLSv1_client_method
Module: U:\extras\lib\libssl.lib(s3_both.obj)
0001:00729080  _ssl3_do_write
0001:007291b7  _ssl3_send_finished
0001:00729380  _ssl3_get_finished
0001:007295cb  _ssl3_send_change_cipher_spec
0001:007296fc  _ssl3_output_cert_chain
0001:007299c0  _ssl3_get_message
0001:00729eda  _ssl_cert_type
0001:00729f8e  _ssl_verify_alarm_type
0001:0072a2b6  _ssl3_setup_read_buffer
0001:0072a3f7  _ssl3_setup_write_buffer
0001:0072a527  _ssl3_setup_buffers
0001:0072a560  _ssl3_release_write_buffer
0001:0072a5c6  _ssl3_release_read_buffer
Module: U:\extras\lib\libssl.lib(s3_enc.obj)
0001:0072a892  _ssl3_change_cipher_state
0001:0072af97  _ssl3_setup_key_block
0001:0072b1cb  _ssl3_cleanup_key_block
0001:0072b23d  _ssl3_enc
0001:0072b45d  _ssl3_init_finished_mac
0001:0072b4ee  _ssl3_free_digest_list
0001:0072b577  _ssl3_finish_mac
0001:0072b60b  _ssl3_digest_cached_records
0001:0072b7e2  _ssl3_cert_verify_mac
0001:0072b813  _ssl3_final_finish_mac
0001:0072bae0  _n_ssl3_mac
0001:0072bd35* _ssl3_record_sequence_update
0001:0072bd69  _ssl3_generate_master_secret
0001:0072befd  _ssl3_alert_code
Module: U:\extras\lib\libssl.lib(s3_lib.obj)
0001:0072c200* _ssl3_version_str
0001:0072c8a8  _ssl3_default_timeout
0001:0072c8b2  _ssl3_num_ciphers
0001:0072c8bc  _ssl3_get_cipher
0001:0072c8e6  _ssl3_pending
0001:0072c92c  _ssl3_new
0001:0072c9db  _ssl3_free
0001:0072cb37  _ssl3_clear
0001:0072cd36  _ssl3_ctrl
0001:0072d57b  _ssl3_callback_ctrl
0001:0072d640  _ssl3_ctx_ctrl
0001:0072dc90  _ssl3_ctx_callback_ctrl
0001:0072dd25  _ssl3_get_cipher_by_char
0001:0072dd8a  _ssl3_put_cipher_by_char
0001:0072ddd4* _ssl3_choose_cipher
0001:0072e4f4* _ssl3_get_req_cert_type
0001:0072e5fe  _ssl3_shutdown
0001:0072e730  _ssl3_write
0001:0072ea06  _ssl3_renegotiate_check
0001:0072e973  _ssl3_read
0001:0072e99c  _ssl3_peek
0001:0072e9c5  _ssl3_renegotiate
0002:000050e0* _ssl3_ciphers
0002:000061c0  _SSLv3_enc_data
Module: U:\extras\lib\libssl.lib(t1_lib.obj)
0001:0072eab0* _tls1_version_str
0001:0072eaf8  _tls1_default_timeout
0001:0072eb02  _tls1_new
0001:0072eb36  _tls1_free
0001:0072eb67  _tls1_clear
0001:0072eb83  _tls1_ec_curve_id2nid
0001:0072eba8  _tls1_ec_nid2curve_id
0001:0072edd6  _ssl_add_clienthello_tlsext
0001:0072f74d* _ssl_add_serverhello_tlsext
0001:0072fbfc* _ssl_parse_clienthello_tlsext
0001:00730651  _ssl_parse_serverhello_tlsext
0001:00730b2a  _ssl_prepare_clienthello_tlsext
0001:00730d76* _ssl_prepare_serverhello_tlsext
0001:00730eb8* _ssl_check_clienthello_tlsext
0001:007310b3  _ssl_check_serverhello_tlsext
0001:007313d7  _tls1_process_ticket
0002:00006200  _TLSv1_enc_data
Module: U:\extras\lib\libssl.lib(s23_pkt.obj)
0001:007319e0  _ssl23_write_bytes
0001:00731a7c  _ssl23_read_bytes
Module: U:\extras\lib\libssl.lib(s2_lib.obj)
0001:00731b20* _ssl2_version_str
0001:00731ba0* _ssl2_ciphers
0001:00731cf0  _ssl2_default_timeout
0001:00731cfa  _ssl2_num_ciphers
0001:00731d04  _ssl2_get_cipher
0001:00731d2e  _ssl2_pending
0001:00731d63  _ssl2_new
0001:00731ee5  _ssl2_clear
0001:00731e73  _ssl2_free
0001:00731f5e  _ssl2_ctrl
0001:00731f84  _ssl2_callback_ctrl
0001:00731f8e  _ssl2_ctx_ctrl
0001:00731f98  _ssl2_ctx_callback_ctrl
0001:00731fa2  _ssl2_get_cipher_by_char
0001:00732017  _ssl2_put_cipher_by_char
0001:007320da  _ssl2_generate_key_material
0001:00732318  _ssl2_return_error
0001:0073237c  _ssl2_write_error
0001:00732486  _ssl2_shutdown
Module: U:\extras\lib\libssl.lib(s23_lib.obj)
0001:007324a0  _ssl23_default_timeout
0001:007324aa  _ssl23_num_ciphers
0001:007324c6  _ssl23_get_cipher
0001:007324ff  _ssl23_get_cipher_by_char
0001:0073252c  _ssl23_put_cipher_by_char
0001:00732578  _ssl23_read
0001:00732629  _ssl23_peek
0001:007326da  _ssl23_write
Module: U:\extras\lib\xmlrpc.lib(queue.obj)
0001:00732790  _Q_Init
0001:007327c3* _Q_AtHead
0001:007327dc* _Q_AtTail
0001:007327f6* _Q_IsEmpty
0001:00732810  _Q_Size
0001:00732821  _Q_Head
0001:0073283f* _Q_Tail
0001:0073285e  _Q_Next
0001:00732881* _Q_Previous
0001:007328a0* _Q_Get
0001:007328b9* _Q_Put
0001:007328de* _Q_Find
0001:00732a56* _Q_Iter_Head
0001:00732a66* _Q_Iter_Tail
0001:00732a77* _Q_Iter_Next
0001:00732a88* _Q_Iter_Prev
0001:00732a99* _Q_Iter_Get
0001:00732aa9* _Q_Iter_Put
0001:00732ac1* _Q_PopTail
0001:00732b3b* _Q_PopHead
0001:00732bb3  _Q_Destroy
0001:00732bd8  _Q_Iter_Del
0001:00732c6d* _Q_DelCur
0001:00732c8d* _Q_Sort
0001:00732dd5* _Q_Seek
0001:00732e86  _Q_PushTail
0001:00732efc* _Q_PushHead
0001:00732f6d* _Q_Insert
Module: U:\extras\lib\xmlrpc.lib(simplestring.obj)
0001:00732fb0  _simplestring_clear
0001:00732fc8  _simplestring_addn
0001:007330ba  _simplestring_add
0001:007330fe  _simplestring_free
0001:0073312d  _simplestring_init
Module: U:\extras\lib\xmlrpc.lib(system_methods.obj)
0001:00733178  _xsm_register
Module: U:\extras\lib\xmlrpc.lib(xml_element.obj)
0001:00735a92* _xml_elem_serialize_to_stream
0001:00735ad3  _xml_elem_serialize_to_string
0001:00735b1a  _xml_elem_new
0001:00735c06  _xml_elem_free_non_recurse
0001:00735d51  _xml_elem_parse_buf
0001:00735fc5  _xml_elem_free
Module: U:\extras\lib\xmlrpc.lib(xml_to_xmlrpc.obj)
0001:00736099* _XMLRPC_to_xml_element_worker
0001:007365f8  _XMLRPC_REQUEST_to_xml_element
0001:0073671f  _XMLRPC_VALUE_to_xml_element
0001:0073674d* _xml_element_to_XMLRPC_REQUEST_worker
0001:00736c85  _xml_element_to_XMLRPC_REQUEST
0001:00736cca* _xml_element_to_XMLRPC_VALUE
Module: U:\extras\lib\xmlrpc.lib(xml_to_soap.obj)
0001:00736e54* _SOAP_to_xml_element_worker
0001:007375e6  _SOAP_REQUEST_to_xml_element
0001:007378c7* _SOAP_VALUE_to_xml_element
0001:007379a4* _xml_element_to_SOAP_REQUEST_worker
0001:00738181  _xml_element_to_SOAP_REQUEST
0001:007381d6* _xml_element_to_SOAP_VALUE
Module: U:\extras\lib\xmlrpc.lib(xml_to_dandarpc.obj)
0001:007382b1* _DANDARPC_to_xml_element_worker
0001:00738791  _DANDARPC_REQUEST_to_xml_element
0001:007388c3* _DANDARPC_VALUE_to_xml_element
0001:007388de* _xml_element_to_DANDARPC_REQUEST_worker
0001:00738d0a  _xml_element_to_DANDARPC_REQUEST
0001:00738d47* _xml_element_to_DANDARPC_VALUE
Module: U:\tmp\ldconv_libgcc_eh_a_3ed14e78ff52199cf0.lib(unwind-dw2-fde.obj)
0001:00739ce1* ___register_frame_info_bases
0001:00739de0* ___register_frame_info
0001:00739e0b* ___register_frame
0001:00739e36* ___register_frame_info_table_bases
0001:00739f28* ___register_frame_info_table
0001:00739f53  ___register_frame_table
0001:00739f76* ___deregister_frame_info_bases
0001:0073a0de* ___deregister_frame_info
0001:0073a0e9  ___deregister_frame
0001:0073a10e* __Unwind_Find_FDE
Module: U:\extras\lib\pthread.lib(my_os2key.obj)
0001:0073a2f0  _pthread_key_create
0001:0073a30c  _pthread_key_delete
0001:0073a318  _pthread_getspecific
0001:0073a324  _pthread_setspecific
Module: U:\extras\lib\pthread.lib(my_os2thread.obj)
0001:0073a374* _LoadExceptq
0001:0073a4ec* __pthreadInit
0001:0073a544* _pthread_exit
0001:0073a620  _pthread_equal
0001:0073a634* _pthread_setprio
0001:0073a660* _pthread_create
0001:0073a794* _pthread_dummy
0001:0073a79c  _pthread_self
0001:0073a80c* _pthread_join
0001:0073a890* _pthread_cleanup_push
0001:0073a898* _pthread_cleanup_pop
0001:0073a8a0  _pthread_once
0001:0073a914* _pthread_yield
0001:0073a928* _pthread_setcancelstate
0001:0073a930* _pthread_setcanceltype
0001:0073a938* _pthread_testcancel
0001:0073a940* _pthread_atfork
0001:0073a948* _pthread_detach
0001:0073a9b8* _pthread_kill
0001:0073a9fc* _pthread_cancel
Module: U:\extras\lib\pthread.lib(my_os2mutex.obj)
0001:0073aa40  _pthread_mutex_init
0001:0073aab0  _pthread_mutex_destroy
0001:0073ab14  _pthread_mutex_lock
0001:0073ab70* _pthread_mutex_trylock
0001:0073abf8  _pthread_mutex_unlock
0001:0073ac44* _pthread_mutexattr_init
0001:0073ac8c* _pthread_mutexattr_destroy
0001:0073acbc* _pthread_mutexattr_settype
0001:0073ace4* _pthread_mutexattr_gettype
Module: U:\extras\lib\pthread.lib(my_os2cond.obj)
0001:0073ad10  _pthread_cond_init
0001:0073adb0  _pthread_cond_destroy
0001:0073ae10  _pthread_cond_wait
0001:0073ae98* _pthread_cond_timedwait
0001:0073af8c  _pthread_cond_signal
0001:0073afe8* _pthread_cond_broadcast
Module: U:\extras\lib\xml2.lib(xmlunicode.obj)
0001:0073b040* _xmlUCSIsAegeanNumbers
0001:0073b056* _xmlUCSIsAlphabeticPresentationForms
0001:0073b06c* _xmlUCSIsArabic
0001:0073b084* _xmlUCSIsArabicPresentationFormsA
0001:0073b09c* _xmlUCSIsArabicPresentationFormsB
0001:0073b0b4* _xmlUCSIsArmenian
0001:0073b0ca* _xmlUCSIsArrows
0001:0073b0e0* _xmlUCSIsBasicLatin
0001:0073b0ee* _xmlUCSIsBengali
0001:0073b104* _xmlUCSIsBlockElements
0001:0073b11a* _xmlUCSIsBopomofo
0001:0073b130* _xmlUCSIsBopomofoExtended
0001:0073b146* _xmlUCSIsBoxDrawing
0001:0073b15c* _xmlUCSIsBraillePatterns
0001:0073b174* _xmlUCSIsBuhid
0001:0073b18a* _xmlUCSIsByzantineMusicalSymbols
0001:0073b1a2* _xmlUCSIsCJKCompatibility
0001:0073b1ba* _xmlUCSIsCJKCompatibilityForms
0001:0073b1d0* _xmlUCSIsCJKCompatibilityIdeographs
0001:0073b1e8* _xmlUCSIsCJKCompatibilityIdeographsSupplement
0001:0073b200* _xmlUCSIsCJKRadicalsSupplement
0001:0073b216* _xmlUCSIsCJKSymbolsandPunctuation
0001:0073b22c* _xmlUCSIsCJKUnifiedIdeographs
0001:0073b244* _xmlUCSIsCJKUnifiedIdeographsExtensionA
0001:0073b25c* _xmlUCSIsCJKUnifiedIdeographsExtensionB
0001:0073b274* _xmlUCSIsCherokee
0001:0073b28a* _xmlUCSIsCombiningDiacriticalMarks
0001:0073b2a0* _xmlUCSIsCombiningDiacriticalMarksforSymbols
0001:0073b2b6* _xmlUCSIsCombiningHalfMarks
0001:0073b2cc* _xmlUCSIsCombiningMarksforSymbols
0001:0073b2e2* _xmlUCSIsControlPictures
0001:0073b2f8* _xmlUCSIsCurrencySymbols
0001:0073b30e* _xmlUCSIsCypriotSyllabary
0001:0073b324* _xmlUCSIsCyrillic
0001:0073b33c* _xmlUCSIsCyrillicSupplement
0001:0073b352* _xmlUCSIsDeseret
0001:0073b368* _xmlUCSIsDevanagari
0001:0073b37e* _xmlUCSIsDingbats
0001:0073b396* _xmlUCSIsEnclosedAlphanumerics
0001:0073b3ae* _xmlUCSIsEnclosedCJKLettersandMonths
0001:0073b3c6* _xmlUCSIsEthiopic
0001:0073b3de* _xmlUCSIsGeneralPunctuation
0001:0073b3f4* _xmlUCSIsGeometricShapes
0001:0073b40a* _xmlUCSIsGeorgian
0001:0073b420* _xmlUCSIsGothic
0001:0073b436* _xmlUCSIsGreek
0001:0073b44e* _xmlUCSIsGreekExtended
0001:0073b466* _xmlUCSIsGreekandCoptic
0001:0073b47e* _xmlUCSIsGujarati
0001:0073b494* _xmlUCSIsGurmukhi
0001:0073b4aa* _xmlUCSIsHalfwidthandFullwidthForms
0001:0073b4c2* _xmlUCSIsHangulCompatibilityJamo
0001:0073b4d8* _xmlUCSIsHangulJamo
0001:0073b4f0* _xmlUCSIsHangulSyllables
0001:0073b508* _xmlUCSIsHanunoo
0001:0073b51e* _xmlUCSIsHebrew
0001:0073b534* _xmlUCSIsHighPrivateUseSurrogates
0001:0073b54a* _xmlUCSIsHighSurrogates
0001:0073b562* _xmlUCSIsHiragana
0001:0073b578* _xmlUCSIsIPAExtensions
0001:0073b58e* _xmlUCSIsIdeographicDescriptionCharacters
0001:0073b5a4* _xmlUCSIsKanbun
0001:0073b5ba* _xmlUCSIsKangxiRadicals
0001:0073b5d2* _xmlUCSIsKannada
0001:0073b5e8* _xmlUCSIsKatakana
0001:0073b5fe* _xmlUCSIsKatakanaPhoneticExtensions
0001:0073b614* _xmlUCSIsKhmer
0001:0073b62a* _xmlUCSIsKhmerSymbols
0001:0073b640* _xmlUCSIsLao
0001:0073b656* _xmlUCSIsLatin1Supplement
0001:0073b66a* _xmlUCSIsLatinExtendedA
0001:0073b680* _xmlUCSIsLatinExtendedB
0001:0073b698* _xmlUCSIsLatinExtendedAdditional
0001:0073b6b0* _xmlUCSIsLetterlikeSymbols
0001:0073b6c6* _xmlUCSIsLimbu
0001:0073b6dc* _xmlUCSIsLinearBIdeograms
0001:0073b6f2* _xmlUCSIsLinearBSyllabary
0001:0073b708* _xmlUCSIsLowSurrogates
0001:0073b720* _xmlUCSIsMalayalam
0001:0073b736* _xmlUCSIsMathematicalAlphanumericSymbols
0001:0073b74e* _xmlUCSIsMathematicalOperators
0001:0073b766* _xmlUCSIsMiscellaneousMathematicalSymbolsA
0001:0073b77c* _xmlUCSIsMiscellaneousMathematicalSymbolsB
0001:0073b792* _xmlUCSIsMiscellaneousSymbols
0001:0073b7aa* _xmlUCSIsMiscellaneousSymbolsandArrows
0001:0073b7c2* _xmlUCSIsMiscellaneousTechnical
0001:0073b7da* _xmlUCSIsMongolian
0001:0073b7f2* _xmlUCSIsMusicalSymbols
0001:0073b80a* _xmlUCSIsMyanmar
0001:0073b822* _xmlUCSIsNumberForms
0001:0073b838* _xmlUCSIsOgham
0001:0073b84e* _xmlUCSIsOldItalic
0001:0073b864* _xmlUCSIsOpticalCharacterRecognition
0001:0073b87a* _xmlUCSIsOriya
0001:0073b890* _xmlUCSIsOsmanya
0001:0073b8a6* _xmlUCSIsPhoneticExtensions
0001:0073b8bc* _xmlUCSIsPrivateUse
0001:0073b8f7* _xmlUCSIsPrivateUseArea
0001:0073b90f* _xmlUCSIsRunic
0001:0073b925* _xmlUCSIsShavian
0001:0073b93b* _xmlUCSIsSinhala
0001:0073b951* _xmlUCSIsSmallFormVariants
0001:0073b967* _xmlUCSIsSpacingModifierLetters
0001:0073b97d* _xmlUCSIsSpecials
0001:0073b993* _xmlUCSIsSuperscriptsandSubscripts
0001:0073b9a9* _xmlUCSIsSupplementalArrowsA
0001:0073b9bf* _xmlUCSIsSupplementalArrowsB
0001:0073b9d5* _xmlUCSIsSupplementalMathematicalOperators
0001:0073b9ed* _xmlUCSIsSupplementaryPrivateUseAreaA
0001:0073ba05* _xmlUCSIsSupplementaryPrivateUseAreaB
0001:0073ba1d* _xmlUCSIsSyriac
0001:0073ba33* _xmlUCSIsTagalog
0001:0073ba49* _xmlUCSIsTagbanwa
0001:0073ba5f* _xmlUCSIsTags
0001:0073ba75* _xmlUCSIsTaiLe
0001:0073ba8b* _xmlUCSIsTaiXuanJingSymbols
0001:0073baa1* _xmlUCSIsTamil
0001:0073bab7* _xmlUCSIsTelugu
0001:0073bacd* _xmlUCSIsThaana
0001:0073bae3* _xmlUCSIsThai
0001:0073baf9* _xmlUCSIsTibetan
0001:0073bb11* _xmlUCSIsUgaritic
0001:0073bb27* _xmlUCSIsUnifiedCanadianAboriginalSyllabics
0001:0073bb3f* _xmlUCSIsVariationSelectors
0001:0073bb55* _xmlUCSIsVariationSelectorsSupplement
0001:0073bb6d* _xmlUCSIsYiRadicals
0001:0073bb83* _xmlUCSIsYiSyllables
0001:0073bb9b* _xmlUCSIsYijingHexagramSymbols
0001:0073bbb1  _xmlUCSIsCatCc
0001:0073bbd0  _xmlUCSIsCatCo
0001:0073bc16* _xmlUCSIsCatCs
0001:0073bc52  _xmlUCSIsCatMe
0001:0073bc92  _xmlUCSIsCatNl
0001:0073bce9  _xmlUCSIsCatPc
0001:0073bd46  _xmlUCSIsCatPf
0001:0073bd7c  _xmlUCSIsCatPi
0001:0073bdb6  _xmlUCSIsCatZl
0001:0073bdc7  _xmlUCSIsCatZp
0001:0073bdd8  _xmlUCSIsCatZs
0001:0073bea2  _xmlUCSIsCatZ
0001:0073bebd  _xmlUCSIsCatSo
0001:0073bed8  _xmlUCSIsCatSm
0001:0073bef3  _xmlUCSIsCatSk
0001:0073bf0e  _xmlUCSIsCatSc
0001:0073bf29  _xmlUCSIsCatS
0001:0073bf44  _xmlUCSIsCatPs
0001:0073bf5f  _xmlUCSIsCatPo
0001:0073bf7a  _xmlUCSIsCatPe
0001:0073bf95  _xmlUCSIsCatPd
0001:0073bfb0  _xmlUCSIsCatP
0001:0073bfcb  _xmlUCSIsCatNo
0001:0073bfe6  _xmlUCSIsCatNd
0001:0073c001  _xmlUCSIsCatN
0001:0073c01c  _xmlUCSIsCatMn
0001:0073c037  _xmlUCSIsCatMc
0001:0073c052  _xmlUCSIsCatM
0001:0073c06d  _xmlUCSIsCatLu
0001:0073c088  _xmlUCSIsCatLt
0001:0073c0a3  _xmlUCSIsCatLo
0001:0073c0be  _xmlUCSIsCatLm
0001:0073c0d9  _xmlUCSIsCatLl
0001:0073c0f4  _xmlUCSIsCatL
0001:0073c10f  _xmlUCSIsCatCf
0001:0073c12a  _xmlUCSIsCatC
0001:0073c145  _xmlUCSIsBlock
0001:0073c175* _xmlUCSIsCat
Module: U:\extras\lib\libcrypto.lib(mem_dbg.obj)
0001:0073f5de  _CRYPTO_mem_ctrl
0001:0073f7d2* _CRYPTO_is_mem_check_on
0001:0073f879* _CRYPTO_dbg_set_options
0001:0073f886* _CRYPTO_dbg_get_options
0001:0073faeb  _CRYPTO_push_info_
0001:0073fbf2  _CRYPTO_pop_info
0001:0073fc35* _CRYPTO_remove_all_info
0001:0073fc76* _CRYPTO_dbg_malloc
0001:0073fea4* _CRYPTO_dbg_free
0001:0073ff37* _CRYPTO_dbg_realloc
0001:0074045b* _CRYPTO_mem_leaks
0001:007405ad* _CRYPTO_mem_leaks_fp
0001:00740698* _CRYPTO_mem_leaks_cb
Module: U:\extras\lib\libcrypto.lib(b_print.obj)
0001:00741b63  _BIO_printf
0001:00741b98* _BIO_vprintf
0001:00741c8c  _BIO_snprintf
0001:00741cc0* _BIO_vsnprintf
Module: U:\extras\lib\libcrypto.lib(mem_clr.obj)
0001:00741d30  _OPENSSL_cleanse
0002:0001f600  _cleanse_ctr
Module: U:\extras\lib\libcrypto.lib(eng_pkey.obj)
0001:00741dc0* _ENGINE_set_load_privkey_function
0001:00741dd3* _ENGINE_set_load_pubkey_function
0001:00741de6* _ENGINE_set_load_ssl_client_cert_function
0001:00741df9* _ENGINE_get_load_privkey_function
0001:00741e04* _ENGINE_get_load_pubkey_function
0001:00741e0f  _ENGINE_get_ssl_client_cert_function
0001:00741e25* _ENGINE_load_private_key
0001:00741fb4* _ENGINE_load_public_key
0001:00742143  _ENGINE_load_ssl_client_cert
Module: U:\extras\lib\libssl.lib(ssl_asn1.obj)
0001:007422b0  _i2d_SSL_SESSION
0001:00742ff9  _d2i_SSL_SESSION
Module: U:\extras\lib\libcrypto.lib(pem_oth.obj)
0001:0074457a  _PEM_ASN1_read_bio
Module: U:\extras\lib\libcrypto.lib(pem_lib.obj)
0001:00744640* _PEM_version
0001:007446bc  _PEM_def_callback
0001:0074480a  _PEM_proc_type
0001:007448a3  _PEM_dek_info
0001:00744993  _PEM_ASN1_read
0001:00746834  _pem_check_suffix
0001:00744e3a  _PEM_bytes_read_bio
0001:00746015  _PEM_read_bio
0001:007457ce  _PEM_get_EVP_CIPHER_INFO
0001:00745594  _PEM_do_header
0001:00744f9d  _PEM_ASN1_write
0001:007450b5  _PEM_ASN1_write_bio
0001:00745c81  _PEM_write_bio
0001:00745bb9* _PEM_write
0001:00745f6a* _PEM_read
Module: U:\extras\lib\libcrypto.lib(ameth_lib.obj)
0001:00746950* _EVP_PKEY_asn1_get_count
0001:0074697b* _EVP_PKEY_asn1_get0
0001:00746a51  _EVP_PKEY_asn1_find
0001:00746ac7  _EVP_PKEY_asn1_find_str
0001:00746bb1* _EVP_PKEY_asn1_add0
0001:00746c15* _EVP_PKEY_asn1_add_alias
0001:00746ce8* _EVP_PKEY_asn1_new
0001:00746c64  _EVP_PKEY_asn1_get0_info
0001:00746cd1* _EVP_PKEY_get0_asn1
0001:00746f5a  _EVP_PKEY_asn1_free
0001:00746e71* _EVP_PKEY_asn1_copy
0001:00746fb0* _EVP_PKEY_asn1_set_public
0001:00746feb* _EVP_PKEY_asn1_set_private
0001:0074700b* _EVP_PKEY_asn1_set_param
0001:00747046* _EVP_PKEY_asn1_set_free
0001:00747054* _EVP_PKEY_asn1_set_ctrl
Module: U:\extras\lib\libcrypto.lib(evp_lib.obj)
0001:00747070  _EVP_CIPHER_param_to_asn1
0001:007470aa  _EVP_CIPHER_asn1_to_param
0001:00747101  _EVP_CIPHER_get_asn1_iv
0001:007473eb  _EVP_CIPHER_CTX_iv_length
0001:007471b3  _EVP_CIPHER_set_asn1_iv
0001:0074721a  _EVP_CIPHER_type
0001:0074740e  _EVP_CIPHER_nid
0001:00747360  _EVP_CIPHER_block_size
0001:0074736b  _EVP_CIPHER_CTX_block_size
0001:00747378  _EVP_Cipher
0001:007473a5  _EVP_CIPHER_CTX_cipher
0001:007473af* _EVP_CIPHER_flags
0001:007473ba  _EVP_CIPHER_CTX_flags
0001:007473c7* _EVP_CIPHER_CTX_get_app_data
0001:007473d2* _EVP_CIPHER_CTX_set_app_data
0001:007473e0  _EVP_CIPHER_iv_length
0001:007473f8  _EVP_CIPHER_key_length
0001:00747403  _EVP_CIPHER_CTX_key_length
0001:00747418* _EVP_CIPHER_CTX_nid
0001:00747424  _EVP_MD_block_size
0001:0074742f  _EVP_MD_type
0001:00747439  _EVP_MD_pkey_type
0001:00747444  _EVP_MD_size
0001:0074748b* _EVP_MD_flags
0001:00747496  _EVP_MD_CTX_md
0001:007474ad  _EVP_MD_CTX_set_flags
0001:007474c3  _EVP_MD_CTX_clear_flags
0001:007474db  _EVP_MD_CTX_test_flags
0001:007474eb* _EVP_CIPHER_CTX_set_flags
0001:00747501* _EVP_CIPHER_CTX_clear_flags
0001:00747519* _EVP_CIPHER_CTX_test_flags
Module: U:\extras\lib\libcrypto.lib(c_zlib.obj)
0001:00747538  _COMP_zlib
0001:0074754a* _COMP_zlib_cleanup
Module: U:\extras\lib\libcrypto.lib(e_null.obj)
0001:00747584  _EVP_enc_null
Module: U:\extras\lib\libcrypto.lib(x509_vfy.obj)
0001:007475d0* _X509_version
0001:0074760b  _X509_verify_cert
0001:0074a344* _X509_get_pubkey_parameters
0001:00749f76* _X509_cmp_time
0001:0074a8c1  _X509_STORE_CTX_init
0001:0074ae24* _X509_STORE_CTX_set0_param
0001:0074ac92  _X509_STORE_CTX_cleanup
0001:00749f5b* _X509_cmp_current_time
0001:0074a26b* _X509_time_adj
0001:0074a249  _X509_gmtime_adj
0001:0074a294* _X509_time_adj_ex
0001:0074a4bc  _X509_STORE_CTX_get_ex_new_index
0001:0074a4f3  _X509_STORE_CTX_set_ex_data
0001:0074a51a* _X509_STORE_CTX_get_ex_data
0001:0074a53a* _X509_STORE_CTX_get_error
0001:0074a545* _X509_STORE_CTX_set_error
0001:0074a553* _X509_STORE_CTX_get_error_depth
0001:0074a55e* _X509_STORE_CTX_get_current_cert
0001:0074a569* _X509_STORE_CTX_get_chain
0001:0074a574* _X509_STORE_CTX_get1_chain
0001:0074a606* _X509_STORE_CTX_get0_current_issuer
0001:0074a611* _X509_STORE_CTX_get0_current_crl
0001:0074a61c* _X509_STORE_CTX_get0_parent_ctx
0001:0074a627* _X509_STORE_CTX_set_cert
0001:0074a635* _X509_STORE_CTX_set_chain
0001:0074a643* _X509_STORE_CTX_set0_crls
0001:0074a651  _X509_STORE_CTX_set_purpose
0001:0074a6a5* _X509_STORE_CTX_purpose_inherit
0001:0074a67b* _X509_STORE_CTX_set_trust
0001:0074a81d* _X509_STORE_CTX_new
0001:0074a89b* _X509_STORE_CTX_free
0001:0074ac7a* _X509_STORE_CTX_trusted_stack
0001:0074ad66* _X509_STORE_CTX_set_depth
0001:0074ad83* _X509_STORE_CTX_set_flags
0001:0074ada0* _X509_STORE_CTX_set_time
0001:0074adbd  _X509_STORE_CTX_set_verify_cb
0001:0074adcb* _X509_STORE_CTX_get0_policy_tree
0001:0074add6* _X509_STORE_CTX_get_explicit_policy
0001:0074ade1  _X509_STORE_CTX_set_default
0001:0074ae19  _X509_STORE_CTX_get0_param
Module: U:\extras\lib\libcrypto.lib(dh_asn1.obj)
0001:0074af20* _DHparams_it
0001:0074af3c  _d2i_DHparams
0001:0074af65  _i2d_DHparams
0001:0074af87  _DHparams_dup
Module: U:\extras\lib\libcrypto.lib(bn_lib.obj)
0001:0074afb0* _BN_version
0001:0074afdd* _BN_set_params
0001:0074b0a4* _BN_get_params
0001:0074b0e2  _BN_value_one
0001:0074b0f6* _BN_options
0001:0074b143  _BN_num_bits_word
0001:0074b1b4  _BN_num_bits
0001:0074b1fe  _BN_clear_free
0001:0074b280  _BN_free
0001:0074b2e8  _BN_init
0001:0074b314  _BN_new
0001:0074b566* _bn_dup_expand
0001:0074b651  _BN_dup
0001:0074b5f2  _bn_expand2
0001:0074b6a6  _BN_copy
0001:0074b7df* _BN_swap
0001:0074b899  _BN_clear
0001:0074b8e4* _BN_get_word
0001:0074b914  _BN_set_word
0001:0074b97b  _BN_bin2bn
0001:0074baea  _BN_bn2bin
0001:0074bb71  _BN_ucmp
0001:0074bbfd  _BN_cmp
0001:0074bd13  _BN_set_bit
0001:0074be0b* _BN_clear_bit
0001:0074bee0  _BN_is_bit_set
0001:0074bf4d  _BN_mask_bits
0001:0074c042  _BN_set_negative
0001:0074c06d  _bn_cmp_words
0001:0074c104  _bn_cmp_part_words
Module: U:\extras\lib\libcrypto.lib(ec_key.obj)
0001:0074c2c9  _EC_KEY_new
0001:0074c37b* _EC_KEY_new_by_curve_name
0001:0074c3c8  _EC_KEY_free
0001:0074c48b* _EC_KEY_copy
0001:0074c6d6  _EC_KEY_dup
0001:0074c71e  _EC_KEY_up_ref
0001:0074c761  _EC_KEY_generate_key
0001:0074c94a* _EC_KEY_check_key
0001:0074ccd1  _EC_KEY_get0_group
0001:0074ccdc  _EC_KEY_set_group
0001:0074cd1b  _EC_KEY_get0_private_key
0001:0074cd26  _EC_KEY_set_private_key
0001:0074cd65  _EC_KEY_get0_public_key
0001:0074cd70  _EC_KEY_set_public_key
0001:0074cdb9  _EC_KEY_get_enc_flags
0001:0074cdc4  _EC_KEY_set_enc_flags
0001:0074cdd2  _EC_KEY_get_conv_form
0001:0074cddd* _EC_KEY_set_conv_form
0001:0074ce0d  _EC_KEY_get_key_method_data
0001:0074ce38  _EC_KEY_insert_key_method_data
0001:0074cede* _EC_KEY_set_asn1_flag
0001:0074cf05* _EC_KEY_precompute_mult
Module: U:\extras\lib\libcrypto.lib(bss_file.obj)
0001:0074cf67  _BIO_new_file
0001:0074d11f  _BIO_s_file
0001:0074d0c3  _BIO_new_fp
Module: U:\extras\lib\libcrypto.lib(pem_x509.obj)
0001:0074d79c  _PEM_read_bio_X509
0001:0074d7d5* _PEM_read_X509
0001:0074d80e  _PEM_write_bio_X509
0001:0074d861* _PEM_write_X509
Module: U:\extras\lib\libcrypto.lib(o_dir.obj)
0001:0074d8c0  _OPENSSL_DIR_read
0001:0074d8d8  _OPENSSL_DIR_end
Module: U:\extras\lib\libcrypto.lib(a_object.obj)
0001:0074d8f0* _i2d_ASN1_OBJECT
0001:0074d9b9  _a2d_ASN1_OBJECT
0001:0074de50  _i2t_ASN1_OBJECT
0001:0074de88  _i2a_ASN1_OBJECT
0001:0074df83  _d2i_ASN1_OBJECT
0001:0074e049  _c2i_ASN1_OBJECT
0001:0074e251  _ASN1_OBJECT_new
0001:0074e2ef  _ASN1_OBJECT_free
0001:0074e3a5  _ASN1_OBJECT_create
Module: U:\extras\lib\libcrypto.lib(x509_trs.obj)
0001:0074e45c* _X509_TRUST_set_default
0001:0074e477  _X509_check_trust
0001:0074e557  _X509_TRUST_get_by_id
0001:0074e510* _X509_TRUST_get0
0001:0074e4e8* _X509_TRUST_get_count
0001:0074e5bc  _X509_TRUST_set
0001:0074e614* _X509_TRUST_add
0001:0074e853* _X509_TRUST_cleanup
0001:0074e8a6* _X509_TRUST_get_flags
0001:0074e8b1* _X509_TRUST_get0_name
0001:0074e8bc* _X509_TRUST_get_trust
Module: U:\extras\lib\libcrypto.lib(obj_lib.obj)
0001:0074ea7a  _OBJ_dup
0001:0074ece7  _OBJ_cmp
Module: U:\extras\lib\libcrypto.lib(tasn_typ.obj)
0001:0074ed50  _ASN1_INTEGER_it
0001:0074ed6c  _d2i_ASN1_INTEGER
0001:0074ed95  _i2d_ASN1_INTEGER
0001:0074edb7  _ASN1_INTEGER_new
0001:0074edcb  _ASN1_INTEGER_free
0001:0074ee00  _ASN1_ENUMERATED_it
0001:0074ee1c  _d2i_ASN1_ENUMERATED
0001:0074ee45* _i2d_ASN1_ENUMERATED
0001:0074ee67* _ASN1_ENUMERATED_new
0001:0074ee7b  _ASN1_ENUMERATED_free
0001:0074eeb0  _ASN1_BIT_STRING_it
0001:0074eecc  _d2i_ASN1_BIT_STRING
0001:0074eef5  _i2d_ASN1_BIT_STRING
0001:0074ef17  _ASN1_BIT_STRING_new
0001:0074ef2b  _ASN1_BIT_STRING_free
0001:0074ef60  _ASN1_OCTET_STRING_it
0001:0074ef7c  _d2i_ASN1_OCTET_STRING
0001:0074efa5  _i2d_ASN1_OCTET_STRING
0001:0074efc7  _ASN1_OCTET_STRING_new
0001:0074efdb  _ASN1_OCTET_STRING_free
0001:0074f000  _ASN1_NULL_it
0001:0074f01c* _d2i_ASN1_NULL
0001:0074f045* _i2d_ASN1_NULL
0001:0074f067  _ASN1_NULL_new
0001:0074f07b* _ASN1_NULL_free
0001:0074f0b0  _ASN1_OBJECT_it
0001:0074f0e0  _ASN1_UTF8STRING_it
0001:0074f0fc* _d2i_ASN1_UTF8STRING
0001:0074f125* _i2d_ASN1_UTF8STRING
0001:0074f147  _ASN1_UTF8STRING_new
0001:0074f15b  _ASN1_UTF8STRING_free
0001:0074f190* _ASN1_PRINTABLESTRING_it
0001:0074f1ac* _d2i_ASN1_PRINTABLESTRING
0001:0074f1d5* _i2d_ASN1_PRINTABLESTRING
0001:0074f1f7* _ASN1_PRINTABLESTRING_new
0001:0074f20b* _ASN1_PRINTABLESTRING_free
0001:0074f240* _ASN1_T61STRING_it
0001:0074f25c* _d2i_ASN1_T61STRING
0001:0074f285* _i2d_ASN1_T61STRING
0001:0074f2a7* _ASN1_T61STRING_new
0001:0074f2bb* _ASN1_T61STRING_free
0001:0074f2f0  _ASN1_IA5STRING_it
0001:0074f30c* _d2i_ASN1_IA5STRING
0001:0074f335* _i2d_ASN1_IA5STRING
0001:0074f357* _ASN1_IA5STRING_new
0001:0074f36b* _ASN1_IA5STRING_free
0001:0074f3a0* _ASN1_GENERALSTRING_it
0001:0074f3bc* _d2i_ASN1_GENERALSTRING
0001:0074f3e5* _i2d_ASN1_GENERALSTRING
0001:0074f407* _ASN1_GENERALSTRING_new
0001:0074f41b* _ASN1_GENERALSTRING_free
0001:0074f450* _ASN1_UTCTIME_it
0001:0074f46c* _d2i_ASN1_UTCTIME
0001:0074f495* _i2d_ASN1_UTCTIME
0001:0074f4b7* _ASN1_UTCTIME_new
0001:0074f4cb* _ASN1_UTCTIME_free
0001:0074f500  _ASN1_GENERALIZEDTIME_it
0001:0074f51c* _d2i_ASN1_GENERALIZEDTIME
0001:0074f545* _i2d_ASN1_GENERALIZEDTIME
0001:0074f567  _ASN1_GENERALIZEDTIME_new
0001:0074f57b* _ASN1_GENERALIZEDTIME_free
0001:0074f5b0* _ASN1_VISIBLESTRING_it
0001:0074f5cc* _d2i_ASN1_VISIBLESTRING
0001:0074f5f5* _i2d_ASN1_VISIBLESTRING
0001:0074f617* _ASN1_VISIBLESTRING_new
0001:0074f62b* _ASN1_VISIBLESTRING_free
0001:0074f660* _ASN1_UNIVERSALSTRING_it
0001:0074f67c* _d2i_ASN1_UNIVERSALSTRING
0001:0074f6a5* _i2d_ASN1_UNIVERSALSTRING
0001:0074f6c7* _ASN1_UNIVERSALSTRING_new
0001:0074f6db* _ASN1_UNIVERSALSTRING_free
0001:0074f710* _ASN1_BMPSTRING_it
0001:0074f72c* _d2i_ASN1_BMPSTRING
0001:0074f755* _i2d_ASN1_BMPSTRING
0001:0074f777* _ASN1_BMPSTRING_new
0001:0074f78b* _ASN1_BMPSTRING_free
0001:0074f7b0  _ASN1_ANY_it
0001:0074f7e0  _ASN1_SEQUENCE_it
0001:0074f7fc  _d2i_ASN1_TYPE
0001:0074f825  _i2d_ASN1_TYPE
0001:0074f847  _ASN1_TYPE_new
0001:0074f85b  _ASN1_TYPE_free
0001:0074f890  _ASN1_PRINTABLE_it
0001:0074f8ac* _d2i_ASN1_PRINTABLE
0001:0074f8d5* _i2d_ASN1_PRINTABLE
0001:0074f8f7* _ASN1_PRINTABLE_new
0001:0074f90b* _ASN1_PRINTABLE_free
0001:0074f940  _DISPLAYTEXT_it
0001:0074f95c* _d2i_DISPLAYTEXT
0001:0074f985* _i2d_DISPLAYTEXT
0001:0074f9a7* _DISPLAYTEXT_new
0001:0074f9bb* _DISPLAYTEXT_free
0001:0074f9f0  _DIRECTORYSTRING_it
0001:0074fa0c* _d2i_DIRECTORYSTRING
0001:0074fa35* _i2d_DIRECTORYSTRING
0001:0074fa57* _DIRECTORYSTRING_new
0001:0074fa6b* _DIRECTORYSTRING_free
0001:0074faa0  _ASN1_BOOLEAN_it
0001:0074fad0* _ASN1_TBOOLEAN_it
0001:0074fb00  _ASN1_FBOOLEAN_it
0001:0074fb40  _ASN1_OCTET_STRING_NDEF_it
0001:0074fb90* _ASN1_SEQUENCE_ANY_it
0001:0074fbe0* _ASN1_SET_ANY_it
0001:0074fbfc  _d2i_ASN1_SEQUENCE_ANY
0001:0074fc25  _i2d_ASN1_SEQUENCE_ANY
0001:0074fc47* _d2i_ASN1_SET_ANY
0001:0074fc70  _i2d_ASN1_SET_ANY
Module: U:\extras\lib\libcrypto.lib(tasn_dec.obj)
0001:0074fd20  _ASN1_tag2bit
0001:0074fd42  _ASN1_item_d2i
0001:0074fe0b  _ASN1_item_ex_d2i
0001:0074fdb0* _ASN1_template_d2i
0001:00751634* _asn1_ex_c2i
Module: U:\extras\lib\libcrypto.lib(tasn_enc.obj)
0001:00752190  _ASN1_item_ndef_i2d
0001:007521b9  _ASN1_item_i2d
0001:007522d4  _ASN1_item_ex_i2d
0001:007527fc* _ASN1_template_i2d
0001:00752fe1* _asn1_ex_i2c
Module: U:\extras\lib\libcrypto.lib(tasn_new.obj)
0001:00753290  _ASN1_item_new
0001:007532bf  _ASN1_item_ex_new
0001:00753810* _ASN1_template_new
0001:00753926* _ASN1_primitive_new
Module: U:\extras\lib\libcrypto.lib(tasn_fre.obj)
0001:00753b20  _ASN1_item_free
0001:00753b42  _ASN1_item_ex_free
0001:00753ef6  _ASN1_template_free
0001:00753f9c  _ASN1_primitive_free
Module: U:\extras\lib\libcrypto.lib(a_dup.obj)
0001:007540e8  _ASN1_dup
0001:007541bc  _ASN1_item_dup
Module: U:\extras\lib\libcrypto.lib(x_algor.obj)
0001:007542d0  _X509_ALGOR_it
0001:00754320  _X509_ALGORS_it
0001:0075433c  _d2i_X509_ALGOR
0001:00754365* _i2d_X509_ALGOR
0001:00754387  _X509_ALGOR_new
0001:0075439b  _X509_ALGOR_free
0001:007543b6* _d2i_X509_ALGORS
0001:007543df  _i2d_X509_ALGORS
0001:00754401* _X509_ALGOR_dup
0001:0075441c  _X509_ALGOR_set0
0001:007544dc  _X509_ALGOR_get0
Module: U:\extras\lib\libcrypto.lib(v3_genn.obj)
0001:00754580* _OTHERNAME_it
0001:0075459c* _d2i_OTHERNAME
0001:007545c5* _i2d_OTHERNAME
0001:007545e7  _OTHERNAME_new
0001:007545fb* _OTHERNAME_free
0001:00754670* _EDIPARTYNAME_it
0001:0075468c* _d2i_EDIPARTYNAME
0001:007546b5* _i2d_EDIPARTYNAME
0001:007546d7* _EDIPARTYNAME_new
0001:007546eb* _EDIPARTYNAME_free
0001:00754860  _GENERAL_NAME_it
0001:0075487c* _d2i_GENERAL_NAME
0001:007548a5* _i2d_GENERAL_NAME
0001:007548c7  _GENERAL_NAME_new
0001:007548db  _GENERAL_NAME_free
0001:00754940  _GENERAL_NAMES_it
0001:0075495c* _d2i_GENERAL_NAMES
0001:00754985* _i2d_GENERAL_NAMES
0001:007549a7  _GENERAL_NAMES_new
0001:007549bb  _GENERAL_NAMES_free
0001:007549d6* _GENERAL_NAME_dup
0001:007549fb  _GENERAL_NAME_cmp
0001:00754b1d* _OTHERNAME_cmp
0001:00754b81* _GENERAL_NAME_set0_value
0001:00754c0b* _GENERAL_NAME_get0_value
0001:00754c8f* _GENERAL_NAME_set0_othername
0001:00754cdc* _GENERAL_NAME_get0_otherName
Module: U:\extras\lib\libcrypto.lib(v3_info.obj)
0001:00754d20  _v3_info
0001:00754ed0* _AUTHORITY_INFO_ACCESS_it
0001:00754d60  _v3_sinfo
0001:00754df0  _ACCESS_DESCRIPTION_it
0001:00754e0c* _d2i_ACCESS_DESCRIPTION
0001:00754e35* _i2d_ACCESS_DESCRIPTION
0001:00754e57* _ACCESS_DESCRIPTION_new
0001:00754e6b* _ACCESS_DESCRIPTION_free
0001:00754eec* _d2i_AUTHORITY_INFO_ACCESS
0001:00754f15* _i2d_AUTHORITY_INFO_ACCESS
0001:00754f37* _AUTHORITY_INFO_ACCESS_new
0001:00754f4b  _AUTHORITY_INFO_ACCESS_free
0001:007553b6* _i2a_ACCESS_DESCRIPTION
Module: U:\extras\lib\libcrypto.lib(a_strex.obj)
0001:0075629c  _X509_NAME_print_ex
0001:007562ed* _X509_NAME_print_ex_fp
0001:00756372  _ASN1_STRING_print_ex
0001:0075639b* _ASN1_STRING_print_ex_fp
0001:007563c4  _ASN1_STRING_to_UTF8
Module: U:\extras\lib\libcrypto.lib(asn1_lib.obj)
0001:00756490* _ASN1_version
0001:00756500* _ASN1_check_infinite_end
0001:0075651a  _ASN1_const_check_infinite_end
0001:0075653f  _ASN1_get_object
0001:00756801  _ASN1_put_object
0001:00756901  _ASN1_put_eoc
0001:007569b4  _ASN1_object_size
0001:00756a8e* _asn1_Finish
0001:00756aa1  _asn1_const_Finish
0001:00756ab4  _asn1_GetSequence
0001:00756bb9  _ASN1_STRING_copy
0001:00756c69  _ASN1_STRING_set
0001:00756c14  _ASN1_STRING_dup
0001:00756dc8  _ASN1_STRING_new
0001:00756e65  _ASN1_STRING_free
0001:00756d97  _ASN1_STRING_set0
0001:00756ddc  _ASN1_STRING_type_new
0001:00756ea6  _ASN1_STRING_cmp
0001:00756f28  _asn1_add_error
0001:00756f9e* _ASN1_STRING_length
0001:00756fa8* _ASN1_STRING_length_set
0001:00756fb5* _ASN1_STRING_type
0001:00756fc0  _ASN1_STRING_data
Module: U:\extras\lib\libcrypto.lib(x509_obj.obj)
0001:00756fe8  _X509_NAME_oneline
Module: U:\extras\lib\libcrypto.lib(m_md5.obj)
0001:007574dc  _EVP_md5
Module: U:\extras\lib\libcrypto.lib(m_sha1.obj)
0001:0075759c  _EVP_sha1
0001:0075766c* _EVP_sha224
0001:007576cc  _EVP_sha256
0001:0075779c* _EVP_sha384
0001:007577fc* _EVP_sha512
Module: U:\extras\lib\libcrypto.lib(x_pubkey.obj)
0001:007578b0  _X509_PUBKEY_it
0001:007578cc* _d2i_X509_PUBKEY
0001:007578f5* _i2d_X509_PUBKEY
0001:00757917* _X509_PUBKEY_new
0001:0075792b* _X509_PUBKEY_free
0001:00757951  _X509_PUBKEY_set
0001:00757a86  _X509_PUBKEY_get
0001:00757c60  _d2i_PUBKEY
0001:00757cd6  _i2d_PUBKEY
0001:00757d32  _d2i_RSA_PUBKEY
0001:00757db8  _i2d_RSA_PUBKEY
0001:00757e43  _d2i_DSA_PUBKEY
0001:00757ec9  _i2d_DSA_PUBKEY
0001:00757f54  _d2i_EC_PUBKEY
0001:00757fda  _i2d_EC_PUBKEY
0001:00758065  _X509_PUBKEY_set0_param
0001:00758104  _X509_PUBKEY_get0_param
Module: U:\extras\lib\libcrypto.lib(x_crl.obj)
0001:007581e0* _X509_REVOKED_it
0001:00758340  _X509_CRL_INFO_it
0001:00758a40  _X509_CRL_it
0001:00758a5c* _d2i_X509_REVOKED
0001:00758a85* _i2d_X509_REVOKED
0001:00758aa7* _X509_REVOKED_new
0001:00758abb* _X509_REVOKED_free
0001:00758ad6* _d2i_X509_CRL_INFO
0001:00758aff* _i2d_X509_CRL_INFO
0001:00758b21* _X509_CRL_INFO_new
0001:00758b35* _X509_CRL_INFO_free
0001:00758b50  _d2i_X509_CRL
0001:00758b79  _i2d_X509_CRL
0001:00758b9b* _X509_CRL_new
0001:00758baf  _X509_CRL_free
0001:00758bca* _X509_CRL_dup
0001:00758c0f* _X509_CRL_add0_revoked
0001:00758ca3  _X509_CRL_verify
0001:00758cd7* _X509_CRL_get0_by_serial
0001:00758d1a  _X509_CRL_get0_by_cert
0001:00758fbe* _X509_CRL_set_default_method
0001:00758fdd* _X509_CRL_METHOD_new
0001:00759041* _X509_CRL_METHOD_free
0001:00759063* _X509_CRL_set_meth_data
0001:00759071* _X509_CRL_get_meth_data
Module: U:\extras\lib\libcrypto.lib(o_names.obj)
0001:007590bf* _OBJ_NAME_init
0001:0075911f* _OBJ_NAME_new_index
0001:007593ae  _OBJ_NAME_get
0001:00759459  _OBJ_NAME_add
0001:0075957e* _OBJ_NAME_remove
0001:0075968f  _OBJ_NAME_do_all
0001:00759736  _OBJ_NAME_do_all_sorted
0001:0075985a  _OBJ_NAME_cleanup
Module: U:\extras\lib\libcrypto.lib(evp_pbe.obj)
0001:00759a95  _EVP_PBE_CipherInit
0001:00759eb6  _EVP_PBE_find
0001:00759d8c* _EVP_PBE_alg_add_type
0001:00759e4c* _EVP_PBE_alg_add
0001:00759f9a  _EVP_PBE_cleanup
Module: U:\extras\lib\libcrypto.lib(obj_xref.obj)
0002:00022410+ _sig_app
0002:00022420+ _sigx_app
0001:0075a2c2  _OBJ_find_sigid_algs
0001:0075a360  _OBJ_find_sigid_by_algs
0001:0075a411* _OBJ_add_sigid
0001:0075a539  _OBJ_sigid_free
Module: U:\extras\lib\libcrypto.lib(tb_rand.obj)
0001:0075a594* _ENGINE_unregister_RAND
0001:0075a5c3* _ENGINE_register_RAND
0001:0075a60f* _ENGINE_register_all_RAND
0001:0075a640* _ENGINE_set_default_RAND
0001:0075a68c  _ENGINE_get_default_RAND
0001:0075a6a9  _ENGINE_get_RAND
0001:0075a6b4* _ENGINE_set_RAND
Module: U:\extras\lib\libcrypto.lib(md_rand.obj)
0001:0075a6d0* _RAND_version
0001:0075a6f7  _RAND_SSLeay
0002:000070b0* _rand_ssleay_meth
Module: U:\extras\lib\libcrypto.lib(x_val.obj)
0001:0075b390  _X509_VAL_it
0001:0075b3ac* _d2i_X509_VAL
0001:0075b3d5* _i2d_X509_VAL
0001:0075b3f7* _X509_VAL_new
0001:0075b40b* _X509_VAL_free
Module: U:\extras\lib\libcrypto.lib(x_x509a.obj)
0001:0075b4d0* _X509_CERT_AUX_it
0001:0075b4ec  _d2i_X509_CERT_AUX
0001:0075b515  _i2d_X509_CERT_AUX
0001:0075b537* _X509_CERT_AUX_new
0001:0075b54b  _X509_CERT_AUX_free
0001:0075b5a7* _X509_alias_set1
0001:0075b65e* _X509_keyid_set1
0001:0075b715* _X509_alias_get0
0001:0075b75a* _X509_keyid_get0
0001:0075b79f* _X509_add1_trust_object
0001:0075b816* _X509_add1_reject_object
0001:0075b891* _X509_trust_clear
0001:0075b8d4* _X509_reject_clear
0001:0075b970* _X509_CERT_PAIR_it
0001:0075b98c  _d2i_X509_CERT_PAIR
0001:0075b9b5  _i2d_X509_CERT_PAIR
0001:0075b9d7* _X509_CERT_PAIR_new
0001:0075b9eb* _X509_CERT_PAIR_free
Module: U:\extras\lib\libcrypto.lib(v3_akeya.obj)
0001:0075ba80  _AUTHORITY_KEYID_it
0001:0075ba9c* _d2i_AUTHORITY_KEYID
0001:0075bac5* _i2d_AUTHORITY_KEYID
0001:0075bae7  _AUTHORITY_KEYID_new
0001:0075bafb  _AUTHORITY_KEYID_free
Module: U:\extras\lib\libcrypto.lib(v3_crld.obj)
0001:0075bb20  _v3_crld
0001:0075c890* _CRL_DIST_POINTS_it
0001:0075bb60  _v3_freshest_crl
0001:0075c727* _DIST_POINT_NAME_new
0001:0075c817* _DIST_POINT_new
0001:0075c82b* _DIST_POINT_free
0001:0075c6c0* _DIST_POINT_NAME_it
0001:0075c6dc* _d2i_DIST_POINT_NAME
0001:0075c705* _i2d_DIST_POINT_NAME
0001:0075c73b* _DIST_POINT_NAME_free
0001:0075c7b0* _DIST_POINT_it
0001:0075c7cc* _d2i_DIST_POINT
0001:0075c7f5* _i2d_DIST_POINT
0001:0075c8ac* _d2i_CRL_DIST_POINTS
0001:0075c8d5* _i2d_CRL_DIST_POINTS
0001:0075c8f7* _CRL_DIST_POINTS_new
0001:0075c90b  _CRL_DIST_POINTS_free
0001:0075c9f0* _ISSUING_DIST_POINT_it
0001:0075ca0c* _d2i_ISSUING_DIST_POINT
0001:0075ca35* _i2d_ISSUING_DIST_POINT
0001:0075ca57* _ISSUING_DIST_POINT_new
0001:0075ca6b  _ISSUING_DIST_POINT_free
0001:0075ca90  _v3_idp
0001:0075d1ca  _DIST_POINT_set_dpname
Module: U:\extras\lib\libcrypto.lib(pcy_cache.obj)
0001:0075d6fa  _policy_cache_free
0001:0075d74d  _policy_cache_set
0001:0075d7b8  _policy_cache_find_data
Module: U:\extras\lib\libcrypto.lib(v3_ncons.obj)
0001:0075d870  _v3_name_constraints
0001:0075d990* _NAME_CONSTRAINTS_it
0001:0075d910* _GENERAL_SUBTREE_it
0001:0075d9ac* _GENERAL_SUBTREE_new
0001:0075d9c0* _GENERAL_SUBTREE_free
0001:0075d9db* _NAME_CONSTRAINTS_new
0001:0075d9ef  _NAME_CONSTRAINTS_free
0001:0075df48  _NAME_CONSTRAINTS_check
Module: U:\extras\lib\libcrypto.lib(eng_lib.obj)
0001:0075e64a  _ENGINE_new
0001:0075e6ef* _engine_set_all_null
0001:0075e79d  _engine_free_util
0001:0075e89a  _ENGINE_free
0001:0075e930  _engine_cleanup_add_first
0001:0075e97b  _engine_cleanup_add_last
0001:0075e9d8* _ENGINE_cleanup
0001:0075ea1c* _ENGINE_get_ex_new_index
0001:0075ea53* _ENGINE_set_ex_data
0001:0075ea77* _ENGINE_get_ex_data
0001:0075ea94* _ENGINE_set_id
0001:0075eae2* _ENGINE_set_name
0001:0075eb31* _ENGINE_set_destroy_function
0001:0075eb44* _ENGINE_set_init_function
0001:0075eb57* _ENGINE_set_finish_function
0001:0075eb6a* _ENGINE_set_ctrl_function
0001:0075eb7d* _ENGINE_set_flags
0001:0075eb90* _ENGINE_set_cmd_defns
0001:0075eba3* _ENGINE_get_id
0001:0075ebad* _ENGINE_get_name
0001:0075ebb8* _ENGINE_get_destroy_function
0001:0075ebc3* _ENGINE_get_init_function
0001:0075ebce* _ENGINE_get_finish_function
0001:0075ebd9* _ENGINE_get_ctrl_function
0001:0075ebe4* _ENGINE_get_flags
0001:0075ebef* _ENGINE_get_cmd_defns
0001:0075ebfa* _ENGINE_get_static_state
Module: U:\extras\lib\libcrypto.lib(rsa_eay.obj)
0001:0075ec28  _RSA_PKCS1_SSLeay
Module: U:\extras\lib\libcrypto.lib(tb_rsa.obj)
0001:00760ce4* _ENGINE_unregister_RSA
0001:00760d13* _ENGINE_register_RSA
0001:00760d5f* _ENGINE_register_all_RSA
0001:00760d90* _ENGINE_set_default_RSA
0001:00760ddc  _ENGINE_get_default_RSA
0001:00760df9  _ENGINE_get_RSA
0001:00760e04* _ENGINE_set_RSA
Module: U:\extras\lib\libcrypto.lib(bn_blind.obj)
0001:00760e2b* _BN_BLINDING_new
0001:00760f67  _BN_BLINDING_free
0001:00760fe1* _BN_BLINDING_update
0001:00761362  _BN_BLINDING_create_param
0001:00761142* _BN_BLINDING_convert
0001:0076116b  _BN_BLINDING_convert_ex
0001:00761220* _BN_BLINDING_invert
0001:00761249  _BN_BLINDING_invert_ex
0001:00761325* _BN_BLINDING_get_thread_id
0001:00761330* _BN_BLINDING_set_thread_id
0001:0076133e  _BN_BLINDING_thread_id
0001:00761349* _BN_BLINDING_get_flags
0001:00761354* _BN_BLINDING_set_flags
Module: U:\extras\lib\libcrypto.lib(bn_ctx.obj)
0001:007615d0* _BN_CTX_init
0001:00761618  _BN_CTX_new
0001:007616b2  _BN_CTX_free
0001:007616e7  _BN_CTX_start
0001:0076176b  _BN_CTX_end
0001:007617d7  _BN_CTX_get
Module: U:\extras\lib\libcrypto.lib(bn_add.obj)
0001:00761cb0  _BN_add
0001:00761f19  _BN_usub
0001:00761d8b  _BN_uadd
0001:00762132  _BN_sub
Module: U:\extras\lib\libcrypto.lib(bn_mul.obj)
0001:007622a0* _bn_sub_part_words
0001:007625e8* _bn_add_part_words
0001:00762a38* _bn_mul_recursive
0001:00764706* _bn_mul_normal
0001:0076316f* _bn_mul_part_recursive
0001:00763994* _bn_mul_low_recursive
0001:007648a9* _bn_mul_low_normal
0001:00763b75* _bn_mul_high
0001:007642ab  _BN_mul
Module: U:\extras\lib\libcrypto.lib(bn_gcd.obj)
0001:007649c0  _BN_gcd
0001:00764cad  _BN_mod_inverse
Module: U:\extras\lib\libcrypto.lib(dh_key.obj)
0001:00765910  _DH_generate_key
0001:00765929  _DH_compute_key
0001:00765962  _DH_OpenSSL
Module: U:\extras\lib\libcrypto.lib(tb_dh.obj)
0001:00765f04* _ENGINE_unregister_DH
0001:00765f33* _ENGINE_register_DH
0001:00765f7f* _ENGINE_register_all_DH
0001:00765fb0* _ENGINE_set_default_DH
0001:00765ffc  _ENGINE_get_default_DH
0001:00766019  _ENGINE_get_DH
0001:00766024* _ENGINE_set_DH
Module: U:\extras\lib\libcrypto.lib(dsa_lib.obj)
0001:00766040* _DSA_version
0001:00766066* _DSA_set_default_method
0001:00766073* _DSA_get_default_method
0001:00766093  _DSA_new
0001:00766122* _DSA_new_method
0001:007660a7* _DSA_set_method
0001:00766382  _DSA_free
0001:007664db  _DSA_up_ref
0001:0076651e  _DSA_size
0001:0076659a* _DSA_get_ex_new_index
0001:007665d1* _DSA_set_ex_data
0001:007665f5* _DSA_get_ex_data
0001:00766612* _DSA_dup_DH
Module: U:\extras\lib\libcrypto.lib(x_attrib.obj)
0001:00766790* _X509_ATTRIBUTE_SET_it
0001:007667f0  _X509_ATTRIBUTE_it
0001:0076680c* _d2i_X509_ATTRIBUTE
0001:00766835* _i2d_X509_ATTRIBUTE
0001:00766857  _X509_ATTRIBUTE_new
0001:0076686b  _X509_ATTRIBUTE_free
0001:00766886  _X509_ATTRIBUTE_dup
0001:007668a1  _X509_ATTRIBUTE_create
Module: U:\extras\lib\libcrypto.lib(x509_v3.obj)
0001:00766980  _X509v3_get_ext_count
0001:007669a0  _X509v3_get_ext_by_NID
0001:007669dc  _X509v3_get_ext_by_OBJ
0001:00766a53  _X509v3_get_ext_by_critical
0001:00766ad2  _X509v3_get_ext
0001:00766b0f  _X509v3_delete_ext
0001:00766b5c  _X509v3_add_ext
0001:00766c92  _X509_EXTENSION_create_by_NID
0001:00766d18  _X509_EXTENSION_create_by_OBJ
0001:00766e00* _X509_EXTENSION_set_object
0001:00766e3d* _X509_EXTENSION_set_critical
0001:00766e6c* _X509_EXTENSION_set_data
0001:00766eb7  _X509_EXTENSION_get_object
0001:00766ece  _X509_EXTENSION_get_data
0001:00766ee6  _X509_EXTENSION_get_critical
Module: U:\extras\lib\libcrypto.lib(x509_ext.obj)
0001:00766f10* _X509_CRL_get_ext_count
0001:00766f28  _X509_CRL_get_ext_by_NID
0001:00766f4e* _X509_CRL_get_ext_by_OBJ
0001:00766f74* _X509_CRL_get_ext_by_critical
0001:00766f9a  _X509_CRL_get_ext
0001:00766fb9* _X509_CRL_delete_ext
0001:00766fd8  _X509_CRL_get_ext_d2i
0001:00767005* _X509_CRL_add1_ext_i2d
0001:00767039* _X509_CRL_add_ext
0001:00767067  _X509_get_ext_count
0001:0076707f  _X509_get_ext_by_NID
0001:007670a5* _X509_get_ext_by_OBJ
0001:007670cb* _X509_get_ext_by_critical
0001:007670f1  _X509_get_ext
0001:00767110* _X509_delete_ext
0001:0076712f* _X509_add_ext
0001:0076715d  _X509_get_ext_d2i
0001:0076718a* _X509_add1_ext_i2d
0001:007671be* _X509_REVOKED_get_ext_count
0001:007671d4* _X509_REVOKED_get_ext_by_NID
0001:007671f8* _X509_REVOKED_get_ext_by_OBJ
0001:0076721c* _X509_REVOKED_get_ext_by_critical
0001:00767240* _X509_REVOKED_get_ext
0001:0076725d* _X509_REVOKED_delete_ext
0001:0076727a* _X509_REVOKED_add_ext
0001:007672a6  _X509_REVOKED_get_ext_d2i
0001:007672d1* _X509_REVOKED_add1_ext_i2d
Module: U:\extras\lib\libcrypto.lib(x_all.obj)
0001:00767310  _X509_verify
0001:0076734d* _X509_REQ_verify
0001:0076738a* _NETSCAPE_SPKI_verify
0001:007673c7* _X509_sign
0001:00767425  _X509_REQ_sign
0001:00767471* _X509_CRL_sign
0001:007674cf* _NETSCAPE_SPKI_sign
0001:0076751b* _d2i_X509_fp
0001:0076753d* _i2d_X509_fp
0001:0076755f  _d2i_X509_bio
0001:00767581* _i2d_X509_bio
0001:007675a3* _d2i_X509_CRL_fp
0001:007675c5* _i2d_X509_CRL_fp
0001:007675e7  _d2i_X509_CRL_bio
0001:00767609* _i2d_X509_CRL_bio
0001:0076762b* _d2i_PKCS7_fp
0001:0076764d* _i2d_PKCS7_fp
0001:0076766f* _d2i_PKCS7_bio
0001:00767691* _i2d_PKCS7_bio
0001:007676b3* _d2i_X509_REQ_fp
0001:007676d5* _i2d_X509_REQ_fp
0001:007676f7* _d2i_X509_REQ_bio
0001:00767719* _i2d_X509_REQ_bio
0001:0076773b* _d2i_RSAPrivateKey_fp
0001:0076775d* _i2d_RSAPrivateKey_fp
0001:0076777f* _d2i_RSAPublicKey_fp
0001:007677a1* _d2i_RSA_PUBKEY_fp
0001:007677cd* _i2d_RSAPublicKey_fp
0001:007677ef* _i2d_RSA_PUBKEY_fp
0001:00767812  _d2i_RSAPrivateKey_bio
0001:00767834* _i2d_RSAPrivateKey_bio
0001:00767856* _d2i_RSAPublicKey_bio
0001:00767878* _d2i_RSA_PUBKEY_bio
0001:007678a4* _i2d_RSAPublicKey_bio
0001:007678c6* _i2d_RSA_PUBKEY_bio
0001:007678e9* _d2i_DSAPrivateKey_fp
0001:00767915* _i2d_DSAPrivateKey_fp
0001:00767938* _d2i_DSA_PUBKEY_fp
0001:00767964* _i2d_DSA_PUBKEY_fp
0001:00767987* _d2i_DSAPrivateKey_bio
0001:007679b3* _i2d_DSAPrivateKey_bio
0001:007679d6* _d2i_DSA_PUBKEY_bio
0001:00767a02* _i2d_DSA_PUBKEY_bio
0001:00767a25* _d2i_EC_PUBKEY_fp
0001:00767a51* _i2d_EC_PUBKEY_fp
0001:00767a74* _d2i_ECPrivateKey_fp
0001:00767aa0* _i2d_ECPrivateKey_fp
0001:00767ac3* _d2i_EC_PUBKEY_bio
0001:00767aef* _i2d_EC_PUBKEY_bio
0001:00767b12* _d2i_ECPrivateKey_bio
0001:00767b3e* _i2d_ECPrivateKey_bio
0001:00767b61* _X509_pubkey_digest
0001:00767bba  _X509_digest
0001:00767bea  _X509_CRL_digest
0001:00767c1a* _X509_REQ_digest
0001:00767c4a* _X509_NAME_digest
0001:00767c7a* _PKCS7_ISSUER_AND_SERIAL_digest
0001:00767caa* _d2i_PKCS8_fp
0001:00767cd6* _i2d_PKCS8_fp
0001:00767cf9  _d2i_PKCS8_bio
0001:00767d25  _i2d_PKCS8_bio
0001:00767d48* _d2i_PKCS8_PRIV_KEY_INFO_fp
0001:00767d74* _i2d_PKCS8_PRIV_KEY_INFO_fp
0001:00767d97* _i2d_PKCS8PrivateKeyInfo_fp
0001:00767ddd* _i2d_PrivateKey_fp
0001:00767e00* _d2i_PrivateKey_fp
0001:00767e2c* _i2d_PUBKEY_fp
0001:00767e4f* _d2i_PUBKEY_fp
0001:00767e7b* _d2i_PKCS8_PRIV_KEY_INFO_bio
0001:00767ea7  _i2d_PKCS8_PRIV_KEY_INFO_bio
0001:00767eca* _i2d_PKCS8PrivateKeyInfo_bio
0001:00767f10* _i2d_PrivateKey_bio
0001:00767f33  _d2i_PrivateKey_bio
0001:00767f5f* _i2d_PUBKEY_bio
0001:00767f82* _d2i_PUBKEY_bio
Module: U:\extras\lib\libcrypto.lib(a_int.obj)
0001:00767fb0* _ASN1_INTEGER_dup
0001:00767fc3  _ASN1_INTEGER_cmp
0001:00768022  _i2c_ASN1_INTEGER
0001:007681f4  _c2i_ASN1_INTEGER
0001:00768426  _d2i_ASN1_UINTEGER
0001:007685f2  _ASN1_INTEGER_set
0001:00768735  _ASN1_INTEGER_get
0001:007687df  _BN_to_ASN1_INTEGER
0001:00768950  _ASN1_INTEGER_to_BN
Module: U:\extras\lib\libcrypto.lib(v3_bcons.obj)
0001:007689d0  _v3_bcons
0001:00768a60* _BASIC_CONSTRAINTS_it
0001:00768a7c* _d2i_BASIC_CONSTRAINTS
0001:00768aa5* _i2d_BASIC_CONSTRAINTS
0001:00768ac7* _BASIC_CONSTRAINTS_new
0001:00768adb  _BASIC_CONSTRAINTS_free
Module: U:\extras\lib\libcrypto.lib(v3_pcia.obj)
0001:00768d40* _PROXY_POLICY_it
0001:00768d5c* _d2i_PROXY_POLICY
0001:00768d85* _i2d_PROXY_POLICY
0001:00768da7* _PROXY_POLICY_new
0001:00768dbb* _PROXY_POLICY_free
0001:00768e50  _PROXY_CERT_INFO_EXTENSION_it
0001:00768e6c* _d2i_PROXY_CERT_INFO_EXTENSION
0001:00768e95* _i2d_PROXY_CERT_INFO_EXTENSION
0001:00768eb7  _PROXY_CERT_INFO_EXTENSION_new
0001:00768ecb  _PROXY_CERT_INFO_EXTENSION_free
Module: U:\extras\lib\libcrypto.lib(a_octet.obj)
0001:00768ef0  _ASN1_OCTET_STRING_dup
0001:00768f03  _ASN1_OCTET_STRING_cmp
0001:00768f1d  _ASN1_OCTET_STRING_set
Module: U:\extras\lib\libcrypto.lib(bn_word.obj)
0001:00768f40  _BN_mod_word
0001:00768fc4  _BN_div_word
0001:007690e4  _BN_add_word
0001:0076923c  _BN_sub_word
0001:007693b6  _BN_mul_word
Module: U:\extras\lib\libcrypto.lib(bn_shift.obj)
0001:00769490  _BN_lshift1
0001:007695ab  _BN_rshift1
0001:007696ec  _BN_lshift
0001:007698d1  _BN_rshift
Module: U:\extras\lib\libcrypto.lib(bn_print.obj)
0001:00769b3c* _BN_bn2hex
0001:00769c70  _BN_bn2dec
0001:00769ef3  _BN_hex2bn
0001:0076a168  _BN_dec2bn
0001:0076a39a  _BN_asc2bn
0001:0076a428* _BN_print_fp
0001:0076a496* _BN_print
Module: U:\extras\lib\libcrypto.lib(tb_cipher.obj)
0001:0076a5a0* _ENGINE_unregister_ciphers
0001:0076a5cf* _ENGINE_register_ciphers
0001:0076a647* _ENGINE_register_all_ciphers
0001:0076a678* _ENGINE_set_default_ciphers
0001:0076a6f0  _ENGINE_get_cipher_engine
0001:0076a717  _ENGINE_get_cipher
0001:0076a78e* _ENGINE_get_ciphers
0001:0076a799* _ENGINE_set_ciphers
Module: U:\extras\lib\libcrypto.lib(by_file.obj)
0001:0076a7c5  _X509_LOOKUP_file
0001:0076ad5f* _X509_load_cert_crl_file
0001:0076a8f1  _X509_load_cert_file
0001:0076ab27  _X509_load_crl_file
0002:00007140* _x509_file_lookup
Module: U:\extras\lib\libcrypto.lib(by_dir.obj)
0001:0076af15  _X509_LOOKUP_hash_dir
0002:00007170* _x509_dir_lookup
Module: U:\extras\lib\libcrypto.lib(tb_digest.obj)
0001:0076b9b0* _ENGINE_unregister_digests
0001:0076b9df* _ENGINE_register_digests
0001:0076ba57* _ENGINE_register_all_digests
0001:0076ba88* _ENGINE_set_default_digests
0001:0076bb00  _ENGINE_get_digest_engine
0001:0076bb27  _ENGINE_get_digest
0001:0076bb9e* _ENGINE_get_digests
0001:0076bba9* _ENGINE_set_digests
Module: U:\extras\lib\libcrypto.lib(pmeth_lib.obj)
0001:0076bc30* _EVP_PKEY_meth_find
0001:0076c29b  _EVP_PKEY_CTX_free
0001:0076bee7* _EVP_PKEY_meth_new
0001:0076c031  _EVP_PKEY_meth_free
0001:0076c057  _EVP_PKEY_CTX_new
0001:0076c079  _EVP_PKEY_CTX_new_id
0001:0076c09b  _EVP_PKEY_CTX_dup
0001:0076c237* _EVP_PKEY_meth_add0
0001:0076c324  _EVP_PKEY_CTX_ctrl
0001:0076c483* _EVP_PKEY_CTX_ctrl_str
0001:0076c596* _EVP_PKEY_CTX_get_operation
0001:0076c5a1* _EVP_PKEY_CTX_set0_keygen_info
0001:0076c5b8* _EVP_PKEY_CTX_set_data
0001:0076c5c6* _EVP_PKEY_CTX_get_data
0001:0076c5d1* _EVP_PKEY_CTX_get0_pkey
0001:0076c5dc* _EVP_PKEY_CTX_get0_peerkey
0001:0076c5e7* _EVP_PKEY_CTX_set_app_data
0001:0076c5f5* _EVP_PKEY_CTX_get_app_data
0001:0076c600* _EVP_PKEY_meth_set_init
0001:0076c60e* _EVP_PKEY_meth_set_copy
0001:0076c61c* _EVP_PKEY_meth_set_cleanup
0001:0076c62a* _EVP_PKEY_meth_set_paramgen
0001:0076c641* _EVP_PKEY_meth_set_keygen
0001:0076c658* _EVP_PKEY_meth_set_sign
0001:0076c66f* _EVP_PKEY_meth_set_verify
0001:0076c686* _EVP_PKEY_meth_set_verify_recover
0001:0076c69d* _EVP_PKEY_meth_set_signctx
0001:0076c6b4* _EVP_PKEY_meth_set_verifyctx
0001:0076c6cb* _EVP_PKEY_meth_set_encrypt
0001:0076c6e2* _EVP_PKEY_meth_set_decrypt
0001:0076c6f9* _EVP_PKEY_meth_set_derive
0001:0076c710* _EVP_PKEY_meth_set_ctrl
0002:0001fc10* _app_pkey_methods
Module: U:\extras\lib\libssl.lib(s2_enc.obj)
0001:0076c7a6  _ssl2_enc_init
0001:0076cac5  _ssl2_enc
0001:0076cb5a  _ssl2_mac
Module: U:\extras\lib\libssl.lib(s2_pkt.obj)
0001:0076d32e  _ssl2_read
0001:0076d357  _ssl2_peek
0001:0076d658  _ssl2_write
0001:0076dd0b  _ssl2_part_read
0001:0076dde7  _ssl2_do_write
Module: U:\extras\lib\libssl.lib(ssl_rsa.obj)
0001:0076df2a  _SSL_use_certificate
0001:0076dfca* _SSL_use_certificate_file
0001:0076e183* _SSL_use_certificate_ASN1
0001:0076e204* _SSL_use_RSAPrivateKey
0001:0076e4ba* _SSL_use_RSAPrivateKey_file
0001:0076e66d* _SSL_use_RSAPrivateKey_ASN1
0001:0076e6f4  _SSL_use_PrivateKey
0001:0076e79a* _SSL_use_PrivateKey_file
0001:0076e94d* _SSL_use_PrivateKey_ASN1
0001:0076e9db* _SSL_CTX_use_certificate
0001:0076ec6b* _SSL_CTX_use_certificate_file
0001:0076ee18* _SSL_CTX_use_certificate_ASN1
0001:0076ee99* _SSL_CTX_use_RSAPrivateKey
0001:0076efb6* _SSL_CTX_use_RSAPrivateKey_file
0001:0076f15d* _SSL_CTX_use_RSAPrivateKey_ASN1
0001:0076f1e4* _SSL_CTX_use_PrivateKey
0001:0076f284* _SSL_CTX_use_PrivateKey_file
0001:0076f42b* _SSL_CTX_use_PrivateKey_ASN1
0001:0076f4b9* _SSL_CTX_use_certificate_chain_file
Module: U:\extras\lib\libcrypto.lib(p_sign.obj)
0001:0076f709  _EVP_SignFinal
Module: U:\extras\lib\libcrypto.lib(ec_curve.obj)
0001:00773a83  _EC_GROUP_new_by_curve_name
0001:00773b3b* _EC_get_builtin_curves
Module: U:\extras\lib\libcrypto.lib(ec_lib.obj)
0001:00773bfe  _EC_GROUP_new
0001:00773d6e  _EC_GROUP_free
0001:00774d06  _EC_EX_DATA_free_all_data
0001:00774ebf  _EC_POINT_free
0001:00773e04  _EC_GROUP_clear_free
0001:00774d5a* _EC_EX_DATA_clear_free_all_data
0001:00774ef7  _EC_POINT_clear_free
0001:00773ee3  _EC_GROUP_copy
0001:00774ab1  _EC_EX_DATA_set_data
0001:00774dae  _EC_POINT_new
0001:00774f60  _EC_POINT_copy
0001:007741e0  _EC_GROUP_dup
0001:00774261  _EC_GROUP_method_of
0001:0077426b  _EC_METHOD_get_field_type
0001:00774275  _EC_GROUP_set_generator
0001:00774385  _EC_GROUP_get0_generator
0001:00774390  _EC_GROUP_get_order
0001:007743c6  _EC_GROUP_get_cofactor
0001:007743fc  _EC_GROUP_set_curve_name
0001:0077440a  _EC_GROUP_get_curve_name
0001:00774415  _EC_GROUP_set_asn1_flag
0001:00774423  _EC_GROUP_get_asn1_flag
0001:0077442e  _EC_GROUP_set_point_conversion_form
0001:0077443c  _EC_GROUP_get_point_conversion_form
0001:00774447  _EC_GROUP_set_seed
0001:007744ea  _EC_GROUP_get0_seed
0001:007744f5  _EC_GROUP_get_seed_len
0001:00774500  _EC_GROUP_set_curve_GFp
0001:00774573  _EC_GROUP_get_curve_GFp
0001:007745e6  _EC_GROUP_set_curve_GF2m
0001:00774659  _EC_GROUP_get_curve_GF2m
0001:007746cc  _EC_GROUP_get_degree
0001:00774723* _EC_GROUP_check_discriminant
0001:00774781  _EC_GROUP_cmp
0001:00775bad  _EC_POINT_cmp
0001:00774bac  _EC_EX_DATA_get_data
0001:00774bf8  _EC_EX_DATA_free_data
0001:00774c7f* _EC_EX_DATA_clear_free_data
0001:0077500e  _EC_POINT_dup
0001:0077506e* _EC_POINT_method_of
0001:00775078  _EC_POINT_set_to_infinity
0001:00775117  _EC_POINT_set_Jprojective_coordinates_GFp
0001:007751d2* _EC_POINT_get_Jprojective_coordinates_GFp
0001:0077528d  _EC_POINT_set_affine_coordinates_GFp
0001:00775341  _EC_POINT_set_affine_coordinates_GF2m
0001:007753f5  _EC_POINT_get_affine_coordinates_GFp
0001:007754a9  _EC_POINT_get_affine_coordinates_GF2m
0001:0077555d  _EC_POINT_set_compressed_coordinates_GFp
0001:00775611  _EC_POINT_set_compressed_coordinates_GF2m
0001:007756c5  _EC_POINT_point2oct
0001:00775780  _EC_POINT_oct2point
0001:00775834  _EC_POINT_add
0001:00775907  _EC_POINT_dbl
0001:007759c2  _EC_POINT_invert
0001:00775a68  _EC_POINT_is_at_infinity
0001:00775b07  _EC_POINT_is_on_curve
0001:00775c68  _EC_POINT_make_affine
0001:00775d0e  _EC_POINTs_make_affine
0001:00775dda* _EC_POINTs_mul
0001:00775e5f  _EC_POINT_mul
0001:00775ebd  _EC_GROUP_precompute_mult
0001:00775f0f  _EC_GROUP_have_precompute_mult
Module: U:\extras\lib\libcrypto.lib(rsa_sign.obj)
0001:00775f6b  _RSA_sign
0001:0077627d  _int_rsa_verify
0001:007766f7  _RSA_verify
Module: U:\extras\lib\libcrypto.lib(m_dss1.obj)
0001:0077683c  _EVP_dss1
Module: U:\extras\lib\libcrypto.lib(p_verify.obj)
0001:0077685b  _EVP_VerifyFinal
Module: U:\extras\lib\libcrypto.lib(m_ecdsa.obj)
0001:00776b2c  _EVP_ecdsa
Module: U:\extras\lib\libcrypto.lib(ech_key.obj)
0001:00776b40  _ECDH_compute_key
Module: U:\extras\lib\libcrypto.lib(pmeth_fn.obj)
0001:00776b9b  _EVP_PKEY_sign_init
0001:00776c34  _EVP_PKEY_sign
0001:00776d6c  _EVP_PKEY_verify_init
0001:00776e05  _EVP_PKEY_verify
0001:00776ec5* _EVP_PKEY_verify_recover_init
0001:00776f5e* _EVP_PKEY_verify_recover
0001:00777096  _EVP_PKEY_encrypt_init
0001:0077712f  _EVP_PKEY_encrypt
0001:00777269  _EVP_PKEY_decrypt_init
0001:00777302  _EVP_PKEY_decrypt
0001:0077743c* _EVP_PKEY_derive_init
0001:007774d5  _EVP_PKEY_derive_set_peer
0001:0077776f* _EVP_PKEY_derive
Module: U:\extras\lib\libcrypto.lib(dsa_sign.obj)
0001:007778a0* _DSA_do_sign
0001:007778c7  _DSA_sign
0001:0077793c  _DSA_sign_setup
Module: U:\extras\lib\libcrypto.lib(ecs_sign.obj)
0001:00777970* _ECDSA_do_sign
0001:007779a1* _ECDSA_do_sign_ex
0001:007779f1  _ECDSA_sign
0001:00777a37* _ECDSA_sign_ex
0001:00777aba  _ECDSA_sign_setup
Module: U:\extras\lib\libcrypto.lib(x509type.obj)
0001:00777b10  _X509_certificate_type
Module: U:\extras\lib\libcrypto.lib(bss_mem.obj)
0001:00777c4e  _BIO_s_mem
0001:00777c62  _BIO_new_mem_buf
Module: U:\extras\lib\libcrypto.lib(rsa_asn1.obj)
0001:007783f0  _RSAPrivateKey_it
0001:00778460  _RSAPublicKey_it
0001:0077847c  _d2i_RSAPrivateKey
0001:007784a5  _i2d_RSAPrivateKey
0001:007784c7  _d2i_RSAPublicKey
0001:007784f0  _i2d_RSAPublicKey
0001:00778512* _RSAPublicKey_dup
0001:0077852d  _RSAPrivateKey_dup
Module: U:\extras\lib\libssl.lib(t1_enc.obj)
0001:00778c88  _tls1_change_cipher_state
0001:007794e8  _tls1_setup_key_block
0001:007797b8  _tls1_enc
0001:00779b94  _tls1_cert_verify_mac
0001:00779cbb  _tls1_final_finish_mac
0001:00779ed3  _tls1_mac
0001:0077a191  _tls1_generate_master_secret
0001:0077a261  _tls1_alert_code
Module: U:\extras\lib\libssl.lib(t1_reneg.obj)
0001:0077a55b  _ssl_add_clienthello_renegotiate_ext
0001:0077a613  _ssl_parse_clienthello_renegotiate_ext
0001:0077a78c  _ssl_add_serverhello_renegotiate_ext
0001:0077a929  _ssl_parse_serverhello_renegotiate_ext
Module: U:\extras\lib\libcrypto.lib(hmac.obj)
0001:0077abf9  _HMAC_Init_ex
0001:0077aeb3* _HMAC_Init
0001:0077afb8  _HMAC_CTX_init
0001:0077aefa  _HMAC_Update
0001:0077af1e  _HMAC_Final
0001:0077afea  _HMAC_CTX_copy
0001:0077b08f  _HMAC_CTX_cleanup
0001:0077b0dc  _HMAC
0001:0077b188* _HMAC_CTX_set_flags
Module: U:\extras\lib\libcrypto.lib(e_aes.obj)
0001:0077b464  _EVP_aes_128_cbc
0001:0077b4a4* _EVP_aes_128_cfb128
0001:0077b4e4* _EVP_aes_128_ofb
0001:0077b524* _EVP_aes_128_ecb
0001:0077b7c4* _EVP_aes_192_cbc
0001:0077b804* _EVP_aes_192_cfb128
0001:0077b844* _EVP_aes_192_ofb
0001:0077b884* _EVP_aes_192_ecb
0001:0077bb24* _EVP_aes_256_cbc
0001:0077bb64* _EVP_aes_256_cfb128
0001:0077bba4* _EVP_aes_256_ofb
0001:0077bbe4* _EVP_aes_256_ecb
0001:0077bce4* _EVP_aes_128_cfb1
0001:0077bde4* _EVP_aes_192_cfb1
0001:0077bee4* _EVP_aes_256_cfb1
0001:0077bfc4* _EVP_aes_128_cfb8
0001:0077c0a4* _EVP_aes_192_cfb8
0001:0077c184* _EVP_aes_256_cfb8
Module: U:\extras\lib\xmlrpc.lib(encodings.obj)
0001:0077c39c  _utf8_decode
0001:0077c3be* _utf8_encode
Module: U:\extras\lib\expat.lib(xmlparse.obj)
0001:0077c413* _XML_UseParserAsHandlerArg
0001:0077c41e* _XML_UseForeignDTD
0001:0077c448* _XML_SetReturnNSTriplet
0001:0077c46c  _XML_SetUserData
0001:0077c487* _XML_GetBase
0001:0077c495* _XML_GetSpecifiedAttributeCount
0001:0077c4a3* _XML_GetIdAttributeIndex
0001:0077c4b1  _XML_SetElementHandler
0001:0077c4c5* _XML_SetStartElementHandler
0001:0077c4d3* _XML_SetEndElementHandler
0001:0077c4e1  _XML_SetCharacterDataHandler
0001:0077c4ef* _XML_SetProcessingInstructionHandler
0001:0077c4fd* _XML_SetCommentHandler
0001:0077c50b* _XML_SetCdataSectionHandler
0001:0077c51f* _XML_SetStartCdataSectionHandler
0001:0077c52d* _XML_SetEndCdataSectionHandler
0001:0077c53b* _XML_SetDefaultHandler
0001:0077c550* _XML_SetDefaultHandlerExpand
0001:0077c565* _XML_SetDoctypeDeclHandler
0001:0077c579* _XML_SetStartDoctypeDeclHandler
0001:0077c587* _XML_SetEndDoctypeDeclHandler
0001:0077c595* _XML_SetUnparsedEntityDeclHandler
0001:0077c5a3* _XML_SetNotationDeclHandler
0001:0077c5b1* _XML_SetNamespaceDeclHandler
0001:0077c5c5* _XML_SetStartNamespaceDeclHandler
0001:0077c5d3* _XML_SetEndNamespaceDeclHandler
0001:0077c5e1* _XML_SetNotStandaloneHandler
0001:0077c5ef* _XML_SetExternalEntityRefHandler
0001:0077c5fd* _XML_SetExternalEntityRefHandlerArg
0001:0077c614* _XML_SetSkippedEntityHandler
0001:0077c622* _XML_SetUnknownEncodingHandler
0001:0077c639* _XML_SetElementDeclHandler
0001:0077c64a* _XML_SetAttlistDeclHandler
0001:0077c65b* _XML_SetEntityDeclHandler
0001:0077c66c* _XML_SetXmlDeclHandler
0001:0077c67d* _XML_SetParamEntityParsing
0001:0077c6a7* _XML_ParseBuffer
0001:0077c7d8* _XML_StopParser
0001:0077c84f* _XML_ResumeParser
0001:0077c938  _XML_GetErrorCode
0001:0077c946  _XML_GetCurrentByteIndex
0001:0077c965  _XML_GetCurrentByteCount
0001:0077c987* _XML_GetInputContext
0001:0077c9b8  _XML_GetCurrentLineNumber
0001:0077ca11  _XML_GetCurrentColumnNumber
0001:0077ca67* _XML_FreeContentModel
0001:0077ca7c* _XML_MemMalloc
0001:0077ca91* _XML_MemRealloc
0001:0077caac* _XML_MemFree
0001:0077cac1  _XML_ErrorString
0001:0077cae6* _XML_ExpatVersion
0001:0077caf0* _XML_ExpatVersionInfo
0001:0077cb0e* _XML_GetFeatureList
0001:0077cc06* _XML_DefaultCurrent
0001:0077d3c9  _XML_ParserFree
0001:0077d81a* _XML_GetParsingStatus
0001:0077d860* _XML_GetBuffer
0001:0077d9e2  _XML_Parse
0001:0077dd35* _XML_SetBase
0001:0077dd7f* _XML_SetEncoding
0001:0077f7ea* _XML_ExternalEntityParserCreate
0001:0077fe0d* _XML_ParserReset
0001:00780161* _XML_ParserCreate_MM
0001:007801ae* _XML_ParserCreateNS
0001:007801d6  _XML_ParserCreate
Module: U:\extras\lib\xmlrpc.lib(base64.obj)
0001:00785990  _buffer_delete
0001:007859c5* _buffer_add
0001:00785a16* _buffer_new
0001:00785a48  _base64_decode
0001:00785bd2  _base64_encode
Module: U:\extras\lib\pthread.lib(my_os2tls.obj)
0002:00022430+ _tls_bits
0001:00785d60  _TlsFree
0001:00785e98* _TlsAllocThreadLocalMemory
0001:00785f50  _TlsSetValue
0001:00785fb8  _TlsGetValue
0001:00786070  _TlsAlloc
0001:007861fc* _TlsFreeThreadLocalMemory
0002:0001fc64* _tls_mutex
0002:0001fc60* _tls_storage
Module: U:\extras\lib\libcrypto.lib(evp_key.obj)
0001:00786290* _EVP_set_pw_prompt
0001:007862c9  _EVP_get_pw_prompt
0001:007862e3* _EVP_read_pw_string
0001:00786313  _EVP_read_pw_string_min
0001:00786436  _EVP_BytesToKey
Module: U:\extras\lib\libcrypto.lib(encode.obj)
0001:00786750  _EVP_EncodeInit
0001:007867a7  _EVP_EncodeUpdate
0001:007869ce  _EVP_EncodeBlock
0001:00786969  _EVP_EncodeFinal
0001:00786b12  _EVP_DecodeInit
0001:00786b5f  _EVP_DecodeUpdate
0001:00786e09  _EVP_DecodeBlock
0001:00786f85  _EVP_DecodeFinal
Module: U:\extras\lib\libcrypto.lib(rsa_ameth.obj)
0001:00787a00  _rsa_asn1_meths
Module: U:\extras\lib\libcrypto.lib(dh_ameth.obj)
0001:00788847* _DHparams_print
0001:007888a0  _dh_asn1_meth
Module: U:\extras\lib\libcrypto.lib(dsa_ameth.obj)
0001:00789bc0  _dsa_asn1_meths
Module: U:\extras\lib\libcrypto.lib(ec_ameth.obj)
0001:0078b110  _eckey_asn1_meth
Module: U:\extras\lib\libcrypto.lib(hm_ameth.obj)
0001:0078b300  _hmac_asn1_meth
Module: U:\extras\lib\libcrypto.lib(tb_asnmth.obj)
0001:0078b360* _ENGINE_unregister_pkey_asn1_meths
0001:0078b38f* _ENGINE_register_pkey_asn1_meths
0001:0078b407* _ENGINE_register_all_pkey_asn1_meths
0001:0078b438* _ENGINE_set_default_pkey_asn1_meths
0001:0078b4b0  _ENGINE_get_pkey_asn1_meth_engine
0001:0078b4d7  _ENGINE_get_pkey_asn1_meth
0001:0078b54e* _ENGINE_get_pkey_asn1_meths
0001:0078b559* _ENGINE_set_pkey_asn1_meths
0001:0078b56c  _engine_pkey_asn1_meths_free
0001:0078b5f7* _ENGINE_get_pkey_asn1_meth_str
0001:0078b79e  _ENGINE_pkey_asn1_find_str
Module: U:\extras\lib\libcrypto.lib(evp_asn1.obj)
0001:0078b840  _ASN1_TYPE_set_octetstring
0001:0078b8b2  _ASN1_TYPE_get_octetstring
0001:0078b94a* _ASN1_TYPE_set_int_octetstring
0001:0078bab7* _ASN1_TYPE_get_int_octetstring
Module: U:\extras\lib\libcrypto.lib(pcy_tree.obj)
0001:0078ca2f  _X509_policy_tree_free
0001:0078cb14  _X509_policy_check
Module: U:\extras\lib\libcrypto.lib(a_utctm.obj)
0001:0078ccd0  _ASN1_UTCTIME_check
0001:0078cf18* _ASN1_UTCTIME_set_string
0001:0078cf8a* _ASN1_UTCTIME_set
0001:0078cfd8  _ASN1_UTCTIME_adj
0001:0078d1ab* _ASN1_UTCTIME_cmp_time_t
Module: U:\extras\lib\libcrypto.lib(a_gentm.obj)
0001:0078d5f0  _ASN1_GENERALIZEDTIME_check
0001:0078d890* _ASN1_GENERALIZEDTIME_set_string
0001:0078d902* _ASN1_GENERALIZEDTIME_set
0001:0078d950  _ASN1_GENERALIZEDTIME_adj
Module: U:\extras\lib\libcrypto.lib(a_time.obj)
0001:0078db70  _ASN1_TIME_it
0001:0078db8c* _d2i_ASN1_TIME
0001:0078dbb5* _i2d_ASN1_TIME
0001:0078dbd7* _ASN1_TIME_new
0001:0078dbeb  _ASN1_TIME_free
0001:0078dc06* _ASN1_TIME_set
0001:0078dc39  _ASN1_TIME_adj
0001:0078dd1c  _ASN1_TIME_check
0001:0078dd5f* _ASN1_TIME_to_generalizedtime
0001:0078de9d* _ASN1_TIME_set_string
Module: U:\extras\lib\libcrypto.lib(x_bignum.obj)
0001:0078df30  _BIGNUM_it
0001:0078df50  _CBIGNUM_it
Module: U:\extras\lib\libcrypto.lib(x_long.obj)
0001:0078e0e0  _LONG_it
0001:0078e110  _ZLONG_it
Module: U:\extras\lib\libcrypto.lib(bn_rand.obj)
0001:0078e642  _BN_rand
0001:0078e672  _BN_pseudo_rand
0001:0078e6a2* _BN_bntest_rand
0001:0078e930  _BN_rand_range
0001:0078e952  _BN_pseudo_rand_range
Module: U:\extras\lib\libcrypto.lib(tasn_utl.obj)
0001:0078e980  _asn1_get_choice_selector
0001:0078e9a0  _asn1_set_choice_selector
0001:0078e9d9  _asn1_do_lock
0001:0078eac9  _asn1_enc_init
0001:0078eb09  _asn1_enc_free
0001:0078eb5f  _asn1_enc_save
0001:0078ec04  _asn1_enc_restore
0001:0078ec88  _asn1_get_field_ptr
0001:0078ecb9  _asn1_do_adb
Module: U:\extras\lib\libcrypto.lib(a_type.obj)
0001:0078edd0  _ASN1_TYPE_get
0001:0078edf5  _ASN1_TYPE_set
0001:0078ee51  _ASN1_TYPE_set1
0001:0078eefb  _ASN1_TYPE_cmp
Module: U:\extras\lib\libcrypto.lib(a_bitstr.obj)
0001:0078ef90  _ASN1_BIT_STRING_set
0001:0078efb1  _i2c_ASN1_BIT_STRING
0001:0078f171  _c2i_ASN1_BIT_STRING
0001:0078f33a  _ASN1_BIT_STRING_set_bit
0001:0078f51c  _ASN1_BIT_STRING_get_bit
0001:0078f591* _ASN1_BIT_STRING_check
Module: U:\extras\lib\libcrypto.lib(v3_alt.obj)
0001:0078f610  _v3_alt
0001:0078f6b8  _i2v_GENERAL_NAMES
0001:0078f795  _i2v_GENERAL_NAME
0001:0078fb41  _GENERAL_NAME_print
0001:007904e1  _v2i_GENERAL_NAME
0001:0079040a  _v2i_GENERAL_NAMES
0001:00790891  _v2i_GENERAL_NAME_ex
0001:00790519* _a2i_GENERAL_NAME
Module: U:\extras\lib\libcrypto.lib(a_utf8.obj)
0001:00790c70  _UTF8_getc
0001:00791120  _UTF8_putc
Module: U:\extras\lib\libcrypto.lib(asn1_par.obj)
0001:0079218b  _ASN1_tag2str
0001:0079157e* _ASN1_parse
0001:007915be  _ASN1_parse_dump
Module: U:\extras\lib\libcrypto.lib(x509name.obj)
0001:007923a0* _X509_NAME_get_text_by_NID
0001:007923e3* _X509_NAME_get_text_by_OBJ
0001:007924d7* _X509_NAME_get_index_by_OBJ
0001:00792556  _X509_NAME_get_entry
0001:00792d0c  _X509_NAME_ENTRY_get_data
0001:00792479  _X509_NAME_entry_count
0001:0079249b  _X509_NAME_get_index_by_NID
0001:00792597  _X509_NAME_delete_entry
0001:00792686* _X509_NAME_add_entry_by_OBJ
0001:00792ae0* _X509_NAME_ENTRY_create_by_OBJ
0001:007927e4  _X509_NAME_add_entry
0001:007926f7* _X509_NAME_add_entry_by_NID
0001:00792a59* _X509_NAME_ENTRY_create_by_NID
0001:00792768  _X509_NAME_add_entry_by_txt
0001:007929af* _X509_NAME_ENTRY_create_by_txt
0001:00792b91* _X509_NAME_ENTRY_set_object
0001:00792c02* _X509_NAME_ENTRY_set_data
0001:00792cf5  _X509_NAME_ENTRY_get_object
Module: U:\extras\lib\libcrypto.lib(t_x509.obj)
0001:00792d30* _X509_print_fp
0001:00792d63* _X509_print_ex_fp
0001:00792fa1* _X509_print_ex
0001:00792e07* _X509_print
0001:00793aa9* _ASN1_TIME_print
0001:00793884* _X509_signature_print
0001:00793674* _X509_ocspid_print
0001:007939a7  _ASN1_STRING_print
0001:00793edd  _ASN1_UTCTIME_print
0001:00793b63  _ASN1_GENERALIZEDTIME_print
0001:00794175  _X509_NAME_print
Module: U:\extras\lib\libcrypto.lib(a_mbstr.obj)
0001:007942f0  _ASN1_mbstring_copy
0001:0079434f  _ASN1_mbstring_ncopy
Module: U:\extras\lib\libcrypto.lib(md5_dgst.obj)
0001:00794d10  _MD5_Update
0001:007950b5* _md5_block_data_order
0001:00794ec7* _MD5_Transform
0001:00794ee9  _MD5_Final
0001:00795040* _MD5_version
0001:00795066  _MD5_Init
Module: U:\extras\lib\libcrypto.lib(sha1dgst.obj)
0001:00795c20* _SHA1_version
0001:00795c47  _SHA1_Update
0001:00795dfe* _SHA1_Transform
0001:00795e20  _SHA1_Final
0001:00796001  _SHA1_Init
Module: U:\extras\lib\libcrypto.lib(sha256.obj)
0001:00798690* _SHA256_version
0001:007986ba  _SHA224_Init
0001:0079873b  _SHA256_Init
0001:007987bc* _SHA224
0001:007988bf  _SHA256_Update
0001:00798a98  _SHA256_Final
0001:00798820* _SHA256
0001:00798884* _SHA224_Update
0001:007988a5* _SHA224_Final
0001:00798a76* _SHA256_Transform
Module: U:\extras\lib\libcrypto.lib(sha512.obj)
0001:0079b0f0* _SHA512_version
0001:0079b11a  _SHA384_Init
0001:0079b1e7  _SHA512_Init
0001:0079b2b4  _SHA512_Final
0001:0079b6c6* _SHA384_Final
0001:0079b6e0  _SHA512_Update
0001:0079b899* _SHA384_Update
0001:0079b8ba* _SHA512_Transform
0001:0079b8dc* _SHA384
0001:0079b94c* _SHA512
Module: U:\extras\lib\libcrypto.lib(a_enum.obj)
0001:0079c5b9* _ASN1_ENUMERATED_set
0001:0079c6fc  _ASN1_ENUMERATED_get
0001:0079c7a6* _BN_to_ASN1_ENUMERATED
0001:0079c8fc  _ASN1_ENUMERATED_to_BN
Module: U:\extras\lib\libcrypto.lib(a_verify.obj)
0001:0079c98b* _ASN1_verify
0001:0079cb51  _ASN1_item_verify
Module: U:\extras\lib\libcrypto.lib(p5_crpt.obj)
0001:0079cdc0* _PKCS5_PBE_add
0001:0079ce2b  _PKCS5_PBE_keyivgen
Module: U:\extras\lib\libcrypto.lib(p12_crpt.obj)
0001:0079d1a0* _PKCS12_PBE_add
0001:0079d1b0  _PKCS12_PBE_keyivgen
Module: U:\extras\lib\libcrypto.lib(p5_crpt2.obj)
0001:0079d440* _PKCS5_PBKDF2_HMAC
0001:0079d62e* _PKCS5_PBKDF2_HMAC_SHA1
0001:0079d694  _PKCS5_v2_PBE_keyivgen
Module: U:\extras\lib\libcrypto.lib(eng_table.obj)
0001:0079dbd0* _ENGINE_get_table_flags
0001:0079dbda* _ENGINE_set_table_flags
0001:0079dca7  _engine_table_register
0001:0079df68  _engine_table_unregister
0001:0079e045  _engine_table_cleanup
0001:0079e0c9  _engine_table_select
0001:0079e2eb  _engine_table_doall
Module: U:\extras\lib\libcrypto.lib(eng_list.obj)
0001:0079e992* _ENGINE_remove
0001:0079e623  _ENGINE_get_first
0001:0079e693* _ENGINE_get_last
0001:0079e703  _ENGINE_get_next
0001:0079e7bf* _ENGINE_get_prev
0001:0079e87b* _ENGINE_add
0001:0079eba8* _ENGINE_by_id
0001:0079ee13* _ENGINE_up_ref
Module: U:\extras\lib\libcrypto.lib(rand_os2.obj)
0001:0079eeab  _RAND_poll
Module: U:\extras\lib\libcrypto.lib(v3_conf.obj)
0001:0079f2bb* _X509V3_EXT_nconf
0001:0079f3a7* _X509V3_EXT_nconf_nid
0001:0079f869  _X509V3_EXT_i2d
0001:0079fc47* _X509V3_EXT_add_nconf_sk
0001:0079fd0f* _X509V3_EXT_add_nconf
0001:0079fd4f* _X509V3_EXT_CRL_add_nconf
0001:0079fd8f* _X509V3_EXT_REQ_add_nconf
0001:0079fe11* _X509V3_get_string
0001:0079fea0  _X509V3_get_section
0001:0079ff2b* _X509V3_string_free
0001:0079ff64  _X509V3_section_free
0001:0079ffd8  _X509V3_set_nconf
0001:0079fff0* _X509V3_set_ctx
0001:007a0021* _X509V3_EXT_conf
0001:007a005b* _X509V3_EXT_conf_nid
0001:007a00d0* _X509V3_set_conf_lhash
0001:007a00e8* _X509V3_EXT_add_conf
0001:007a0122* _X509V3_EXT_CRL_add_conf
0001:007a015c* _X509V3_EXT_REQ_add_conf
Module: U:\extras\lib\libcrypto.lib(v3_utl.obj)
0001:007a022b  _X509V3_add_value
0001:007a0372  _X509V3_add_value_uchar
0001:007a0393  _X509V3_conf_free
0001:007a0400  _X509V3_add_value_bool
0001:007a0444* _X509V3_add_value_bool_nf
0001:007a0473  _i2s_ASN1_ENUMERATED
0001:007a0500  _i2s_ASN1_INTEGER
0001:007a058d  _s2i_ASN1_INTEGER
0001:007a073d  _X509V3_add_value_int
0001:007a07d8  _X509V3_get_value_bool
0001:007a099d  _X509V3_get_value_int
0001:007a0a19  _X509V3_parse_list
0001:007a0d88  _hex_to_string
0001:007a0e6f  _string_to_hex
0001:007a10c3  _name_cmp
0001:007a1141* _X509_get1_email
0001:007a11a3* _X509_get1_ocsp
0001:007a1264* _X509_REQ_get1_email
0001:007a14b0* _X509_email_free
0001:007a14cc  _a2i_IPADDRESS
0001:007a166b* _a2i_ipadd
0001:007a153d  _a2i_IPADDRESS_NC
0001:007a1aff  _X509V3_NAME_from_section
Module: U:\extras\lib\libcrypto.lib(pcy_data.obj)
0001:007a1c30  _policy_data_free
0001:007a1c96  _policy_data_new
Module: U:\extras\lib\libcrypto.lib(v3_cpols.obj)
0001:007a1dc0  _v3_cpols
0001:007a1e30* _CERTIFICATEPOLICIES_it
0001:007a1f20* _POLICYINFO_it
0001:007a1e4c* _d2i_CERTIFICATEPOLICIES
0001:007a1e75* _i2d_CERTIFICATEPOLICIES
0001:007a1e97* _CERTIFICATEPOLICIES_new
0001:007a1eab* _CERTIFICATEPOLICIES_free
0001:007a2090* _POLICYQUALINFO_it
0001:007a1f3c* _d2i_POLICYINFO
0001:007a1f65* _i2d_POLICYINFO
0001:007a1f87* _POLICYINFO_new
0001:007a1f9b  _POLICYINFO_free
0001:007a2180* _USERNOTICE_it
0001:007a20ac* _d2i_POLICYQUALINFO
0001:007a20d5* _i2d_POLICYQUALINFO
0001:007a20f7* _POLICYQUALINFO_new
0001:007a210b  _POLICYQUALINFO_free
0001:007a2270* _NOTICEREF_it
0001:007a219c* _d2i_USERNOTICE
0001:007a21c5* _i2d_USERNOTICE
0001:007a21e7* _USERNOTICE_new
0001:007a21fb* _USERNOTICE_free
0001:007a228c* _d2i_NOTICEREF
0001:007a22b5* _i2d_NOTICEREF
0001:007a22d7* _NOTICEREF_new
0001:007a22eb* _NOTICEREF_free
0001:007a33dd* _X509_POLICY_NODE_print
Module: U:\extras\lib\libcrypto.lib(pcy_map.obj)
0001:007a34d0  _policy_cache_set_mapping
Module: U:\extras\lib\libcrypto.lib(v3_pcons.obj)
0001:007a36a0  _v3_policy_constraints
0001:007a3750* _POLICY_CONSTRAINTS_it
0001:007a376c* _POLICY_CONSTRAINTS_new
0001:007a3780  _POLICY_CONSTRAINTS_free
Module: U:\extras\lib\libcrypto.lib(tb_pkmeth.obj)
0001:007a3a00* _ENGINE_unregister_pkey_meths
0001:007a3a2f* _ENGINE_register_pkey_meths
0001:007a3aa7* _ENGINE_register_all_pkey_meths
0001:007a3ad8* _ENGINE_set_default_pkey_meths
0001:007a3b50  _ENGINE_get_pkey_meth_engine
0001:007a3b77  _ENGINE_get_pkey_meth
0001:007a3bee* _ENGINE_get_pkey_meths
0001:007a3bf9* _ENGINE_set_pkey_meths
0001:007a3c0c  _engine_pkey_meths_free
Module: U:\extras\lib\libcrypto.lib(bn_exp.obj)
0001:007a3ca9* _BN_exp
0001:007a3e66  _BN_mod_exp
0001:007a50c9  _BN_mod_exp_mont_word
0001:007a440d  _BN_mod_exp_mont
0001:007a3f50* _BN_mod_exp_recp
0001:007a4b4f* _BN_mod_exp_mont_consttime
0001:007a55ef* _BN_mod_exp_simple
Module: U:\extras\lib\libcrypto.lib(rsa_pk1.obj)
0001:007a5a0a  _RSA_padding_add_PKCS1_type_1
0001:007a5abb  _RSA_padding_check_PKCS1_type_1
0001:007a5c5b  _RSA_padding_add_PKCS1_type_2
0001:007a5d53  _RSA_padding_check_PKCS1_type_2
Module: U:\extras\lib\libcrypto.lib(rsa_oaep.obj)
0001:007a5ecb  _RSA_padding_add_PKCS1_OAEP
0001:007a6156  _RSA_padding_check_PKCS1_OAEP
0001:007a6469  _PKCS1_MGF1
Module: U:\extras\lib\libcrypto.lib(rsa_ssl.obj)
0001:007a65fa  _RSA_padding_add_SSLv23
0001:007a6714  _RSA_padding_check_SSLv23
Module: U:\extras\lib\libcrypto.lib(rsa_none.obj)
0001:007a68eb  _RSA_padding_add_none
0001:007a6987  _RSA_padding_check_none
Module: U:\extras\lib\libcrypto.lib(bn_mont.obj)
0001:007a6a20  _BN_mod_mul_montgomery
0001:007a6fb0  _BN_from_montgomery
0001:007a7028  _BN_MONT_CTX_new
0001:007a7074* _BN_MONT_CTX_init
0001:007a70cf  _BN_MONT_CTX_free
0001:007a7122  _BN_MONT_CTX_set
0001:007a7393  _BN_MONT_CTX_copy
0001:007a7439  _BN_MONT_CTX_set_locked
Module: U:\extras\lib\libcrypto.lib(rsa_x931.obj)
0001:007a757b  _RSA_padding_add_X931
0001:007a7649  _RSA_padding_check_X931
0001:007a77d3  _RSA_X931_hash_id
Module: U:\extras\lib\libcrypto.lib(bn_div.obj)
0001:007a7839  _BN_div
Module: U:\extras\lib\libcrypto.lib(bn_mod.obj)
0001:007a85c0  _BN_nnmod
0001:007a8638  _BN_mod_add
0001:007a8684  _BN_mod_add_quick
0001:007a86e6* _BN_mod_sub
0001:007a8732  _BN_mod_sub_quick
0001:007a8788  _BN_mod_mul
0001:007a8843  _BN_mod_sqr
0001:007a8897* _BN_mod_lshift1
0001:007a88dc  _BN_mod_lshift1_quick
0001:007a8937* _BN_mod_lshift
0001:007a89eb  _BN_mod_lshift_quick
Module: U:\extras\lib\libcrypto.lib(bn_asm.obj)
0001:007a8b30  _bn_mul_add_words
0001:007a8fb2  _bn_mul_words
0001:007a93ae  _bn_sqr_words
0001:007a9605  _bn_div_words
0001:007a9792  _bn_add_words
0001:007a9944  _bn_sub_words
0001:007a9aeb  _bn_mul_comba8
0001:007aea5a  _bn_mul_comba4
0001:007afae7  _bn_sqr_comba8
0001:007b2929  _bn_sqr_comba4
Module: U:\extras\lib\libcrypto.lib(dh_check.obj)
0001:007b32b0* _DH_check
0001:007b3487  _DH_check_pub_key
Module: U:\extras\lib\libcrypto.lib(dsa_ossl.obj)
0001:007b3573  _DSA_OpenSSL
Module: U:\extras\lib\libcrypto.lib(tb_dsa.obj)
0001:007b4094* _ENGINE_unregister_DSA
0001:007b40c3* _ENGINE_register_DSA
0001:007b410f* _ENGINE_register_all_DSA
0001:007b4140* _ENGINE_set_default_DSA
0001:007b418c  _ENGINE_get_default_DSA
0001:007b41a9  _ENGINE_get_DSA
0001:007b41b4* _ENGINE_set_DSA
Module: U:\extras\lib\libcrypto.lib(v3_lib.obj)
0001:007b41d9* _X509V3_EXT_add
0001:007b42f8  _X509V3_EXT_get_nid
0001:007b438c  _X509V3_EXT_get
0001:007b43bc* _X509V3_EXT_add_list
0001:007b43ef* _X509V3_EXT_add_alias
0001:007b44db* _X509V3_EXT_cleanup
0001:007b4523* _X509V3_add_standard_extensions
0001:007b452d  _X509V3_EXT_d2i
0001:007b45b3  _X509V3_get_d2i
0001:007b46db  _X509V3_add1_i2d
Module: U:\extras\lib\libcrypto.lib(x_req.obj)
0001:007b49b0  _X509_REQ_INFO_it
0001:007b49cc* _d2i_X509_REQ_INFO
0001:007b49f5* _i2d_X509_REQ_INFO
0001:007b4a17* _X509_REQ_INFO_new
0001:007b4a2b* _X509_REQ_INFO_free
0001:007b4ae0  _X509_REQ_it
0001:007b4afc  _d2i_X509_REQ
0001:007b4b25  _i2d_X509_REQ
0001:007b4b47  _X509_REQ_new
0001:007b4b5b  _X509_REQ_free
0001:007b4b76* _X509_REQ_dup
Module: U:\extras\lib\libcrypto.lib(x_spki.obj)
0001:007b4c00  _NETSCAPE_SPKAC_it
0001:007b4c1c* _d2i_NETSCAPE_SPKAC
0001:007b4c45* _i2d_NETSCAPE_SPKAC
0001:007b4c67* _NETSCAPE_SPKAC_new
0001:007b4c7b* _NETSCAPE_SPKAC_free
0001:007b4d00* _NETSCAPE_SPKI_it
0001:007b4d1c* _d2i_NETSCAPE_SPKI
0001:007b4d45* _i2d_NETSCAPE_SPKI
0001:007b4d67* _NETSCAPE_SPKI_new
0001:007b4d7b* _NETSCAPE_SPKI_free
Module: U:\extras\lib\libcrypto.lib(a_sign.obj)
0001:007b4da9* _ASN1_sign
0001:007b5114  _ASN1_item_sign
Module: U:\extras\lib\libcrypto.lib(a_d2i_fp.obj)
0001:007b549b  _ASN1_d2i_fp
0001:007b553f  _ASN1_d2i_bio
0001:007b55ad  _ASN1_item_d2i_bio
0001:007b5622  _ASN1_item_d2i_fp
Module: U:\extras\lib\libcrypto.lib(a_i2d_fp.obj)
0001:007b5a2b  _ASN1_i2d_fp
0001:007b5ac8  _ASN1_i2d_bio
0001:007b5bb6  _ASN1_item_i2d_fp
0001:007b5c53  _ASN1_item_i2d_bio
Module: U:\extras\lib\libcrypto.lib(pk7_asn1.obj)
0001:007b60f0* _PKCS7_SIGNED_it
0001:007b64b0* _PKCS7_ENVELOPE_it
0001:007b6850* _PKCS7_SIGN_ENVELOPE_it
0001:007b6a30* _PKCS7_DIGEST_it
0001:007b6930* _PKCS7_ENCRYPT_it
0001:007b5f50  _PKCS7_it
0001:007b5f6c  _d2i_PKCS7
0001:007b5f95  _i2d_PKCS7
0001:007b5fb7  _PKCS7_new
0001:007b5fcb  _PKCS7_free
0001:007b5fe6* _i2d_PKCS7_NDEF
0001:007b6008* _PKCS7_dup
0001:007b62c0* _PKCS7_SIGNER_INFO_it
0001:007b610c* _d2i_PKCS7_SIGNED
0001:007b6135* _i2d_PKCS7_SIGNED
0001:007b6157  _PKCS7_SIGNED_new
0001:007b616b  _PKCS7_SIGNED_free
0001:007b63b0  _PKCS7_ISSUER_AND_SERIAL_it
0001:007b62dc* _d2i_PKCS7_SIGNER_INFO
0001:007b6305* _i2d_PKCS7_SIGNER_INFO
0001:007b6327  _PKCS7_SIGNER_INFO_new
0001:007b633b  _PKCS7_SIGNER_INFO_free
0001:007b63cc* _d2i_PKCS7_ISSUER_AND_SERIAL
0001:007b63f5* _i2d_PKCS7_ISSUER_AND_SERIAL
0001:007b6417* _PKCS7_ISSUER_AND_SERIAL_new
0001:007b642b* _PKCS7_ISSUER_AND_SERIAL_free
0001:007b6610* _PKCS7_RECIP_INFO_it
0001:007b6710* _PKCS7_ENC_CONTENT_it
0001:007b64cc* _d2i_PKCS7_ENVELOPE
0001:007b64f5* _i2d_PKCS7_ENVELOPE
0001:007b6517  _PKCS7_ENVELOPE_new
0001:007b652b* _PKCS7_ENVELOPE_free
0001:007b662c* _d2i_PKCS7_RECIP_INFO
0001:007b6655* _i2d_PKCS7_RECIP_INFO
0001:007b6677  _PKCS7_RECIP_INFO_new
0001:007b668b  _PKCS7_RECIP_INFO_free
0001:007b672c* _d2i_PKCS7_ENC_CONTENT
0001:007b6755* _i2d_PKCS7_ENC_CONTENT
0001:007b6777* _PKCS7_ENC_CONTENT_new
0001:007b678b* _PKCS7_ENC_CONTENT_free
0001:007b686c* _d2i_PKCS7_SIGN_ENVELOPE
0001:007b6895* _i2d_PKCS7_SIGN_ENVELOPE
0001:007b68b7  _PKCS7_SIGN_ENVELOPE_new
0001:007b68cb* _PKCS7_SIGN_ENVELOPE_free
0001:007b694c* _d2i_PKCS7_ENCRYPT
0001:007b6975* _i2d_PKCS7_ENCRYPT
0001:007b6997  _PKCS7_ENCRYPT_new
0001:007b69ab* _PKCS7_ENCRYPT_free
0001:007b6a4c* _d2i_PKCS7_DIGEST
0001:007b6a75* _i2d_PKCS7_DIGEST
0001:007b6a97  _PKCS7_DIGEST_new
0001:007b6aab* _PKCS7_DIGEST_free
0001:007b6b10  _PKCS7_ATTR_SIGN_it
0001:007b6b60  _PKCS7_ATTR_VERIFY_it
0001:007b6b7c* _PKCS7_print_ctx
Module: U:\extras\lib\libcrypto.lib(dsa_asn1.obj)
0001:007b6ca0* _DSA_SIG_it
0001:007b6cbc  _d2i_DSA_SIG
0001:007b6ce5  _i2d_DSA_SIG
0001:007b6d07  _DSA_SIG_new
0001:007b6d1b  _DSA_SIG_free
0001:007b6e50* _DSAPrivateKey_it
0001:007b6e6c  _d2i_DSAPrivateKey
0001:007b6e95  _i2d_DSAPrivateKey
0001:007b6f20* _DSAparams_it
0001:007b6f3c  _d2i_DSAparams
0001:007b6f65  _i2d_DSAparams
0001:007b6fe0* _dsa_pub_internal_it
0001:007b7050* _DSAPublicKey_it
0001:007b706c* _d2i_DSAPublicKey
0001:007b7095  _i2d_DSAPublicKey
0001:007b70b7* _DSAparams_dup
Module: U:\extras\lib\libcrypto.lib(ec_asn1.obj)
0001:007b70e0  _EC_GROUP_get_basis_type
0001:007b7150* _EC_GROUP_get_trinomial_basis
0001:007b71e3* _EC_GROUP_get_pentanomial_basis
0001:007b7310* _X9_62_PENTANOMIAL_it
0001:007b732c* _X9_62_PENTANOMIAL_new
0001:007b7340* _X9_62_PENTANOMIAL_free
0001:007b7480* _X9_62_CHARACTERISTIC_TWO_it
0001:007b749c* _X9_62_CHARACTERISTIC_TWO_new
0001:007b74b0* _X9_62_CHARACTERISTIC_TWO_free
0001:007b75a0* _X9_62_FIELDID_it
0001:007b7620* _X9_62_CURVE_it
0001:007b7700* _ECPARAMETERS_it
0001:007b771c* _ECPARAMETERS_new
0001:007b7730* _ECPARAMETERS_free
0001:007b77e0* _ECPKPARAMETERS_it
0001:007b77fc* _d2i_UC_ECPKPARAMETERS
0001:007b7825* _i2d_UC_ECPKPARAMETERS
0001:007b7847* _ECPKPARAMETERS_new
0001:007b785b* _ECPKPARAMETERS_free
0001:007b7900* _EC_PRIVATEKEY_it
0001:007b791c* _d2i_EC_PRIVATEKEY
0001:007b7945* _i2d_EC_PRIVATEKEY
0001:007b7967* _EC_PRIVATEKEY_new
0001:007b797b* _EC_PRIVATEKEY_free
0001:007b957c  _d2i_ECPKParameters
0001:007b9672  _i2d_ECPKParameters
0001:007b9737  _d2i_ECPrivateKey
0001:007b9aba  _i2d_ECPrivateKey
0001:007b9f64  _i2d_ECParameters
0001:007b9fba  _d2i_ECParameters
0001:007ba0c5  _o2i_ECPublicKey
0001:007ba21e  _i2o_ECPublicKey
Module: U:\extras\lib\libcrypto.lib(a_digest.obj)
0001:007ba3eb* _ASN1_digest
0001:007ba4b7  _ASN1_item_digest
Module: U:\extras\lib\libcrypto.lib(x_sig.obj)
0001:007ba580  _X509_SIG_it
0001:007ba59c  _d2i_X509_SIG
0001:007ba5c5  _i2d_X509_SIG
0001:007ba5e7  _X509_SIG_new
0001:007ba5fb  _X509_SIG_free
Module: U:\extras\lib\libcrypto.lib(p8_pkey.obj)
0001:007ba720  _PKCS8_PRIV_KEY_INFO_it
0001:007ba73c  _d2i_PKCS8_PRIV_KEY_INFO
0001:007ba765  _i2d_PKCS8_PRIV_KEY_INFO
0001:007ba787  _PKCS8_PRIV_KEY_INFO_new
0001:007ba79b  _PKCS8_PRIV_KEY_INFO_free
0001:007ba7b6  _PKCS8_pkey_set0
0001:007ba89e  _PKCS8_pkey_get0
Module: U:\extras\lib\libcrypto.lib(evp_pkey.obj)
0001:007ba971  _EVP_PKCS82PKEY
0001:007bab1d  _EVP_PKEY2PKCS8
0001:007bab38* _EVP_PKEY2PKCS8_broken
0001:007baca3* _PKCS8_set_broken
0001:007bad12* _EVP_PKEY_get_attr_count
0001:007bad28* _EVP_PKEY_get_attr_by_NID
0001:007bad4c* _EVP_PKEY_get_attr_by_OBJ
0001:007bad70* _EVP_PKEY_get_attr
0001:007bad8d* _EVP_PKEY_delete_attr
0001:007badaa* _EVP_PKEY_add1_attr
0001:007badd7* _EVP_PKEY_add1_attr_by_OBJ
0001:007bae19* _EVP_PKEY_add1_attr_by_NID
0001:007bae5b* _EVP_PKEY_add1_attr_by_txt
Module: U:\extras\lib\libcrypto.lib(i2d_pr.obj)
0001:007baea9  _i2d_PrivateKey
Module: U:\extras\lib\libcrypto.lib(d2i_pr.obj)
0001:007baf69  _d2i_PrivateKey
0001:007bb12e  _d2i_AutoPrivateKey
Module: U:\extras\lib\libcrypto.lib(x509_def.obj)
0001:007bb290* _X509_get_default_private_dir
0001:007bb2a2  _X509_get_default_cert_area
0001:007bb2ba  _X509_get_default_cert_dir
0001:007bb2d5  _X509_get_default_cert_file
0001:007bb2ec  _X509_get_default_cert_dir_env
0001:007bb304  _X509_get_default_cert_file_env
Module: U:\extras\lib\libcrypto.lib(pem_xaux.obj)
0001:007bb324  _PEM_read_bio_X509_AUX
0001:007bb35d* _PEM_read_X509_AUX
0001:007bb396* _PEM_write_bio_X509_AUX
0001:007bb3e9* _PEM_write_X509_AUX
0001:007bb44d* _PEM_read_bio_X509_CERT_PAIR
0001:007bb486* _PEM_read_X509_CERT_PAIR
0001:007bb4bf* _PEM_write_bio_X509_CERT_PAIR
0001:007bb512* _PEM_write_X509_CERT_PAIR
Module: U:\extras\lib\libcrypto.lib(pem_all.obj)
0001:007bb584* _PEM_read_bio_X509_REQ
0001:007bb5bd* _PEM_read_X509_REQ
0001:007bb5f6* _PEM_write_bio_X509_REQ
0001:007bb649* _PEM_write_X509_REQ
0001:007bb6b4* _PEM_write_bio_X509_REQ_NEW
0001:007bb707* _PEM_write_X509_REQ_NEW
0001:007bb763  _PEM_read_bio_X509_CRL
0001:007bb79c* _PEM_read_X509_CRL
0001:007bb7d5* _PEM_write_bio_X509_CRL
0001:007bb828* _PEM_write_X509_CRL
0001:007bb881* _PEM_read_bio_PKCS7
0001:007bb8ba* _PEM_read_PKCS7
0001:007bb8f3* _PEM_write_bio_PKCS7
0001:007bb946* _PEM_write_PKCS7
0001:007bb9a5* _PEM_read_bio_NETSCAPE_CERT_SEQUENCE
0001:007bb9de* _PEM_read_NETSCAPE_CERT_SEQUENCE
0001:007bba17* _PEM_write_bio_NETSCAPE_CERT_SEQUENCE
0001:007bba6a* _PEM_write_NETSCAPE_CERT_SEQUENCE
0001:007bbb16  _PEM_read_bio_RSAPrivateKey
0001:007bbb54* _PEM_read_RSAPrivateKey
0001:007bbba2  _PEM_write_bio_RSAPrivateKey
0001:007bbbf0* _PEM_write_RSAPrivateKey
0001:007bbc4d* _PEM_read_bio_RSAPublicKey
0001:007bbc86* _PEM_read_RSAPublicKey
0001:007bbcbf* _PEM_write_bio_RSAPublicKey
0001:007bbd12* _PEM_write_RSAPublicKey
0001:007bbd70* _PEM_read_bio_RSA_PUBKEY
0001:007bbda9* _PEM_read_RSA_PUBKEY
0001:007bbde2* _PEM_write_bio_RSA_PUBKEY
0001:007bbe35* _PEM_write_RSA_PUBKEY
0001:007bbee1* _PEM_read_bio_DSAPrivateKey
0001:007bbf2f* _PEM_write_bio_DSAPrivateKey
0001:007bbf7d* _PEM_write_DSAPrivateKey
0001:007bbfcb* _PEM_read_bio_DSA_PUBKEY
0001:007bc004* _PEM_read_DSA_PUBKEY
0001:007bc03d* _PEM_write_bio_DSA_PUBKEY
0001:007bc090* _PEM_write_DSA_PUBKEY
0001:007bc0e3* _PEM_read_DSAPrivateKey
0001:007bc130* _PEM_read_bio_DSAparams
0001:007bc169* _PEM_read_DSAparams
0001:007bc1a2* _PEM_write_bio_DSAparams
0001:007bc1f5* _PEM_write_DSAparams
0001:007bc2a1* _PEM_read_bio_ECPrivateKey
0001:007bc2ed* _PEM_read_bio_ECPKParameters
0001:007bc326* _PEM_read_ECPKParameters
0001:007bc35f* _PEM_write_bio_ECPKParameters
0001:007bc3b2* _PEM_write_ECPKParameters
0001:007bc414* _PEM_write_bio_ECPrivateKey
0001:007bc462* _PEM_write_ECPrivateKey
0001:007bc4b0* _PEM_read_bio_EC_PUBKEY
0001:007bc4e9* _PEM_read_EC_PUBKEY
0001:007bc522* _PEM_write_bio_EC_PUBKEY
0001:007bc575* _PEM_write_EC_PUBKEY
0001:007bc5c8* _PEM_read_ECPrivateKey
0001:007bc614* _PEM_read_bio_DHparams
0001:007bc64d* _PEM_read_DHparams
0001:007bc686* _PEM_write_bio_DHparams
0001:007bc6d9* _PEM_write_DHparams
0001:007bc72c* _PEM_read_bio_PUBKEY
0001:007bc765* _PEM_read_PUBKEY
0001:007bc79e* _PEM_write_bio_PUBKEY
0001:007bc7f1* _PEM_write_PUBKEY
Module: U:\extras\lib\libcrypto.lib(pem_info.obj)
0001:007bc85b* _PEM_X509_INFO_read
0001:007bc968  _PEM_X509_INFO_read_bio
0001:007bd0ad* _PEM_X509_INFO_write_bio
Module: U:\extras\lib\libcrypto.lib(x_info.obj)
0001:007bd359  _X509_INFO_new
0001:007bd408  _X509_INFO_free
Module: U:\extras\lib\libcrypto.lib(rsa_pmeth.obj)
0001:007be590  _rsa_pkey_meth
Module: U:\extras\lib\libcrypto.lib(dh_pmeth.obj)
0001:007bea40  _dh_pkey_meth
Module: U:\extras\lib\libcrypto.lib(dsa_pmeth.obj)
0001:007bf1b0  _dsa_pkey_meth
Module: U:\extras\lib\libcrypto.lib(ec_pmeth.obj)
0001:007bf930  _ec_pkey_meth
Module: U:\extras\lib\libcrypto.lib(hm_pmeth.obj)
0001:007bfe20  _hmac_pkey_meth
Module: U:\extras\lib\libcrypto.lib(pem_pkey.obj)
0001:007bfecd  _PEM_read_bio_PrivateKey
0001:007c01f2* _PEM_write_bio_PrivateKey
0001:007c02c3* _PEM_read_bio_Parameters
0001:007c0446* _PEM_write_bio_Parameters
0001:007c04e5  _PEM_read_PrivateKey
0001:007c0589* _PEM_write_PrivateKey
Module: U:\extras\lib\libcrypto.lib(ec_cvt.obj)
0001:007c0630  _EC_GROUP_new_curve_GFp
0001:007c0743  _EC_GROUP_new_curve_GF2m
Module: U:\extras\lib\libcrypto.lib(ec_mult.obj)
0001:007c0dc2  _ec_wNAF_mul
0001:007c1b98  _ec_wNAF_precompute_mult
0001:007c21cf  _ec_wNAF_have_precompute_mult
Module: U:\extras\lib\libcrypto.lib(dsa_vrf.obj)
0001:007c2210* _DSA_do_verify
0001:007c223e  _DSA_verify
Module: U:\extras\lib\libcrypto.lib(ecs_vrf.obj)
0001:007c22c0* _ECDSA_do_verify
0001:007c2309  _ECDSA_verify
Module: U:\extras\lib\libcrypto.lib(ech_lib.obj)
0001:007c2380* _ECDH_version
0001:007c23a7* _ECDH_set_default_method
0001:007c23b4* _ECDH_get_default_method
0001:007c23d4* _ECDH_set_method
0001:007c25fe  _ecdh_check
0001:007c267c* _ECDH_get_ex_new_index
0001:007c26b3* _ECDH_set_ex_data
0001:007c26f2* _ECDH_get_ex_data
Module: U:\extras\lib\libcrypto.lib(ecs_lib.obj)
0001:007c2730* _ECDSA_version
0001:007c2758* _ECDSA_set_default_method
0001:007c2765* _ECDSA_get_default_method
0001:007c2785* _ECDSA_set_method
0001:007c29af  _ecdsa_check
0001:007c2a2d  _ECDSA_size
0001:007c2b2e* _ECDSA_get_ex_new_index
0001:007c2b65* _ECDSA_set_ex_data
0001:007c2ba4* _ECDSA_get_ex_data
Module: U:\extras\lib\libcrypto.lib(ecs_asn1.obj)
0001:007c2c30* _ECDSA_SIG_it
0001:007c2c4c  _d2i_ECDSA_SIG
0001:007c2c75  _i2d_ECDSA_SIG
0001:007c2c97  _ECDSA_SIG_new
0001:007c2cab  _ECDSA_SIG_free
Module: U:\extras\lib\libcrypto.lib(pmeth_gn.obj)
0001:007c2cdb* _EVP_PKEY_paramgen_init
0001:007c2d74* _EVP_PKEY_paramgen
0001:007c2e66* _EVP_PKEY_keygen_init
0001:007c2eff* _EVP_PKEY_keygen
0001:007c2ff1* _EVP_PKEY_CTX_set_cb
0001:007c2fff* _EVP_PKEY_CTX_get_cb
0001:007c3042  _evp_pkey_set_cb_translate
0001:007c306c* _EVP_PKEY_CTX_get_keygen_info
0001:007c30a7  _EVP_PKEY_new_mac_key
Module: U:\extras\lib\libcrypto.lib(m_sigver.obj)
0001:007c335e  _EVP_DigestSignInit
0001:007c3395  _EVP_DigestVerifyInit
0001:007c33cc  _EVP_DigestSignFinal
0001:007c3566  _EVP_DigestVerifyFinal
Module: U:\extras\lib\libcrypto.lib(aes_cbc.obj)
0001:007c3660  _AES_cbc_encrypt
Module: U:\extras\lib\libcrypto.lib(aes_cfb.obj)
0001:007c36d0  _AES_cfb128_encrypt
0001:007c3716  _AES_cfb1_encrypt
0001:007c375c  _AES_cfb8_encrypt
Module: U:\extras\lib\libcrypto.lib(aes_ecb.obj)
0001:007c37b0  _AES_ecb_encrypt
Module: U:\extras\lib\libcrypto.lib(aes_ofb.obj)
0001:007c3800  _AES_ofb128_encrypt
Module: U:\extras\lib\libcrypto.lib(aes_core.obj)
0001:007c5968  _AES_set_encrypt_key
0001:007c6005  _AES_set_decrypt_key
0001:007c63c8  _AES_encrypt
0001:007c6a27  _AES_decrypt
Module: U:\extras\lib\expat.lib(xmlrole.obj)
0001:007c89f0  _XmlPrologStateInit
0001:007c8a13  _XmlPrologStateInitExternalEntity
Module: U:\extras\lib\expat.lib(xmltok.obj)
0001:007d7a0f  _XmlUtf8Encode
0001:007d7aaf* _XmlUtf16Encode
0001:007d7af7  _XmlSizeOfUnknownEncoding
0001:007d7d2c  _XmlInitUnknownEncoding
0001:007d8252  _XmlGetUtf8InternalEncoding
0001:007d825c* _XmlGetUtf16InternalEncoding
0001:007d82c3  _XmlInitEncoding
0001:007d83b5  _XmlParseXmlDecl
0001:007d8405  _XmlGetUtf8InternalEncodingNS
0001:007d840f* _XmlGetUtf16InternalEncodingNS
0001:007d8476  _XmlInitEncodingNS
0001:007d8568  _XmlParseXmlDeclNS
0001:007d85b8  _XmlInitUnknownEncodingNS
Module: U:\extras\lib\libcrypto.lib(ui_lib.obj)
0001:007da4c0  _UI_new
0001:007da4dd* _UI_new_method
0001:007db514* _UI_get_default_method
0001:007da5fa  _UI_free
0001:007da971  _UI_add_input_string
0001:007da9bf* _UI_dup_input_string
0001:007daa61  _UI_add_verify_string
0001:007daaae* _UI_dup_verify_string
0001:007dab4f* _UI_add_input_boolean
0001:007dab9c* _UI_dup_input_boolean
0001:007dad79* _UI_add_info_string
0001:007dadcb* _UI_dup_info_string
0001:007dae71* _UI_add_error_string
0001:007daec3* _UI_dup_error_string
0001:007daf72* _UI_construct_prompt
0001:007db0dd* _UI_add_user_data
0001:007db0fa* _UI_get0_user_data
0001:007db105* _UI_get0_result
0001:007db799  _UI_get0_result_string
0001:007db20c  _UI_process
0001:007db3bb* _UI_ctrl
0001:007db48f* _UI_get_ex_new_index
0001:007db4c6* _UI_set_ex_data
0001:007db4ea* _UI_get_ex_data
0001:007db507* _UI_set_default_method
0001:007db534* _UI_get_method
0001:007db53e* _UI_set_method
0001:007db550* _UI_create_method
0001:007db5ab* _UI_destroy_method
0001:007db5d4* _UI_method_set_opener
0001:007db5f4* _UI_method_set_writer
0001:007db614* _UI_method_set_flusher
0001:007db634* _UI_method_set_reader
0001:007db654* _UI_method_set_closer
0001:007db674* _UI_method_set_prompt_constructor
0001:007db694* _UI_method_get_opener
0001:007db6ac* _UI_method_get_writer
0001:007db6c4* _UI_method_get_flusher
0001:007db6dc* _UI_method_get_reader
0001:007db6f4* _UI_method_get_closer
0001:007db70c* _UI_method_get_prompt_constructor
0001:007db724  _UI_get_string_type
0001:007db73b  _UI_get_input_flags
0001:007db753  _UI_get0_output_string
0001:007db76b  _UI_get0_action_string
0001:007db7c3  _UI_get0_test_string
0001:007db7ec* _UI_get_result_minsize
0001:007db816* _UI_get_result_maxsize
0001:007db866  _UI_set_result
Module: U:\extras\lib\libcrypto.lib(t_pkey.obj)
0001:007dbb79  _ASN1_bn_print
Module: U:\extras\lib\libcrypto.lib(pk7_lib.obj)
0001:007dbdca  _PKCS7_ctrl
0001:007dbf4b* _PKCS7_content_new
0001:007dc071  _PKCS7_set_type
0001:007dbfb8* _PKCS7_set_content
0001:007dc30d* _PKCS7_set0_type_other
0001:007dc334* _PKCS7_add_signer
0001:007dc4fd* _PKCS7_add_certificate
0001:007dc625* _PKCS7_add_crl
0001:007dc74d* _PKCS7_SIGNER_INFO_set
0001:007dc902* _PKCS7_add_signature
0001:007dc9e8* _PKCS7_set_digest
0001:007dcabf* _PKCS7_get_signer_info
0001:007dcb08  _PKCS7_SIGNER_INFO_get0_algs
0001:007dcb40  _PKCS7_RECIP_INFO_get0_alg
0001:007dcb56* _PKCS7_add_recipient
0001:007dcc51* _PKCS7_RECIP_INFO_set
0001:007dcbba* _PKCS7_add_recipient_info
0001:007dce3f* _PKCS7_cert_from_signer_info
0001:007dce8b* _PKCS7_set_cipher
0001:007dcf55  _PKCS7_stream
Module: U:\extras\lib\libcrypto.lib(cms_sd.obj)
0001:007dd18c* _CMS_SignedData_init
0001:007ddd5a* _CMS_get0_SignerInfos
0001:007dd4bf  _cms_set1_SignerIdentifier
0001:007dd627  _cms_SignerIdentifier_get0_signer_id
0001:007dd687  _cms_SignerIdentifier_cert_cmp
0001:007dd73c* _CMS_add1_signer
0001:007dec8f* _CMS_add_standard_smimecap
0001:007deab1* _CMS_add_smimecap
0001:007de362* _CMS_SignerInfo_sign
0001:007ddd83* _CMS_get0_signers
0001:007dde24* _CMS_SignerInfo_set1_signer_cert
0001:007ddeaa* _CMS_SignerInfo_get0_signer_id
0001:007dded5* _CMS_SignerInfo_cert_cmp
0001:007ddef2* _CMS_set1_signers_certs
0001:007de067  _CMS_SignerInfo_get0_algs
0001:007de2e2  _cms_SignedData_final
0001:007de616* _CMS_SignerInfo_verify
0001:007de7b4  _cms_SignedData_init_bio
0001:007de883* _CMS_SignerInfo_verify_content
0001:007deb1c* _CMS_add_simple_smimecap
Module: U:\extras\lib\libcrypto.lib(cms_env.obj)
0001:007def0d* _CMS_get0_RecipientInfos
0001:007def36* _CMS_RecipientInfo_type
0001:007def40* _CMS_EnvelopedData_create
0001:007defe1* _CMS_add1_recipient_cert
0001:007df278  _CMS_RecipientInfo_ktri_get0_algs
0001:007df2fd* _CMS_RecipientInfo_ktri_get0_signer_id
0001:007df36d* _CMS_RecipientInfo_ktri_cert_cmp
0001:007df3c9* _CMS_RecipientInfo_set0_pkey
0001:007df89c* _CMS_RecipientInfo_kekri_id_cmp
0001:007df952* _CMS_add0_recipient_key
0001:007dfbf8* _CMS_RecipientInfo_kekri_get0_id
0001:007dfcd7* _CMS_RecipientInfo_set0_key
0001:007e0197* _CMS_RecipientInfo_decrypt
0001:007e0208  _cms_EnvelopedData_init_bio
Module: U:\extras\lib\libcrypto.lib(ec_print.obj)
0001:007e03ab  _EC_POINT_point2bn
0001:007e0496* _EC_POINT_bn2point
0001:007e05c8* _EC_POINT_point2hex
0001:007e0737* _EC_POINT_hex2point
Module: U:\extras\lib\libcrypto.lib(eck_prn.obj)
0001:007e07aa* _ECPKParameters_print_fp
0001:007e0aac  _ECPKParameters_print
0001:007e0847* _EC_KEY_print_fp
0001:007e097a* _EC_KEY_print
0001:007e08e4* _ECParameters_print_fp
0001:007e09df* _ECParameters_print
Module: U:\extras\lib\libcrypto.lib(a_bytes.obj)
0001:007e148a* _d2i_ASN1_type_bytes
0001:007e167b  _i2d_ASN1_bytes
0001:007e1767* _d2i_ASN1_bytes
Module: U:\extras\lib\libcrypto.lib(pcy_node.obj)
0001:007e1c18  _policy_node_cmp_new
0001:007e1c2d  _tree_find_sk
0001:007e1c75  _level_find_node
0001:007e1cef  _level_add_node
0001:007e1e24  _policy_node_free
0001:007e1e37  _policy_node_match
Module: U:\extras\lib\libcrypto.lib(pcy_lib.obj)
0001:007e1ef0* _X509_policy_tree_level_count
0001:007e1f08* _X509_policy_tree_get0_level
0001:007e1f38* _X509_policy_tree_get0_policies
0001:007e1f50  _X509_policy_tree_get0_user_policies
0001:007e1f7d* _X509_policy_level_node_count
0001:007e1fca* _X509_policy_level_get0_node
0001:007e200f* _X509_policy_node_get0_policy
0001:007e2029* _X509_policy_node_get0_qualifiers
0001:007e2043* _X509_policy_node_get0_parent
Module: U:\extras\lib\libcrypto.lib(o_time.obj)
0001:007e2060  _OPENSSL_gmtime
0001:007e20ad  _OPENSSL_gmtime_adj
Module: U:\extras\lib\libcrypto.lib(asn1_gen.obj)
0001:007e2580* _ASN1_generate_nconf
0001:007e25d2  _ASN1_generate_v3
Module: U:\extras\lib\libcrypto.lib(a_bool.obj)
0001:007e3f70* _i2d_ASN1_BOOLEAN
0001:007e3ff5  _d2i_ASN1_BOOLEAN
Module: U:\extras\lib\libcrypto.lib(b_dump.obj)
0001:007e40d0* _BIO_dump_cb
0001:007e4133* _BIO_dump_indent_cb
0001:007e44ea* _BIO_dump_fp
0001:007e4513* _BIO_dump_indent_fp
0001:007e4564* _BIO_dump
0001:007e458d  _BIO_dump_indent
Module: U:\extras\lib\libcrypto.lib(a_strnid.obj)
0001:007e45c0* _ASN1_STRING_set_default_mask
0001:007e45cd* _ASN1_STRING_get_default_mask
0001:007e45fb* _ASN1_STRING_set_default_mask_asc
0001:007e4706  _ASN1_STRING_set_by_NID
0001:007e49e1* _ASN1_STRING_TABLE_get
0001:007e4a6b* _ASN1_STRING_TABLE_add
0001:007e4bb7* _ASN1_STRING_TABLE_cleanup
Module: U:\extras\lib\libcrypto.lib(a_print.obj)
0001:007e4c10  _ASN1_PRINTABLE_type
0001:007e4d1e* _ASN1_UNIVERSALSTRING_to_string
Module: U:\extras\lib\libcrypto.lib(err_prn.obj)
0001:007e4e32  _ERR_print_errors_cb
0001:007e4fa5* _ERR_print_errors_fp
0001:007e4fe1  _ERR_print_errors
Module: U:\extras\lib\libcrypto.lib(v3_prn.obj)
0001:007e5019* _X509V3_EXT_val_prn
0001:007e518a* _X509V3_EXT_print
0001:007e53fd  _X509V3_extensions_print
0001:007e56d6* _X509V3_EXT_print_fp
Module: U:\extras\lib\libcrypto.lib(t_x509a.obj)
0001:007e57bf  _X509_CERT_AUX_print
Module: U:\extras\lib\libcrypto.lib(p5_pbe.obj)
0001:007e5b10* _PBEPARAM_it
0001:007e5b2c  _d2i_PBEPARAM
0001:007e5b55* _i2d_PBEPARAM
0001:007e5b77* _PBEPARAM_new
0001:007e5b8b  _PBEPARAM_free
0001:007e5baf* _PKCS5_pbe_set0_algor
0001:007e5dc4  _PKCS5_pbe_set
Module: U:\extras\lib\libcrypto.lib(p12_key.obj)
0001:007e5e5a  _PKCS12_key_gen_asc
0001:007e5f4b* _PKCS12_key_gen_uni
Module: U:\extras\lib\libcrypto.lib(p5_pbev2.obj)
0001:007e64b0* _PBE2PARAM_it
0001:007e64cc  _d2i_PBE2PARAM
0001:007e64f5* _i2d_PBE2PARAM
0001:007e6517* _PBE2PARAM_new
0001:007e652b  _PBE2PARAM_free
0001:007e65c0* _PBKDF2PARAM_it
0001:007e65dc  _d2i_PBKDF2PARAM
0001:007e6605* _i2d_PBKDF2PARAM
0001:007e6627* _PBKDF2PARAM_new
0001:007e663b  _PBKDF2PARAM_free
0001:007e6661* _PKCS5_pbe2_set_iv
0001:007e6b9d  _PKCS5_pbe2_set
Module: U:\extras\lib\libcrypto.lib(eng_ctrl.obj)
0001:007e7012* _ENGINE_ctrl
0001:007e71fb* _ENGINE_cmd_is_executable
0001:007e7293* _ENGINE_ctrl_cmd
0001:007e7396  _ENGINE_ctrl_cmd_string
Module: U:\extras\lib\libcrypto.lib(conf_lib.obj)
0001:007e7710* _CONF_version
0001:007e7737  _CONF_set_nconf
0001:007e776b* _CONF_set_default_method
0001:007e778b* _CONF_load
0001:007e7894* _CONF_load_bio
0001:007e7813* _CONF_load_fp
0001:007e7c36* _NCONF_load_bio
0001:007e78da  _CONF_get_section
0001:007e7c95  _NCONF_get_section
0001:007e7913  _CONF_get_string
0001:007e7d2f  _NCONF_get_string
0001:007e7968* _CONF_get_number
0001:007e7df5* _NCONF_get_number_e
0001:007e79e6  _CONF_free
0001:007e7b35* _NCONF_free_data
0001:007e7a0b* _CONF_dump_fp
0001:007e7a85* _CONF_dump_bio
0001:007e7f48* _NCONF_dump_bio
0001:007e7ab1  _NCONF_new
0001:007e7b14  _NCONF_free
0001:007e7b56  _NCONF_load
0001:007e7bb5* _NCONF_load_fp
0001:007e7ece* _NCONF_dump_fp
Module: U:\extras\lib\libcrypto.lib(x509_req.obj)
0001:007e7fab* _X509_to_X509_REQ
0001:007e80e1* _X509_REQ_get_pubkey
0001:007e810f* _X509_REQ_check_private_key
0001:007e8284* _X509_REQ_extension_nid
0001:007e82c6* _X509_REQ_get_extension_nids
0001:007e82d0* _X509_REQ_set_extension_nids
0001:007e82dd  _X509_REQ_get_extensions
0001:007e8575* _X509_REQ_get_attr_by_NID
0001:007e85c1* _X509_REQ_get_attr
0001:007e83f7* _X509_REQ_add_extensions_nid
0001:007e853b  _X509_REQ_add_extensions
0001:007e855d* _X509_REQ_get_attr_count
0001:007e859b* _X509_REQ_get_attr_by_OBJ
0001:007e85e0* _X509_REQ_delete_attr
0001:007e85ff* _X509_REQ_add1_attr
0001:007e862e* _X509_REQ_add1_attr_by_OBJ
0001:007e8672* _X509_REQ_add1_attr_by_NID
0001:007e86b6* _X509_REQ_add1_attr_by_txt
Module: U:\extras\lib\libcrypto.lib(conf_mod.obj)
0001:007e875f* _CONF_modules_load
0001:007e8880* _CONF_modules_load_file
0001:007e9200* _CONF_get1_default_config_file
0001:007e8faa* _CONF_modules_unload
0001:007e9084* _CONF_modules_finish
0001:007e9128* _CONF_module_add
0001:007e9161* _CONF_modules_free
0001:007e917a* _CONF_imodule_get_name
0001:007e9185* _CONF_imodule_get_value
0001:007e9190* _CONF_imodule_get_usr_data
0001:007e919b* _CONF_imodule_set_usr_data
0001:007e91a9* _CONF_imodule_get_module
0001:007e91b3* _CONF_imodule_get_flags
0001:007e91be* _CONF_imodule_set_flags
0001:007e91cc* _CONF_module_get_usr_data
0001:007e91d7* _CONF_module_set_usr_data
0001:007e92d1  _CONF_parse_list
Module: U:\extras\lib\libcrypto.lib(v3_pmaps.obj)
0001:007e9430  _v3_policy_mappings
0001:007e9520* _POLICY_MAPPINGS_it
0001:007e94d0* _POLICY_MAPPING_it
0001:007e953c* _POLICY_MAPPING_new
0001:007e9550  _POLICY_MAPPING_free
Module: U:\extras\lib\libcrypto.lib(bn_sqr.obj)
0001:007e98a0  _BN_sqr
0001:007e9b43* _bn_sqr_normal
0001:007e9c72* _bn_sqr_recursive
Module: U:\extras\lib\libcrypto.lib(bn_recp.obj)
0001:007e9f20  _BN_RECP_CTX_init
0001:007e9f5f* _BN_RECP_CTX_new
0001:007e9fab  _BN_RECP_CTX_free
0001:007e9fed  _BN_RECP_CTX_set
0001:007ea048  _BN_mod_mul_reciprocal
0001:007ea118* _BN_div_recp
0001:007ea443* _BN_reciprocal
Module: U:\extras\lib\libcrypto.lib(bn_prime.obj)
0001:007eb4d0  _BN_GENCB_call
0001:007eb550  _BN_generate_prime_ex
0001:007eb89b  _BN_is_prime_fasttest_ex
0001:007eb86b  _BN_is_prime_ex
Module: U:\extras\lib\libcrypto.lib(bn_exp2.obj)
0001:007ec34a  _BN_mod_exp2_mont
Module: U:\extras\lib\libcrypto.lib(v3_bitst.obj)
0001:007eccd0  _v3_nscert
0001:007ecd48* _i2v_ASN1_BIT_STRING
0001:007ecdc4* _v2i_ASN1_BIT_STRING
0001:007ecd10  _v3_key_usage
Module: U:\extras\lib\libcrypto.lib(v3_ia5.obj)
0001:007ecfa0  _v3_ns_ia5_list
Module: U:\extras\lib\libcrypto.lib(v3_skey.obj)
0001:007ed2e0  _v3_skey_id
0001:007ed318* _i2s_ASN1_OCTET_STRING
0001:007ed341* _s2i_ASN1_OCTET_STRING
Module: U:\extras\lib\libcrypto.lib(v3_pku.obj)
0001:007ed5c0  _v3_pkey_usage_period
0001:007ed650* _PKEY_USAGE_PERIOD_it
0001:007ed66c* _d2i_PKEY_USAGE_PERIOD
0001:007ed695* _i2d_PKEY_USAGE_PERIOD
0001:007ed6b7* _PKEY_USAGE_PERIOD_new
0001:007ed6cb* _PKEY_USAGE_PERIOD_free
Module: U:\extras\lib\libcrypto.lib(v3_int.obj)
0001:007ed7d0  _v3_crl_num
0001:007ed810  _v3_delta_crl
0001:007ed870  _v3_inhibit_anyp
Module: U:\extras\lib\libcrypto.lib(v3_akey.obj)
0001:007ed8b0  _v3_akey_id
Module: U:\extras\lib\libcrypto.lib(v3_extku.obj)
0001:007edd90  _v3_ext_ku
0001:007ede40* _EXTENDED_KEY_USAGE_it
0001:007eddd0  _v3_ocsp_accresp
0001:007ede5c* _d2i_EXTENDED_KEY_USAGE
0001:007ede85* _i2d_EXTENDED_KEY_USAGE
0001:007edea7* _EXTENDED_KEY_USAGE_new
0001:007edebb* _EXTENDED_KEY_USAGE_free
Module: U:\extras\lib\libcrypto.lib(v3_enum.obj)
0001:007ee210  _v3_crl_reason
0001:007ee248* _i2s_ASN1_ENUMERATED_TABLE
Module: U:\extras\lib\libcrypto.lib(v3_ocsp.obj)
0001:007ee2b0  _v3_ocsp_crlid
0001:007ee2f0  _v3_ocsp_acutoff
0001:007ee330  _v3_crl_invdate
0001:007ee370  _v3_crl_hold
0001:007ee3b0  _v3_ocsp_nonce
0001:007ee3f0  _v3_ocsp_nocheck
0001:007ee430  _v3_ocsp_serviceloc
Module: U:\extras\lib\libcrypto.lib(v3_sxnet.obj)
0001:007ee9c0  _v3_sxnet
0001:007eeb20* _SXNET_it
0001:007eea40* _SXNETID_it
0001:007eea5c* _d2i_SXNETID
0001:007eea85* _i2d_SXNETID
0001:007eeaa7* _SXNETID_new
0001:007eeabb* _SXNETID_free
0001:007eeb3c* _d2i_SXNET
0001:007eeb65* _i2d_SXNET
0001:007eeb87* _SXNET_new
0001:007eeb9b* _SXNET_free
0001:007eed50* _SXNET_add_id_asc
0001:007eee66* _SXNET_add_id_INTEGER
0001:007eedce* _SXNET_add_id_ulong
0001:007ef18d* _SXNET_get_id_INTEGER
0001:007ef071* _SXNET_get_id_asc
0001:007ef0f2* _SXNET_get_id_ulong
Module: U:\extras\lib\libcrypto.lib(v3_pci.obj)
0001:007ef200  _v3_pci
Module: U:\extras\lib\libcrypto.lib(pk7_doit.obj)
0001:007f07b3  _PKCS7_dataInit
0001:007f0da6* _PKCS7_dataDecode
0001:007f2535  _PKCS7_get_signed_attribute
0001:007f1c82* _PKCS7_SIGNER_INFO_sign
0001:007f16d8  _PKCS7_dataFinal
0001:007f1ef9* _PKCS7_dataVerify
0001:007f20c1* _PKCS7_signatureVerify
0001:007f2624* _PKCS7_digest_from_attributes
0001:007f249d* _PKCS7_get_issuer_and_serial
0001:007f2552* _PKCS7_get_attribute
0001:007f2655* _PKCS7_set_signed_attributes
0001:007f2701* _PKCS7_set_attributes
0001:007f27ad  _PKCS7_add_signed_attribute
0001:007f27d8* _PKCS7_add_attribute
Module: U:\extras\lib\libcrypto.lib(tasn_prn.obj)
0001:007f296b* _ASN1_PCTX_new
0001:007f29ff* _ASN1_PCTX_free
0001:007f2a12* _ASN1_PCTX_get_flags
0001:007f2a1c* _ASN1_PCTX_set_flags
0001:007f2a29* _ASN1_PCTX_get_nm_flags
0001:007f2a34* _ASN1_PCTX_set_nm_flags
0001:007f2a42* _ASN1_PCTX_get_cert_flags
0001:007f2a4d* _ASN1_PCTX_set_cert_flags
0001:007f2a5b* _ASN1_PCTX_get_oid_flags
0001:007f2a66* _ASN1_PCTX_set_oid_flags
0001:007f2a74* _ASN1_PCTX_get_str_flags
0001:007f2a7f* _ASN1_PCTX_set_str_flags
0001:007f2a8d  _ASN1_item_print
0001:007f30df* _asn1_template_print_ctx
0002:000087b0* _default_pctx
Module: U:\extras\lib\libcrypto.lib(ec2_smpl.obj)
0001:007f3a70  _EC_GF2m_simple_method
0001:007f3a7a* _ec_GF2m_simple_group_init
0001:007f3ab3* _ec_GF2m_simple_group_finish
0001:007f3ae7* _ec_GF2m_simple_group_clear_finish
0001:007f3b57* _ec_GF2m_simple_group_copy
0001:007f3d5e  _ec_GF2m_simple_group_set_curve
0001:007f3f78* _ec_GF2m_simple_group_get_curve
0001:007f3ffd* _ec_GF2m_simple_group_get_degree
0001:007f4014* _ec_GF2m_simple_group_check_discriminant
0001:007f40f5* _ec_GF2m_simple_point_init
0001:007f412c* _ec_GF2m_simple_point_finish
0001:007f415e* _ec_GF2m_simple_point_clear_finish
0001:007f419a* _ec_GF2m_simple_point_copy
0001:007f421c* _ec_GF2m_simple_point_set_to_infinity
0001:007f4249* _ec_GF2m_simple_point_set_affine_coordinates
0001:007f434a* _ec_GF2m_simple_point_get_affine_coordinates
0001:007f4467* _ec_GF2m_simple_set_compressed_coordinates
0001:007f47b3* _ec_GF2m_simple_point2oct
0001:007f4bfe* _ec_GF2m_simple_oct2point
0001:007f5085* _ec_GF2m_simple_add
0001:007f5616* _ec_GF2m_simple_dbl
0001:007f5645* _ec_GF2m_simple_invert
0001:007f56ba* _ec_GF2m_simple_is_at_infinity
0001:007f56cd* _ec_GF2m_simple_is_on_curve
0001:007f58e8* _ec_GF2m_simple_cmp
0001:007f5ae0* _ec_GF2m_simple_make_affine
0001:007f5c27* _ec_GF2m_simple_points_make_affine
0001:007f5c79* _ec_GF2m_simple_field_mul
0001:007f5cab* _ec_GF2m_simple_field_sqr
0001:007f5cd6* _ec_GF2m_simple_field_div
Module: U:\extras\lib\libcrypto.lib(x509_att.obj)
0001:007f5db0  _X509at_get_attr_count
0001:007f5dc3  _X509at_get_attr_by_NID
0001:007f5dff  _X509at_get_attr_by_OBJ
0001:007f5e76  _X509at_get_attr
0001:007f5eb3  _X509at_delete_attr
0001:007f5f01  _X509at_add1_attr
0001:007f6006  _X509at_add1_attr_by_OBJ
0001:007f626c* _X509_ATTRIBUTE_create_by_OBJ
0001:007f6069  _X509at_add1_attr_by_NID
0001:007f61df* _X509_ATTRIBUTE_create_by_NID
0001:007f60cc  _X509at_add1_attr_by_txt
0001:007f634f* _X509_ATTRIBUTE_create_by_txt
0001:007f612f  _X509at_get0_data_by_OBJ
0001:007f6614* _X509_ATTRIBUTE_count
0001:007f6663* _X509_ATTRIBUTE_get0_data
0001:007f63f9* _X509_ATTRIBUTE_set1_object
0001:007f6436* _X509_ATTRIBUTE_set1_data
0001:007f664c* _X509_ATTRIBUTE_get0_object
0001:007f66d6* _X509_ATTRIBUTE_get0_type
Module: U:\extras\lib\libcrypto.lib(nsseq.obj)
0001:007f67d0* _NETSCAPE_CERT_SEQUENCE_it
0001:007f67ec  _d2i_NETSCAPE_CERT_SEQUENCE
0001:007f6815  _i2d_NETSCAPE_CERT_SEQUENCE
0001:007f6837* _NETSCAPE_CERT_SEQUENCE_new
0001:007f684b* _NETSCAPE_CERT_SEQUENCE_free
Module: U:\extras\lib\libcrypto.lib(x_pkey.obj)
0001:007f6870* _i2d_X509_PKEY
0001:007f6883* _d2i_X509_PKEY
0001:007f6b13  _X509_PKEY_new
0001:007f6c2b  _X509_PKEY_free
Module: U:\extras\lib\libcrypto.lib(rsa_pss.obj)
0001:007f6d02  _RSA_verify_PKCS1_PSS
0001:007f7153  _RSA_padding_add_PKCS1_PSS
Module: U:\extras\lib\libcrypto.lib(rsa_gen.obj)
0001:007f7480  _RSA_generate_key_ex
Module: U:\extras\lib\libcrypto.lib(dh_gen.obj)
0001:007f7d00  _DH_generate_parameters_ex
Module: U:\extras\lib\libcrypto.lib(dsa_gen.obj)
0001:007f8000* _DSA_generate_parameters_ex
0001:007f80d9  _dsa_builtin_paramgen
Module: U:\extras\lib\libcrypto.lib(dsa_key.obj)
0001:007f8a20  _DSA_generate_key
Module: U:\extras\lib\libcrypto.lib(p12_p8d.obj)
0001:007f8c10  _PKCS8_decrypt
Module: U:\extras\lib\libcrypto.lib(pem_pk8.obj)
0001:007f8c50* _PEM_write_bio_PKCS8PrivateKey_nid
0001:007f8c9d  _PEM_write_bio_PKCS8PrivateKey
0001:007f8cea* _i2d_PKCS8PrivateKey_bio
0001:007f8d37* _i2d_PKCS8PrivateKey_nid_bio
0001:007f93e5* _PEM_write_bio_PKCS8
0001:007f9509* _PEM_write_bio_PKCS8_PRIV_KEY_INFO
0001:007f8f94* _d2i_PKCS8PrivateKey_bio
0001:007f90f6* _i2d_PKCS8PrivateKey_fp
0001:007f9143* _i2d_PKCS8PrivateKey_nid_fp
0001:007f9190* _PEM_write_PKCS8PrivateKey_nid
0001:007f91dd* _PEM_write_PKCS8PrivateKey
0001:007f92d5* _d2i_PKCS8PrivateKey_fp
0001:007f9373* _PEM_read_bio_PKCS8
0001:007f93ac* _PEM_read_PKCS8
0001:007f9438* _PEM_write_PKCS8
0001:007f9497* _PEM_read_bio_PKCS8_PRIV_KEY_INFO
0001:007f94d0* _PEM_read_PKCS8_PRIV_KEY_INFO
0001:007f955c* _PEM_write_PKCS8_PRIV_KEY_INFO
Module: U:\extras\lib\libcrypto.lib(ecp_nist.obj)
0001:007f95b0  _EC_GFp_nist_method
0001:007f95ba* _ec_GFp_nist_group_copy
0001:007f95f1* _ec_GFp_nist_group_set_curve
0001:007f9791* _ec_GFp_nist_field_mul
0001:007f987c* _ec_GFp_nist_field_sqr
Module: U:\extras\lib\libcrypto.lib(ecp_mont.obj)
0001:007f9a00  _EC_GFp_mont_method
0001:007f9a0a* _ec_GFp_mont_group_init
0001:007f9a3d* _ec_GFp_mont_group_finish
0001:007f9aa6* _ec_GFp_mont_group_clear_finish
0001:007f9b0f* _ec_GFp_mont_group_copy
0001:007f9c5d* _ec_GFp_mont_group_set_curve
0001:007f9e66* _ec_GFp_mont_field_mul
0001:007f9edb* _ec_GFp_mont_field_sqr
0001:007f9f50* _ec_GFp_mont_field_encode
0001:007f9fce* _ec_GFp_mont_field_decode
0001:007fa03c* _ec_GFp_mont_field_set_to_one
Module: U:\extras\lib\libcrypto.lib(ech_ossl.obj)
0001:007fa164  _ECDH_OpenSSL
Module: U:\extras\lib\libcrypto.lib(tb_ecdh.obj)
0001:007fa604* _ENGINE_unregister_ECDH
0001:007fa633* _ENGINE_register_ECDH
0001:007fa67f* _ENGINE_register_all_ECDH
0001:007fa6b0* _ENGINE_set_default_ECDH
0001:007fa6fc  _ENGINE_get_default_ECDH
0001:007fa719  _ENGINE_get_ECDH
0001:007fa724* _ENGINE_set_ECDH
Module: U:\extras\lib\libcrypto.lib(ecs_ossl.obj)
0001:007fa755  _ECDSA_OpenSSL
Module: U:\extras\lib\libcrypto.lib(tb_ecdsa.obj)
0001:007fb794* _ENGINE_unregister_ECDSA
0001:007fb7c3* _ENGINE_register_ECDSA
0001:007fb80f* _ENGINE_register_all_ECDSA
0001:007fb840* _ENGINE_set_default_ECDSA
0001:007fb88c  _ENGINE_get_default_ECDSA
0001:007fb8a9  _ENGINE_get_ECDSA
0001:007fb8b4* _ENGINE_set_ECDSA
Module: U:\extras\lib\libcrypto.lib(cbc128.obj)
0001:007fb8d0  _CRYPTO_cbc128_encrypt
0001:007fb9fc  _CRYPTO_cbc128_decrypt
Module: U:\extras\lib\libcrypto.lib(cfb128.obj)
0001:007fbbc0  _CRYPTO_cfb128_encrypt
0001:007fbfc1  _CRYPTO_cfb128_1_encrypt
0001:007fc09e  _CRYPTO_cfb128_8_encrypt
Module: U:\extras\lib\libcrypto.lib(ofb128.obj)
0001:007fc100  _CRYPTO_ofb128_encrypt
Module: U:\extras\lib\libcrypto.lib(ui_openssl.obj)
0001:007fc22f  _UI_OpenSSL
Module: U:\extras\lib\libcrypto.lib(cms_asn1.obj)
0001:007fca10  _CMS_IssuerAndSerialNumber_it
0001:007fcaa0* _CMS_OtherCertificateFormat_it
0001:007fcb90  _CMS_CertificateChoices_it
0001:007fcc20* _CMS_SignerIdentifier_it
0001:007fccb0* _CMS_EncapsulatedContentInfo_it
0001:007fce30  _CMS_SignerInfo_it
0001:007fcec0* _CMS_OtherRevocationInfoFormat_it
0001:007fcf40  _CMS_RevocationInfoChoice_it
0001:007fd030  _CMS_SignedData_it
0001:007fd090* _CMS_OriginatorInfo_it
0001:007fd150* _CMS_EncryptedContentInfo_it
0001:007fd210  _CMS_KeyTransRecipientInfo_it
0001:007fd280  _CMS_OtherKeyAttribute_it
0001:007fd320* _CMS_RecipientKeyIdentifier_it
0001:007fd3a0* _CMS_KeyAgreeRecipientIdentifier_it
0001:007fd410* _CMS_RecipientEncryptedKey_it
0001:007fd480* _CMS_OriginatorPublicKey_it
0001:007fd510* _CMS_OriginatorIdentifierOrKey_it
0001:007fd5e0* _CMS_KeyAgreeRecipientInfo_it
0001:007fd660* _CMS_KEKIdentifier_it
0001:007fd700  _CMS_KEKRecipientInfo_it
0001:007fd7b0* _CMS_PasswordRecipientInfo_it
0001:007fd820* _CMS_OtherRecipientInfo_it
0001:007fd9b0  _CMS_RecipientInfo_it
0001:007fda90  _CMS_EnvelopedData_it
0001:007fdb30  _CMS_DigestedData_it
0001:007fdba0  _CMS_EncryptedData_it
0001:007fdcc0* _CMS_AuthenticatedData_it
0001:007fdd50* _CMS_CompressedData_it
0001:007fdfe0  _CMS_ContentInfo_it
0001:007fe040  _CMS_Attributes_Sign_it
0001:007fe090  _CMS_Attributes_Verify_it
0001:007fe110* _CMS_ReceiptsFrom_it
0001:007fe1b0* _CMS_ReceiptRequest_it
0001:007fe250* _CMS_Receipt_it
Module: U:\extras\lib\libcrypto.lib(cms_att.obj)
0001:007fe270  _CMS_signed_get_attr_count
0001:007fe286  _CMS_signed_get_attr_by_NID
0001:007fe2aa* _CMS_signed_get_attr_by_OBJ
0001:007fe2ce* _CMS_signed_get_attr
0001:007fe2eb* _CMS_signed_delete_attr
0001:007fe308* _CMS_signed_add1_attr
0001:007fe335* _CMS_signed_add1_attr_by_OBJ
0001:007fe377  _CMS_signed_add1_attr_by_NID
0001:007fe3b9* _CMS_signed_add1_attr_by_txt
0001:007fe3fb  _CMS_signed_get0_data_by_OBJ
0001:007fe426* _CMS_unsigned_get_attr_count
0001:007fe43c* _CMS_unsigned_get_attr_by_NID
0001:007fe460* _CMS_unsigned_get_attr_by_OBJ
0001:007fe484* _CMS_unsigned_get_attr
0001:007fe4a1* _CMS_unsigned_delete_attr
0001:007fe4be* _CMS_unsigned_add1_attr
0001:007fe4eb* _CMS_unsigned_add1_attr_by_OBJ
0001:007fe52d* _CMS_unsigned_add1_attr_by_NID
0001:007fe56f* _CMS_unsigned_add1_attr_by_txt
0001:007fe5b1* _CMS_unsigned_get0_data_by_OBJ
Module: U:\extras\lib\libcrypto.lib(cms_lib.obj)
0001:007fe5e0  _d2i_CMS_ContentInfo
0001:007fe609  _i2d_CMS_ContentInfo
0001:007fe62b  _CMS_ContentInfo_new
0001:007fe63f  _CMS_ContentInfo_free
0001:007fe65a* _CMS_ContentInfo_print_ctx
0001:007fe68a* _CMS_get0_type
0001:007fe694* _priv_cms_Data_create
0001:007fecc3* _CMS_set_detached
0001:007fe6d1* _cms_content_bio
0001:007fea58  _CMS_get0_content
0001:007fe756  _CMS_dataInit
0001:007fe899  _CMS_dataFinal
0001:007febfe  _CMS_get0_eContentType
0001:007fec26* _CMS_set1_eContentType
0001:007fec8b* _CMS_is_detached
0001:007fed7c  _cms_DigestAlgorithm_set
0001:007fedd2  _cms_DigestAlgorithm_init_bio
0001:007feeda  _cms_DigestAlgorithm_find_ctx
0001:007ff047* _CMS_add0_CertificateChoices
0001:007ff0e0* _CMS_add0_cert
0001:007ff1d6  _CMS_add1_cert
0001:007ff295* _CMS_add0_RevocationInfoChoice
0001:007ff32e* _CMS_add0_crl
0001:007ff368* _CMS_add1_crl
0001:007ff3bc* _CMS_get1_certs
0001:007ff4b8* _CMS_get1_crls
Module: U:\extras\lib\libcrypto.lib(cms_enc.obj)
0001:007ff5ca  _cms_EncryptedContent_init_bio
0001:007ffa7d  _cms_EncryptedContent_init
0001:007ffb09* _CMS_EncryptedData_set1_key
0001:007ffc3d  _cms_EncryptedData_init_bio
Module: U:\extras\lib\libcrypto.lib(aes_wrap.obj)
0001:007ffc88  _AES_wrap_key
0001:007ffe18  _AES_unwrap_key
Module: U:\extras\lib\libcrypto.lib(asn_pack.obj)
0001:007fffeb* _ASN1_seq_unpack
0001:00800069* _ASN1_seq_pack
0001:0080018f* _ASN1_unpack_string
0001:008001f4* _ASN1_pack_string
0001:00800333  _ASN1_item_pack
0001:00800465  _ASN1_item_unpack
Module: U:\extras\lib\libcrypto.lib(p12_utl.obj)
0001:008004ea  _OPENSSL_asc2uni
0001:008005a3* _OPENSSL_uni2asc
0001:00800633* _i2d_PKCS12_bio
0001:00800655* _i2d_PKCS12_fp
0001:00800677* _d2i_PKCS12_bio
0001:00800699* _d2i_PKCS12_fp
0001:008006bb* _PKCS12_x5092certbag
0001:008006e6* _PKCS12_x509crl2certbag
0001:00800711* _PKCS12_certbag2x509
0001:0080076b* _PKCS12_certbag2x509crl
Module: U:\extras\lib\libcrypto.lib(conf_def.obj)
0001:008007d0* _CONF_def_version
0001:00800811  _NCONF_default
0001:0080081b* _NCONF_WIN32
Module: U:\extras\lib\libcrypto.lib(conf_api.obj)
0001:00801dcf  __CONF_get_section
0001:00801e12  __CONF_get_section_values
0001:00801e42  __CONF_add_string
0001:00801ee9  __CONF_get_string
0001:008020c3  __CONF_new_data
0001:00802114  __CONF_free_data
0001:0080225e  __CONF_new_section
Module: U:\extras\lib\libcrypto.lib(x509rset.obj)
0001:008023a0* _X509_REQ_set_version
0001:008023cc  _X509_REQ_set_subject_name
0001:00802401  _X509_REQ_set_pubkey
Module: U:\extras\lib\libcrypto.lib(dso_lib.obj)
0001:00802440* _DSO_new
0001:0080249a* _DSO_new_method
0001:00802454* _DSO_set_default_method
0001:00802461* _DSO_get_default_method
0001:0080246b* _DSO_get_method
0001:00802475* _DSO_set_method
0001:008025da  _DSO_free
0001:00802756* _DSO_flags
0001:0080276e* _DSO_up_ref
0001:008027e2  _DSO_load
0001:00802bcf* _DSO_ctrl
0001:00802d6f* _DSO_set_filename
0001:00802a03* _DSO_bind_var
0001:00802ae9  _DSO_bind_func
0001:00802cc8* _DSO_set_name_converter
0001:00802d28* _DSO_get_filename
0001:00802ea1* _DSO_merge
0001:00802f57* _DSO_convert_filename
0001:008030d3* _DSO_get_loaded_filename
0001:0080311a* _DSO_pathbyaddr
0001:00803191* _DSO_global_lookup
Module: U:\extras\lib\libcrypto.lib(f_int.obj)
0001:00803208  _i2a_ASN1_INTEGER
0001:00803379* _a2i_ASN1_INTEGER
Module: U:\extras\lib\libcrypto.lib(f_string.obj)
0001:00803795  _i2a_ASN1_STRING
0001:008038cf* _a2i_ASN1_STRING
Module: U:\extras\lib\libcrypto.lib(bio_md.obj)
0001:00803ccf  _BIO_f_md
Module: U:\extras\lib\libcrypto.lib(bio_enc.obj)
0001:00804167  _BIO_f_cipher
0001:00804aaa* _BIO_set_cipher
Module: U:\extras\lib\libcrypto.lib(bss_null.obj)
0001:00804b95  _BIO_s_null
Module: U:\extras\lib\libcrypto.lib(pk7_attr.obj)
0001:00804c9b* _PKCS7_add_attrib_smimecap
0001:00804d28* _PKCS7_get_smimecap
0001:00804d90* _PKCS7_simple_smimecap
0001:00804f07* _PKCS7_add_attrib_content_type
0001:00804f64  _PKCS7_add0_attrib_signing_time
0001:00804fe4  _PKCS7_add1_attrib_digest
Module: U:\extras\lib\libcrypto.lib(bn_gf2m.obj)
0001:00805321  _BN_GF2m_add
0001:00805466  _BN_GF2m_mod_arr
0001:008058d0* _BN_GF2m_mod
0001:00806d1e  _BN_GF2m_poly2arr
0001:008059a7  _BN_GF2m_mod_mul_arr
0001:00805d13  _BN_GF2m_mod_sqr_arr
0001:00805c2a* _BN_GF2m_mod_mul
0001:00805f57* _BN_GF2m_mod_sqr
0001:00806035* _BN_GF2m_mod_inv
0001:00806270* _BN_GF2m_mod_inv_arr
0001:00806dda* _BN_GF2m_arr2poly
0001:008062eb  _BN_GF2m_mod_div
0001:0080638d* _BN_GF2m_mod_div_arr
0001:0080640f* _BN_GF2m_mod_exp_arr
0001:0080657a* _BN_GF2m_mod_exp
0001:00806663  _BN_GF2m_mod_sqrt_arr
0001:0080670b* _BN_GF2m_mod_sqrt
0001:008067e9  _BN_GF2m_mod_solve_quad_arr
0001:00806c40* _BN_GF2m_mod_solve_quad
Module: U:\extras\lib\libcrypto.lib(ec2_mult.obj)
0001:00807a60  _ec_GF2m_simple_mul
0001:00807d25  _ec_GF2m_precompute_mult
0001:00807d3f  _ec_GF2m_have_precompute_mult
Module: U:\extras\lib\libcrypto.lib(p12_decr.obj)
0001:00807d6b* _PKCS12_pbe_crypt
0001:00807f1d  _PKCS12_item_decrypt_d2i
0001:00808025  _PKCS12_item_i2d_encrypt
Module: U:\extras\lib\libcrypto.lib(p12_p8e.obj)
0001:0080818a  _PKCS8_encrypt
Module: U:\extras\lib\libcrypto.lib(ecp_smpl.obj)
0001:00808310* _EC_GFp_simple_method
0001:0080831a  _ec_GFp_simple_group_init
0001:00808360  _ec_GFp_simple_group_finish
0001:00808394  _ec_GFp_simple_group_clear_finish
0001:008083c8  _ec_GFp_simple_group_copy
0001:00808460  _ec_GFp_simple_group_set_curve
0001:008086c8  _ec_GFp_simple_group_get_curve
0001:00808825  _ec_GFp_simple_group_get_degree
0001:0080883b  _ec_GFp_simple_group_check_discriminant
0001:00808b16  _ec_GFp_simple_point_init
0001:00808b57  _ec_GFp_simple_point_finish
0001:00808b89  _ec_GFp_simple_point_clear_finish
0001:00808bc5  _ec_GFp_simple_point_copy
0001:00808c47  _ec_GFp_simple_point_set_to_infinity
0001:00808c74  _ec_GFp_simple_set_Jprojective_coordinates_GFp
0001:00808ec4  _ec_GFp_simple_get_Jprojective_coordinates_GFp
0001:00809045  _ec_GFp_simple_point_set_affine_coordinates
0001:008090bc  _ec_GFp_simple_point_get_affine_coordinates
0001:008094ea  _ec_GFp_simple_set_compressed_coordinates
0001:00809b00  _ec_GFp_simple_point2oct
0001:00809f02  _ec_GFp_simple_oct2point
0001:0080a340  _ec_GFp_simple_add
0001:0080ab3e  _ec_GFp_simple_dbl
0001:0080b1e6  _ec_GFp_simple_invert
0001:0080b237  _ec_GFp_simple_is_at_infinity
0001:0080b24a  _ec_GFp_simple_is_on_curve
0001:0080b692  _ec_GFp_simple_cmp
0001:0080ba3c  _ec_GFp_simple_make_affine
0001:0080bb8e  _ec_GFp_simple_points_make_affine
0001:0080c281* _ec_GFp_simple_field_mul
0001:0080c2b3* _ec_GFp_simple_field_sqr
Module: U:\extras\lib\libcrypto.lib(bn_nist.obj)
0001:0080c824  _BN_get0_nist_prime_192
0001:0080c82e  _BN_get0_nist_prime_224
0001:0080c838  _BN_get0_nist_prime_256
0001:0080c842  _BN_get0_nist_prime_384
0001:0080c84c  _BN_get0_nist_prime_521
0001:0080c8eb  _BN_nist_mod_192
0001:0080cbfd  _BN_nist_mod_224
0001:0080d030  _BN_nist_mod_256
0001:0080d5ce  _BN_nist_mod_384
0001:0080dc79  _BN_nist_mod_521
Module: U:\extras\lib\libcrypto.lib(cms_io.obj)
0001:0080dfc9  _CMS_stream
0001:0080e076* _d2i_CMS_bio
0001:0080e098* _i2d_CMS_bio
0001:0080e0be* _PEM_read_bio_CMS
0001:0080e0f7* _PEM_read_CMS
0001:0080e130* _PEM_write_bio_CMS
0001:0080e183* _PEM_write_CMS
0001:0080e1d6* _BIO_new_CMS
0001:0080e1f8* _i2d_CMS_bio_stream
0001:0080e228* _PEM_write_bio_CMS_stream
0001:0080e260* _SMIME_write_CMS
0001:0080e2e6* _SMIME_read_CMS
Module: U:\extras\lib\libcrypto.lib(cms_dd.obj)
0001:0080e310* _cms_DigestedData_create
0001:0080e3af  _cms_DigestedData_init_bio
0001:0080e3d7  _cms_DigestedData_do_final
Module: U:\extras\lib\libcrypto.lib(a_set.obj)
0001:0080e59c  _i2d_ASN1_SET
0001:0080e8c7  _d2i_ASN1_SET
Module: U:\extras\lib\libcrypto.lib(p12_asn.obj)
0001:0080ed20* _PKCS12_MAC_DATA_it
0001:0080ec20  _PKCS12_it
0001:0080ec3c* _d2i_PKCS12
0001:0080ec65* _i2d_PKCS12
0001:0080ec87* _PKCS12_new
0001:0080ec9b* _PKCS12_free
0001:0080ed3c* _d2i_PKCS12_MAC_DATA
0001:0080ed65* _i2d_PKCS12_MAC_DATA
0001:0080ed87* _PKCS12_MAC_DATA_new
0001:0080ed9b* _PKCS12_MAC_DATA_free
0001:0080eec0* _PKCS12_BAGS_it
0001:0080eedc* _d2i_PKCS12_BAGS
0001:0080ef05* _i2d_PKCS12_BAGS
0001:0080ef27  _PKCS12_BAGS_new
0001:0080ef3b* _PKCS12_BAGS_free
0001:0080f0c0* _PKCS12_SAFEBAG_it
0001:0080f0dc* _d2i_PKCS12_SAFEBAG
0001:0080f105* _i2d_PKCS12_SAFEBAG
0001:0080f127  _PKCS12_SAFEBAG_new
0001:0080f13b* _PKCS12_SAFEBAG_free
0001:0080f190  _PKCS12_SAFEBAGS_it
0001:0080f1e0  _PKCS12_AUTHSAFES_it
Module: U:\extras\lib\libcrypto.lib(p12_add.obj)
0001:0080f20a  _PKCS12_item_pack_safebag
0001:0080f316* _PKCS12_MAKE_KEYBAG
0001:0080f37c* _PKCS12_MAKE_SHKEYBAG
0001:0080f47e* _PKCS12_pack_p7data
0001:0080f582* _PKCS12_unpack_p7data
0001:0080f5e6* _PKCS12_pack_p7encdata
0001:0080f7d4* _PKCS12_unpack_p7encdata
0001:0080f838* _PKCS12_decrypt_skey
0001:0080f85c* _PKCS12_pack_authsafes
0001:0080f894* _PKCS12_unpack_authsafes
Module: U:\extras\lib\libcrypto.lib(dso_openssl.obj)
0001:0080f900  _DSO_METHOD_openssl
Module: U:\extras\lib\libcrypto.lib(bn_sqrt.obj)
0001:0080f91a  _BN_mod_sqrt
Module: U:\extras\lib\libcrypto.lib(bn_kron.obj)
0001:00810480  _BN_kronecker
Module: U:\extras\lib\libcrypto.lib(bio_ndef.obj)
0001:0081080b  _BIO_new_NDEF
Module: U:\extras\lib\libcrypto.lib(asn_mime.obj)
0001:00810cfd  _i2d_ASN1_bio_stream
0001:00812066* _SMIME_crlf_copy
0001:00810ee2  _PEM_write_bio_ASN1_stream
0001:008114bd  _SMIME_write_ASN1
0001:00811ae6  _SMIME_read_ASN1
0001:008121ee* _SMIME_text
Module: U:\extras\lib\libcrypto.lib(dso_null.obj)
0001:00812e4b  _DSO_METHOD_null
Module: U:\extras\lib\libcrypto.lib(bio_asn1.obj)
0001:00812e65  _BIO_f_asn1
0001:008137ab  _BIO_asn1_set_prefix
0001:008137d4* _BIO_asn1_get_prefix
0001:008137fd  _BIO_asn1_set_suffix
0001:00813826* _BIO_asn1_get_suffix
Module: U:\extras\lib\libcrypto.lib(bio_b64.obj)
0001:00813860  _BIO_f_base64


                        +----------------------+
                        |   Imported Symbols   |
                        +----------------------+

Symbol                              Module
======                              ======

___libc_ForkRegisterModule          libc063
___init_dll                         libc063
___libc_Back_termDll                libc063
___libc_ForkDeregisterModule        libc063
__atfork_callback                   libc063
___libc_GLocaleCtype                libc063
__assert                            libc063
_strlcat                            libc063
DosReleaseMutexSem                  doscalls
DosRequestMutexSem                  doscalls
DosCloseMutexSem                    doscalls
DosSleep                            doscalls
DosGetDateTime                      doscalls
DosQuerySysInfo                     doscalls
DosGetInfoBlocks                    doscalls
DosFreeModule                       doscalls
DosQueryProcAddr                    doscalls
DosSetFileLocks                     doscalls
DosQueryFileInfo                    doscalls
DosResetBuffer                      doscalls
DosSetFileSize                      doscalls
DosSetFilePtr                       doscalls
DosWrite                            doscalls
DosRead                             doscalls
DosClose                            doscalls
DosForceDelete                      doscalls
UniCreateUconvObject                uconv
UniStrToUcs                         uconv
UniStrFromUcs                       uconv
DosLoadModule                       doscalls
DosQueryPathInfo                    doscalls
DosDelete                           doscalls
DosFreeMem                          doscalls
UniFreeUconvObject                  uconv
DosCreateMutexSem                   doscalls
DosGetNamedSharedMem                doscalls
DosAllocSharedMem                   doscalls
DosDupHandle                        doscalls
DosOpen                             doscalls
DosScanEnv                          doscalls
DosQueryCurrentDisk                 doscalls
___stderrp                          libc063
__errno                             libc063
_strlcpy                            libc063
_initgroups                         libc063
_getgrgid_r                         libc063
_getgrnam_r                         libc063
_getpwuid_r                         libc063
_getpwnam_r                         libc063
_getprotobyname                     tcpip32
_hstrerror                          tcpip32
_gethostbyname                      tcpip32
_inet_aton                          tcpip32
_tcp_h_errno1                       tcpip32
_inet_ntoa                          tcpip32
_getprotobynumber                   tcpip32
_getservbyport                      tcpip32
_getservbyname                      tcpip32
_inet_ntop                          tcpip32
_inet_pton                          tcpip32
_gethostname                        tcpip32
_inet_addr                          tcpip32
_gethostbyaddr                      tcpip32
DosQueryFSInfo                      doscalls
___isfinite                         libc063
___stdinp                           libc063
___stdoutp                          libc063
__exit                              libc063
DosAllocThreadLocalMemory           doscalls
___threadid                         libc063
DosFreeThreadLocalMemory            doscalls
_isspace                            libc063
___flt_rounds                       libc063
__CRT_init                          libc063
__std_strnicmp                      libc063
__std_strdup                        libc063
__std_memcpy                        libc063
__std_time                          libc063
__std_getenv                        libc063
__std_free                          libc063
__std_floor                         libc063
__std_malloc                        libc063
__std_strftime                      libc063
__std_sin                           libc063
__std_cos                           libc063
__std_atan2                         libc063
__std_acos                          libc063
__std_sqrt                          libc063
__std_stricmp                       libc063
__std_strchr                        libc063
__std_calloc                        libc063
__std_strtoll                       libc063
__std_strtol                        libc063
__std_realloc                       libc063
__std_strtod                        libc063
__std_memset                        libc063
__std_pow                           libc063
__std_setlocale                     libc063
__std_printf                        libc063
__std_putchar                       libc063
__std_strcmp                        libc063
__std_strncat                       libc063
__std_strncpy                       libc063
__std_strncmp                       libc063
__std_memmove                       libc063
__std_strcpy                        libc063
__std_memcmp                        libc063
__std_localtime                     libc063
__std_sprintf                       libc063
__std_qsort                         libc063
__std_memchr                        libc063
__std_dup                           libc063
__std_fwrite                        libc063
__std_exit                          libc063
___signbit                          libc063
__std_fprintf                       libc063
__std_abort                         libc063
__std_strstr                        libc063
__std_strtoull                      libc063
__std_stat                          libc063
__std_opendir                       libc063
__std_readdir                       libc063
__std_closedir                      libc063
__std_fputc                         libc063
__std_lseek                         libc063
__std_read                          libc063
__std_mktime                        libc063
__std_write                         libc063
__std_mkstemp                       libc063
__std_unlink                        libc063
__std_dup2                          libc063
__std_close                         libc063
__std_strerror                      libc063
__std_utimes                        libc063
__std_access                        libc063
__std_vasprintf                     libc063
__std_gmtime                        libc063
__std_asctime                       libc063
__std_strcspn                       libc063
__std_ctime                         libc063
__std_atoi                          libc063
__std_strpbrk                       libc063
___libc_FH                          libc063
__libsocket_set_errno               tcpip32
__libsocket_accept                  tcpip32
___libc_TcpipAllocFH44              libc063
__libsocket_soclose                 tcpip32
__libsocket_sock_errno              tcpip32
__libsocket_send                    tcpip32
__libsocket_recv                    tcpip32
__libsocket_getsockname             tcpip32
__std_strrchr                       libc063
__std_sscanf                        libc063
__libsocket_socket                  tcpip32
__libsocket_bind                    tcpip32
__libsocket_listen                  tcpip32
__std_gmtime_r                      libc063
__std_localtime_r                   libc063
__std_getuid                        libc063
__std_getgid                        libc063
__std_getgroups                     libc063
__std_sigsetjmp                     libc063
__std_strtok_r                      libc063
__std_strtok                        libc063
__std_mknod                         libc063
__std_mkfifo                        libc063
__std_isatty                        libc063
__std_ttyname                       libc063
__std_times                         libc063
__std_uname                         libc063
__std_getsid                        libc063
__std_getpgid                       libc063
__std_setpgid                       libc063
__std_setsid                        libc063
__std_getpgrp                       libc063
__std_getlogin                      libc063
__std_setegid                       libc063
__std_seteuid                       libc063
__std_setgid                        libc063
__std_setuid                        libc063
__std_getegid                       libc063
__std_geteuid                       libc063
__std_getppid                       libc063
__std_getpid                        libc063
__std_kill                          libc063
__std_getrlimit                     libc063
__std_sysconf                       libc063
__std_gettimeofday                  libc063
__std_readdir_r                     libc063
__std_fstat                         libc063
__std_flock                         libc063
__std_fcntl                         libc063
__std_pwrite                        libc063
__std_ftruncate                     libc063
__std_pread                         libc063
__std_timezone                      libc063
__std_strcat                        libc063
__std_open                          libc063
__libsocket_shutdown                tcpip32
__libsocket_getsockopt              tcpip32
__libsocket_sendto                  tcpip32
__libsocket_connect                 tcpip32
__std_select                        libc063
__libsocket_socketpair              tcpip32
___libc_FHClose                     libc063
__libsocket_getpeername             tcpip32
__libsocket_recvfrom                tcpip32
__libsocket_setsockopt              tcpip32
__std_readlink                      libc063
__std_strtoul                       libc063
__std_getloadavg                    libc063
__std_umask                         libc063
__std_nanosleep                     libc063
__std_usleep                        libc063
__std_sleep                         libc063
__std_environ                       libc063
__std_putenv                        libc063
__std_tzset                         libc063
__std_unsetenv                      libc063
__std_strptime                      libc063
__std_glob                          libc063
__std_globfree                      libc063
__std_dlopen                        libc063
__std_dlsym                         libc063
__std_dlclose                       libc063
__std_dlerror                       libc063
__std_mblen                         libc063
__std_nice                          libc063
__std_fnmatch                       libc063
__std_fclose                        libc063
__std_localeconv                    libc063
__std_nl_langinfo                   libc063
__std_getc                          libc063
__std_fileno                        libc063
__std_symlink                       libc063
__std_link                          libc063
__std_popen                         libc063
__std_pclose                        libc063
__std_log10                         libc063
__std_ceil                          libc063
__std_tan                           libc063
__std_asin                          libc063
__std_atan                          libc063
__std_sinh                          libc063
__std_cosh                          libc063
__std_tanh                          libc063
__std_asinh                         libc063
__std_acosh                         libc063
__std_atanh                         libc063
__std_exp                           libc063
__std_expm1                         libc063
__std_log1p                         libc063
__std_log                           libc063
__std_hypot                         libc063
__std_fmod                          libc063
__std_rand_r                        libc063
__std_strcoll                       libc063
__std_ctime_r                       libc063
__getprogname                       libc063
__std_vsnprintf                     libc063
__std_writev                        libc063
__std_getdtablesize                 libc063
__std_strspn                        libc063
__std_ftok                          libc063
__std_waitpid                       libc063
__std_fork                          libc063
__std_chdir                         libc063
__std_execle                        libc063
__std_perror                        libc063
__std_execl                         libc063
__std_fseek                         libc063
__std_fopen                         libc063
__std_ftell                         libc063
__std_clearerr                      libc063
__std_fread                         libc063
__std_remove                        libc063
__std_fdopen                        libc063
__std_rename                        libc063
__std_chmod                         libc063
__std_putc                          libc063
__std_atol                          libc063
__std_atof                          libc063
__std_lstat                         libc063
__std_getcwd                        libc063
__std_utime                         libc063
__std_chown                         libc063
__std_lchown                        libc063
__std_creat                         libc063
__std_mkdir                         libc063
__std_rmdir                         libc063
__std_asctime_r                     libc063
__std_fputs                         libc063
___strnlen                          libc063
__std_vsprintf                      libc063
__std_setmode                       libc063
__std_fflush                        libc063
__std_rewind                        libc063
__std_rewinddir                     libc063
__std_setvbuf                       libc063
__std_setitimer                     libc063
__std_signal                        libc063
__std_sigemptyset                   libc063
__std_sigaddset                     libc063
__std_sigprocmask                   libc063
__std_siglongjmp                    libc063
__std_snprintf                      libc063
DosTrueGetMessage                   msg
___ctordtorInit1                    libc063
___ctordtorTerm1                    libc063
__std_vfprintf                      libc063
__std_iconv                         libc063
__std_iconv_open                    libc063
__std_iconv_close                   libc063
__std_strlen                        libc063
__std_puts                          libc063
__fmutex_create                     libc063
___libc_Back_threadSleep            libc063
___fmutex_request_internal          libc063
___fmutex_release_internal          libc063
___libc_GpFIBLIS                    libc063
___fmutex_request_internal_must_complete libc063
___fmutex_release_internal_must_complete libc063
DosQueryModuleName                  doscalls
__endthread                         libc063
DosUnsetExceptionHandler            doscalls
DosSetPriority                      doscalls
__beginthread                       libc063
__gettid                            libc063
DosWaitThread                       doscalls
DosEnterCritSec                     doscalls
DosExitCritSec                      doscalls
DosCreateEventSem                   doscalls
DosCloseEventSem                    doscalls
DosPostEventSem                     doscalls
DosWaitEventSem                     doscalls
__std_ftime                         libc063
__std_ferror                        libc063
__std_feof                          libc063
__std_fgets                         libc063
DosTmrQueryTime                     doscalls
DosPerfSysCall                      doscalls
DosAllocMem                         doscalls
DosQuerySysState                    doscalls
__std_random                        libc063
__std_tcgetattr                     libc063
__std_tcsetattr                     libc063
__std_sigaction                     libc063


                        +--------------------+
                        |   Libraries Used   |
                        +--------------------+

U:\extras\lib\libz.lib
U:\extras\lib\xmlrpc.lib
U:\extras\lib\libcrypto.lib
U:\extras\lib\libssl.lib
U:\extras\lib\pthread.lib
U:\extras\lib\expat.lib
U:\extras\lib\poll.lib
U:\extras\lib\xml2.lib
U:\tmp\ldconv_libgcc_eh_a_3ed14e78ff52199cf0.lib
U:\tmp\ldconv_libgcc_a_3ed14e78ff521a1dd8.lib
U:\usr\lib\libc_alias.lib
U:\usr\lib\libc_dll.lib
U:\usr\lib\libos2.lib
U:\usr\lib\libend.lib


                        +-----------------------+
                        |   Linker Statistics   |
                        +-----------------------+

Stack size:  0000 (0.)
Memory size:  00836ec0 (8613568.)
Link time: 00:00.76
